** EXPERIMENTAL (HLL) ** Open Watcom Linker Version 1.6beta1 Limited Availability
Portions Copyright (c) 1985-2002 Sybase, Inc. All Rights Reserved.
Created on:       10/07/24 13:03:15
Executable Image: .libs/php5.dll
creating an OS/2 EMX dynamic link library


                        +------------+
                        |   Groups   |
                        +------------+

Group                           Address              Size
=====                           =======              ====

CGROUP                          0001:00000000        00883ff0
DGROUP                          0002:00000000        00021cc0



                        +--------------+
                        |   Segments   |
                        +--------------+

Segment                Class          Group          Address         Size
=======                =====          =====          =======         ====

TEXT32                 CODE           CGROUP         0001:00000000   00883fe8
________TEXT           CODE           CGROUP         0001:00883ff0   00000000
DATA32                 DATA           DGROUP         0002:00000000   000088a0
SET1__os2dll           DATA           DGROUP         0002:000088a0   00000004
SET2__os2dll           DATA           DGROUP         0002:000088a4   00000000
SET3__os2dll           DATA           DGROUP         0002:000088a4   00000004
SET1___CTOR_LIST__     DATA           DGROUP         0002:000088a8   00000004
SET2___CTOR_LIST__     DATA           DGROUP         0002:000088ac   00000000
SET3___CTOR_LIST__     DATA           DGROUP         0002:000088ac   00000004
SET1___DTOR_LIST__     DATA           DGROUP         0002:000088b0   00000004
SET2___DTOR_LIST__     DATA           DGROUP         0002:000088b4   00000000
SET3___DTOR_LIST__     DATA           DGROUP         0002:000088b4   00000004
SET1___crtinit1__      DATA           DGROUP         0002:000088b8   00000004
SET2___crtinit1__      DATA           DGROUP         0002:000088bc   00000000
SET3___crtinit1__      DATA           DGROUP         0002:000088bc   00000004
SET1___crtexit1__      DATA           DGROUP         0002:000088c0   00000004
SET2___crtexit1__      DATA           DGROUP         0002:000088c4   00000000
SET3___crtexit1__      DATA           DGROUP         0002:000088c4   00000004
SET1___eh_frame__      DATA           DGROUP         0002:000088c8   00000004
SET2___eh_frame__      DATA           DGROUP         0002:000088cc   00000014
SET3___eh_frame__      DATA           DGROUP         0002:000088e0   00000004
SET1___eh_init__       DATA           DGROUP         0002:000088e4   00000004
SET2___eh_init__       DATA           DGROUP         0002:000088e8   00000004
SET3___eh_init__       DATA           DGROUP         0002:000088ec   00000004
SET1___eh_term__       DATA           DGROUP         0002:000088f0   00000004
SET2___eh_term__       DATA           DGROUP         0002:000088f4   00000004
SET3___eh_term__       DATA           DGROUP         0002:000088f8   00000004
SET1___fork_parent1__  DATA           DGROUP         0002:000088fc   00000004
SET2___fork_parent1__  DATA           DGROUP         0002:00008900   00000000
SET3___fork_parent1__  DATA           DGROUP         0002:00008900   00000004
SET1___fork_child1__   DATA           DGROUP         0002:00008904   00000004
SET2___fork_child1__   DATA           DGROUP         0002:00008908   00000000
SET3___fork_child1__   DATA           DGROUP         0002:00008908   00000004
________DATA           DATA           DGROUP         0002:00008910   00000000
BSS32                  BSS            DGROUP         0002:00008910   00017120
c_common               BSS            DGROUP         0002:0001fa30   00002290
________BSS            BSS            DGROUP         0002:00021cc0   00000000


                        +----------------+
                        |   Memory Map   |
                        +----------------+

* = unreferenced symbol
+ = symbol only referenced locally

Address        Symbol
=======        ======

Module: U:\usr\lib\dll0.obj({standard input})
0001:00000000* __text
0002:00000000* __data
0002:00000000* ___data_start
0002:00008910* ___bss_start
0002:000088a0+ __os2dll
0002:000088a8  ___CTOR_LIST__
0002:000088b0  ___DTOR_LIST__
0002:000088b8* ___crtinit1__
0002:000088c0* ___crtexit1__
0002:000088c8  ___eh_frame__
0002:000088e4  ___eh_init__
0002:000088f0  ___eh_term__
0002:000088fc+ ___fork_parent1__
0002:00008904+ ___fork_child1__
Module: U:\dev\php-5.3.3\ext\date\php_date.o(php_date.o)
0002:0001fa30  _date_ce_date
0002:0001fa40  _date_ce_timezone
0002:0001fa50  _date_globals_id
0002:0001fa60  _php_date_global_timezone_db
0002:0001fa70  _date_ce_interval
0002:0001fa80  _php_date_global_timezone_db_enabled
0002:0001fa90  _date_ce_period
0001:000000a0  _php_date_get_date_ce
0001:000000aa  _php_date_get_timezone_ce
0001:000002fb  _zm_activate_date
0001:0000035c  _zif_timezone_version_get
0001:000003c3  _zif_date_default_timezone_set
0001:000004cf  _zif_timezone_abbreviations_list
0001:00000761  _zif_timezone_identifiers_list
0001:00000c09  _zim_DatePeriod___construct
0001:00001047  _zim_DateInterval___construct
0001:0000120e  _zif_date_timestamp_get
0001:000012d1  _zif_date_timezone_get
0001:00001474  _zif_date_interval_format
0001:00001aba  _zif_date_interval_create_from_date_string
0001:00001b9c  _php_parse_date
0001:00001ccf  _zif_timezone_location_get
0001:00001e13  _zif_timezone_offset_get
0001:00001f76  _zif_date_offset_get
0001:000020a2  _zif_timezone_name_from_abbr
0001:0000215e  _zif_timezone_name_get
0001:00002517  _zim_DateTimeZone___construct
0001:000025cb  _zif_timezone_open
0001:00002a38  _zif_date_diff
0001:00002bb3  _zif_date_timezone_set
0001:00002d10  _php_date_short_day_name
0001:00002d58  _php_date_full_day_name
0001:000040b3  _zif_date_format
0001:000046db  _php_date_do_return_parsed_time
0001:00004d83  _zif_date_parse_from_format
0001:00004e48  _zif_date_parse
0001:00004ef8  _zif_date_get_last_errors
0001:00004f5a  _zif_time
0001:00004fb1  _date_object_period_get_iterator
0001:00005021  _zif_checkdate
0001:000050be  _php_date_set_tzdb
0001:000053d3  _get_timezone_info
0001:000054fe  _zif_date_sun_info
0001:0000600a  _zif_date_sunset
0001:00006048  _zif_date_sunrise
0001:00006086  _zif_date_default_timezone_get
0001:0000667a  _zim_DateTime___wakeup
0001:000066c7  _zim_DateTime___set_state
0001:0000677e  _zim_DateTime___construct
0001:0000685c  _zif_date_create_from_format
0001:0000694f  _zif_date_create
0001:00006a4d  _zif_getdate
0001:00006d24  _zif_localtime
0001:0000703b  _php_strftime
0001:000072c8  _zif_gmstrftime
0001:00007306  _zif_strftime
0001:000073a3  _php_mktime
0001:00007671  _zif_gmmktime
0001:000076af  _zif_mktime
0001:000076f9  _zif_strtotime
0001:0000797e  _php_idate
0001:00007f68  _zif_idate
0001:00008037  _php_format_date
0001:000080eb  _zif_timezone_transitions_get
0001:00008a43  _zif_gmdate
0001:00008a81  _zif_date
0001:00008b33  _zm_info_date
0001:00008bfb  _zm_shutdown_date
0001:0000c1f0  _date_funcs_date
0001:0000c3c0  _date_funcs_timezone
0001:0000c480  _date_funcs_interval
0001:0000adfe  _date_interval_read_property
0001:0000b068  _date_interval_write_property
0001:0000c4d0  _date_funcs_period
0001:00009861  _zm_startup_date
0001:0000a00d  _zm_deactivate_date
0001:0000a0be  _zif_date_timestamp_set
0001:0000a1c8  _zif_date_date_set
0001:0000a2ea  _zif_date_time_set
0001:0000a40e  _zif_date_isodate_set
0001:0000a585  _zif_date_modify
0001:0000a7a2  _zif_date_add
0001:0000aabc  _zif_date_sub
0001:0000bd90  _date_functions
0002:000000b0  _date_period_it_funcs
0002:00000050  _date_module_entry
Module: U:\dev\php-5.3.3\ext\date\lib\astro.o(astro.o)
0001:0000dc80  _timelib_ts_to_juliandate
0001:0000dc9a  _timelib_astro_rise_set_altitude
Module: U:\dev\php-5.3.3\ext\date\lib\dow.o(dow.o)
0001:0000e530  _timelib_day_of_week
0001:0000e56e  _timelib_iso_day_of_week
0001:0000e5ac  _timelib_day_of_year
0001:0000e646  _timelib_days_in_month
0001:0000e6bd  _timelib_isoweek_from_date
0001:0000e9a5  _timelib_daynr_from_weeknr
0001:0000ea57  _timelib_valid_time
0001:0000eab2  _timelib_valid_date
Module: U:\dev\php-5.3.3\ext\date\lib\parse_date.o(parse_date.o)
0001:0000ecc0  _timelib_timezone_abbreviations_list
0001:0000edbf  _timelib_timezone_id_from_abbr
0001:0000edeb  _timelib_fill_holes
0001:00010267  _timelib_parse_from_format
0001:0001164c  _timelib_strtotime
Module: U:\dev\php-5.3.3\ext\date\lib\parse_tz.o(parse_tz.o)
0001:00036d10  _timelib_builtin_db
0001:00036d1a  _timelib_timezone_builtin_identifiers_list
0001:00039c80  _timezonedb_idx_builtin
0001:00036e83  _timelib_timestamp_is_in_dst
0001:00036ebd  _timelib_get_time_zone_info
0001:0003701c  _timelib_get_current_offset
0001:00037199  _timelib_timezone_id_is_valid
0001:000371ba  _timelib_parse_tzfile
0001:000378fe  _timelib_dump_tzinfo
0001:0003ae30  _timelib_timezone_db_data_builtin
0001:0007a2b0  _timezonedb_builtin
Module: U:\dev\php-5.3.3\ext\date\lib\timelib.o(timelib.o)
0001:0007a2d0  _timelib_date_to_int
0001:0007a386  _timelib_dump_rel_time
0001:0007a534  _timelib_dump_date
0001:0007a8be  _timelib_decimal_hour_to_hms
0001:0007a94c  _timelib_error_container_dtor
0001:0007a9c5  _timelib_tzinfo_dtor
0001:0007aa74  _timelib_time_offset_dtor
0001:0007aaa1  _timelib_rel_time_dtor
0001:0007aab6  _timelib_time_dtor
0001:0007aae3  _timelib_get_tz_abbr_ptr
0001:0007ab10  _timelib_time_offset_ctor
0001:0007ab2c  _timelib_rel_time_ctor
0001:0007ab48  _timelib_rel_time_clone
0001:0007ab62  _timelib_time_ctor
0001:0007ab7e  _timelib_tzinfo_ctor
0001:0007abb0  _timelib_tzinfo_clone
0001:0007acca  _timelib_time_tz_abbr_update
Module: U:\dev\php-5.3.3\ext\date\lib\tm2unixtime.o(tm2unixtime.o)
0001:0007aeba  _timelib_do_rel_normalize
0001:0007b631  _timelib_update_ts
Module: U:\dev\php-5.3.3\ext\date\lib\unixtime2tm.o(unixtime2tm.o)
0001:0007c230  _timelib_unixtime2gmt
0001:0007c7ea  _timelib_set_timezone
0001:0007c866  _timelib_update_from_sse
0001:0007c963  _timelib_unixtime2local
0001:0007ca75  _timelib_apply_localtime
Module: U:\dev\php-5.3.3\ext\date\lib\parse_iso_intervals.o(parse_iso_intervals.o)
0001:0007cda3  _timelib_strtointerval
Module: U:\dev\php-5.3.3\ext\date\lib\interval.o(interval.o)
0001:0007dfa0  _timelib_diff
Module: U:\dev\php-5.3.3\ext\ereg\ereg.o(ereg.o)
0002:0001faa0  _ereg_globals_id
0001:0007e2a2  _zm_shutdown_ereg
0001:0007e2ab  _zif_sql_regcase
0001:0007e98f  _zif_spliti
0001:0007e9cd  _zif_split
0001:0007ea0b  _php_ereg_replace
0001:0007f184  _zif_eregi_replace
0001:0007f1c2  _zif_ereg_replace
0001:0007f639  _zif_eregi
0001:0007f677  _zif_ereg
0001:0007f6db  _zm_info_ereg
0001:0007f708  _zm_startup_ereg
0001:0007f7c0  _ereg_functions
0002:00000130  _ereg_module_entry
Module: U:\dev\php-5.3.3\ext\ereg\regex\regcomp.o(regcomp.o)
0001:00081c34  _php_regcomp
Module: U:\dev\php-5.3.3\ext\ereg\regex\regexec.o(regexec.o)
0001:00084d95  _php_regexec
Module: U:\dev\php-5.3.3\ext\ereg\regex\regerror.o(regerror.o)
0001:00085eee  _php_regerror
Module: U:\dev\php-5.3.3\ext\ereg\regex\regfree.o(regfree.o)
0001:000863d0  _php_regfree
Module: U:\dev\php-5.3.3\ext\libxml\libxml.o(libxml.o)
0001:00086473  _php_libxml_switch_context
0001:0008648e  _php_libxml_xmlCheckUTF8
0001:000868a7  _php_libxml_increment_doc_ref
0001:00086d3d  _php_libxml_decrement_node_ptr
0001:00086d91  _php_libxml_increment_node_ptr
0001:00088302  _php_libxml_structured_error_handler
0001:00088287  _php_libxml_error_handler
0001:00087401  _php_libxml_decrement_doc_ref
0001:00087611  _php_libxml_node_free_resource
0001:000876f4  _php_libxml_node_decrement_resource
0001:00087766  _php_libxml_import_node
0001:000877ce  _php_libxml_shutdown
0001:00087810  _php_libxml_initialize
0001:00087e74  _php_libxml_register_export
0001:000882b0  _php_libxml_ctx_warning
0001:000882d9  _php_libxml_ctx_error
0001:0008831b  _php_libxml_issue_error
0002:00000190  _libxml_module_entry
Module: U:\dev\php-5.3.3\ext\pcre\pcrelib\pcre_chartables.o(pcre_chartables.o)
0001:000885c0  _php__pcre_default_tables
Module: U:\dev\php-5.3.3\ext\pcre\pcrelib\pcre_ucd.o(pcre_ucd.o)
0001:00088a00  _php__pcre_ucd_records
0001:00089a30  _php__pcre_ucd_stage1
0001:0008bc30  _php__pcre_ucd_stage2
Module: U:\dev\php-5.3.3\ext\pcre\pcrelib\pcre_compile.o(pcre_compile.o)
0001:000972bc  __pcre_find_bracket
0001:0009ec55  _php_pcre_compile2
0001:0009f6f4  _php_pcre_compile
Module: U:\dev\php-5.3.3\ext\pcre\pcrelib\pcre_config.o(pcre_config.o)
0001:000a0460  _php_pcre_config
Module: U:\dev\php-5.3.3\ext\pcre\pcrelib\pcre_exec.o(pcre_exec.o)
0001:000a0686  _php_pcre_exec
Module: U:\dev\php-5.3.3\ext\pcre\pcrelib\pcre_fullinfo.o(pcre_fullinfo.o)
0001:000ad310  _php_pcre_fullinfo
Module: U:\dev\php-5.3.3\ext\pcre\pcrelib\pcre_get.o(pcre_get.o)
0001:000ad540  _php_pcre_free_substring_list
0001:000ad54e  _php_pcre_free_substring
0001:000ad55c  _php_pcre_get_substring
0001:000ad5c7  _php_pcre_get_substring_list
0001:000ad67b  _php_pcre_copy_substring
0001:000ad6d3  _php_pcre_get_stringtable_entries
0001:000ad870  _php_pcre_get_stringnumber
0001:000ada1c  _php_pcre_get_named_substring
0001:000ada74  _php_pcre_copy_named_substring
Module: U:\dev\php-5.3.3\ext\pcre\pcrelib\pcre_globals.o(pcre_globals.o)
0002:000001f0  _php_pcre_malloc
0002:000001f4  _php_pcre_free
0002:000001f8  _php_pcre_stack_malloc
0002:000001fc  _php_pcre_stack_free
0002:00008b50  _php_pcre_callout
Module: U:\dev\php-5.3.3\ext\pcre\pcrelib\pcre_info.o(pcre_info.o)
0001:000adae0  _php_pcre_info
Module: U:\dev\php-5.3.3\ext\pcre\pcrelib\pcre_maketables.o(pcre_maketables.o)
0001:000adb7d  _php_pcre_maketables
Module: U:\dev\php-5.3.3\ext\pcre\pcrelib\pcre_newline.o(pcre_newline.o)
0001:000adf10  _php__pcre_is_newline
0001:000ae00d  _php__pcre_was_newline
Module: U:\dev\php-5.3.3\ext\pcre\pcrelib\pcre_ord2utf8.o(pcre_ord2utf8.o)
0001:000ae130  _php__pcre_ord2utf8
Module: U:\dev\php-5.3.3\ext\pcre\pcrelib\pcre_refcount.o(pcre_refcount.o)
0001:000ae1a0  _php_pcre_refcount
Module: U:\dev\php-5.3.3\ext\pcre\pcrelib\pcre_study.o(pcre_study.o)
0001:000aefb4  _php_pcre_study
Module: U:\dev\php-5.3.3\ext\pcre\pcrelib\pcre_tables.o(pcre_tables.o)
0001:000af1c0  _php__pcre_OP_lengths
0001:000af240  _php__pcre_utf8_table1
0001:000af258  _php__pcre_utf8_table1_size
0001:000af260  _php__pcre_utf8_table2
0001:000af280  _php__pcre_utf8_table3
0001:000af2a0  _php__pcre_utf8_table4
0001:000af2e0  _php__pcre_ucp_gentype
0001:000af360  _php__pcre_utt_names
0001:000af700  _php__pcre_utt
0001:000afa14  _php__pcre_utt_size
Module: U:\dev\php-5.3.3\ext\pcre\pcrelib\pcre_try_flipped.o(pcre_try_flipped.o)
0001:000afa62  _php__pcre_try_flipped
Module: U:\dev\php-5.3.3\ext\pcre\pcrelib\pcre_valid_utf8.o(pcre_valid_utf8.o)
0001:000afc30  _php__pcre_valid_utf8
Module: U:\dev\php-5.3.3\ext\pcre\pcrelib\pcre_version.o(pcre_version.o)
0001:000afda0  _php_pcre_version
Module: U:\dev\php-5.3.3\ext\pcre\pcrelib\pcre_xclass.o(pcre_xclass.o)
0001:000afdb0  _php__pcre_xclass
Module: U:\dev\php-5.3.3\ext\pcre\php_pcre.o(php_pcre.o)
0002:0001fab0  _pcre_globals_id
0001:000b0ec4  _pcre_get_compiled_regex_cache
0001:000b15fc  _pcre_get_compiled_regex_ex
0001:000b1676  _pcre_get_compiled_regex
0001:000b16fd  _php_pcre_grep_impl
0001:000b1bb3  _php_pcre_replace_impl
0001:000b2a0d  _php_pcre_replace
0001:000b3687  _php_pcre_split_impl
0001:000b3dde  _php_pcre_match_impl
0002:00000200  _pcre_module_entry
Module: U:\dev\php-5.3.3\ext\sqlite3\sqlite3.o(sqlite3.o)
0002:0001fac0  _php_sqlite3_sc_entry
0002:0001fad0  _php_sqlite3_stmt_entry
0002:0001fae0  _php_sqlite3_result_entry
0002:0001faf0  _sqlite3_globals_id
0001:000b52a5  _zm_info_sqlite3
0001:000b531b  _zm_shutdown_sqlite3
0001:000b545c  _zm_startup_sqlite3
0001:000b5eee  _zim_sqlite3result___construct
0001:000b5f1f  _zim_sqlite3stmt_close
0001:000b5f8e  _zim_sqlite3_enableExceptions
0001:000b60dc  _zim_sqlite3result_finalize
0001:000b618d  _zim_sqlite3result_reset
0001:000b6253  _zim_sqlite3stmt_reset
0001:000b62ee  _zim_sqlite3result_columnType
0001:000b638a  _zim_sqlite3result_columnName
0001:000b647e  _zim_sqlite3_lastErrorMsg
0001:000b669c  _zim_sqlite3result_fetchArray
0001:000b6853  _zim_sqlite3result_numColumns
0001:000b6904  _zim_sqlite3stmt___construct
0001:000b6b12  _zim_sqlite3stmt_execute
0001:000b6f06  _zim_sqlite3_prepare
0001:000b7207  _zim_sqlite3stmt_bindValue
0001:000b732e  _zim_sqlite3stmt_bindParam
0001:000b7469  _zim_sqlite3stmt_clear
0001:000b7502  _zim_sqlite3stmt_paramCount
0001:000b757d  _zim_sqlite3_openBlob
0001:000b77c9  _zim_sqlite3_createAggregate
0001:000b7a55  _zim_sqlite3_createFunction
0001:000b82f3  _zim_sqlite3_querySingle
0001:000b85f5  _zim_sqlite3_query
0001:000b88ad  _zim_sqlite3_exec
0001:000b8997  _zim_sqlite3_escapeString
0001:000b8a4e  _zim_sqlite3_changes
0001:000b8bac  _zim_sqlite3_loadExtension
0001:000b8efb  _zim_sqlite3_busyTimeout
0001:000b8fc0  _zim_sqlite3_lastErrorCode
0001:000b903e  _zim_sqlite3_lastInsertRowID
0001:000b90d8  _zim_sqlite3_version
0001:000b9185  _zim_sqlite3_close
0001:000b9366  _zim_sqlite3_open
0002:00000260  _sqlite3_module_entry
Module: U:\dev\php-5.3.3\ext\sqlite3\libsqlite\sqlite3.o(sqlite3.o)
0001:000b9db8  _sqlite3_compileoption_used
0001:000b9f6d  _sqlite3_compileoption_get
0001:000b9f83  _sqlite3_db_status
0001:000ba43f  _sqlite3_mutex_free
0001:000ba456  _sqlite3_mutex_enter
0001:000ba46d  _sqlite3_mutex_try
0001:000ba487  _sqlite3_mutex_leave
0001:000ba49e  _sqlite3_vfs_unregister
0001:000ba518  _sqlite3_release_memory
0001:000ba56c  _sqlite3_memory_alarm
0001:000ba759  _sqlite3_free
0001:000baba2  _sqlite3_strnicmp
0001:000bcacb  _sqlite3_enable_shared_cache
0001:000bd0bc  _sqlite3_backup_remaining
0001:000bd0c7  _sqlite3_backup_pagecount
0001:000bd0d2  _sqlite3_sql
0001:000bd731  _sqlite3_expired
0001:000bd74b  _sqlite3_value_type
0001:000bd757  _sqlite3_user_data
0001:000bd764  _sqlite3_context_db_handle
0001:000bd76f  _sqlite3_get_auxdata
0001:000bd792  _sqlite3_aggregate_count
0001:000bd7a0  _sqlite3_column_count
0001:000bd7b2  _sqlite3_data_count
0001:000bd840  _sqlite3_column_name
0001:000bd86a  _sqlite3_column_name16
0001:000bd894  _sqlite3_column_decltype
0001:000bd8be  _sqlite3_column_decltype16
0001:000bd8e8  _sqlite3_column_database_name
0001:000bd912  _sqlite3_column_database_name16
0001:000bd93c  _sqlite3_column_table_name
0001:000bd966  _sqlite3_column_table_name16
0001:000bd990  _sqlite3_column_origin_name
0001:000bd9ba  _sqlite3_column_origin_name16
0001:000bd9e4  _sqlite3_bind_parameter_count
0001:000bda6f  _sqlite3_bind_parameter_name
0001:000bdaa7  _sqlite3_db_handle
0001:000bdab7  _sqlite3_next_stmt
0001:000bdaf3  _sqlite3_stmt_status
0001:000bdb4c  _sqlite3_blob_bytes
0001:000be786  _sqlite3_set_authorizer
0001:000bf86e  _sqlite3_enable_load_extension
0001:000bfb9e  _sqlite3_free_table
0001:000c0d10  _sqlite3_complete
0001:000c15f3  _sqlite3_libversion
0001:000c163d  _sqlite3_sourceid
0001:000c1647  _sqlite3_libversion_number
0001:000c1651  _sqlite3_threadsafe
0001:000c17c4  _sqlite3_db_mutex
0001:000c1881  _sqlite3_last_insert_rowid
0001:000c188f  _sqlite3_changes
0001:000c189a  _sqlite3_total_changes
0001:000c193f  _sqlite3_busy_handler
0001:000c1983  _sqlite3_progress_handler
0001:000c19f1  _sqlite3_busy_timeout
0001:000c1a3b  _sqlite3_interrupt
0001:000c1a4d  _sqlite3_trace
0001:000c1a8f  _sqlite3_profile
0001:000c1ad1  _sqlite3_commit_hook
0001:000c1b13  _sqlite3_update_hook
0001:000c1b55  _sqlite3_rollback_hook
0001:000c1b97  _sqlite3_limit
0001:000c1bcf  _sqlite3_collation_needed
0001:000c1c13  _sqlite3_collation_needed16
0001:000c1c57  _sqlite3_global_recover
0001:000c1c5e  _sqlite3_get_autocommit
0001:000c1c6a  _sqlite3_thread_cleanup
0001:000c1c6f  _sqlite3_extended_result_codes
0001:000c2975  _fts3SnippetShift
0001:000c2c30  _sqlite3_db_config
0001:000c8493  _sqlite3_log
0001:000c88ba  _sqlite3_config
0001:000c8acb  _sqlite3_status
0001:000c8b16  _sqlite3_memory_highwater
0001:000c8b43  _sqlite3_memory_used
0001:000c8bf1  _sqlite3_extended_errcode
0001:000c8c37  _sqlite3_errcode
0001:000c8d9a  _sqlite3_snprintf
0001:000dd572  _sqlite3_value_text
0001:000dd557  _sqlite3_value_text16
0001:00126f09  _sqlite3_version
0001:000ce65e  _sqlite3_file_control
0001:000cf095  _sqlite3_bind_parameter_index
0001:000cf7b0  _sqlite3_os_end
0001:000cf7f0  _os2CurrentTime
0001:000d0324  _sqlite3_os_init
0001:000d59fd  _sqlite3_vfs_register
0001:000d0347  _sqlite3_initialize
0001:000d3a0e  _sqlite3_malloc
0001:000d07d3  _sqlite3_reset_auto_extension
0001:000d0828  _sqlite3_shutdown
0001:000d08da  _sqlite3_vmprintf
0001:000d0957  _sqlite3_mprintf
0001:000d0980  _sqlite3_realloc
0001:000d22cd  _sqlite3_set_auxdata
0001:000d3961  _sqlite3_auto_extension
0001:000d5916  _sqlite3_soft_heap_limit
0001:000d5990  _sqlite3_mutex_alloc
0001:000d5aae  _sqlite3_vfs_find
0001:000d5b21  _sqlite3_sleep
0001:000d5b71  _sqlite3_randomness
0001:000d5ce5  _sqlite3_test_control
0001:000dd521  _sqlite3_value_text16le
0001:000dd53c  _sqlite3_value_text16be
0001:000dd5a9  _sqlite3_errmsg
0001:000dd658  _sqlite3_value_blob
0001:000dd696  _sqlite3_value_bytes16
0001:000dd6df  _sqlite3_value_bytes
0001:000dd7a1  _sqlite3_value_double
0001:000de5ea  _sqlite3_value_int64
0001:000de5f6  _sqlite3_value_int
0001:000dfdc3  _sqlite3_result_int64
0001:000dfe13  _sqlite3_result_int
0001:000dffa1  _sqlite3_transfer_bindings
0001:000dfff2  _sqlite3_result_zeroblob
0001:000e00c3  _sqlite3_clear_bindings
0001:000e05db  _sqlite3_result_value
0001:000e06d6  _sqlite3_aggregate_context
0001:000e0e40  _sqlite3_create_module_v2
0001:000e0e4c  _sqlite3_create_module
0001:000e0f04  _sqlite3_load_extension
0001:000e1417  _sqlite3_create_collation_v2
0001:000e1483  _sqlite3_create_collation
0001:000e179e  _sqlite3_overload_function
0001:000e186b  _sqlite3_create_function
0001:000e1961  _sqlite3_column_type
0001:000e1990  _sqlite3_column_value
0001:000e19d0  _sqlite3_column_text16
0001:000e1a05  _sqlite3_column_text
0001:000e1a3a  _sqlite3_column_blob
0001:000e1a6f  _sqlite3_column_bytes16
0001:000e1aa4  _sqlite3_column_bytes
0001:000e1ad9  _sqlite3_column_double
0001:000e1b0e  _sqlite3_column_int64
0001:000e1b90  _sqlite3_column_int
0001:000e1d3c  _sqlite3_bind_null
0001:000e1d72  _sqlite3_bind_int64
0001:000e1ddd  _sqlite3_bind_int
0001:000e1e03  _sqlite3_bind_zeroblob
0001:000e2313  _sqlite3_result_error_toobig
0001:000e239c  _sqlite3_result_error_code
0001:000e2446  _sqlite3_result_text16le
0001:000e2476  _sqlite3_result_text16be
0001:000e24a6  _sqlite3_result_text16
0001:000e24d6  _sqlite3_result_text
0001:000e2c79  _sqlite3_result_blob
0001:000e306b  _sqlite3_result_error16
0001:000e30a6  _sqlite3_result_error
0001:000e35e5  _sqlite3_create_collation16
0001:000e3688  _sqlite3_create_function16
0001:000e3813  _sqlite3_value_numeric_type
0001:000e39f3  _sqlite3_errmsg16
0001:000e622e  _sqlite3_bind_text16
0001:000e6265  _sqlite3_bind_text
0001:000e629c  _sqlite3_bind_blob
0001:000e632b  _sqlite3_bind_double
0001:000e6382  _sqlite3_bind_value
0001:000e6470  _sqlite3_result_double
0001:000e6605  _sqlite3_result_error_nomem
0001:000e7921  _sqlite3_result_null
0001:000e7bb3  _sqlite3_close
0001:000e8266  _sqlite3_backup_finish
0001:000e8f9e  _sqlite3_backup_step
0001:000ed661  _sqlite3_blob_write
0001:000ed691  _sqlite3_blob_read
0001:000ed701  _sqlite3_finalize
0001:000ed843  _sqlite3_blob_close
0001:000ed891  _sqlite3_reset
0001:000ed97e  _sqlite3_complete16
0001:000edbd9  _convertCpPathToUtf8
0001:000f0bd4  _sqlite3_backup_init
0001:000f15fd  _sqlite3_open16
0001:000f16c4  _sqlite3_open_v2
0001:000f16d0  _sqlite3_open
0001:00103c6b  _sqlite3_declare_vtab
0001:00106150  _sqlite3_prepare16_v2
0001:00106187  _sqlite3_prepare16
0001:001061be  _sqlite3_prepare_v2
0001:00106387  _sqlite3_prepare
0001:00106449  _sqlite3_step
0001:0010920b  _sqlite3_exec
0001:0010961e  _fts3DbExec
0001:0010a364  _sqlite3_table_column_metadata
0001:00118bc1  _sqlite3_get_table
0001:0011c954  _sqlite3_blob_open
0002:00008cb0  _sqlite3_temp_directory
Module: U:\dev\php-5.3.3\ext\zlib\zlib.o(zlib.o)
0002:0001fb00  _zlib_globals_id
0001:0012d6de  _php_ob_gzhandler_check
0002:00000f60  _php_zlib_module_entry
Module: U:\dev\php-5.3.3\ext\zlib\zlib_fopen_wrapper.o(zlib_fopen_wrapper.o)
0001:0012e569  _php_stream_gzopen
0002:00000fc0  _php_stream_gzip_wrapper
Module: U:\dev\php-5.3.3\ext\zlib\zlib_filter.o(zlib_filter.o)
0002:00001040  _php_zlib_filter_factory
Module: U:\dev\php-5.3.3\ext\ctype\ctype.o(ctype.o)
0002:00001060  _ctype_module_entry
Module: U:\dev\php-5.3.3\ext\dom\php_dom.o(php_dom.o)
0002:0001fb10  _dom_domimplementation_class_entry
0002:0001fb20  _dom_nodelist_class_entry
0002:0001fb30  _dom_namednodemap_class_entry
0002:0001fb40  _dom_object_handlers
0002:0001fbb0  _dom_namespace_node_class_entry
0002:0001fbc0  _dom_entity_class_entry
0002:0001fbd0  _dom_notation_class_entry
0002:0001fbe0  _dom_documentfragment_class_entry
0002:0001fbf0  _dom_documenttype_class_entry
0002:0001fc00  _dom_document_class_entry
0002:0001fc10  _dom_comment_class_entry
0002:0001fc20  _dom_processinginstruction_class_entry
0002:0001fc30  _dom_entityreference_class_entry
0002:0001fc40  _dom_cdatasection_class_entry
0002:0001fc50  _dom_text_class_entry
0002:0001fc60  _dom_attr_class_entry
0002:0001fc70  _dom_element_class_entry
0002:0001fc80  _dom_xpath_class_entry
0002:0001fc90  _dom_node_class_entry
0002:0001fca0  _dom_domexception_class_entry
0002:0001fcb0  _dom_domstringlist_class_entry
0002:0001fcc0  _dom_namelist_class_entry
0002:0001fcd0  _dom_domimplementationlist_class_entry
0002:0001fce0  _dom_domimplementationsource_class_entry
0002:0001fcf0  _dom_characterdata_class_entry
0002:0001fd00  _dom_typeinfo_class_entry
0002:0001fd10  _dom_userdatahandler_class_entry
0002:0001fd20  _dom_domerror_class_entry
0002:0001fd30  _dom_domerrorhandler_class_entry
0002:0001fd40  _dom_domlocator_class_entry
0002:0001fd50  _dom_domconfiguration_class_entry
0002:0001fd60  _dom_string_extend_class_entry
0001:00130d00  _dom_node_is_read_only
0001:00130d61  _dom_node_children_valid
0001:00130d7d  _dom_object_get_node
0001:00130d96  _php_dom_object_get_data
0001:00130db1  _dom_hierarchy
0001:00130dee  _dom_get_nsdecl
0001:00130e75  _dom_get_elements_by_tag_name_ns_raw
0001:00131001  _dom_get_ns
0001:001310da  _dom_check_qname
0001:0013115c  _dom_set_old_ns
0001:001311db  _node_list_unlink
0001:00131298  _dom_normalize
0001:0013138a  _dom_has_feature
0001:00131414  _php_dom_create_implementation
0001:00131439  _php_dom_create_interator
0001:00131475  _dom_get_doc_props
0001:001315b8  _dom_namednode_iter
0001:0013162d  _dom_get_doc_classmap
0001:0013169f  _php_dom_create_object
0001:001319a4  _dom_nnodemap_objects_new
0001:00131bf2  _dom_objects_clone
0001:00131b1b  _dom_nnodemap_objects_free_storage
0001:00131a33  _dom_objects_new
0001:00131d75  _dom_objects_free_storage
0001:00131ae7  _dom_get_strict_error
0001:00131b4f  _dom_xpath_objects_new
0001:00131de4  _dom_xpath_objects_free_storage
0001:00131e62  _zm_shutdown_dom
0001:00131ff6  _zm_info_dom
0001:00132992  _zm_startup_dom
0001:00136f75  _dom_read_property
0001:00136e5c  _dom_write_property
0001:001370fe  _dom_objects_store_clone_obj
0001:001371c9  _php_dom_export_node
0001:00137235  _zif_dom_import_simplexml
0001:00137319  _dom_set_doc_classmap
0002:000010c0  _dom_module_entry
Module: U:\dev\php-5.3.3\ext\dom\attr.o(attr.o)
0001:00137524  _zif_dom_attr_is_id
0001:001375ec  _dom_attr_schema_type_info_read
0001:00137635  _dom_attr_specified_read
0001:00137686  _dom_attr_owner_element_read
0001:0013774f  _dom_attr_value_write
0001:00137839  _dom_attr_value_read
0001:00137911  _dom_attr_name_read
0001:001379a0  _zim_domattr___construct
0001:00137b30  _php_dom_attr_class_functions
Module: U:\dev\php-5.3.3\ext\dom\document.o(document.o)
0001:00137c04  _zif_dom_document_rename_node
0001:00137c2b  _zif_dom_document_adopt_node
0001:00137ced  _zim_domdocument_registerNodeClass
0001:00137f87  _zif_dom_document_save_html
0001:001380aa  _zif_dom_document_save_html_file
0001:0013846e  _zim_domdocument_loadHTML
0001:001384ac  _zim_domdocument_loadHTMLFile
0001:001384ea  _zif_dom_document_validate
0001:00138676  _zif_dom_document_xinclude
0001:00138799  _zif_dom_document_savexml
0001:00138a99  _zif_dom_document_save
0001:00138c26  __dom_get_valid_file_path
0001:00138fe1  _zif_dom_document_relaxNG_validate_xml
0001:0013901f  _zif_dom_document_relaxNG_validate_file
0001:0013932a  _zif_dom_document_schema_validate_xml
0001:00139368  _zif_dom_document_schema_validate_file
0001:0013989a  _zim_domdocument_loadXML
0001:001398d8  _zim_domdocument_load
0001:0013991b  _zim_domdocument___construct
0001:00139ab6  _zif_dom_document_normalize_document
0001:00139b57  _zif_dom_document_get_element_by_id
0001:00139c7f  _zif_dom_document_get_elements_by_tag_name_ns
0001:00139db6  _zif_dom_document_get_elements_by_tag_name
0001:00139ec1  _zif_dom_document_create_attribute
0001:0013a05a  _zif_dom_document_create_attribute_ns
0001:0013a318  _zif_dom_document_create_element
0001:0013a4b1  _zif_dom_document_create_element_ns
0001:0013a797  _zif_dom_document_import_node
0001:0013aa1f  _zif_dom_document_create_entity_reference
0001:0013ab85  _zif_dom_document_create_processing_instruction
0001:0013ad15  _zif_dom_document_create_cdatasection
0001:0013ae37  _zif_dom_document_create_comment
0001:0013af52  _zif_dom_document_create_text_node
0001:0013b06d  _zif_dom_document_create_document_fragment
0001:0013b173  _dom_document_config_read
0001:0013b199  _dom_document_document_uri_read
0001:0013b235  _dom_document_substitue_entities_read
0001:0013b295  _dom_document_recover_read
0001:0013b2f5  _dom_document_preserve_whitespace_read
0001:0013b355  _dom_document_resolve_externals_read
0001:0013b3b5  _dom_document_validate_on_parse_read
0001:0013b415  _dom_document_format_output_read
0001:0013b474  _dom_document_strict_error_checking_read
0001:0013b4d4  _dom_document_version_read
0001:0013b571  _dom_document_standalone_read
0001:0013b5dc  _dom_document_encoding_read
0001:0013b679  _dom_document_document_element_read
0001:0013b74b  _dom_document_implementation_read
0001:0013b781  _dom_document_doctype_read
0001:0013b853  _dom_document_format_output_write
0001:0013b8e6  _dom_document_encoding_write
0001:0013b9f8  _dom_document_strict_error_checking_write
0001:0013ba72  _dom_document_standalone_write
0001:0013bb36  _dom_document_document_uri_write
0001:0013bc06  _dom_document_version_write
0001:0013bcd6  _dom_document_substitue_entities_write
0001:0013bd4d  _dom_document_recover_write
0001:0013bdc7  _dom_document_preserve_whitespace_write
0001:0013be42  _dom_document_resolve_externals_write
0001:0013bebc  _dom_document_validate_on_parse_write
0001:0013c120  _php_dom_document_class_functions
Module: U:\dev\php-5.3.3\ext\dom\domerrorhandler.o(domerrorhandler.o)
0001:0013cc44  _zif_dom_domerrorhandler_handle_error
0001:0013cc80  _php_dom_domerrorhandler_class_functions
Module: U:\dev\php-5.3.3\ext\dom\domstringlist.o(domstringlist.o)
0001:0013cd04  _zif_dom_domstringlist_item
0001:0013cd30  _dom_domstringlist_length_read
0001:0013cd90  _php_dom_domstringlist_class_functions
Module: U:\dev\php-5.3.3\ext\dom\domexception.o(domexception.o)
0001:0013cdf0  _php_dom_throw_error_with_message
0001:0013ce39  _php_dom_throw_error
0001:0013ce80  _php_dom_domexception_class_functions
Module: U:\dev\php-5.3.3\ext\dom\namelist.o(namelist.o)
0001:0013d034  _zif_dom_namelist_get_namespace_uri
0001:0013d05b  _zif_dom_namelist_get_name
0001:0013d087  _dom_namelist_length_read
0001:0013d0f0  _php_dom_namelist_class_functions
Module: U:\dev\php-5.3.3\ext\dom\processinginstruction.o(processinginstruction.o)
0001:0013d1a0  _dom_processinginstruction_data_write
0001:0013d277  _dom_processinginstruction_data_read
0001:0013d34f  _dom_processinginstruction_target_read
0001:0013d3de  _zim_domprocessinginstruction___construct
0001:0013d570  _php_dom_processinginstruction_class_functions
Module: U:\dev\php-5.3.3\ext\dom\cdatasection.o(cdatasection.o)
0001:0013d603  _zim_domcdatasection___construct
0001:0013d740  _php_dom_cdatasection_class_functions
Module: U:\dev\php-5.3.3\ext\dom\documentfragment.o(documentfragment.o)
0001:0013d829  _zim_domdocumentfragment_appendXML
0001:0013d9a6  _zim_domdocumentfragment___construct
0001:0013dac0  _php_dom_documentfragment_class_functions
Module: U:\dev\php-5.3.3\ext\dom\domimplementation.o(domimplementation.o)
0001:0013db64  _zim_domimplementation_getFeature
0001:0013dbf2  _zim_domimplementation_createDocument
0001:0013dfac  _zim_domimplementation_createDocumentType
0001:0013e1a5  _zim_domimplementation_hasFeature
0001:0013e260  _php_dom_domimplementation_class_functions
Module: U:\dev\php-5.3.3\ext\dom\element.o(element.o)
0001:0013e502  _zif_dom_element_set_id_attribute_node
0001:0013e669  _zif_dom_element_set_id_attribute_ns
0001:0013e7c3  _zif_dom_element_set_id_attribute
0001:0013e92f  _zif_dom_element_has_attribute_ns
0001:0013ebad  _zif_dom_element_has_attribute
0001:0013ec80  _zif_dom_element_get_elements_by_tag_name_ns
0001:0013edb7  _zif_dom_element_get_elements_by_tag_name
0001:0013ef02  _zif_dom_element_set_attribute_node_ns
0001:0013f201  _zif_dom_element_get_attribute_node_ns
0001:0013f333  _zif_dom_element_remove_attribute_node
0001:0013f504  _zif_dom_element_set_attribute_node
0001:0013f7b4  _zif_dom_element_remove_attribute_ns
0001:0013f984  _zif_dom_element_remove_attribute
0001:0013fb2b  _zif_dom_element_set_attribute
0001:0013fdec  _zif_dom_element_set_attribute_ns
0001:0014048d  _zif_dom_element_get_attribute_ns
0001:00140619  _zif_dom_element_get_attribute
0001:0014078f  _zif_dom_element_get_attribute_node
0001:0014094d  _dom_element_schema_type_info_read
0001:00140975  _dom_element_tag_name_read
0001:00140a87  _zim_domelement___construct
0001:00140ee0  _php_dom_element_class_functions
Module: U:\dev\php-5.3.3\ext\dom\node.o(node.o)
0001:00141610  _dom_node_text_content_write
0001:0014162b  _zif_dom_node_get_user_data
0001:00141652  _zif_dom_node_set_user_data
0001:00141679  _zif_dom_node_get_feature
0001:001416a0  _zif_dom_node_is_equal_node
0001:001416c7  _zif_dom_node_compare_document_position
0001:0014171b  _zim_domnode_getLineNo
0001:001417dd  _zim_domnode_getNodePath
0001:001418ca  _zif_dom_node_is_same_node
0001:001419a8  _zif_dom_node_has_attributes
0001:00142149  _zim_domnode_C14NFile
0001:00142187  _zim_domnode_C14N
0001:001421c9  _zif_dom_node_lookup_namespace_uri
0001:001422ec  _zif_dom_node_is_default_namespace
0001:00142402  _zif_dom_node_lookup_prefix
0001:00142580  _zif_dom_node_is_supported
0001:00142612  _zif_dom_node_normalize
0001:001426da  _zif_dom_node_clone_node
0001:001428eb  _zif_dom_node_has_child_nodes
0001:001429b6  _zif_dom_node_remove_child
0001:00142d89  _zif_dom_node_append_child
0001:00143207  _zif_dom_node_replace_child
0001:0014363c  _zif_dom_node_insert_before
0001:00143d2a  _dom_node_text_content_read
0001:00143dfd  _dom_node_local_name_read
0001:00143eaa  _dom_node_prefix_read
0001:00143f93  _dom_node_namespace_uri_read
0001:0014406f  _dom_node_owner_document_read
0001:0014415c  _dom_node_next_sibling_read
0001:0014421a  _dom_node_previous_sibling_read
0001:001442e3  _dom_node_last_child_read
0001:001443d3  _dom_node_first_child_read
0001:001444c3  _dom_node_parent_node_read
0001:0014458c  _dom_node_node_type_read
0001:00144607  _dom_node_node_value_read
0001:00144725  _dom_node_base_uri_read
0001:0014482d  _dom_node_prefix_write
0001:00144abb  _dom_node_attributes_read
0001:00144b89  _dom_node_child_nodes_read
0001:00144c5f  _dom_node_node_value_write
0001:00144dde  _dom_node_node_name_read
0001:00145120  _php_dom_node_class_functions
Module: U:\dev\php-5.3.3\ext\dom\string_extend.o(string_extend.o)
0001:001458e4  _zif_dom_string_extend_find_offset32
0001:0014590b  _zif_dom_string_extend_find_offset16
0001:00145950  _php_dom_string_extend_class_functions
Module: U:\dev\php-5.3.3\ext\dom\characterdata.o(characterdata.o)
0001:00145a27  _zif_dom_characterdata_replace_data
0001:00145c8c  _zif_dom_characterdata_delete_data
0001:00145e82  _zif_dom_characterdata_insert_data
0001:00146038  _zif_dom_characterdata_append_data
0001:001460ff  _zif_dom_characterdata_substring_data
0001:001462c5  _dom_characterdata_length_read
0001:00146350  _dom_characterdata_data_read
0001:00146428  _dom_characterdata_data_write
0001:00146540  _php_dom_characterdata_class_functions
Module: U:\dev\php-5.3.3\ext\dom\documenttype.o(documenttype.o)
0001:00146751  _dom_documenttype_internal_subset_read
0001:00146867  _dom_documenttype_system_id_read
0001:0014690d  _dom_documenttype_public_id_read
0001:001469b3  _dom_documenttype_name_read
0001:00146a3d  _dom_documenttype_notations_read
0001:00146afe  _dom_documenttype_entities_read
0001:00146bc0  _php_dom_documenttype_class_functions
Module: U:\dev\php-5.3.3\ext\dom\domimplementationlist.o(domimplementationlist.o)
0001:00146bf4  _zif_dom_domimplementationlist_item
0001:00146c20  _dom_domimplementationlist_length_read
0001:00146c80  _php_dom_domimplementationlist_class_functions
Module: U:\dev\php-5.3.3\ext\dom\entity.o(entity.o)
0001:00146ce0  _dom_entity_actual_encoding_write
0001:00146ce7  _dom_entity_encoding_write
0001:00146cee  _dom_entity_version_write
0001:00146cf5  _dom_entity_version_read
0001:00146d1b  _dom_entity_encoding_read
0001:00146d41  _dom_entity_actual_encoding_read
0001:00146d67  _dom_entity_notation_name_read
0001:00146e1a  _dom_entity_system_id_read
0001:00146eb8  _dom_entity_public_id_read
0001:00146f60  _php_dom_entity_class_functions
Module: U:\dev\php-5.3.3\ext\dom\nodelist.o(nodelist.o)
0001:00146fa6  _zif_dom_nodelist_item
0001:001471e0  _dom_nodelist_length_read
0001:00147320  _php_dom_nodelist_class_functions
Module: U:\dev\php-5.3.3\ext\dom\text.o(text.o)
0001:00147394  _zif_dom_text_replace_whole_text
0001:001473cf  _zif_dom_text_is_whitespace_in_element_content
0001:00147491  _zif_dom_text_split_text
0001:00147677  _dom_text_whole_text_read
0001:001477aa  _zim_domtext___construct
0001:00147920  _php_dom_text_class_functions
Module: U:\dev\php-5.3.3\ext\dom\comment.o(comment.o)
0001:00147a64  _zim_domcomment___construct
0001:00147b90  _php_dom_comment_class_functions
Module: U:\dev\php-5.3.3\ext\dom\domconfiguration.o(domconfiguration.o)
0001:00147c04  _zif_dom_domconfiguration_can_set_parameter
0001:00147c2b  _zif_dom_domconfiguration_get_parameter
0001:00147c52  _zif_dom_domconfiguration_set_parameter
0001:00147cb0  _php_dom_domconfiguration_class_functions
Module: U:\dev\php-5.3.3\ext\dom\domimplementationsource.o(domimplementationsource.o)
0001:00147df4  _zif_dom_domimplementationsource_get_domimplementations
0001:00147e1b  _zif_dom_domimplementationsource_get_domimplementation
0001:00147e70  _php_dom_domimplementationsource_class_functions
Module: U:\dev\php-5.3.3\ext\dom\entityreference.o(entityreference.o)
0001:00147f23  _zim_domentityreference___construct
0001:001480a0  _php_dom_entityreference_class_functions
Module: U:\dev\php-5.3.3\ext\dom\notation.o(notation.o)
0001:00148101  _dom_notation_system_id_read
0001:001481a7  _dom_notation_public_id_read
0001:00148250  _php_dom_notation_class_functions
Module: U:\dev\php-5.3.3\ext\dom\xpath.o(xpath.o)
0001:0014828e  _zif_dom_xpath_register_php_functions
0001:001485fa  _dom_xpath_document_read
0001:00148bb9  _zif_dom_xpath_evaluate
0001:00148bf7  _zif_dom_xpath_query
0001:00148c39  _zif_dom_xpath_register_ns
0001:00148d44  _zim_domxpath___construct
0001:001499c0  _php_dom_xpath_class_functions
Module: U:\dev\php-5.3.3\ext\dom\dom_iterators.o(dom_iterators.o)
0001:00149cf9  _php_dom_libxml_hash_iter
0001:00149d67  _create_notation
0001:00149e08  _php_dom_libxml_notation_iter
0001:0014a0c1  _php_dom_get_iterator
0002:00001120  _php_dom_iterator_funcs
Module: U:\dev\php-5.3.3\ext\dom\typeinfo.o(typeinfo.o)
0001:0014a2d0  _dom_typeinfo_type_namespace_read
0001:0014a2f6  _dom_typeinfo_type_name_read
0001:0014a320  _php_dom_typeinfo_class_functions
Module: U:\dev\php-5.3.3\ext\dom\domerror.o(domerror.o)
0001:0014a345  _dom_domerror_location_read
0001:0014a393  _dom_domerror_related_data_read
0001:0014a3e1  _dom_domerror_related_exception_read
0001:0014a42f  _dom_domerror_type_read
0001:0014a47d  _dom_domerror_message_read
0001:0014a4cb  _dom_domerror_severity_read
0001:0014a520  _php_dom_domerror_class_functions
Module: U:\dev\php-5.3.3\ext\dom\domlocator.o(domlocator.o)
0001:0014a545  _dom_domlocator_uri_read
0001:0014a593  _dom_domlocator_related_node_read
0001:0014a5e1  _dom_domlocator_offset_read
0001:0014a62f  _dom_domlocator_column_number_read
0001:0014a67d  _dom_domlocator_line_number_read
0001:0014a6d0  _php_dom_domlocator_class_functions
Module: U:\dev\php-5.3.3\ext\dom\namednodemap.o(namednodemap.o)
0001:0014a704  _zif_dom_namednodemap_remove_named_item_ns
0001:0014a72b  _zif_dom_namednodemap_set_named_item_ns
0001:0014a752  _zif_dom_namednodemap_remove_named_item
0001:0014a779  _zif_dom_namednodemap_set_named_item
0001:0014a7ca  _zif_dom_namednodemap_get_named_item_ns
0001:0014a949  _zif_dom_namednodemap_item
0001:0014aaa8  _zif_dom_namednodemap_get_named_item
0001:0014ac0a  _dom_namednodemap_length_read
0001:0014ad10  _php_dom_namednodemap_class_functions
Module: U:\dev\php-5.3.3\ext\dom\userdatahandler.o(userdatahandler.o)
0001:0014afa4  _zif_dom_userdatahandler_handle
0001:0014afe0  _php_dom_userdatahandler_class_functions
Module: U:\dev\php-5.3.3\ext\fileinfo\fileinfo.o(fileinfo.o)
0002:0001fd70  _finfo_class_entry
0001:0014b05d  _zif_finfo_set_flags
0001:0014b91f  _zif_mime_content_type
0001:0014b965  _zif_finfo_buffer
0001:0014b9ab  _zif_finfo_file
0001:0014b9f3  _zif_finfo_close
0001:0014ba93  _finfo_resource_destructor
0001:0014bb03  _zif_finfo_open
0001:0014bd29  _zm_info_fileinfo
0001:0014be17  _zm_startup_finfo
0001:0014c113  _finfo_objects_new
0002:00001140  _finfo_class_functions
0002:000011b0  _fileinfo_functions
0002:00001240  _fileinfo_module_entry
Module: U:\dev\php-5.3.3\ext\fileinfo\libmagic\apprentice.o(apprentice.o)
0002:0001fd80  _file_formats
0002:0001fe30  _file_names
0001:0014c682  _file_showstr
0001:0014c7f3  _file_signextend
0001:0014f2a5  _file_delmagic
0001:00150680  _php_magic_database
0001:00150500  _file_apprentice
0001:00150678  _file_nformats
0001:0015067c  _file_nnames
Module: U:\dev\php-5.3.3\ext\fileinfo\libmagic\ascmagic.o(ascmagic.o)
0001:002fc6ce  _file_ascmagic_with_encoding
0001:002fcf2a  _file_ascmagic
Module: U:\dev\php-5.3.3\ext\fileinfo\libmagic\cdf.o(cdf.o)
0001:002fd740  _cdf_tole2
0001:002fd761  _cdf_tole4
0001:002fd788  _cdf_tole8
0001:002fd7da  _cdf_swap_header
0001:002fda4a  _cdf_swap_dir
0001:002fdbe0  _cdf_swap_class
0001:002fdc73  _cdf_print_elapsed_time
0001:002fde42  _cdf_print_property_name
0001:002fded9  _cdf_print_classid
0001:002fdf54  _cdf_count_chain
0001:002fdffe  _cdf_read_short_sector
0001:002fe037  _cdf_unpack_dir
0001:002fe0c7  _cdf_unpack_header
0001:002fe18a  _cdf_read_property_info
0001:002fe95a  _cdf_unpack_summary_info
0001:002feb70  _cdf_read_short_sector_chain
0001:002fed9f  _cdf_read_sector
0001:002fedd0  _cdf_read_ssat
0001:002fef32  _cdf_read_dir
0001:002ff151  _cdf_read_long_sector_chain
0001:002ff2c8  _cdf_read_short_stream
0001:002ff361  _cdf_read_sector_chain
0001:002ff3cf  _cdf_read_summary_info
0001:002ff4fd  _cdf_read_sat
0001:002ff7e7  _cdf_read_header
Module: U:\dev\php-5.3.3\ext\fileinfo\libmagic\cdf_time.o(cdf_time.o)
0001:002ffaa0  _cdf_timespec_to_timestamp
0001:002ffaa7  _cdf_timestamp_to_timespec
Module: U:\dev\php-5.3.3\ext\fileinfo\libmagic\compress.o(compress.o)
0001:002ffe7d  _sread
0001:002fff8f  _file_pipe2file
Module: U:\dev\php-5.3.3\ext\fileinfo\libmagic\encoding.o(encoding.o)
0001:00300180  _file_looks_utf8
0001:003003f1  _file_encoding
Module: U:\dev\php-5.3.3\ext\fileinfo\libmagic\fsmagic.o(fsmagic.o)
0001:00300bf2  _file_fsmagic
Module: U:\dev\php-5.3.3\ext\fileinfo\libmagic\funcs.o(funcs.o)
0001:00300f50  _file_check_mem
0001:00300fc3  _file_getbuffer
0001:00301094  _file_printf
0001:003011d8  _file_buffer
0001:003016a4  _file_magerror
0001:003016d4  _file_error
0001:0030171a  _file_reset
0001:00301796  _file_badread
0001:003017ca  _file_badseek
0001:0030180a  _file_oomem
Module: U:\dev\php-5.3.3\ext\fileinfo\libmagic\is_tar.o(is_tar.o)
0001:003018a3  _file_is_tar
Module: U:\dev\php-5.3.3\ext\fileinfo\libmagic\magic.o(magic.o)
0001:00301af0  _magic_error
0001:00301b03  _magic_errno
0001:00301b16  _magic_setflags
0001:00301b26  _magic_buffer
0001:00301f4d  _magic_stream
0001:00301f6f  _magic_file
0001:00301f91  _magic_descriptor
0001:0030200b  _magic_compile
0001:00302041  _magic_load
0001:00302083  _magic_close
0001:003020dd  _magic_open
Module: U:\dev\php-5.3.3\ext\fileinfo\libmagic\print.o(print.o)
0001:003021a1  _file_fmttime
0001:0030220a  _file_magwarn
Module: U:\dev\php-5.3.3\ext\fileinfo\libmagic\readcdf.o(readcdf.o)
0001:00302808  _file_trycdf
Module: U:\dev\php-5.3.3\ext\fileinfo\libmagic\softmagic.o(softmagic.o)
0001:0030628b  _file_softmagic
Module: U:\dev\php-5.3.3\ext\filter\filter.o(filter.o)
0002:0001fee0  _filter_globals_id
0001:003068a9  _zif_filter_id
0001:0030693d  _zif_filter_list
0001:00306b71  _zif_filter_has_var
0001:00306ca4  _zm_info_filter
0001:00306cfd  _zm_deactivate_filter
0001:00306df4  _zm_shutdown_filter
0001:003072a4  _zm_startup_filter
0001:00308bec  _zif_filter_var
0001:00308cdc  _zif_filter_input
0001:00309368  _zif_filter_var_array
0001:00309413  _zif_filter_input_array
0002:000012a0  _filter_module_entry
Module: U:\dev\php-5.3.3\ext\filter\sanitizing_filters.o(sanitizing_filters.o)
0001:00309bd0  _php_filter_magic_quotes
0001:00309ce8  _php_filter_number_float
0001:00309db8  _php_filter_number_int
0001:00309e7f  _php_filter_url
0001:00309f61  _php_filter_email
0001:0030a106  _php_filter_encoded
0001:0030a515  _php_filter_unsafe_raw
0001:0030a5b7  _php_filter_special_chars
0001:0030a656  _php_filter_full_special_chars
0001:0030a6d2  _php_filter_string
Module: U:\dev\php-5.3.3\ext\filter\logical_filters.o(logical_filters.o)
0001:0030a93b  _php_filter_validate_url
0001:0030ab3d  _php_filter_validate_regexp
0001:0030b1bb  _php_filter_validate_email
0001:0030b2f6  _php_filter_int
0001:0030b895  _php_filter_float
0001:0030bf4b  _php_filter_boolean
0001:0030c120  _php_filter_validate_ip
Module: U:\dev\php-5.3.3\ext\filter\callback_filter.o(callback_filter.o)
0001:0030c512  _php_filter_callback
Module: U:\dev\php-5.3.3\ext\ftp\php_ftp.o(php_ftp.o)
0001:0030c703  _zif_ftp_get_option
0001:0030c880  _zif_ftp_set_option
0001:0030ca09  _zif_ftp_close
0001:0030cabb  _zif_ftp_site
0001:0030cb97  _zif_ftp_delete
0001:0030cc77  _zif_ftp_rename
0001:0030cd68  _zif_ftp_mdtm
0001:0030ce10  _zif_ftp_size
0001:0030ceeb  _zif_ftp_nb_put
0001:0030d151  _zif_ftp_put
0001:0030d3c5  _zif_ftp_nb_fput
0001:0030d63d  _zif_ftp_fput
0001:0030d8b6  _zif_ftp_nb_continue
0001:0030da2b  _zif_ftp_nb_fget
0001:0030dcb4  _zif_ftp_nb_get
0001:0030e01c  _zif_ftp_get
0001:0030e36b  _zif_ftp_fget
0001:0030e5b2  _zif_ftp_pasv
0001:0030e661  _zif_ftp_systype
0001:0030e74a  _zif_ftp_rawlist
0001:0030e84a  _zif_ftp_nlist
0001:0030e93c  _zif_ftp_alloc
0001:0030ea51  _zif_ftp_chmod
0001:0030eb45  _zif_ftp_rmdir
0001:0030ec21  _zif_ftp_mkdir
0001:0030ed0e  _zif_ftp_raw
0001:0030edb4  _zif_ftp_exec
0001:0030ee90  _zif_ftp_chdir
0001:0030ef6c  _zif_ftp_cdup
0001:0030f033  _zif_ftp_pwd
0001:0030f117  _zif_ftp_login
0001:0030f211  _zif_ftp_ssl_connect
0001:0030f2fe  _zif_ftp_connect
0001:0030f3ff  _zm_info_ftp
0001:0030f4a5  _zm_startup_ftp
0001:0030f820  _php_ftp_functions
0002:00001300  _php_ftp_module_entry
Module: U:\dev\php-5.3.3\ext\ftp\ftp.o(ftp.o)
0001:003108bd  _ftp_gc
0001:00310909  _ftp_close
0001:00310e81  _data_writeable
0001:00310ee1  _data_available
0001:0031124f  _ftp_nb_continue_write
0001:0031144d  _ftp_site
0001:003114b2  _ftp_rename
0001:00311538  _ftp_delete
0001:0031158e  _ftp_rmdir
0001:003115e5  _ftp_cdup
0001:00311658  _ftp_chdir
0001:003116d0  _ftp_exec
0001:00311727  _ftp_reinit
0001:00311791  _ftp_quit
0001:00311885  _ftp_login
0001:00311b71  _ftp_mdtm
0001:00311cb1  _ftp_size
0001:00311d44  _ftp_pasv
0001:00312368  _ftp_nb_put
0001:003124a3  _ftp_put
0001:003126f8  _ftp_alloc
0001:00312795  _ftp_chmod
0001:0031283a  _ftp_syst
0001:003128f2  _ftp_mkdir
0001:00312993  _ftp_pwd
0001:00312a56  _ftp_open
0001:00312c00  _ftp_raw
0001:00312cf6  _ftp_nb_continue_read
0001:00312ede  _ftp_nb_get
0001:00313019  _ftp_get
0001:00313646  _ftp_list
0001:00313681  _ftp_nlist
Module: U:\dev\php-5.3.3\ext\hash\hash.o(hash.o)
0002:0001fef0  _php_hash_hashtable
0001:003136d9  _zm_info_hash
0001:003137b6  _zm_shutdown_hash
0001:0031384a  _zif_hash_algos
0001:003138f9  _zif_hash_update
0001:003139af  _php_hash_copy
0001:003139d7  _zif_hash_copy
0001:00313b0c  _zif_hash_final
0001:00313d68  _zif_hash_update_file
0001:00313f3b  _zif_hash_update_stream
0001:003140e7  _php_hash_register_algo
0001:003142f3  _zm_startup_hash
0001:003146cd  _php_hash_fetch_ops
0001:00314770  _zif_hash_init
0001:00314d40  _zif_hash_hmac
0001:00314d59  _zif_hash_hmac_file
0001:0031500c  _zif_hash
0001:00315025  _zif_hash_file
0001:003150c0  _hash_functions
0002:00001360  _hash_module_entry
Module: U:\dev\php-5.3.3\ext\hash\hash_md.o(hash_md.o)
0001:00315af2  _PHP_MD4Init
0001:00315b9a  _PHP_MD2Init
0001:00315be1  _PHP_MD2Final
0001:00315c4a  _PHP_MD2Update
0001:00315d5a  _PHP_MD4Update
0001:00315e34  _PHP_MD4Final
0001:00315f00  _php_hash_md5_ops
0001:00315f20  _php_hash_md4_ops
0001:00315f40  _php_hash_md2_ops
Module: U:\dev\php-5.3.3\ext\hash\hash_sha.o(hash_sha.o)
0001:003160a0  _PHP_SHA256Init
0001:003160ed  _PHP_SHA224Init
0001:003161bc  _PHP_SHA384Init
0001:0031624f  _PHP_SHA512Init
0001:00316cd3  _PHP_SHA512Update
0001:00316dea  _PHP_SHA512Final
0001:00316f2a  _PHP_SHA384Update
0001:00317041  _PHP_SHA384Final
0001:00317181  _PHP_SHA256Update
0001:0031725b  _PHP_SHA256Final
0001:00317327  _PHP_SHA224Update
0001:00317401  _PHP_SHA224Final
0001:003174d0  _php_hash_sha1_ops
0001:003174f0  _php_hash_sha256_ops
0001:00317510  _php_hash_sha224_ops
0001:00317530  _php_hash_sha384_ops
0001:00317550  _php_hash_sha512_ops
Module: U:\dev\php-5.3.3\ext\hash\hash_ripemd.o(hash_ripemd.o)
0001:00317af0  _PHP_RIPEMD128Init
0001:00317b21  _PHP_RIPEMD256Init
0001:00317b6e  _PHP_RIPEMD160Init
0001:00317ba6  _PHP_RIPEMD320Init
0001:00318b01  _PHP_RIPEMD320Update
0001:00318bdb  _PHP_RIPEMD320Final
0001:00318c8f  _PHP_RIPEMD160Update
0001:00318d69  _PHP_RIPEMD160Final
0001:00318e1d  _PHP_RIPEMD256Update
0001:00318ef7  _PHP_RIPEMD256Final
0001:00318fab  _PHP_RIPEMD128Update
0001:00319085  _PHP_RIPEMD128Final
0001:00319140  _php_hash_ripemd128_ops
0001:00319160  _php_hash_ripemd160_ops
0001:00319180  _php_hash_ripemd256_ops
0001:003191a0  _php_hash_ripemd320_ops
Module: U:\dev\php-5.3.3\ext\hash\hash_haval.o(hash_haval.o)
0001:00319381  _PHP_3HAVAL128Init
0001:003193c5  _PHP_3HAVAL160Init
0001:00319409  _PHP_3HAVAL192Init
0001:0031944d  _PHP_3HAVAL224Init
0001:00319491  _PHP_3HAVAL256Init
0001:003194d5  _PHP_4HAVAL128Init
0001:00319519  _PHP_4HAVAL160Init
0001:0031955d  _PHP_4HAVAL192Init
0001:003195a1  _PHP_4HAVAL224Init
0001:003195e5  _PHP_4HAVAL256Init
0001:00319629  _PHP_5HAVAL128Init
0001:0031966d  _PHP_5HAVAL160Init
0001:003196b1  _PHP_5HAVAL192Init
0001:003196f5  _PHP_5HAVAL224Init
0001:00319739  _PHP_5HAVAL256Init
0001:0031a47e  _PHP_HAVALUpdate
0001:0031a55a  _PHP_HAVAL256Final
0001:0031a60f  _PHP_HAVAL224Final
0001:0031a70b  _PHP_HAVAL192Final
0001:0031a848  _PHP_HAVAL160Final
0001:0031a99e  _PHP_HAVAL128Final
0001:0031ab00  _php_hash_3haval128_ops
0001:0031ab20  _php_hash_3haval160_ops
0001:0031ab40  _php_hash_3haval192_ops
0001:0031ab60  _php_hash_3haval224_ops
0001:0031ab80  _php_hash_3haval256_ops
0001:0031aba0  _php_hash_4haval128_ops
0001:0031abc0  _php_hash_4haval160_ops
0001:0031abe0  _php_hash_4haval192_ops
0001:0031ac00  _php_hash_4haval224_ops
0001:0031ac20  _php_hash_4haval256_ops
0001:0031ac40  _php_hash_5haval128_ops
0001:0031ac60  _php_hash_5haval160_ops
0001:0031ac80  _php_hash_5haval192_ops
0001:0031aca0  _php_hash_5haval224_ops
0001:0031acc0  _php_hash_5haval256_ops
Module: U:\dev\php-5.3.3\ext\hash\hash_tiger.o(hash_tiger.o)
0001:0031b280  _PHP_4TIGERInit
0001:0031b2c2  _PHP_3TIGERInit
0001:00320612  _PHP_TIGER192Final
0001:0032072e  _PHP_TIGER160Final
0001:00320814  _PHP_TIGER128Final
0001:003208dd  _PHP_TIGERUpdate
0001:003268e0  _php_hash_3tiger128_ops
0001:00326900  _php_hash_3tiger160_ops
0001:00326920  _php_hash_3tiger192_ops
0001:00326940  _php_hash_4tiger128_ops
0001:00326960  _php_hash_4tiger160_ops
0001:00326980  _php_hash_4tiger192_ops
Module: U:\dev\php-5.3.3\ext\hash\hash_gost.o(hash_gost.o)
0001:00329bb6  _PHP_GOSTInit
0001:00329bcb  _PHP_GOSTUpdate
0001:00329deb  _PHP_GOSTFinal
0001:00329f20  _php_hash_gost_ops
Module: U:\dev\php-5.3.3\ext\hash\hash_snefru.o(hash_snefru.o)
0001:0032af40  _PHP_SNEFRUInit
0001:0032af55  _PHP_SNEFRUUpdate
0001:0032b9b8  _PHP_SNEFRUFinal
0001:0032c1f0  _php_hash_snefru_ops
Module: U:\dev\php-5.3.3\ext\hash\hash_whirlpool.o(hash_whirlpool.o)
0001:00331b45  _PHP_WHIRLPOOLUpdate
0001:00331d6a  _PHP_WHIRLPOOLInit
0001:00331d7f  _PHP_WHIRLPOOLFinal
0001:00331ed0  _php_hash_whirlpool_ops
Module: U:\dev\php-5.3.3\ext\hash\hash_adler32.o(hash_adler32.o)
0001:00335f50  _PHP_ADLER32Init
0001:00335f5e  _PHP_ADLER32Update
0001:00335fdb  _PHP_ADLER32Final
0001:00336006  _PHP_ADLER32Copy
0001:00336020  _php_hash_adler32_ops
Module: U:\dev\php-5.3.3\ext\hash\hash_crc32.o(hash_crc32.o)
0001:00336040  _PHP_CRC32Init
0001:0033604e  _PHP_CRC32Update
0001:0033608b  _PHP_CRC32BUpdate
0001:003360c4  _PHP_CRC32Final
0001:003360f4  _PHP_CRC32BFinal
0001:00336124  _PHP_CRC32Copy
0001:00336140  _php_hash_crc32_ops
0001:00336160  _php_hash_crc32b_ops
Module: U:\dev\php-5.3.3\ext\hash\hash_salsa.o(hash_salsa.o)
0001:00336eef  _PHP_SALSA20Init
0001:00336f0e  _PHP_SALSA10Init
0001:00336f2d  _PHP_SALSAUpdate
0001:00337168  _PHP_SALSAFinal
0001:00337230  _php_hash_salsa10_ops
0001:00337250  _php_hash_salsa20_ops
Module: U:\dev\php-5.3.3\ext\json\json.o(json.o)
0002:0001ff20  _json_globals_id
0001:0033904d  _php_json_encode
0001:0033a256  _php_json_decode
0002:000013c0  _json_module_entry
Module: U:\dev\php-5.3.3\ext\json\utf8_to_utf16.o(utf8_to_utf16.o)
0001:0033a9e0  _utf8_to_utf16
Module: U:\dev\php-5.3.3\ext\json\utf8_decode.o(utf8_decode.o)
0001:0033aa70  _utf8_decode_init
0001:0033aa98  _utf8_decode_at_byte
0001:0033aaa3  _utf8_decode_at_character
0001:0033aab7  _utf8_decode_next
Module: U:\dev\php-5.3.3\ext\json\JSON_parser.o(JSON_parser.o)
0001:0033ad10  _free_JSON_parser
0001:0033b564  _parse_JSON
0001:0033c4b4  _new_JSON_parser
Module: U:\dev\php-5.3.3\ext\pdo\pdo.o(pdo.o)
0002:0001ff30  _pdo_dbh_ce
0002:0001ff40  _pdo_exception_ce
0002:0001ff50  _pdo_driver_hash
0002:0001ff80  _pdo_globals_id
0002:0001ff90  _pdo_dbstmt_ce
0002:0001ffa0  _pdo_row_ce
0001:0033d600  _php_pdo_list_entry
0001:0033d60a  _php_pdo_get_dbh_ce
0001:0033d614  _php_pdo_get_exception
0001:0033d62c  _php_pdo_int64_to_str
0001:0033d80f  _zm_info_pdo
0001:0033d91b  _zm_shutdown_pdo
0001:0033d936  _php_pdo_parse_data_source
0001:0033db3d  _pdo_find_driver
0001:0033db7c  _php_pdo_unregister_driver
0001:0033dc4d  _php_pdo_register_driver
0001:0033dd06  _zif_pdo_drivers
0001:0033ddbc  _php_pdo_get_exception_base
0001:0033de5a  _zm_startup_pdo
0001:0033e027  _php_pdo_str_tolower_dup
0001:0033e070  _pdo_functions
0002:00001420  _pdo_module_entry
Module: U:\dev\php-5.3.3\ext\pdo\pdo_dbh.o(pdo_dbh.o)
0001:0033e10a  _php_pdo_dbh_addref
0001:0033e5bf  _php_pdo_pdbh_dtor
0001:0033e671  _php_pdo_dbh_delref
0001:0033e67d  _pdo_dbh_new
0001:0033eb7e  _pdo_dbh_init
0001:003431b0  _pdo_dbh_functions
0001:0033f859  _pdo_handle_error
0001:0033fb8a  _pdo_raise_impl_error
0001:00342d44  _pdo_hash_methods
Module: U:\dev\php-5.3.3\ext\pdo\pdo_stmt.o(pdo_stmt.o)
0002:0001ffb0  _pdo_dbstmt_object_handlers
0001:003435ba  _php_pdo_stmt_addref
0001:0034508b  _pdo_row_new
0001:003460e3  _pdo_row_free_storage
0001:0034615e  _php_pdo_stmt_delref
0001:0034617c  _pdo_dbstmt_free_storage
0001:00346185  _pdo_stmt_describe_columns
0001:0034654c  _pdo_dbstmt_new
0001:00346754  _pdo_stmt_init
0001:00349910  _pdo_dbstmt_functions
0001:0034873d  _pdo_stmt_iter_get
0001:00349ad0  _pdo_row_functions
0001:00346c85  _pdo_stmt_setup_fetch_mode
0002:00001480  _pdo_row_object_handlers
Module: U:\dev\php-5.3.3\ext\pdo\pdo_sql_parser.o(pdo_sql_parser.o)
0001:0034a072  _pdo_parse_params
Module: U:\dev\php-5.3.3\ext\pdo\pdo_sqlstate.o(pdo_sqlstate.o)
0001:0034ac20  _pdo_sqlstate_state_to_description
0001:0034ac5a  _pdo_sqlstate_init_error_table
0001:0034acfb  _pdo_sqlstate_fini_error_table
Module: U:\dev\php-5.3.3\ext\phar\util.o(util.o)
0001:0034d665  _phar_compress_filter
0001:0034d6be  _phar_decompress_filter
0001:0034d704  _phar_free_alias
0001:0034d795  _phar_copy_on_write
0001:0034dcc1  _phar_add_virtual_dirs
0001:0034de24  _phar_create_writeable_entry
0001:0034df14  _phar_open_archive_fp
0001:0034e053  _phar_mount_entry
0001:0034e551  _phar_get_entry_info_dir
0001:0034eaf5  _phar_get_entry_info
0001:0034eb39  _phar_get_link_source
0001:0034ec6b  _phar_get_efp
0001:0034ee35  _phar_seek_efp
0001:0034f3af  _phar_create_signature
0001:0034f894  _phar_verify_signature
0001:0034ff9b  _phar_get_archive
0001:00350a8f  _phar_find_in_include_path
0001:0035106d  _phar_open_entry_fp
0001:003518a3  _phar_open_jit
0001:003519b7  _phar_separate_entry_fp
0001:00351b82  _phar_copy_entry_fp
0001:00351edd  _phar_get_entry_data
0001:00352586  _phar_get_or_create_entry_data
Module: U:\dev\php-5.3.3\ext\phar\tar.o(tar.o)
0001:003533dd  _phar_tar_setmetadata
0001:0035395b  _phar_tar_flush
0001:003552cf  _phar_parse_tarfile
0001:00356bca  _phar_open_or_create_tar
0001:00356ca2  _phar_is_tar
Module: U:\dev\php-5.3.3\ext\phar\zip.o(zip.o)
0001:003587c0  _phar_zip_flush
0001:00359bff  _phar_open_or_create_zip
0001:0035a6ab  _phar_parse_zipfile
Module: U:\dev\php-5.3.3\ext\phar\stream.o(stream.o)
0001:0035e6fa  _phar_dostat
0001:0035e9a0  _phar_parse_url
0002:00001510  _phar_ops
0002:00001540  _phar_stream_wops
0002:00001570  _php_stream_phar_wrapper
Module: U:\dev\php-5.3.3\ext\phar\func_interceptors.o(func_interceptors.o)
0001:00361120  _phar_intercept_functions
0001:00361159  _phar_release_functions
0001:00361174  _phar_save_orig_functions
0001:0036128f  _phar_restore_orig_functions
0001:00361478  _phar_intercept_functions_shutdown
0001:00361e5d  _phar_intercept_functions_init
0001:003657d4  _phar_is_dir
0001:003658ad  _phar_file_exists
0001:003662d9  _phar_fileperms
0001:00366200  _phar_fileinode
0001:00366127  _phar_filesize
0001:0036604e  _phar_fileowner
0001:00365f75  _phar_filegroup
0001:00365e9c  _phar_fileatime
0001:00365dc3  _phar_filemtime
0001:00365cea  _phar_filectime
0001:00365c11  _phar_filetype
0001:00365b38  _phar_is_writable
0001:00365a5f  _phar_is_readable
0001:00365986  _phar_is_executable
0001:003656fb  _phar_lstat
0001:00365622  _phar_stat
Module: U:\dev\php-5.3.3\ext\phar\dirstream.o(dirstream.o)
0001:003667b4  _phar_wrapper_rmdir
0001:00366fd9  _phar_wrapper_mkdir
0001:00367b19  _phar_wrapper_open_dir
0002:00001590  _phar_dir_ops
Module: U:\dev\php-5.3.3\ext\phar\phar.o(phar.o)
0002:00020020  _phar_globals_id
0002:00020030  _cached_phars
0002:00020060  _cached_alias
0002:00020090  _phar_orig_compile_file
0002:000200a0  _phar_save_resolve_path
0001:0036801f  _zm_globals_dtor_phar
0001:0036807e  _zm_deactivate_phar
0001:0036826a  _phar_request_initialize
0001:003686e5  _zm_info_phar
0001:003689b1  _zm_shutdown_phar
0001:00368b13  _phar_create_default_stub
0001:00368ce6  _zm_startup_phar
0001:00368f32  _zm_globals_ctor_phar
0001:00369fc5  _phar_flush
0001:0036c0ff  _phar_postprocess_file
0001:0036c635  _phar_fix_filepath
0001:0036cd1b  _phar_detect_phar_fname_ext
0001:0036d340  _phar_split_fname
0001:0036d489  _phar_parse_metadata
0001:0036d64e  _phar_open_parsed_phar
0001:0036d7b6  _destroy_phar_manifest_entry
0001:0036d905  _phar_destroy_phar_data
0001:00371405  _phar_open_executed_filename
0001:003716cb  _phar_open_from_filename
0001:00371d06  _phar_create_or_parse_filename
0001:00372401  _phar_open_or_create_filename
0001:003727ea  _phar_archive_delref
0001:0037292b  _phar_entry_delref
0001:003729d2  _phar_entry_remove
0001:00372ab0  _phar_ini_cache_list
0001:00372fe2  _phar_ini_modify_handler
0002:000015c0  _phar_module_entry
0002:00009700  _phar_functions
Module: U:\dev\php-5.3.3\ext\phar\phar_object.o(phar_object.o)
0001:00375190  _zim_Phar_canWrite
0001:003752d2  _phar_object_init
0001:003759b3  _zim_PharFileInfo_hasMetadata
0001:00375a16  _zim_PharFileInfo_getPharFlags
0001:00375a76  _zim_PharFileInfo_isCRCChecked
0001:00375b27  _zim_PharFileInfo_getCRC32
0001:00375ba2  _zim_PharFileInfo_getCompressedSize
0001:00375c33  _zim_Phar_hasMetadata
0001:00375c99  _zim_Phar_getModified
0001:00375cfd  _zim_Phar_isBuffering
0001:00375d62  _zim_Phar_startBuffering
0001:00375db2  _zim_Phar_isCompressed
0001:00375fd4  _zim_PharFileInfo_decompress
0001:00376268  _zim_PharFileInfo___destruct
0001:003762f5  _zim_Phar_stopBuffering
0001:003764b0  _zim_PharFileInfo_chmod
0001:0037677b  _zim_PharFileInfo_isCompressed
0001:0037688c  _zim_Phar_isFileFormat
0001:00376cb5  _zim_PharFileInfo_compress
0001:0037716b  _zim_PharFileInfo_getContent
0001:00377364  _zim_Phar_getPath
0001:003773cd  _zim_Phar_getAlias
0001:00377445  _zim_Phar_apiVersion
0001:00377519  _zim_PharFileInfo_delMetadata
0001:003776e9  _zim_Phar_delMetadata
0001:0037791f  _zim_PharFileInfo___construct
0001:00377c4e  _zim_Phar_isWritable
0001:00377d1a  _zim_Phar_count
0001:003788f5  _zim_Phar_extractTo
0001:00378ef3  _zim_Phar_getStub
0001:003795dd  _zim_Phar_addFromString
0001:0037973e  _zim_Phar_addEmptyDir
0001:00379a60  _zim_Phar_addFile
0001:00379c7b  _zim_Phar_offsetUnset
0001:00379e82  _zim_Phar_offsetExists
0001:00379fda  _zim_Phar_delete
0001:0037a2e3  _zim_Phar_offsetSet
0001:0037a566  _zim_Phar_setSignatureAlgorithm
0001:0037a81d  _zim_Phar_setStub
0001:0037abf1  _zim_Phar_offsetGet
0001:0037af1a  _zim_Phar_getVersion
0001:0037b140  _zim_Phar_copy
0001:0037b7ad  _zim_Phar_decompressFiles
0001:0037bb2f  _zim_Phar_compressFiles
0001:0037bd88  _zim_Phar_isValidPharFilename
0001:0037be56  _zim_Phar_getSignature
0001:0037c148  _zim_Phar_setDefaultStub
0001:0037c458  _zim_Phar_createDefaultStub
0001:0037c527  _zim_Phar___destruct
0001:0037c66f  _zim_Phar_setAlias
0001:0037cccc  _zim_Phar_buildFromIterator
0001:0037cfbc  _zim_Phar_buildFromDirectory
0001:0037e24b  _zim_Phar_running
0001:0037e501  _zim_Phar_unlinkArchive
0001:0037e7f7  _zim_Phar_canCompress
0001:0037e8c7  _zim_Phar_loadPhar
0001:0037e9ac  _zim_Phar_getSupportedCompression
0001:0037ea52  _zim_Phar_getSupportedSignatures
0001:0037ec02  _zim_Phar___construct
0001:0037f10c  _zim_Phar_mapPhar
0001:0037f1c9  _zim_Phar_interceptFileFuncs
0001:0037f3f0  _zim_Phar_mungServer
0001:003808fe  _zim_Phar_webPhar
0001:00381a4b  _zim_Phar_mount
0001:0038329d  _zim_Phar_setMetadata
0001:003834e9  _zim_PharFileInfo_getMetadata
0001:00383605  _zim_Phar_getMetadata
0001:0038378e  _zim_PharFileInfo_setMetadata
0001:00383a70  _zim_Phar_decompress
0001:00383d2f  _zim_Phar_compress
0001:0038409f  _zim_Phar_convertToExecutable
0001:00384401  _zim_Phar_convertToData
0002:00001620  _php_archive_methods
0002:00001aa0  _php_entry_methods
0002:00009720  _phar_exception_methods
Module: U:\dev\php-5.3.3\ext\phar\phar_path_check.o(phar_path_check.o)
0001:00385445  _phar_path_check
Module: U:\dev\php-5.3.3\ext\posix\posix.o(posix.o)
0002:000200b0  _posix_globals_id
0001:0038589f  _zif_posix_get_last_error
0001:003858e7  _zif_posix_initgroups
0001:00385964  _zif_posix_strerror
0001:003859f9  _zif_posix_getrlimit
0001:00385c38  _php_posix_passwd_to_array
0001:00385d9b  _zif_posix_getpwuid
0001:00385ec2  _zif_posix_getpwnam
0001:00385ff8  _zif_posix_access
0001:00386161  _php_posix_group_to_array
0001:003862ce  _zif_posix_getgrgid
0001:0038641b  _zif_posix_getgrnam
0001:003865e6  _zif_posix_mknod
0001:00386760  _zif_posix_mkfifo
0001:0038683a  _zif_posix_getcwd
0001:00386a9f  _zif_posix_isatty
0001:00386bbc  _zif_posix_ttyname
0001:00386d2f  _zif_posix_times
0001:00386e74  _zif_posix_uname
0001:00386fb5  _zif_posix_getsid
0001:0038702b  _zif_posix_getpgid
0001:003870a4  _zif_posix_setpgid
0001:00387129  _zif_posix_setsid
0001:00387163  _zif_posix_getpgrp
0001:0038719d  _zif_posix_getlogin
0001:00387221  _zif_posix_getgroups
0001:003872d2  _zif_posix_setegid
0001:00387349  _zif_posix_seteuid
0001:003873c0  _zif_posix_setgid
0001:00387437  _zif_posix_setuid
0001:003874ae  _zif_posix_getegid
0001:003874e8  _zif_posix_geteuid
0001:00387522  _zif_posix_getgid
0001:0038755c  _zif_posix_getuid
0001:00387596  _zif_posix_getppid
0001:003875d0  _zif_posix_getpid
0001:0038760a  _zif_posix_kill
0001:00387880  _posix_functions
0002:00001c50  _limits
0002:00001bf0  _posix_module_entry
Module: U:\dev\php-5.3.3\ext\reflection\php_reflection.o(php_reflection.o)
0002:000200c0  _reflection_exception_ptr
0002:000200d0  _reflection_ptr
0002:000200e0  _reflector_ptr
0002:000200f0  _reflection_function_abstract_ptr
0002:00020100  _reflection_function_ptr
0002:00020110  _reflection_parameter_ptr
0002:00020120  _reflection_method_ptr
0002:00020130  _reflection_class_ptr
0002:00020140  _reflection_object_ptr
0002:00020150  _reflection_property_ptr
0002:00020160  _reflection_extension_ptr
0001:003882a5  _zm_info_reflection
0001:0038846f  _zm_startup_reflection
0001:003896a7  _zim_reflection_property_setAccessible
0001:00389700  _zim_reflection_method_setAccessible
0001:00389795  _zim_reflection_property_getModifiers
0001:003898ec  _zim_reflection_property_isDefault
0001:0038992a  _zim_reflection_property_isStatic
0001:00389968  _zim_reflection_property_isProtected
0001:003899a6  _zim_reflection_property_isPrivate
0001:003899e4  _zim_reflection_property_isPublic
0001:00389a22  _zim_reflection_class_getModifiers
0001:00389b79  _zim_reflection_class_isAbstract
0001:00389bb7  _zim_reflection_class_isFinal
0001:00389bf5  _zim_reflection_class_isInterface
0001:00389c33  _zim_reflection_class_isInstantiable
0001:00389d1c  _zim_reflection_class_getEndLine
0001:00389de2  _zim_reflection_class_getStartLine
0001:00389ea8  _zim_reflection_class_isUserDefined
0001:00389f55  _zim_reflection_class_isInternal
0001:0038a002  _zim_reflection_method_getModifiers
0001:0038a0a9  _zim_reflection_method_isDestructor
0001:0038a156  _zim_reflection_method_isConstructor
0001:0038a2dc  _zim_reflection_function_isDeprecated
0001:0038a31a  _zim_reflection_method_isStatic
0001:0038a358  _zim_reflection_method_isProtected
0001:0038a396  _zim_reflection_method_isPrivate
0001:0038a3d4  _zim_reflection_method_isPublic
0001:0038a412  _zim_reflection_method_isAbstract
0001:0038a450  _zim_reflection_method_isFinal
0001:0038a48e  _zim_reflection_parameter_isDefaultValueAvailable
0001:0038a5a6  _zim_reflection_parameter_isOptional
0001:0038a655  _zim_reflection_parameter_getPosition
0001:0038a6fb  _zim_reflection_parameter_isPassedByReference
0001:0038a7ac  _zim_reflection_parameter_allowsNull
0001:0038a85d  _zim_reflection_parameter_isArray
0001:0038a90e  _zim_reflection_function_getEndLine
0001:0038a9d1  _zim_reflection_function_getStartLine
0001:0038aa94  _zim_reflection_function_isUserDefined
0001:0038ab41  _zim_reflection_function_isInternal
0001:0038abee  _zim_reflection_function_isClosure
0001:0038ac9b  _zim_reflection_extension_info
0001:0038ad58  _zim_reflection_extension_getDependencies
0001:0038aeec  _zim_reflection_extension_getClassNames
0001:0038afe1  _zim_reflection_extension_getClasses
0001:0038b0d6  _zim_reflection_extension_getINIEntries
0001:0038b1c8  _zim_reflection_extension_getConstants
0001:0038b2e9  _zim_reflection_class_getInterfaceNames
0001:0038b411  _zim_reflection_getModifierNames
0001:0038b66d  _zim_reflection_class_inNamespace
0001:0038b71e  _zim_reflection_function_inNamespace
0001:0038b7ce  _zim_reflection_extension_getVersion
0001:0038b8af  _zim_reflection_property_getDocComment
0001:0038b989  _zim_reflection_class_getNamespaceName
0001:0038ba76  _zim_reflection_class_getDocComment
0001:0038bb5c  _zim_reflection_class_getFileName
0001:0038bc39  _zim_reflection_function_getNamespaceName
0001:0038bd26  _zim_reflection_function_getDocComment
0001:0038be03  _zim_reflection_function_getFileName
0001:0038c07f  _zim_reflection_extension_getFunctions
0001:0038c3ca  _zim_reflection_class_getConstructor
0001:0038c4a3  _zend_reflection_class_factory
0001:0038c637  _zim_reflection_class_getParentClass
0001:0038c702  _zim_reflection_class_getInterfaces
0001:0038c845  _zim_reflection_parameter_getDeclaringClass
0001:0038ca13  _zim_reflection_parameter_getDefaultValue
0001:0038ce68  _zim_reflection_class_getConstants
0001:0038cf66  _zim_reflection_function_getStaticVariables
0001:0038d234  _zim_reflection_property___toString
0001:0038d31b  _zim_reflection_property_getDeclaringClass
0001:0038d6fb  _zim_reflection_extension___construct
0001:0038da94  _zim_reflection___clone
0001:0038de70  _zim_reflection_extension_export
0001:0038deb7  _zim_reflection_property_export
0001:0038defe  _zim_reflection_object_export
0001:0038df45  _zim_reflection_class_export
0001:0038df8c  _zim_reflection_method_export
0001:0038dfd3  _zim_reflection_parameter_export
0001:0038e01a  _zim_reflection_function_export
0001:0038e085  _zim_reflection_class_getExtensionName
0001:0038e1ad  _zim_reflection_class_getExtension
0001:0038e2b0  _zim_reflection_class_isIterateable
0001:0038e453  _zim_reflection_class_newInstance
0001:0038e72e  _zim_reflection_class_isInstance
0001:0038e875  _zim_reflection_class_hasConstant
0001:0038e9c7  _zim_reflection_class_getProperties
0001:0038eb94  _zim_reflection_class_hasProperty
0001:0038eda7  _zim_reflection_class_getMethod
0001:0038f0e3  _zim_reflection_class_hasMethod
0001:0038f2bc  _zim_reflection_method_getPrototype
0001:0038f3fa  _zim_reflection_method_getDeclaringClass
0001:0038f5e5  _zim_reflection_method_invoke
0001:0038f994  _zim_reflection_function_getExtensionName
0001:0038fab8  _zim_reflection_function_getExtension
0001:0038fbc7  _zim_reflection_function_getNumberOfRequiredParameters
0001:0038fcb1  _zim_reflection_function_getNumberOfParameters
0001:0038fd9b  _zim_reflection_function_returnsReference
0001:0038feaf  _zim_reflection_function_invoke
0001:00390126  _zim_reflection_function_isDisabled
0001:003902a4  _zim_reflection_property___construct
0001:0039085e  _zim_reflection_class_implementsInterface
0001:00390aa3  _zim_reflection_class_isSubclassOf
0001:00390cde  _zim_reflection_class_newInstanceArgs
0001:00391036  _zim_reflection_method_invokeArgs
0001:00391431  _zim_reflection_function_invokeArgs
0001:003918f1  _zim_reflection_class_getMethods
0001:00391b98  _zim_reflection_class_getProperty
0001:00391f47  _zim_reflection_method___construct
0001:003924a0  _zim_reflection_parameter_getClass
0001:003926d1  _zim_reflection_parameter_getDeclaringFunction
0001:003927e0  _zim_reflection_function_getParameters
0001:00392b9b  _zim_reflection_parameter___construct
0001:00393353  _zim_reflection_function___construct
0001:00393661  _zim_reflection_class_getDefaultProperties
0001:003938dd  _zim_reflection_class_getStaticProperties
0001:00393bbf  _zim_reflection_class_setStaticPropertyValue
0001:00393d38  _zim_reflection_class_getShortName
0001:00393e46  _zim_reflection_function_getShortName
0001:0039403e  _zim_reflection_property_setValue
0001:0039442d  _zim_reflection_function_getName
0001:00394478  _zim_reflection_parameter_getName
0001:003944c3  _zim_reflection_class_getName
0001:0039450e  _zim_reflection_property_getName
0001:00394559  _zim_reflection_extension_getName
0001:0039460b  _zim_reflection_export
0001:00394889  _zim_reflection_property_getValue
0001:00394bf0  _zim_reflection_class_getStaticPropertyValue
0001:00394d73  _zim_reflection_class_getConstant
0001:00395a27  _zim_reflection_method___toString
0001:00395b10  _zim_reflection_function___toString
0001:003969be  _zim_reflection_class___toString
0001:00396b9e  _zim_reflection_extension___toString
0001:00397172  _zim_reflection_parameter___toString
0001:0039755e  _zim_reflection_object___construct
0001:0039759c  _zim_reflection_class___construct
0001:003975e0  _reflection_ext_functions
0002:00001cb0  _reflection_module_entry
Module: U:\dev\php-5.3.3\ext\session\session.o(session.o)
0002:00020170  _ps_globals_id
0001:003990b0  _php_session_register_serializer
0001:0039910a  _php_session_register_module
0001:0039929f  _php_get_session_var
0001:0039b84a  _session_adapt_url
0001:0039b89f  __php_find_ps_serializer
0001:0039b9d0  __php_find_ps_module
0001:0039bb09  _ps_srlzr_encode_php
0001:0039c028  _ps_srlzr_encode_php_binary
0001:0039c535  _php_session_create_id
0001:0039cec5  _php_session_start
0001:0039e689  _php_set_session_var
0001:0039f74d  _php_add_session_var
0001:0039fe64  _ps_srlzr_decode_php
0001:003a0033  _ps_srlzr_decode_php_binary
0002:00001d10  _session_module_entry
Module: U:\dev\php-5.3.3\ext\session\mod_files.o(mod_files.o)
0001:003a146c  _ps_gc_files
0001:003a14a0  _ps_close_files
0001:003a155d  _ps_open_files
0001:003a1c32  _ps_write_files
0001:003a1d6c  _ps_read_files
0001:003a1eca  _ps_delete_files
0002:00001e60  _ps_mod_files
Module: U:\dev\php-5.3.3\ext\session\mod_user.o(mod_user.o)
0001:003a200f  _ps_gc_user
0001:003a20aa  _ps_close_user
0001:003a2114  _ps_delete_user
0001:003a21e0  _ps_write_user
0001:003a22ea  _ps_read_user
0001:003a23d9  _ps_open_user
0002:00001e80  _ps_mod_user
Module: U:\dev\php-5.3.3\ext\simplexml\simplexml.o(simplexml.o)
0001:003a24f0  _sxe_get_element_class_entry
0001:003a251e  _zm_shutdown_simplexml
0001:003a272b  _sxe_object_new
0001:003a2a1d  _php_sxe_get_iterator
0001:003a2bcc  _zm_info_simplexml
0001:003a2c42  _zm_startup_simplexml
0001:003a380b  _simplexml_export_node
0001:003a2e3f  _zif_simplexml_import_dom
0001:003a2f92  _zif_simplexml_load_file
0001:003a30e5  _zif_simplexml_load_string
0001:003a3272  _zim_simplexml_element___construct
0001:003a341b  _zim_simplexml_element_registerXPathNamespace
0001:003a3871  _zim_simplexml_element_getName
0001:003a3935  _zim_simplexml_element_attributes
0001:003a3a1e  _zim_simplexml_element_children
0001:003a3b8b  _zim_simplexml_element_addChild
0001:003a3e99  _zim_simplexml_element_addAttribute
0001:003a412e  _zim_simplexml_element_asXML
0001:003a43c9  _zim_simplexml_element_xpath
0001:003a48d0  _zim_simplexml_element_count
0001:003a4937  _php_sxe_move_forward_iterator
0001:003a5d65  _zim_simplexml_element_getDocNamespaces
0001:003a6802  _zim_simplexml_element___toString
0001:003a6aef  _zim_simplexml_element_getNamespaces
0001:003a7c50  _simplexml_functions
0002:00001ea0  _php_sxe_iterator_funcs
0002:00001ec0  _simplexml_module_entry
0002:00009810  _sxe_class_entry
Module: U:\dev\php-5.3.3\ext\simplexml\sxe.o(sxe.o)
0002:00020180  _ce_SimpleXMLElement
0001:003a80a3  _zm_startup_sxe
0001:003a8276  _zim_ce_SimpleXMLIterator_next
0001:003a82b0  _zim_ce_SimpleXMLIterator_valid
0001:003a82e3  _zim_ce_SimpleXMLIterator_rewind
0001:003a831d  _zim_ce_SimpleXMLIterator_getChildren
0001:003a8386  _zim_ce_SimpleXMLIterator_current
0001:003a83ff  _zim_ce_SimpleXMLIterator_hasChildren
0001:003a84a3  _zim_ce_SimpleXMLIterator_key
0002:00009820  _ce_SimpleXMLIterator
Module: U:\dev\php-5.3.3\ext\soap\soap.o(soap.o)
0002:00020190  _soap_globals_id
0002:000201a0  _soap_var_class_entry
0001:003a866c  _zm_activate_soap
0001:003a8bd2  _add_soap_fault
0001:003a8c7c  _zif_use_soap_error_handler
0001:003a8d02  _zim_SoapClient___getLastResponseHeaders
0001:003a8daa  _zim_SoapClient___getLastRequestHeaders
0001:003a8e4b  _zim_SoapClient___getLastResponse
0001:003a8eeb  _zim_SoapClient___getLastRequest
0001:003a8f88  _zim_SoapClient___setLocation
0001:003a90ae  _zif_is_soap_fault
0001:003a915c  _zim_SoapParam_SoapParam
0001:003a92fb  _zim_SoapClient___setSoapHeaders
0001:003a94fe  _zim_SoapClient___setCookie
0001:003a970a  _zim_SoapClient___doRequest
0001:003a98f4  _zim_SoapServer_setPersistence
0001:003ac1e9  _zim_SoapClient___getTypes
0001:003ac60b  _zim_SoapClient___getFunctions
0001:003ad5e0  _zim_SoapFault_SoapFault
0001:003af080  _zim_SoapHeader_SoapHeader
0001:003af9fe  _zim_SoapServer_SoapServer
0001:003b201c  _zim_SoapServer_fault
0001:003b262f  _zim_SoapServer_addFunction
0001:003b2b70  _zim_SoapServer_getFunctions
0001:003b2e17  _zim_SoapServer_setClass
0001:003b3096  _zim_SoapVar_SoapVar
0001:003b335f  _zim_SoapFault___toString
0001:003b3550  _zm_info_soap
0001:003b3bda  _zm_startup_soap
0001:003b5d88  _zm_shutdown_soap
0001:003b5e2d  _OnUpdateCacheMode
0001:003b5e98  _OnUpdateCacheEnabled
0001:003b5f7b  _zim_SoapServer_addSoapHeader
0001:003b615e  _zim_SoapServer_setObject
0001:003b67d1  _zim_SoapServer_handle
0001:003baa19  _zim_SoapClient___call
0001:003bb0de  _zim_SoapClient_SoapClient
0002:00001f90  _soap_module_entry
0002:00009830  _le_url
Module: U:\dev\php-5.3.3\ext\soap\php_encoding.o(php_encoding.o)
0001:003bd100  _whiteSpace_replace
0001:003bd128  _whiteSpace_collapse
0001:003bdefa  _delete_encoder
0001:003be8eb  _get_conversion
0001:003bef5d  _master_to_zval
0001:003c0bac  _delete_encoder_persistent
0001:003c0be3  _encode_finish
0001:003c0c65  _encode_reset_ns
0001:003c0d07  _encode_add_ns
0001:003c3ef8  _master_to_xml
0001:003c7abd  _sdl_guess_convert_xml
0001:003c7c2e  _to_zval_user
0001:003c7e48  _to_xml_user
0001:003c895d  _sdl_guess_convert_zval
0002:00001ff0  _defaultEncoding
0002:00002840  _numDefaultEncodings
Module: U:\dev\php-5.3.3\ext\soap\php_http.o(php_http.o)
0001:003c9289  _proxy_authentication
0001:003c9727  _basic_authentication
0001:003ca8fb  _make_http_soap_request
Module: U:\dev\php-5.3.3\ext\soap\php_packet_soap.o(php_packet_soap.o)
0001:003d2433  _parse_packet_soap
Module: U:\dev\php-5.3.3\ext\soap\php_schema.o(php_schema.o)
0001:003d3510  _delete_restriction_var_char_persistent
0001:003d3541  _delete_restriction_var_int_persistent
0001:003d355b  _delete_extra_attribute_persistent
0001:003d3591  _delete_restriction_var_char
0001:003d35c2  _delete_restriction_var_int
0001:003d35dc  _delete_extra_attribute
0001:003d3612  _delete_attribute_persistent
0001:003d368f  _delete_attribute
0001:003d370c  _delete_model_persistent
0001:003d3764  _delete_type_persistent
0001:003d38ca  _delete_model
0001:003d3922  _delete_type
0001:003d42c7  _schema_pass2
0001:003d46d7  _schema_min_max
0001:003db44e  _load_schema
Module: U:\dev\php-5.3.3\ext\soap\php_sdl.o(php_sdl.o)
0001:003dbef0  _delete_sdl_impl
0001:003dbfc9  _delete_sdl
0001:003dd82e  _get_binding_from_name
0001:003dda72  _sdl_restore_uri_credentials
0001:003df999  _get_binding_from_type
0001:003e42cd  _sdl_set_uri_credentials
0001:003e5030  _get_encoder_ex
0001:003e605b  _get_encoder
0001:003e636a  _get_encoder_from_prefix
0001:003e93b8  _get_sdl
Module: U:\dev\php-5.3.3\ext\soap\php_xml.o(php_xml.o)
0001:003eda7a  _parse_namespace
0001:003edaea  _node_find_ns
0001:003edb15  _node_is_equal_ex
0001:003edb79  _get_node_recurisve_ex
0001:003edbdd  _get_node_ex
0001:003edc1a  _attr_find_ns
0001:003edc4f  _attr_is_equal_ex
0001:003edcb3  _get_attribute_ex
0001:003edcf0  _get_node_with_attribute_recursive_ex
0001:003edda6  _get_node_with_attribute_ex
0001:003ede27  _soap_xmlParseMemory
0001:003edf6e  _soap_xmlParseFile
Module: U:\dev\php-5.3.3\ext\sockets\sockets.o(sockets.o)
0002:000201b0  _sockets_globals_id
0001:003ee060  _php_sockets_le_socket
0001:003ee089  _zif_socket_clear_error
0001:003ee137  _zif_socket_last_error
0001:003ee24c  _zif_socket_shutdown
0001:003ee36f  _zm_deactivate_sockets
0001:003ee3ef  _zif_socket_get_option
0001:003ee886  _zif_socket_sendto
0001:003eeb41  _zif_socket_strerror
0001:003eebb6  _zif_socket_send
0001:003eed5b  _zif_socket_bind
0001:003eeffe  _zif_socket_connect
0001:003ef359  _zif_socket_create
0001:003ef4f2  _zif_socket_write
0001:003ef64b  _zif_socket_close
0001:003ef6fc  _zif_socket_listen
0001:003ef81f  _zif_socket_set_block
0001:003ef8d1  _zif_socket_set_nonblock
0001:003ef9a9  _zif_socket_accept
0001:003efb68  _zif_socket_create_listen
0001:003f014c  _zm_info_sockets
0001:003f071c  _zm_startup_sockets
0001:003f18f2  _zif_socket_read
0001:003f1ca3  _zif_socket_select
0001:003f2002  _zif_socket_create_pair
0001:003f22d1  _zif_socket_getpeername
0001:003f258f  _zif_socket_getsockname
0001:003f2831  _zif_socket_recv
0001:003f2a23  _zif_socket_recvfrom
0001:003f2f08  _zif_socket_set_option
0001:003f3800  _sockets_functions
0002:00002850  _sockets_module_entry
0002:00009960  _inet_ntoa_lock
Module: U:\dev\php-5.3.3\ext\spl\php_spl.o(php_spl.o)
0002:000201c0  _spl_globals_id
0001:003f4463  _zm_activate_spl
0001:003f4494  _zm_deactivate_spl
0001:003f4520  _zm_startup_spl
0001:003f45bc  _zif_spl_classes
0001:003f4f81  _zm_info_spl
0001:003f63c5  _spl_build_class_list_string
0001:003f641d  _php_spl_object_hash
0001:003f654e  _zif_spl_object_hash
0001:003f65df  _zif_spl_autoload_functions
0001:003f68a8  _zif_spl_autoload_unregister
0001:003f6d0e  _zif_spl_autoload_register
0001:003f740c  _zif_spl_autoload_call
0001:003f767d  _zif_spl_autoload_extensions
0001:003f7793  _zif_spl_autoload
0001:003f7d77  _zif_class_implements
0001:003f7e69  _zif_class_parents
0001:003f8040  _spl_functions
0002:000028b0  _spl_module_entry
Module: U:\dev\php-5.3.3\ext\spl\spl_functions.o(spl_functions.o)
0001:003f8510  _spl_gen_private_prop_name
0001:003f8554  _spl_add_class_name
0001:003f8637  _spl_add_interfaces
0001:003f8694  _spl_add_classes
0001:003f8734  _spl_register_property
0001:003f8740  _spl_register_sub_class
0001:003f8891  _spl_register_std_class
0001:003f89bc  _spl_register_interface
Module: U:\dev\php-5.3.3\ext\spl\spl_engine.o(spl_engine.o)
0001:003f8ad0  _spl_offset_convert_to_long
0001:003f8bf5  _spl_instantiate
Module: U:\dev\php-5.3.3\ext\spl\spl_iterators.o(spl_iterators.o)
0002:000201d0  _spl_ce_RecursiveIterator
0002:000201e0  _spl_ce_RecursiveIteratorIterator
0002:000201f0  _spl_ce_OuterIterator
0002:00020200  _spl_ce_IteratorIterator
0002:00020210  _spl_ce_FilterIterator
0002:00020220  _spl_ce_RecursiveFilterIterator
0002:00020230  _spl_ce_ParentIterator
0002:00020240  _spl_ce_Countable
0002:00020250  _spl_ce_SeekableIterator
0002:00020260  _spl_ce_LimitIterator
0002:00020270  _spl_ce_CachingIterator
0002:00020280  _spl_ce_RecursiveCachingIterator
0002:00020290  _spl_ce_NoRewindIterator
0002:000202a0  _spl_ce_AppendIterator
0002:000202b0  _spl_ce_InfiniteIterator
0002:000202c0  _spl_ce_RegexIterator
0002:000202d0  _spl_ce_RecursiveRegexIterator
0002:000202e0  _spl_ce_EmptyIterator
0002:000202f0  _spl_ce_RecursiveTreeIterator
0001:003f8cbe  _zim_spl_RecursiveIteratorIterator_beginIteration
0001:003f8cc3  _zim_spl_RecursiveIteratorIterator_endIteration
0001:003f8cc8  _zim_spl_RecursiveIteratorIterator_beginChildren
0001:003f8ccd  _zim_spl_RecursiveIteratorIterator_endChildren
0001:003f8cd2  _zim_spl_RecursiveIteratorIterator_nextElement
0001:003f8cd7  _zim_spl_NoRewindIterator_rewind
0001:003f8cdc  _zim_spl_EmptyIterator_rewind
0001:003f8ce1  _zim_spl_EmptyIterator_valid
0001:003f8cf3  _zim_spl_EmptyIterator_next
0001:003f8df2  _spl_iterator_apply
0001:003f990c  _zim_spl_EmptyIterator_current
0001:003f995a  _zim_spl_EmptyIterator_key
0001:003f9d3b  _zm_startup_spl_iterators
0001:00401e50  _spl_funcs_RecursiveIterator
0001:003fb396  _zim_spl_AppendIterator_valid
0001:003fb3c9  _zim_spl_NoRewindIterator_next
0001:003fb3f8  _zim_spl_NoRewindIterator_key
0001:003fb47e  _zim_spl_NoRewindIterator_valid
0001:003fb4c0  _zim_spl_RecursiveCachingIterator_hasChildren
0001:003fb4f3  _zim_spl_CachingIterator_getFlags
0001:003fb51e  _zim_spl_CachingIterator_valid
0001:003fb54d  _zim_spl_LimitIterator_getPosition
0001:003fb578  _zim_spl_LimitIterator_valid
0001:003fb5c3  _zim_spl_RegexIterator_getPregFlags
0001:003fb5f5  _zim_spl_RegexIterator_getFlags
0001:003fb620  _zim_spl_RegexIterator_getMode
0001:003fb64b  _zim_spl_RecursiveFilterIterator_hasChildren
0001:003fb70d  _zim_spl_dual_it_valid
0001:003fb740  _zim_spl_RecursiveTreeIterator_getPrefix
0001:003fb771  _zim_spl_RecursiveIteratorIterator_getMaxDepth
0001:003fb7b1  _zim_spl_RecursiveIteratorIterator_callGetChildren
0001:003fb878  _zim_spl_RecursiveIteratorIterator_callHasChildren
0001:003fb951  _zim_spl_RecursiveIteratorIterator_getDepth
0001:003fb97c  _zim_spl_RecursiveIteratorIterator_next
0001:003fb9aa  _zim_spl_RecursiveIteratorIterator_key
0001:003fba39  _zim_spl_RecursiveIteratorIterator_valid
0001:003fba7d  _zim_spl_RecursiveIteratorIterator_rewind
0001:003fbc8c  _zif_iterator_count
0001:003fbd12  _zim_spl_RegexIterator_setPregFlags
0001:003fbd65  _zim_spl_RegexIterator_setFlags
0001:003fbdd6  _zim_spl_RecursiveIteratorIterator_setMaxDepth
0001:003fbe57  _zif_iterator_apply
0001:003fc101  _zim_spl_RegexIterator_setMode
0001:003fc1b1  _zim_spl_RecursiveTreeIterator_setPrefixPart
0001:003fc37c  _zim_spl_AppendIterator_getIteratorIndex
0001:003fc3e8  _zim_spl_dual_it_key
0001:003fc44f  _zim_spl_RecursiveTreeIterator_getPostfix
0001:003fcd6f  _zim_spl_AppendIterator___construct
0001:003fcdbf  _zim_spl_InfiniteIterator___construct
0001:003fce0f  _zim_spl_NoRewindIterator___construct
0001:003fce5f  _zim_spl_IteratorIterator___construct
0001:003fceaf  _zim_spl_RecursiveCachingIterator___construct
0001:003fceff  _zim_spl_CachingIterator___construct
0001:003fcf4f  _zim_spl_LimitIterator___construct
0001:003fcf9f  _zim_spl_RecursiveRegexIterator___construct
0001:003fcfef  _zim_spl_RegexIterator___construct
0001:003fd03f  _zim_spl_ParentIterator___construct
0001:003fd08f  _zim_spl_RecursiveFilterIterator___construct
0001:003fd0df  _zim_spl_FilterIterator___construct
0001:003fd170  _zim_spl_CachingIterator_count
0001:003fd2d5  _zim_spl_CachingIterator_setFlags
0001:003fd48a  _zim_spl_CachingIterator_offsetExists
0001:003fd662  _zim_spl_CachingIterator_offsetUnset
0001:003fd8e1  _zim_spl_RecursiveRegexIterator_getChildren
0001:003fda1b  _zim_spl_RecursiveFilterIterator_getChildren
0001:003fdb56  _zim_spl_RegexIterator_accept
0001:003fdf82  _zim_spl_CachingIterator_hasNext
0001:003fdfc9  _zim_spl_RecursiveIteratorIterator_getInnerIterator
0001:003fe034  _zif_iterator_to_array
0001:003fe0e9  _zim_spl_AppendIterator_getArrayIterator
0001:003fe18b  _zim_spl_NoRewindIterator_current
0001:003fe20b  _zim_spl_RecursiveIteratorIterator_current
0001:003fe294  _zim_spl_CachingIterator_getCache
0001:003fe33e  _zim_spl_dual_it_current
0001:003fe3ac  _zim_spl_RecursiveCachingIterator_getChildren
0001:003fe41a  _zim_spl_dual_it_getInnerIterator
0001:003fe49d  _zim_spl_CachingIterator_offsetGet
0001:003fe715  _zim_spl_RecursiveIteratorIterator_getSubIterator
0001:003fe7c0  _zim_spl_RecursiveTreeIterator_key
0001:003feaf2  _zim_spl_RecursiveTreeIterator_current
0001:003fecc3  _zim_spl_RecursiveTreeIterator_getEntry
0001:003fed36  _zim_spl_CachingIterator___toString
0001:003fee44  _zim_spl_CachingIterator_offsetSet
0001:003ff815  _zim_spl_RecursiveTreeIterator___construct
0001:003ff865  _zim_spl_RecursiveIteratorIterator___construct
0001:00400048  _zim_spl_CachingIterator_next
0001:00400071  _zim_spl_CachingIterator_rewind
0001:00400172  _zim_spl_dual_it_rewind
0001:004009a8  _zim_spl_LimitIterator_seek
0001:00400a0f  _zim_spl_LimitIterator_rewind
0001:00400ae7  _spl_append_it_next_iterator
0001:00400d0f  _spl_append_it_fetch
0001:00400e59  _zim_spl_AppendIterator_rewind
0001:00400ead  _zim_spl_AppendIterator_append
0001:00400fba  _spl_append_it_next
0001:0040108f  _zim_spl_AppendIterator_next
0001:004010bf  _zim_spl_FilterIterator_rewind
0001:00401435  _zim_spl_InfiniteIterator_next
0001:004016ea  _zim_spl_LimitIterator_next
0001:004018e4  _zim_spl_dual_it_next
0001:00401ac6  _zim_spl_FilterIterator_next
0002:00002910  _spl_recursive_it_iterator_funcs
Module: U:\dev\php-5.3.3\ext\spl\spl_array.o(spl_array.o)
0002:00020300  _spl_ce_ArrayObject
0002:00020310  _spl_handler_ArrayObject
0002:00020380  _spl_ce_ArrayIterator
0002:00020390  _spl_handler_ArrayIterator
0002:00020400  _spl_ce_RecursiveArrayIterator
0001:00403363  _zim_spl_Array_getFlags
0001:00403528  _zm_startup_spl_array
0001:00407d15  _spl_array_serialize
0001:00403e3e  _spl_array_unserialize
0001:004063fb  _spl_array_object_count_elements
0001:00403901  _spl_array_get_iterator
0001:00403ae2  _zim_spl_Array_setFlags
0001:00403b40  _zim_spl_Array_setIteratorClass
0001:00403bb4  _spl_array_unserialize_helper
0001:00403f98  _zim_spl_Array_unserialize
0001:004040a3  _zim_spl_Array_getIteratorClass
0001:00404e0e  _zim_spl_Array_offsetGet
0001:0040510a  _zim_spl_Array_natcasesort
0001:00405160  _zim_spl_Array_natsort
0001:004051b5  _zim_spl_Array_uksort
0001:0040520a  _zim_spl_Array_uasort
0001:0040525e  _zim_spl_Array_ksort
0001:004052b2  _zim_spl_Array_asort
0001:00405529  _zim_spl_Array_rewind
0001:00405552  _spl_hash_verify_pos_ex
0001:00405623  _spl_array_iterator_key
0001:004057b5  _zim_spl_Array_key
0001:004057cd  _spl_hash_verify_pos
0001:004058ea  _zim_spl_Array_next
0001:00405ec3  _zim_spl_Array_hasChildren
0001:004063b5  _zim_spl_Array_count
0001:00407005  _zim_spl_Array_exchangeArray
0001:00407192  _zim_spl_Array___construct
0001:00407273  _zim_spl_Array_valid
0001:004073d3  _zim_spl_Array_current
0001:00407566  _zim_spl_Array_getArrayCopy
0001:00407681  _zim_spl_Array_getIterator
0001:004077ca  _zim_spl_Array_seek
0001:0040796a  _spl_array_serialize_helper
0001:00407dbf  _zim_spl_Array_serialize
0001:00407ea7  _zim_spl_Array_getChildren
0001:0040871f  _zim_spl_Array_offsetUnset
0001:00408d0d  _spl_array_iterator_append
0001:00408e80  _zim_spl_Array_append
0001:00408ecc  _zim_spl_Array_offsetSet
0001:0040941b  _zim_spl_Array_offsetExists
0002:00002930  _spl_array_it_funcs
Module: U:\dev\php-5.3.3\ext\spl\spl_directory.o(spl_directory.o)
0002:00020410  _spl_ce_SplFileObject
0002:00020420  _spl_ce_SplFileInfo
0002:00020430  _spl_ce_DirectoryIterator
0002:00020440  _spl_ce_FilesystemIterator
0002:00020450  _spl_ce_RecursiveDirectoryIterator
0002:00020460  _spl_ce_GlobIterator
0002:00020470  _spl_ce_SplTempFileObject
0001:00409bf6  _zim_spl_SplFileObject_hasChildren
0001:00409c08  _zim_spl_SplFileObject_getChildren
0001:0040a314  _zm_startup_spl_directory
0001:0040c496  _spl_filesystem_dir_get_iterator
0001:0040c439  _spl_filesystem_tree_get_iterator
0001:0040a971  _zim_spl_SplFileObject_fseek
0001:0040aa5a  _zim_spl_SplFileObject_setCsvControl
0001:0040abaa  _zim_spl_SplFileObject_getMaxLineLen
0001:0040ac0f  _zim_spl_SplFileObject_setMaxLineLen
0001:0040ac82  _zim_spl_SplFileObject_getFlags
0001:0040acb0  _zim_spl_SplFileObject_setFlags
0001:0040aceb  _zim_spl_SplFileObject_key
0001:0040ad1d  _zim_spl_RecursiveDirectoryIterator_getSubPathname
0001:0040adc7  _zim_spl_RecursiveDirectoryIterator_getSubPath
0001:0040ae35  _zim_spl_FilesystemIterator_setFlags
0001:0040ae8c  _zim_spl_FilesystemIterator_getFlags
0001:0040aebf  _zim_spl_SplFileInfo_setInfoClass
0001:0040af40  _zim_spl_SplFileInfo_setFileClass
0001:0040afc1  _zim_spl_DirectoryIterator_getFilename
0001:0040b00d  _zim_spl_DirectoryIterator_valid
0001:0040b03f  _zim_spl_DirectoryIterator_key
0001:0040b084  _zim_spl_DirectoryIterator_rewind
0001:0040b0e6  _zim_spl_SplFileObject_valid
0001:0040b151  _zim_spl_SplFileObject_eof
0001:0040b192  _zim_spl_DirectoryIterator_current
0001:0040b514  _zim_spl_SplFileObject_fgetcsv
0001:0040b672  _zim_spl_SplFileObject_fgets
0001:0040b6f7  _zim_spl_SplFileObject_ftruncate
0001:0040b98b  _zim_spl_SplFileObject_fstat
0001:0040ba43  _zim_spl_SplFileObject_fscanf
0001:0040bb0b  _zim_spl_SplFileObject_fgetss
0001:0040bc27  _zim_spl_SplFileObject_flock
0001:0040bcdc  _zim_spl_SplFileObject_fwrite
0001:0040be12  _zim_spl_SplFileObject_fpassthru
0001:0040be4b  _zim_spl_SplFileObject_fgetc
0001:0040bed7  _zim_spl_SplFileObject_ftell
0001:0040bf26  _zim_spl_SplFileObject_fflush
0001:0040bf6f  _zim_spl_SplFileObject_getCsvControl
0001:0040c020  _zim_spl_SplTempFileObject___construct
0001:0040c15a  _zim_spl_SplFileObject___construct
0001:0040c2aa  _spl_filesystem_info_set_filename
0001:0040c36a  _zim_spl_SplFileInfo___construct
0001:0040c50c  _zim_spl_GlobIterator_count
0001:0040c58d  _zim_spl_DirectoryIterator_seek
0001:0040c7c6  _zim_spl_SplFileInfo_getLinkTarget
0001:0040c8bf  _zim_spl_DirectoryIterator_getBasename
0001:0040c96d  _spl_filesystem_object_get_path
0001:0040ca72  _zim_spl_SplFileInfo_getRealPath
0001:0040cb94  _zim_spl_SplFileInfo_getBasename
0001:0040cc6f  _zim_spl_SplFileInfo_getFilename
0001:0040ccfd  _zim_spl_SplFileInfo_getPath
0001:0040d00d  _zim_spl_SplFileObject_current
0001:0040d0e3  _zim_spl_SplFileObject_next
0001:0040d20c  _zim_spl_SplFileObject_seek
0001:0040d2c9  _zim_spl_SplFileObject_rewind
0001:0040d43f  _zim_spl_FilesystemIterator_rewind
0001:0040d4d8  _zim_spl_DirectoryIterator_next
0001:0040d90c  _spl_filesystem_object_construct
0001:0040daf9  _zim_spl_GlobIterator___construct
0001:0040db37  _zim_spl_RecursiveDirectoryIterator___construct
0001:0040db75  _zim_spl_FilesystemIterator___construct
0001:0040dbb3  _zim_spl_DirectoryIterator___construct
0001:0040dbf1  _zim_spl_DirectoryIterator_isDot
0001:0040dc53  _zim_spl_SplFileInfo_getOwner
0001:0040dd68  _zim_spl_SplFileInfo_getSize
0001:0040de7d  _zim_spl_SplFileInfo_getInode
0001:0040df92  _zim_spl_SplFileInfo_getPerms
0001:0040e0a8  _zim_spl_RecursiveDirectoryIterator_getChildren
0001:0040e318  _zim_spl_SplFileInfo_isLink
0001:0040e42d  _zim_spl_SplFileInfo_isDir
0001:0040e542  _zim_spl_SplFileInfo_isFile
0001:0040e658  _zim_spl_SplFileInfo_isExecutable
0001:0040e76d  _zim_spl_SplFileInfo_isReadable
0001:0040e882  _zim_spl_SplFileInfo_isWritable
0001:0040e998  _zim_spl_SplFileInfo_getType
0001:0040eaad  _zim_spl_SplFileInfo_getCTime
0001:0040ebc2  _zim_spl_SplFileInfo_getMTime
0001:0040ecd8  _zim_spl_SplFileInfo_getATime
0001:0040eded  _zim_spl_SplFileInfo_getGroup
0001:0040f034  _zim_spl_FilesystemIterator_key
0001:0040f223  _zim_spl_SplFileInfo_getPathInfo
0001:0040f465  _zim_spl_SplFileInfo_getPathname
0001:0040f979  _zim_spl_RecursiveDirectoryIterator_hasChildren
0001:004102c0  _zim_spl_SplFileInfo_getFileInfo
0001:00410365  _zim_spl_SplFileInfo_openFile
0001:004103ac  _zim_spl_FilesystemIterator_current
0002:00002970  _spl_filesystem_tree_it_funcs
0002:00002950  _spl_filesystem_dir_it_funcs
Module: U:\dev\php-5.3.3\ext\spl\spl_exceptions.o(spl_exceptions.o)
0002:00020480  _spl_ce_LogicException
0002:00020490  _spl_ce_BadFunctionCallException
0002:000204a0  _spl_ce_BadMethodCallException
0002:000204b0  _spl_ce_DomainException
0002:000204c0  _spl_ce_InvalidArgumentException
0002:000204d0  _spl_ce_LengthException
0002:000204e0  _spl_ce_OutOfRangeException
0002:000204f0  _spl_ce_RuntimeException
0002:00020500  _spl_ce_OutOfBoundsException
0002:00020510  _spl_ce_OverflowException
0002:00020520  _spl_ce_RangeException
0002:00020530  _spl_ce_UnderflowException
0002:00020540  _spl_ce_UnexpectedValueException
0001:004115bf  _zm_startup_spl_exceptions
Module: U:\dev\php-5.3.3\ext\spl\spl_observer.o(spl_observer.o)
0002:00020550  _spl_ce_SplObserver
0002:00020560  _spl_ce_SplSubject
0002:00020570  _spl_ce_SplObjectStorage
0002:00020580  _spl_handler_SplObjectStorage
0002:000205f0  _spl_ce_MultipleIterator
0001:004118d3  _zm_startup_spl_observer
0001:00411af8  _zim_spl_MultipleIterator_getFlags
0001:00411b23  _zim_spl_SplObjectStorage_key
0001:00411c1a  _zim_spl_SplObjectStorage_count
0001:00411c4d  _zim_spl_SplObjectStorage_rewind
0001:00411c87  _zim_spl_SplObjectStorage_next
0001:0041205b  _zim_spl_MultipleIterator_valid
0001:004121cd  _zim_spl_MultipleIterator_next
0001:004122c5  _zim_spl_MultipleIterator_rewind
0001:0041280f  _zim_spl_MultipleIterator_key
0001:00412847  _zim_spl_MultipleIterator_current
0001:00412881  _zim_spl_MultipleIterator_setFlags
0001:004128be  _zim_spl_SplObjectStorage_setInfo
0001:00412940  _zim_spl_MultipleIterator___construct
0001:004129bd  _zim_spl_SplObjectStorage_serialize
0001:00412fd9  _zim_spl_SplObjectStorage_valid
0001:0041301c  _zim_spl_SplObjectStorage_getInfo
0001:0041309c  _zim_spl_SplObjectStorage_current
0001:0041311b  _spl_object_storage_contains
0001:00413139  _zim_spl_SplObjectStorage_contains
0001:004131ac  _spl_object_storage_detach
0001:004131e3  _zim_spl_SplObjectStorage_removeAll
0001:004132d3  _zim_spl_SplObjectStorage_detach
0001:00413345  _spl_object_storage_get
0001:0041338d  _zim_spl_SplObjectStorage_offsetGet
0001:0041344d  _spl_object_storage_attach
0001:0041355b  _zim_spl_MultipleIterator_attachIterator
0001:004136b9  _zim_spl_SplObjectStorage_attach
0001:00413727  _spl_object_storage_addall
0001:00413e4b  _spl_SplOjectStorage_free_storage
0001:00413936  _zim_spl_SplObjectStorage_addAll
0001:00413a04  _zim_spl_SplObjectStorage_unserialize
Module: U:\dev\php-5.3.3\ext\spl\spl_dllist.o(spl_dllist.o)
0002:00020600  _spl_ce_SplDoublyLinkedList
0002:00020610  _spl_handler_SplDoublyLinkedList
0002:00020680  _spl_ce_SplQueue
0002:00020690  _spl_ce_SplStack
0001:0041491a  _zm_startup_spl_dllist
0001:00415505  _spl_dllist_get_iterator
0001:00414b1d  _zim_spl_SplDoublyLinkedList_rewind
0001:00414b99  _zim_spl_SplDoublyLinkedList_valid
0001:00414bcc  _zim_spl_SplDoublyLinkedList_next
0001:00414c0a  _zim_spl_SplDoublyLinkedList_prev
0001:00414c4b  _zim_spl_SplDoublyLinkedList_key
0001:004155a3  _zim_spl_SplDoublyLinkedList_getIteratorMode
0001:00415634  _zim_spl_SplDoublyLinkedList_setIteratorMode
0001:004156bf  _zim_spl_SplDoublyLinkedList_count
0001:00415711  _zim_spl_SplDoublyLinkedList_unshift
0001:0041582c  _zim_spl_SplDoublyLinkedList_offsetUnset
0001:0041598e  _zim_spl_SplDoublyLinkedList_offsetExists
0001:00415a00  _zim_spl_SplDoublyLinkedList_current
0001:00415bb4  _zim_spl_SplDoublyLinkedList_isEmpty
0001:00415c31  _zim_spl_SplDoublyLinkedList_bottom
0001:00415ce0  _zim_spl_SplDoublyLinkedList_top
0001:00415db8  _zim_spl_SplDoublyLinkedList_shift
0001:00415e9a  _zim_spl_SplDoublyLinkedList_pop
0001:00415f77  _zim_spl_SplDoublyLinkedList_offsetGet
0001:0041609a  _zim_spl_SplDoublyLinkedList_push
0001:00416154  _zim_spl_SplDoublyLinkedList_offsetSet
0002:00002990  _spl_dllist_it_funcs
Module: U:\dev\php-5.3.3\ext\spl\spl_heap.o(spl_heap.o)
0002:000206a0  _spl_ce_SplHeap
0002:000206b0  _spl_handler_SplHeap
0002:00020720  _spl_ce_SplMinHeap
0002:00020730  _spl_ce_SplMaxHeap
0002:00020740  _spl_ce_SplPriorityQueue
0002:00020750  _spl_handler_SplPriorityQueue
0001:0041685f  _zim_spl_SplHeap_rewind
0001:00416b46  _zm_startup_spl_heap
0001:00416f0f  _spl_heap_get_iterator
0001:00416e89  _spl_pqueue_get_iterator
0001:00416da5  _zim_spl_SplHeap_valid
0001:00416ddb  _zim_spl_SplHeap_next
0001:00416e21  _zim_spl_SplHeap_key
0001:00417bc4  _zim_spl_SplMaxHeap_compare
0001:00417c27  _zim_spl_SplMinHeap_compare
0001:00417c8a  _zim_spl_SplPriorityQueue_compare
0001:00417cee  _zim_spl_SplHeap_recoverFromCorruption
0001:00417d41  _zim_spl_SplPriorityQueue_setExtractFlags
0001:00417d97  _zim_spl_SplHeap_isEmpty
0001:00417def  _zim_spl_SplHeap_count
0001:00417f2a  _zim_spl_SplHeap_insert
0001:0041818f  _zim_spl_SplHeap_top
0001:00418257  _zim_spl_SplPriorityQueue_current
0001:004182f7  _zim_spl_SplHeap_current
0001:0041836e  _zim_spl_SplPriorityQueue_top
0001:004184ad  _zim_spl_SplHeap_extract
0001:00418597  _zim_spl_SplPriorityQueue_extract
0001:004186e3  _zim_spl_SplPriorityQueue_insert
0002:000029d0  _spl_pqueue_it_funcs
0002:000029b0  _spl_heap_it_funcs
Module: U:\dev\php-5.3.3\ext\spl\spl_fixedarray.o(spl_fixedarray.o)
0002:000207c0  _spl_ce_SplFixedArray
0002:000207d0  _spl_handler_SplFixedArray
0001:00418e21  _zm_startup_spl_fixedarray
0001:00418f65  _spl_fixedarray_get_iterator
0001:004197a9  _zim_spl_SplFixedArray_rewind
0001:004197ef  _zim_spl_SplFixedArray_valid
0001:00419855  _zim_spl_SplFixedArray_next
0001:00419898  _zim_spl_SplFixedArray_key
0001:004198e5  _zim_spl_SplFixedArray_getSize
0001:00419945  _zim_spl_SplFixedArray_count
0001:004199cc  _zim_spl_SplFixedArray___construct
0001:00419a75  _zim_spl_SplFixedArray_setSize
0001:00419c63  _zim_spl_SplFixedArray_toArray
0001:00419f24  _zim_spl_SplFixedArray_fromArray
0001:0041aa23  _zim_spl_SplFixedArray_offsetExists
0001:0041aab2  _zim_spl_SplFixedArray_offsetUnset
0001:0041ab6f  _zim_spl_SplFixedArray_current
0001:0041ac99  _zim_spl_SplFixedArray_offsetGet
0001:0041ae67  _zim_spl_SplFixedArray_offsetSet
0002:000029f0  _spl_fixedarray_it_funcs
Module: U:\dev\php-5.3.3\ext\standard\crypt_freesec.o(crypt_freesec.o)
0001:0041b140  __crypt_extended_init
0001:0041bcb9  __crypt_extended_r
Module: U:\dev\php-5.3.3\ext\standard\crypt_blowfish.o(crypt_blowfish.o)
0001:0041c490  _php_crypt_gensalt_blowfish_rn
0001:0041c5fb  _php_crypt_blowfish_rn
Module: U:\dev\php-5.3.3\ext\standard\crypt_sha512.o(crypt_sha512.o)
0001:00420e7e  _php_sha512_crypt_r
0001:00421f56  _php_sha512_crypt
Module: U:\dev\php-5.3.3\ext\standard\crypt_sha256.o(crypt_sha256.o)
0001:00422947  ___php_mempcpy
0001:0042296f  ___php_stpncpy
0001:004229ba  _php_sha256_crypt_r
0001:00423a5d  _php_sha256_crypt
Module: U:\dev\php-5.3.3\ext\standard\php_crypt_r.o(php_crypt_r.o)
0002:00020840  _php_crypt_extended_init_lock
0001:00423c64  _php_md5_crypt_r
0001:0042417f  __crypt_extended_init_r
0001:004241af  _php_shutdown_crypt_r
0001:004241c4  _php_init_crypt_r
Module: U:\dev\php-5.3.3\ext\standard\array.o(array.o)
0002:00020850  _array_globals_id
0001:00424322  _php_multisort_compare
0001:004244e5  _zif_array_chunk
0001:0042474f  _zif_array_key_exists
0001:00424965  _zif_array_filter
0001:00424bdd  _zif_array_values
0001:00424d00  _zif_array_push
0001:00424e48  _zif_array_fill
0001:004250e1  _zif_array_search
0001:0042511f  _zif_in_array
0001:0042515f  _zif_key
0001:00425254  _zif_array_rand
0001:00425510  _zif_array_multisort
0001:00425c38  _zif_shuffle
0001:0042600e  _zif_array_slice
0001:00426706  _zif_array_udiff_assoc
0001:00426744  _zif_array_diff_assoc
0001:00426782  _zif_array_diff_key
0001:00426b2a  _zif_array_uintersect_assoc
0001:00426b68  _zif_array_intersect_assoc
0001:00426ba6  _zif_array_intersect_key
0001:00426be4  _php_splice
0001:00426f8c  _zif_array_change_key_case
0001:0042713a  _zif_array_unshift
0001:0042724a  _zif_array_reverse
0001:00427571  _zif_array_keys
0001:00427784  _zif_array_splice
0001:004279ae  _zif_compact
0001:00427acd  _php_prefix_varname
0001:00427b93  _zif_uksort
0001:00427d53  _zif_uasort
0001:00427f13  _zif_usort
0001:004280d3  _zif_rsort
0001:00428171  _zif_sort
0001:0042820f  _zif_arsort
0001:004282ad  _zif_asort
0001:004283d8  _zif_natcasesort
0001:00428416  _zif_natsort
0001:00428454  _zif_ksort
0001:004284f2  _zif_krsort
0001:0042859a  _zif_count
0001:0042876d  _zm_shutdown_array
0001:00428880  _zm_startup_array
0001:00428e6e  _zif_array_count_values
0001:00429326  _zif_extract
0001:00429af7  _zif_array_sum
0001:00429c2c  _php_array_replace_recursive
0001:00429f76  _zif_array_map
0001:0042a647  _zif_array_combine
0001:0042a855  _zif_array_product
0001:0042ad71  _zif_array_walk_recursive
0001:0042aef5  _zif_array_walk
0001:0042b0b2  _zif_array_pad
0001:0042b490  _zif_min
0001:0042b673  _zif_max
0001:0042baa4  _zif_array_shift
0001:0042bae2  _zif_array_pop
0001:0042bb20  _zif_current
0001:0042bc00  _zif_array_reduce
0001:0042be82  _php_array_merge
0001:0042c699  _zif_array_replace_recursive
0001:0042c6df  _zif_array_replace
0001:0042c725  _zif_array_merge_recursive
0001:0042c76b  _zif_array_merge
0001:0042c7b1  _zif_end
0001:0042c870  _zif_reset
0001:0042c92f  _zif_prev
0001:0042c9ee  _zif_next
0001:0042d916  _zif_array_udiff_uassoc
0001:0042d964  _zif_array_diff_uassoc
0001:0042d9b2  _zif_array_udiff
0001:0042da00  _zif_array_diff
0001:0042da4e  _zif_array_diff_ukey
0001:0042e875  _zif_array_uintersect_uassoc
0001:0042e8c3  _zif_array_intersect_uassoc
0001:0042e911  _zif_array_uintersect
0001:0042e95f  _zif_array_intersect
0001:0042e9ad  _zif_array_intersect_ukey
0001:0042ea25  _zif_range
0001:0042f486  _zif_array_fill_keys
0001:0042f781  _zif_array_flip
0001:0042fa95  _zif_array_unique
Module: U:\dev\php-5.3.3\ext\standard\base64.o(base64.o)
0001:0042fd90  _php_base64_encode
0001:0042ff13  _zif_base64_encode
0001:0042ff89  _php_base64_decode_ex
0001:00430141  _zif_base64_decode
0001:004301ca  _php_base64_decode
Module: U:\dev\php-5.3.3\ext\standard\basic_functions.o(basic_functions.o)
0002:00020860  _basic_globals_id
0001:00430450  _php_get_nan
0001:0043045b  _php_get_inf
0001:00430466  _zif_get_magic_quotes_runtime
0001:00430487  _zif_get_magic_quotes_gpc
0001:004304a7  _zif_connection_aborted
0001:004304ce  _zif_connection_status
0001:004304f2  _zif_sys_getloadavg
0001:00430581  _zif_set_magic_quotes_runtime
0001:0043060c  _zif_import_request_variables
0001:0043099d  _zif_parse_ini_string
0001:00430b5e  _zif_parse_ini_file
0001:00430cbc  _zif_is_uploaded_file
0001:00430d7d  _zif_move_uploaded_file
0001:00430fb4  _zif_unregister_tick_function
0001:004311e4  _zif_getprotobynumber
0001:00431263  _zif_getprotobyname
0001:004312c7  _zif_getservbyport
0001:00431361  _zif_getservbyname
0001:004313f1  _zif_ignore_user_abort
0001:004314a2  _zif_print_r
0001:0043157d  _zif_restore_include_path
0001:004315bf  _zif_ini_restore
0001:00431611  _zif_get_include_path
0001:0043169a  _zif_ini_get
0001:00431755  _zif_ini_get_all
0001:00431a77  _zif_php_strip_whitespace
0001:00431c28  _php_get_highlight_struct
0001:00431d22  _zif_register_shutdown_function
0001:00431fca  _php_free_shutdown_functions
0001:00432078  _php_call_shutdown_functions
0001:00432128  _zif_error_get_last
0001:00432292  __php_error_log_ex
0001:004323cf  __php_error_log
0001:00432426  _zif_error_log
0001:00432500  _zif_get_cfg_var
0001:004326de  _zif_get_current_user
0001:0043276e  _zif_time_sleep_until
0001:00432902  _zif_time_nanosleep
0001:00432a42  _zif_usleep
0001:00432af1  _zif_sleep
0001:00432b6f  _zif_flush
0001:00432c43  _zif_putenv
0001:0043307f  _zif_getenv
0001:0043313f  _zif_long2ip
0001:00433231  _php_inet_ntop
0001:00433302  _zif_ip2long
0001:0043339d  _php_inet_pton
0001:004334ad  _zif_constant
0001:0043354c  _zm_info_basic
0001:0043358f  _zm_deactivate_basic
0001:00433759  _zm_activate_basic
0001:0043397e  _zm_shutdown_basic
0001:00433c43  _zm_startup_basic
0001:00434890  _zif_highlight_string
0001:00434b04  _zif_forward_static_call
0001:00434cc7  _zif_call_user_method_array
0001:00434f25  _zif_call_user_method
0001:004350fd  _zif_call_user_func
0001:00435214  _zif_forward_static_call_array
0001:00435371  _zif_call_user_func_array
0001:0043548a  _zif_set_include_path
0001:004357ba  _zif_register_tick_function
0001:00436120  _zif_ini_set
0001:00436372  _zif_highlight_file
0001:00436dec  _zif_getopt
0001:00439220  _basic_functions
0002:00002be0  _basic_functions_module
Module: U:\dev\php-5.3.3\ext\standard\browscap.o(browscap.o)
0001:004451bb  _zif_get_browser
0001:00445791  _zm_shutdown_browscap
0001:004457f3  _zm_startup_browscap
Module: U:\dev\php-5.3.3\ext\standard\crc32.o(crc32.o)
0001:00446042  _php_if_crc32
Module: U:\dev\php-5.3.3\ext\standard\crypt.o(crypt.o)
0001:004464da  _zif_crypt
0001:00446a24  _zm_shutdown_crypt
0001:00446a94  _zm_startup_crypt
Module: U:\dev\php-5.3.3\ext\standard\cyr_convert.o(cyr_convert.o)
0001:00446c80  _zif_convert_cyr_string
Module: U:\dev\php-5.3.3\ext\standard\datetime.o(datetime.o)
0001:00447759  _zif_strptime
0001:00447964  _php_std_date
0002:00002c70  _mon_short_names
0002:00002ca0  _day_full_names
0002:00002cc0  _day_short_names
0002:00002c40  _mon_full_names
Module: U:\dev\php-5.3.3\ext\standard\dir.o(dir.o)
0002:00020870  _dir_globals_id
0001:00447b70  _zm_activate_dir
0001:00447bd1  _zif_scandir
0001:00447e2d  _zif_glob
0001:004482d5  _php_if_readdir
0001:0044851e  _zif_getcwd
0001:004485af  _zif_rewinddir
0001:004487b2  _zif_chdir
0001:00448a08  _zif_closedir
0001:00448da5  _zif_getdir
0001:00448de3  _zif_opendir
0001:00448eab  _zm_startup_dir
Module: U:\dev\php-5.3.3\ext\standard\dl.o(dl.o)
0001:00449280  _zm_info_dl
0001:0044949d  _php_load_extension
0001:00449880  _php_dl
0001:004499e6  _zif_dl
Module: U:\dev\php-5.3.3\ext\standard\dns.o(dns.o)
0001:00449b72  _zif_gethostbynamel
0001:00449c26  _zif_gethostbyname
0001:00449cd7  _zif_gethostbyaddr
0001:00449dd3  _zif_gethostname
Module: U:\dev\php-5.3.3\ext\standard\exec.o(exec.o)
0001:00449ef8  _zif_proc_nice
0001:00449fd9  _zif_shell_exec
0001:0044a11b  _php_escape_shell_arg
0001:0044a258  _zif_escapeshellarg
0001:0044a2c1  _php_escape_shell_cmd
0001:0044a66a  _zif_escapeshellcmd
0001:0044a74a  _php_exec
0001:0044adcf  _zif_passthru
0001:0044ae0d  _zif_system
0001:0044ae4b  _zif_exec
Module: U:\dev\php-5.3.3\ext\standard\file.o(file.o)
0002:00020880  _file_globals_id
0001:0044ae90  _php_le_stream_context
0001:0044aec7  _zm_shutdown_file
0001:0044aece  _zif_sys_get_temp_dir
0001:0044af90  _zif_fnmatch
0001:0044b074  _php_next_meta_token
0001:0044b4af  _zif_realpath
0001:0044b637  _php_fgetcsv
0001:0044bca9  _zif_fgetc
0001:0044bd79  _zif_feof
0001:0044bf19  _zif_fgetcsv
0001:0044c2a5  _zif_fputcsv
0001:0044cac5  _zif_fwrite
0001:0044cc80  _zif_fread
0001:0044ce33  _php_copy_file_ex
0001:0044d0ec  _php_copy_file
0001:0044d129  _zif_copy
0001:0044d263  _php_if_fopen
0001:0044d3c0  _php_if_fstat
0001:0044e135  _php_if_ftruncate
0001:0044e288  _zif_unlink
0001:0044e482  _zif_rename
0001:0044e650  _zif_fpassthru
0001:0044e6fc  _zif_readfile
0001:0044e835  _zif_umask
0001:0044e8d8  _zif_rmdir
0001:0044e9c5  _zif_mkdir
0001:0044eaf1  _zif_flock
0001:0044ec77  _php_mkdir_ex
0001:0044ed25  _php_mkdir
0001:0044ed53  _zif_fseek
0001:0044ee25  _zif_rewind
0001:0044eef0  _zif_ftell
0001:0044ef9b  _zif_fflush
0001:0044f061  _zif_fscanf
0001:0044f1b3  _zif_fgetss
0001:0044f35f  _zif_fgets
0001:0044f57e  _zif_pclose
0001:0044f65a  _zif_fclose
0001:0044f763  _zif_popen
0001:0044fa6c  _php_if_tmpfile
0001:0044facb  _zif_tempnam
0001:0044fc71  _zif_file_get_contents
0001:0044ff39  _zif_file
0001:004504ef  _zif_file_put_contents
0001:00450c8e  _zif_get_meta_tags
0001:004517b0  _zm_startup_file
Module: U:\dev\php-5.3.3\ext\standard\filestat.o(filestat.o)
0001:004524c0  _zm_activate_filestat
0001:00452507  _zif_realpath_cache_get
0001:004526a1  _zif_realpath_cache_size
0001:004526e0  _zm_deactivate_filestat
0001:00452817  _php_stat
0001:00453d5f  _php_if_stat
0001:00453dbe  _php_if_lstat
0001:00453e1d  _zif_file_exists
0001:00453e7c  _zif_is_link
0001:00453edb  _zif_is_dir
0001:00453f3a  _zif_is_file
0001:00453f99  _zif_is_executable
0001:00453ff8  _zif_is_readable
0001:00454057  _zif_is_writable
0001:004540b6  _zif_filetype
0001:00454115  _zif_filectime
0001:00454174  _zif_filemtime
0001:004541d3  _zif_fileatime
0001:00454232  _zif_filegroup
0001:00454291  _zif_fileowner
0001:004542f0  _zif_filesize
0001:0045434f  _zif_fileinode
0001:004543ae  _zif_fileperms
0001:0045440d  _php_clear_stat_cache
0001:004544bc  _zif_clearstatcache
0001:00454569  _zif_touch
0001:0045475f  _zif_chmod
0001:00454b77  _zif_lchown
0001:00454bbf  _zif_chown
0001:00454e45  _zif_lchgrp
0001:00454e83  _zif_chgrp
0001:00454ec1  _zif_disk_free_space
0001:00454f8a  _zif_disk_total_space
Module: U:\dev\php-5.3.3\ext\standard\flock_compat.o(flock_compat.o)
0001:00455060  _php_flock
Module: U:\dev\php-5.3.3\ext\standard\formatted_print.o(formatted_print.o)
0001:00456fd8  _zif_vfprintf
0001:004570e4  _zif_fprintf
0001:004571f3  _zif_vsprintf
0001:0045724c  _zif_user_sprintf
0001:004572a5  _zif_vprintf
0001:0045731d  _zif_user_printf
Module: U:\dev\php-5.3.3\ext\standard\fsock.o(fsock.o)
0001:0045773c  _zif_pfsockopen
0001:0045777a  _zif_fsockopen
Module: U:\dev\php-5.3.3\ext\standard\head.o(head.o)
0001:004577c1  _zif_headers_list
0001:0045785b  _zif_headers_sent
0001:00457b03  _php_setcookie
0001:00457eee  _zif_setrawcookie
0001:00458023  _zif_setcookie
0001:0045815b  _zif_header_remove
0001:004581cd  _zif_header
0001:00458249  _php_header
Module: U:\dev\php-5.3.3\ext\standard\html.o(html.o)
0001:00458280  _php_utf32_utf8
0001:004586cb  _zif_get_html_translation_table
0001:004588ac  _zif_htmlspecialchars_decode
0001:00458b7d  _register_html_constants
0001:00458cc4  _php_escape_html_entities_ex
0001:00459609  _zif_htmlentities
0001:00459647  _zif_htmlspecialchars
0001:00459685  _php_escape_html_entities
0001:004596e2  _php_unescape_html_entities
0001:00459d83  _zif_html_entity_decode
Module: U:\dev\php-5.3.3\ext\standard\image.o(image.o)
0001:0045c3fc  _php_image_type_to_mime_type
0001:0045d06f  _php_getimagetype
0001:0045ebfb  _php_sig_gif
0001:0045ec0a  _php_sig_jpg
0001:0045ec0d  _php_sig_png
0001:0045ec04  _php_sig_swf
0001:0045ec07  _php_sig_swc
0001:0045ebfe  _php_sig_psd
0001:0045ec02  _php_sig_bmp
0001:0045ec1d  _php_sig_jpc
0001:0045ec15  _php_sig_tif_ii
0001:0045ec19  _php_sig_tif_mm
0001:0045ec2c  _php_sig_iff
0001:0045ec30  _php_sig_ico
0001:0045ec20  _php_sig_jp2
0001:0045d3da  _zif_getimagesize
0001:0045e366  _zif_image_type_to_extension
0001:0045e6c5  _zif_image_type_to_mime_type
0001:0045e874  _zm_startup_imagetypes
0001:0045ec40  _php_tiff_bytes_per_format
Module: U:\dev\php-5.3.3\ext\standard\info.o(info.o)
0001:0045ed71  _zif_php_ini_scanned_files
0001:0045edaa  _zif_php_ini_loaded_file
0001:0045ee1b  _zif_php_sapi_name
0001:0045eeb4  _zif_zend_logo_guid
0001:0045ef2c  _zif_php_egg_logo_guid
0001:0045efa4  _zif_php_real_logo_guid
0001:0045eff4  _php_logo_guid
0001:0045f042  _zif_php_logo_guid
0001:0045f096  _zif_phpcredits
0001:0045f0f6  _zif_phpversion
0001:0045f333  _register_phpinfo_constants
0001:0045f641  _php_info_print_table_colspan_header
0001:0045f70d  _php_info_print_hr
0001:0045f749  _php_info_print_table_end
0001:0045f775  _php_info_print_box_end
0001:0045f7c6  _php_info_print_table_start
0001:0045f81a  _php_info_print_box_start
0001:0045f8a0  _php_info_print_table_header
0001:0045fa7c  _php_info_html_esc
0001:0045fce9  _php_info_print_table_row_ex
0001:0045fd0c  _php_info_print_table_row
0001:0045fd77  _php_info_print_module
0001:0045feb2  _php_info_html_esc_write
0001:00460403  _php_get_uname
0001:004604a5  _zif_php_uname
0001:0046053e  _php_info_print_style
0001:00460659  _php_print_info_htmlhead
0001:00461441  _php_print_info
0001:004627e5  _zif_phpinfo
Module: U:\dev\php-5.3.3\ext\standard\iptc.o(iptc.o)
0001:0046288a  _zif_iptcparse
0001:00462c6a  _zif_iptcembed
Module: U:\dev\php-5.3.3\ext\standard\lcg.o(lcg.o)
0002:00020890  _lcg_globals_id
0001:0046320b  _zm_startup_lcg
0001:00463239  _php_combined_lcg
0001:004633a9  _zif_lcg_value
Module: U:\dev\php-5.3.3\ext\standard\link.o(link.o)
0001:00463418  _zif_link
0001:00463637  _zif_symlink
0001:0046389d  _zif_linkinfo
0001:00463945  _zif_readlink
Module: U:\dev\php-5.3.3\ext\standard\mail.o(mail.o)
0001:00463a8f  _zm_info_mail
0001:00463bf9  _php_mail
0001:0046400c  _zif_ezmlm_hash
0001:0046413e  _zif_mail
Module: U:\dev\php-5.3.3\ext\standard\math.o(math.o)
0001:00464640  _zif_pi
0001:00464654  __php_math_basetozval
0001:0046477a  _zif_rad2deg
0001:004647c5  _zif_deg2rad
0001:00464810  _zif_is_nan
0001:0046485d  _zif_fmod
0001:004648d5  __php_math_longtobase
0001:0046495d  __php_math_zvaltobase
0001:00464b96  __php_math_basetolong
0001:00464c79  _zif_hypot
0001:00464cce  _zif_sqrt
0001:00464d2e  _zif_log10
0001:00464d95  _zif_log
0001:00464e5f  _zif_log1p
0001:00464ea6  _zif_expm1
0001:00464eed  _zif_exp
0001:00464f39  _zif_pow
0001:004650a2  _zif_is_infinite
0001:004650f6  _zif_is_finite
0001:0046514a  _zif_atanh
0001:00465191  _zif_acosh
0001:004651d8  _zif_asinh
0001:0046521f  _zif_tanh
0001:00465266  _zif_cosh
0001:004652ad  _zif_sinh
0001:004652f4  _zif_atan2
0001:00465349  _zif_atan
0001:00465390  _zif_acos
0001:004653d7  _zif_asin
0001:0046541e  _zif_tan
0001:00465465  _zif_cos
0001:004654ac  _zif_sin
0001:004654f5  _zif_octdec
0001:004655ee  _zif_hexdec
0001:004656e7  _zif_bindec
0001:004657e0  _zif_dechex
0001:004658ca  _zif_decoct
0001:004659b4  _zif_decbin
0001:00465ad4  _zif_base_convert
0001:00465c5f  _zif_abs
0001:00465d8d  _zif_ceil
0001:00465f1b  _zif_floor
0001:004660b1  __php_math_round
0001:004666af  __php_math_number_format
0001:004668d1  _zif_number_format
0001:00466a0e  _zif_round
Module: U:\dev\php-5.3.3\ext\standard\md5.o(md5.o)
0001:00466de0  _make_digest_ex
0001:00466e29  _make_digest
0001:00467575  _PHP_MD5Init
0001:004675a6  _PHP_MD5Final
0001:004676ff  _PHP_MD5Update
0001:004677e6  _php_if_md5_file
0001:004679c4  _php_if_md5
Module: U:\dev\php-5.3.3\ext\standard\metaphone.o(metaphone.o)
0001:00467b14  _zif_metaphone
0002:00002d50  __codes
Module: U:\dev\php-5.3.3\ext\standard\microtime.o(microtime.o)
0001:00468d75  _zif_gettimeofday
0001:00468db3  _zif_microtime
Module: U:\dev\php-5.3.3\ext\standard\pack.o(pack.o)
0002:000208a0  _machine_little_endian
0001:00468e00  _zm_startup_pack
0001:00469074  _zif_unpack
0001:00469ed7  _zif_pack
Module: U:\dev\php-5.3.3\ext\standard\pageinfo.o(pageinfo.o)
0001:0046b220  _zif_getmypid
0001:0046b24f  _php_statpage
0001:0046b2da  _php_getlastmod
0001:0046b304  _zif_getlastmod
0001:0046b339  _zif_getmyinode
0001:0046b383  _php_getgid
0001:0046b3c0  _zif_getmygid
0001:0046b3ef  _php_getuid
0001:0046b42c  _zif_getmyuid
Module: U:\dev\php-5.3.3\ext\standard\quot_print.o(quot_print.o)
0001:0046b463  _zif_quoted_printable_decode
0001:0046b713  _php_quot_print_encode
0001:0046b878  _zif_quoted_printable_encode
0001:0046b904  _php_quot_print_decode
Module: U:\dev\php-5.3.3\ext\standard\rand.o(rand.o)
0001:0046bf00  _php_srand
0001:0046bf24  _php_mt_rand
0001:0046c09d  _zif_mt_getrandmax
0001:0046c0d6  _zif_getrandmax
0001:0046c112  _zif_srand
0001:0046c1b3  _php_rand
0001:0046c246  _zif_rand
0001:0046c2f4  _php_mt_srand
0001:0046c455  _zif_mt_rand
0001:0046c571  _zif_mt_srand
Module: U:\dev\php-5.3.3\ext\standard\soundex.o(soundex.o)
0001:0046c622  _zif_soundex
Module: U:\dev\php-5.3.3\ext\standard\string.o(string.o)
0001:0046c780  _php_strtoupper
0001:0046c7a8  _php_strtolower
0001:0046c7d0  _php_strspn
0001:0046c80b  _php_strcspn
0001:0046c84a  _php_strtr
0001:0046c9f2  _zif_ord
0001:0046cc15  _zif_strcspn
0001:0046cc53  _zif_strspn
0001:0046ccf7  _zif_substr_compare
0001:0046cea3  _zif_strpbrk
0001:0046cf69  _zif_str_rot13
0001:0046cfe9  _zif_ucwords
0001:0046d0a4  _zif_lcfirst
0001:0046d133  _zif_ucfirst
0001:0046d1c7  _zif_substr
0001:0046d302  _zif_strtolower
0001:0046d37d  _zif_strtoupper
0001:0046d431  _zif_str_split
0001:0046d56f  _zif_str_shuffle
0001:0046d63a  _zif_sscanf
0001:0046d6fc  _zif_nl2br
0001:0046d8a5  _zif_strrev
0001:0046d99c  _zif_str_pad
0001:0046dc85  _zif_strnatcasecmp
0001:0046dcfe  _zif_strnatcmp
0001:0046dd77  _php_stripslashes
0001:0046decd  _zif_stripslashes
0001:0046df47  _zif_count_chars
0001:0046e122  _php_char_to_str_ex
0001:0046e423  _php_char_to_str
0001:0046ec28  _zif_hebrevc
0001:0046ec66  _zif_hebrev
0001:0046ecd5  _zif_chunk_split
0001:0046ef5f  _zif_bin2hex
0001:0046f051  _zif_str_repeat
0001:0046f1b7  _zif_str_getcsv
0001:0046f2cf  _php_addslashes_ex
0001:0046f440  _php_addslashes
0001:0046f477  _zif_addslashes
0001:0046f525  _zif_quotemeta
0001:0046f706  _php_tag_find
0001:0046f83a  _php_strip_tags_ex
0001:0047039d  _php_strip_tags
0001:004703d8  _zif_parse_str
0001:00470503  _php_stripcslashes
0001:004707c8  _zif_stripcslashes
0001:00470834  _zif_similar_text
0001:00470989  _zif_chr
0001:00470a16  _zif_strtok
0001:00470ca4  _php_dirname
0001:00470cb0  _zif_dirname
0001:00470d1b  _php_basename
0001:00470e9a  _zif_basename
0001:00470f7f  _zif_wordwrap
0001:004714f1  _zif_strcoll
0001:0047156c  _zif_nl_langinfo
0001:004717e1  _zm_startup_nl_langinfo
0001:00472283  _register_string_constants
0001:0047252c  _zm_shutdown_localeconv
0001:0047254d  _zm_startup_localeconv
0001:00472561  _localeconv_r
0001:004726a1  _zif_localeconv
0001:00472b6e  _zif_setlocale
0001:0047304c  _zif_strtr
0001:00473818  _php_implode
0001:00473fc6  _zif_implode
0001:004742d3  _zif_pathinfo
0001:004747ca  _zif_strrchr
0001:0047491d  _zif_strripos
0001:00474c85  _zif_strrpos
0001:00474edb  _zif_stripos
0001:004750ea  _zif_strip_tags
0001:004752eb  _zif_substr_replace
0001:00476224  _php_addcslashes
0001:00476593  _zif_addcslashes
0001:0047666f  _php_trim
0001:00476ade  _zif_ltrim
0001:00476b1c  _zif_rtrim
0001:00476b5a  _zif_trim
0001:00476c43  _zif_substr_count
0001:00476ecc  _php_explode_negative_limit
0001:00477150  _php_stristr
0001:00477267  _zif_stristr
0001:00477414  _php_explode
0001:0047763d  _zif_explode
0001:004777ac  _php_str_to_str_ex
0001:004780e8  _php_str_to_str
0001:00478c89  _zif_str_ireplace
0001:00478cc7  _zif_str_replace
0001:00478d1e  _zif_str_word_count
0001:0047914c  _zif_strstr
0001:00479355  _zif_strpos
Module: U:\dev\php-5.3.3\ext\standard\scanf.o(scanf.o)
0001:00479699  _ValidateFormat
0001:00479cdd  _php_sscanf_internal
Module: U:\dev\php-5.3.3\ext\standard\syslog.o(syslog.o)
0001:0047b086  _zif_syslog
0001:0047b0ef  _zif_closelog
0001:0047b163  _zm_shutdown_syslog
0001:0047b1ad  _zif_openlog
0001:0047b3be  _zm_startup_syslog
0001:0047e16f  _zif_define_syslog_variables
0001:0047e1d6  _zm_activate_syslog
Module: U:\dev\php-5.3.3\ext\standard\type.o(type.o)
0001:0047e242  _zif_is_scalar
0001:0047e2ac  _zif_is_callable
0001:0047e3ea  _zif_is_numeric
0001:0047e6c9  _zif_is_object
0001:0047e707  _zif_is_array
0001:0047e745  _zif_is_string
0001:0047e783  _zif_is_float
0001:0047e7c1  _zif_is_long
0001:0047e7ff  _zif_is_bool
0001:0047e83d  _zif_is_resource
0001:0047e87b  _zif_is_null
0001:0047e8b9  _zif_strval
0001:0047e97b  _zif_floatval
0001:0047e9fb  _zif_intval
0001:0047eb4d  _zif_settype
0001:0047ed73  _zif_gettype
Module: U:\dev\php-5.3.3\ext\standard\uniqid.o(uniqid.o)
0001:0047ef6f  _zif_uniqid
Module: U:\dev\php-5.3.3\ext\standard\url.o(url.o)
0001:0047f0b0  _php_replace_controlchars_ex
0001:0047f13a  _php_url_decode
0001:0047f1f4  _php_raw_url_decode
0001:0047f2b0  _zif_get_headers
0001:0047f6cd  _zif_rawurldecode
0001:0047f738  _zif_urldecode
0001:0047f7a3  _php_raw_url_encode
0001:0047f87a  _zif_rawurlencode
0001:0047f8dc  _php_url_encode
0001:0047f993  _zif_urlencode
0001:0047f9f5  _php_replace_controlchars
0001:0047fa3a  _php_url_parse_ex
0001:00480335  _php_url_parse
0001:00480361  _php_url_free
0001:00480434  _zif_parse_url
Module: U:\dev\php-5.3.3\ext\standard\var.o(var.o)
0001:00480773  _zif_memory_get_peak_usage
0001:004807d6  _zif_memory_get_usage
0001:0048085c  _zif_unserialize
0001:0048118f  _php_var_export_ex
0001:004820b6  _zif_var_export
0001:00482180  _php_var_export
0001:00482fb8  _php_debug_zval_dump
0001:00483476  _zif_debug_zval_dump
0001:0048375c  _php_var_dump
0001:00483bad  _zif_var_dump
0001:00487a9f  _php_var_serialize
0001:00487add  _zif_serialize
Module: U:\dev\php-5.3.3\ext\standard\versioning.o(versioning.o)
0001:00487c9b  _php_canonicalize_version
0001:00487e8e  _php_version_compare
0001:0048819f  _zif_version_compare
Module: U:\dev\php-5.3.3\ext\standard\assert.o(assert.o)
0002:000208a8  _assert_globals_id
0001:004885a6  _zm_deactivate_assert
0001:004885ff  _zif_assert_options
0001:00488b47  _zif_assert
0001:004890ac  _zm_info_assert
0001:004890b8  _zm_shutdown_assert
0001:00489143  _zm_startup_assert
Module: U:\dev\php-5.3.3\ext\standard\strnatcmp.o(strnatcmp.o)
0001:00489610  _strnatcmp_ex
Module: U:\dev\php-5.3.3\ext\standard\levenshtein.o(levenshtein.o)
0001:00489c2d  _zif_levenshtein
Module: U:\dev\php-5.3.3\ext\standard\incomplete_class.o(incomplete_class.o)
0001:00489e1c  _php_store_class_name
0001:00489ecf  _php_lookup_class_name
0001:00489f6e  _php_create_incomplete_class
Module: U:\dev\php-5.3.3\ext\standard\url_scanner_ex.o(url_scanner_ex.o)
0001:0048a3e0  _php_url_scanner_reset_vars
0001:0048a40a  _zm_activate_url_scanner_ex
0001:0048a42a  _zm_deactivate_url_scanner_ex
0001:0048a5ad  _zm_shutdown_url_scanner_ex
0001:0048a5c9  _zm_startup_url_scanner_ex
0001:0048ae62  _php_url_scanner_adapt_single_url
0001:0048b11d  _php_url_scanner_add_var
Module: U:\dev\php-5.3.3\ext\standard\ftp_fopen_wrapper.o(ftp_fopen_wrapper.o)
0001:00490002  _php_stream_ftp_opendir
0001:004905d4  _php_stream_url_wrap_ftp
0002:00002df0  _php_stream_ftp_wrapper
Module: U:\dev\php-5.3.3\ext\standard\http_fopen_wrapper.o(http_fopen_wrapper.o)
0001:00491430  _php_stream_url_wrap_http_ex
0001:0049447d  _php_stream_url_wrap_http
0002:00002e70  _php_stream_http_wrapper
Module: U:\dev\php-5.3.3\ext\standard\php_fopen_wrapper.o(php_fopen_wrapper.o)
0001:004948ec  _php_stream_url_wrap_php
0002:00002ef0  _php_stream_input_ops
0002:00002ec0  _php_stream_output_ops
0002:00002f20  _php_stream_php_wrapper
Module: U:\dev\php-5.3.3\ext\standard\credits.o(credits.o)
0001:0049699a  _php_print_credits
Module: U:\dev\php-5.3.3\ext\standard\css.o(css.o)
0001:00497c61  _php_info_print_css
Module: U:\dev\php-5.3.3\ext\standard\var_unserializer.o(var_unserializer.o)
0001:00497e40  _var_replace
0001:00497ee1  _var_push_dtor
0001:00497f65  _var_destroy
0001:004981fe  _php_var_unserialize
Module: U:\dev\php-5.3.3\ext\standard\ftok.o(ftok.o)
0001:00499e48  _zif_ftok
Module: U:\dev\php-5.3.3\ext\standard\sha1.o(sha1.o)
0001:00499f90  _PHP_SHA1Init
0001:0049b696  _PHP_SHA1Update
0001:0049b770  _PHP_SHA1Final
0001:0049b83c  _make_sha1_digest
0001:0049b865  _zif_sha1_file
0001:0049ba4d  _zif_sha1
Module: U:\dev\php-5.3.3\ext\standard\user_filters.o(user_filters.o)
0001:0049bb90  _zif_user_filter_nop
0001:0049bbd4  _zif_stream_filter_register
0001:0049c39d  _zif_stream_get_filters
0001:0049c4a5  _zif_stream_bucket_new
0001:0049c6fd  _zif_stream_bucket_make_writeable
0001:0049cb1e  _zif_stream_bucket_append
0001:0049cb5c  _zif_stream_bucket_prepend
0001:0049cc0a  _userfilter_filter
0001:0049d00e  _zm_deactivate_user_filters
0001:0049d0f4  _zm_startup_user_filters
Module: U:\dev\php-5.3.3\ext\standard\uuencode.o(uuencode.o)
0001:0049d580  _php_uuencode
0001:0049d864  _zif_convert_uuencode
0001:0049d8da  _php_uudecode
0001:0049db34  _zif_convert_uudecode
Module: U:\dev\php-5.3.3\ext\standard\filters.o(filters.o)
0001:0049e516  _zm_shutdown_standard_filters
0001:0049f528  _zm_startup_standard_filters
0002:00002fc0  _consumed_filter_factory
Module: U:\dev\php-5.3.3\ext\standard\proc_open.o(proc_open.o)
0001:004a1446  _zif_proc_get_status
0001:004a16aa  _zif_proc_close
0001:004a1865  _zif_proc_terminate
0001:004a1917  _zm_startup_proc_open
0001:004a1c07  _zif_proc_open
Module: U:\dev\php-5.3.3\ext\standard\streamsfuncs.o(streamsfuncs.o)
0001:004a2f6a  _zif_stream_socket_shutdown
0001:004a302e  _zif_stream_supports_lock
0001:004a30f8  _zif_stream_set_read_buffer
0001:004a31f7  _zif_stream_set_write_buffer
0001:004a32fb  _zif_stream_set_timeout
0001:004a3419  _zif_stream_set_blocking
0001:004a34f2  _zif_stream_is_local
0001:004a3672  _zif_stream_resolve_include_path
0001:004a373e  _zif_stream_socket_enable_crypto
0001:004a3939  _zif_stream_get_line
0001:004a3afa  _zif_stream_filter_remove
0001:004a3f17  _zif_stream_filter_append
0001:004a3f55  _zif_stream_filter_prepend
0001:004a4246  _zif_stream_context_create
0001:004a44ec  _zif_stream_context_set_default
0001:004a458a  _zif_stream_context_get_default
0001:004a46e6  _zif_stream_context_get_params
0001:004a4856  _zif_stream_context_set_params
0001:004a48fa  _zif_stream_context_get_options
0001:004a49f3  _zif_stream_context_set_option
0001:004a4ef2  _zif_stream_select
0001:004a54b9  _zif_stream_get_wrappers
0001:004a559c  _zif_stream_get_transports
0001:004a56d1  _zif_stream_get_meta_data
0001:004a59c5  _zif_stream_copy_to_stream
0001:004a5b60  _zif_stream_get_contents
0001:004a5d56  _zif_stream_socket_sendto
0001:004a5edd  _zif_stream_socket_get_name
0001:004a5fef  _zif_stream_socket_pair
0001:004a6151  _zif_stream_socket_accept
0001:004a63a8  _zif_stream_socket_recvfrom
0001:004a660c  _zif_stream_socket_client
0001:004a6a12  _zif_stream_socket_server
Module: U:\dev\php-5.3.3\ext\standard\http.o(http.o)
0001:004a6d46  _php_url_encode_hash_ex
0001:004a79d8  _zif_http_build_query
Module: U:\dev\php-5.3.3\ext\tokenizer\tokenizer.o(tokenizer.o)
0001:004a7ba2  _zif_token_name
0001:004a7c0f  _zif_token_get_all
0001:004a7f43  _zm_info_tokenizer
0001:004a7f70  _zm_startup_tokenizer
0001:004a7fb0  _tokenizer_functions
0002:000030f0  _tokenizer_module_entry
Module: U:\dev\php-5.3.3\ext\tokenizer\tokenizer_data.o(tokenizer_data.o)
0001:004a8088  _get_token_type_name
0001:004a8627  _tokenizer_register_constants
Module: U:\dev\php-5.3.3\ext\xml\xml.o(xml.o)
0002:000208b8  _xml_globals_id
0001:004a9df4  _zif_xml_parser_get_option
0001:004a9fbd  _zif_xml_parser_set_option
0001:004aa3d8  _zif_xml_parser_free
0001:004aa4a3  _zif_xml_get_current_byte_index
0001:004aa539  _zif_xml_get_current_column_number
0001:004aa5cf  _zif_xml_get_current_line_number
0001:004aa667  _zif_xml_error_string
0001:004aa6d5  _zif_xml_get_error_code
0001:004aa770  _zif_xml_parse
0001:004aa853  _zif_xml_parse_into_struct
0001:004ac068  __xml_defaultHandler
0001:004ad5d1  __xml_endElementHandler
0001:004ad136  __xml_startElementHandler
0001:004ac19b  __xml_characterDataHandler
0001:004aaa21  _zif_xml_set_object
0001:004aabef  _zif_xml_set_end_namespace_decl_handler
0001:004abc82  __xml_endNamespaceDeclHandler
0001:004aacac  _zif_xml_set_default_handler
0001:004aad69  _zif_xml_set_character_data_handler
0001:004aae2a  _zif_xml_set_element_handler
0001:004aaf0c  _zif_xml_set_start_namespace_decl_handler
0001:004abcfe  __xml_startNamespaceDeclHandler
0001:004aafc9  _zif_xml_set_external_entity_ref_handler
0001:004abd9b  __xml_externalEntityRefHandler
0001:004ab086  _zif_xml_set_notation_decl_handler
0001:004abe95  __xml_notationDeclHandler
0001:004ab143  _zif_xml_set_unparsed_entity_decl_handler
0001:004abf70  __xml_unparsedEntityDeclHandler
0001:004ab200  _zif_xml_set_processing_instruction_handler
0001:004ac0e3  __xml_processingInstructionHandler
0001:004ab509  _zif_xml_parser_create_ns
0001:004ab547  _zif_xml_parser_create
0001:004ab99a  __xml_zval_strdup
0001:004ab9eb  _xml_utf8_decode
0001:004abb85  _zif_utf8_decode
0001:004ac59d  _xml_utf8_encode
0001:004ac6e9  _zif_utf8_encode
0001:004ac7a3  _zm_info_xml
0001:004acad1  _zm_startup_xml
0001:004ada50  _xml_functions
0002:000031b0  _xml_encodings
0002:00003150  _xml_module_entry
Module: U:\dev\php-5.3.3\ext\xml\compat.o(compat.o)
0001:004ae46c  _php_XML_SetUserData
0001:004ae47a  _XML_GetUserData
0001:004ae485  _php_XML_SetElementHandler
0001:004ae499  _php_XML_SetCharacterDataHandler
0001:004ae4a7  _php_XML_SetProcessingInstructionHandler
0001:004ae4b5  _php_XML_SetCommentHandler
0001:004ae4c3  _php_XML_SetDefaultHandler
0001:004ae4d1  _php_XML_SetUnparsedEntityDeclHandler
0001:004ae4df  _php_XML_SetNotationDeclHandler
0001:004ae4ed  _php_XML_SetExternalEntityRefHandler
0001:004ae4fb  _php_XML_SetStartNamespaceDeclHandler
0001:004ae509  _php_XML_SetEndNamespaceDeclHandler
0001:004ae517  _php_XML_GetErrorCode
0001:004ae52d  _php_XML_ErrorString
0001:004ae546  _php_XML_GetCurrentLineNumber
0001:004ae557  _php_XML_GetCurrentColumnNumber
0001:004ae568  _php_XML_GetCurrentByteIndex
0001:004ae57f  _php_XML_GetCurrentByteCount
0001:004ae59a  _php_XML_ExpatVersion
0001:004ae5a4  _php_XML_ParserFree
0001:004ae5f5  _php_XML_Parse
0001:004ae640  _php_XML_ParserCreate_MM
0001:004ae6ea  _php_XML_ParserCreateNS
0001:004ae716  _php_XML_ParserCreate
Module: U:\dev\php-5.3.3\ext\xmlreader\php_xmlreader.o(php_xmlreader.o)
0002:000208c8  _xmlreader_class_entry
0001:004afd80  _xmlreader_objects_clone
0001:004afd97  _zm_info_xmlreader
0001:004afdc4  _zm_shutdown_xmlreader
0001:004afe2c  _zim_xmlreader_moveToNextAttribute
0001:004afe6a  _zim_xmlreader_moveToFirstAttribute
0001:004afea8  _zim_xmlreader_moveToElement
0001:004afee6  _zim_xmlreader_isValid
0001:004affc2  _zim_xmlreader_expand
0001:004b020e  _zim_xmlreader_XML
0001:004b04ac  _zim_xmlreader_close
0001:004b04fb  _zim_xmlreader_setParserProperty
0001:004b061f  _zim_xmlreader_setSchema
0001:004b077c  _zim_xmlreader_readString
0001:004b07ba  _zim_xmlreader_readOuterXml
0001:004b07f8  _zim_xmlreader_readInnerXml
0001:004b0947  _zim_xmlreader_lookupNamespace
0001:004b0985  _zim_xmlreader_getAttribute
0001:004b0a08  _zim_xmlreader_next
0001:004b0b34  _zim_xmlreader_read
0001:004b0bed  _zim_xmlreader_moveToAttributeNs
0001:004b0cd4  _zim_xmlreader_moveToAttributeNo
0001:004b0d6b  _zim_xmlreader_moveToAttribute
0001:004b0e2d  _zim_xmlreader_getParserProperty
0001:004b0ecd  _zim_xmlreader_getAttributeNs
0001:004b0ff4  _zim_xmlreader_getAttributeNo
0001:004b10b4  _xmlreader_objects_new
0001:004b116e  _xmlreader_objects_free_storage
0001:004b11b9  __xmlreader_get_valid_file_path
0001:004b12ad  _zim_xmlreader_open
0001:004b14a7  _xmlreader_write_property
0001:004b15bb  _xmlreader_read_property
0001:004b17db  _xmlreader_get_property_ptr_ptr
0001:004b1a5d  _zim_xmlreader_setRelaxNGSchemaSource
0001:004b1a9b  _zim_xmlreader_setRelaxNGSchema
0001:004b1c9a  _zm_startup_xmlreader
0002:00003260  _xmlreader_module_entry
Module: U:\dev\php-5.3.3\ext\xmlrpc\xmlrpc-epi-php.o(xmlrpc-epi-php.o)
0001:004b2caf  _xmlrpc_type_as_str
0001:004b2d80  _zif_xmlrpc_is_fault
0001:004b2f13  _set_zval_xmlrpc_type
0001:004b3146  _xmlrpc_str_as_vector_type
0001:004b3225  _xmlrpc_str_as_type
0001:004b3332  _zif_xmlrpc_set_type
0001:004b33d6  _get_zval_xmlrpc_type
0001:004b3536  _zif_xmlrpc_get_type
0001:004b3bd7  _zif_xmlrpc_parse_method_descriptions
0001:004b3d0c  _zif_xmlrpc_server_register_introspection_callback
0001:004b4225  _zif_xmlrpc_server_add_introspection_data
0001:004b479f  _zif_xmlrpc_encode_request
0001:004b4923  _zif_xmlrpc_server_register_method
0001:004b4a2f  _zif_xmlrpc_server_destroy
0001:004b4ab2  _zif_xmlrpc_server_create
0001:004b4b9b  _zif_xmlrpc_encode
0001:004b4ce4  _zm_info_xmlrpc
0001:004b4d90  _zm_startup_xmlrpc
0001:004b539c  _decode_request_worker
0001:004b548a  _zif_xmlrpc_decode
0001:004b555a  _zif_xmlrpc_decode_request
0001:004b5633  _zif_xmlrpc_server_call_method
0001:004b5b20  _xmlrpc_functions
0002:000032c0  _xmlrpc_module_entry
Module: U:\dev\php-5.3.3\ext\xmlwriter\php_xmlwriter.o(php_xmlwriter.o)
0002:00003320  _xmlwriter_module_entry
Module: U:\dev\php-5.3.3\ext\zip\php_zip.o(php_zip.o)
0001:004be8b2  _php_zip_pcre
0001:004bec94  _php_zip_glob
0002:00003380  _zip_module_entry
Module: U:\dev\php-5.3.3\ext\zip\zip_stream.o(zip_stream.o)
0001:004c163c  _php_stream_zip_open
0001:004c173e  _php_stream_zip_opener
0002:000033e0  _php_stream_zipio_ops
0002:00003410  _php_stream_zip_wrapper
Module: U:\dev\php-5.3.3\ext\zip\lib\zip_add.o(zip_add.o)
0001:004c1960  _zip_add
Module: U:\dev\php-5.3.3\ext\zip\lib\zip_error.o(zip_error.o)
0001:004c19c0  __zip_error_clear
0001:004c19d5  __zip_error_copy
0001:004c19ea  __zip_error_init
0001:004c1a06  __zip_error_set
0001:004c1a1d  __zip_error_get
0001:004c1a61  __zip_error_fini
Module: U:\dev\php-5.3.3\ext\zip\lib\zip_fclose.o(zip_fclose.o)
0001:004c1a90  _zip_fclose
Module: U:\dev\php-5.3.3\ext\zip\lib\zip_fread.o(zip_fread.o)
0001:004c1b40  _zip_fread
Module: U:\dev\php-5.3.3\ext\zip\lib\zip_open.o(zip_open.o)
0001:004c2097  _zip_open
Module: U:\dev\php-5.3.3\ext\zip\lib\zip_source_filep.o(zip_source_filep.o)
0001:004c2a20  __zip_source_file_or_p
0001:004c2b4d  _zip_source_filep
Module: U:\dev\php-5.3.3\ext\zip\lib\zip_strerror.o(zip_strerror.o)
0001:004c2e80  _zip_strerror
Module: U:\dev\php-5.3.3\ext\zip\lib\zip_close.o(zip_close.o)
0001:004c33b7  _zip_close
Module: U:\dev\php-5.3.3\ext\zip\lib\zip_error_get.o(zip_error_get.o)
0001:004c43e0  _zip_error_get
Module: U:\dev\php-5.3.3\ext\zip\lib\zip_file_error_get.o(zip_file_error_get.o)
0001:004c4400  _zip_file_error_get
Module: U:\dev\php-5.3.3\ext\zip\lib\zip_free.o(zip_free.o)
0001:004c4420  __zip_free
Module: U:\dev\php-5.3.3\ext\zip\lib\zip_rename.o(zip_rename.o)
0001:004c4510  _zip_rename
Module: U:\dev\php-5.3.3\ext\zip\lib\zip_source_free.o(zip_source_free.o)
0001:004c45d0  _zip_source_free
Module: U:\dev\php-5.3.3\ext\zip\lib\zip_unchange_all.o(zip_unchange_all.o)
0001:004c4620  _zip_unchange_all
Module: U:\dev\php-5.3.3\ext\zip\lib\zip_delete.o(zip_delete.o)
0001:004c4670  _zip_delete
Module: U:\dev\php-5.3.3\ext\zip\lib\zip_error_get_sys_type.o(zip_error_get_sys_type.o)
0001:004c46f0  _zip_error_get_sys_type
Module: U:\dev\php-5.3.3\ext\zip\lib\zip_file_get_offset.o(zip_file_get_offset.o)
0001:004c4710  __zip_file_get_offset
Module: U:\dev\php-5.3.3\ext\zip\lib\zip_get_name.o(zip_get_name.o)
0001:004c47e0  __zip_get_name
0001:004c4873  _zip_get_name
Module: U:\dev\php-5.3.3\ext\zip\lib\zip_replace.o(zip_replace.o)
0001:004c48a0  __zip_replace
0001:004c4931  _zip_replace
Module: U:\dev\php-5.3.3\ext\zip\lib\zip_source_function.o(zip_source_function.o)
0001:004c49a0  _zip_source_function
Module: U:\dev\php-5.3.3\ext\zip\lib\zip_unchange.o(zip_unchange.o)
0001:004c4a00  __zip_unchange
0001:004c4b15  _zip_unchange
Module: U:\dev\php-5.3.3\ext\zip\lib\zip_dirent.o(zip_dirent.o)
0001:004c4b40  __zip_dirent_init
0001:004c4bbc  __zip_read2
0001:004c4bd9  __zip_read4
0001:004c4c9a  __zip_dirent_write
0001:004c4f1a  __zip_dirent_torrent_normalize
0001:004c5002  __zip_dirent_finalize
0001:004c5048  __zip_cdir_free
0001:004c515a  __zip_cdir_new
0001:004c527e  __zip_dirent_read
0001:004c5814  __zip_cdir_write
0001:004c5975  __zip_cdir_grow
Module: U:\dev\php-5.3.3\ext\zip\lib\zip_error_strerror.o(zip_error_strerror.o)
0001:004c5a1c  __zip_error_strerror
Module: U:\dev\php-5.3.3\ext\zip\lib\zip_filerange_crc.o(zip_filerange_crc.o)
0001:004c5b60  __zip_filerange_crc
Module: U:\dev\php-5.3.3\ext\zip\lib\zip_file_strerror.o(zip_file_strerror.o)
0001:004c5ca0  _zip_file_strerror
Module: U:\dev\php-5.3.3\ext\zip\lib\zip_get_num_files.o(zip_get_num_files.o)
0001:004c5cb0  _zip_get_num_files
Module: U:\dev\php-5.3.3\ext\zip\lib\zip_get_archive_flag.o(zip_get_archive_flag.o)
0001:004c5cd0  _zip_get_archive_flag
Module: U:\dev\php-5.3.3\ext\zip\lib\zip_set_archive_flag.o(zip_set_archive_flag.o)
0001:004c5d00  _zip_set_archive_flag
Module: U:\dev\php-5.3.3\ext\zip\lib\zip_set_name.o(zip_set_name.o)
0001:004c5d20  __zip_set_name
Module: U:\dev\php-5.3.3\ext\zip\lib\zip_source_zip.o(zip_source_zip.o)
0001:004c5e20  _zip_source_zip
Module: U:\dev\php-5.3.3\ext\zip\lib\zip_unchange_data.o(zip_unchange_data.o)
0001:004c62c0  __zip_unchange_data
Module: U:\dev\php-5.3.3\ext\zip\lib\zip_entry_free.o(zip_entry_free.o)
0001:004c6320  __zip_entry_free
Module: U:\dev\php-5.3.3\ext\zip\lib\zip_error_to_str.o(zip_error_to_str.o)
0001:004c638c  _zip_error_to_str
Module: U:\dev\php-5.3.3\ext\zip\lib\zip_fopen.o(zip_fopen.o)
0001:004c6440  _zip_fopen
Module: U:\dev\php-5.3.3\ext\zip\lib\zip_name_locate.o(zip_name_locate.o)
0001:004c6490  __zip_name_locate
0001:004c65b9  _zip_name_locate
Module: U:\dev\php-5.3.3\ext\zip\lib\zip_source_buffer.o(zip_source_buffer.o)
0001:004c65f0  _zip_source_buffer
Module: U:\dev\php-5.3.3\ext\zip\lib\zip_stat.o(zip_stat.o)
0001:004c67d0  _zip_stat
Module: U:\dev\php-5.3.3\ext\zip\lib\zip_entry_new.o(zip_entry_new.o)
0001:004c6820  __zip_entry_new
Module: U:\dev\php-5.3.3\ext\zip\lib\zip_err_str.o(zip_err_str.o)
0001:004c6b10  __zip_err_str
0001:004c6b70  __zip_nerr_str
0001:004c6b80  __zip_err_type
Module: U:\dev\php-5.3.3\ext\zip\lib\zip_fopen_index.o(zip_fopen_index.o)
0001:004c6be0  __zip_file_fillbuf
0001:004c6ceb  _zip_fopen_index
Module: U:\dev\php-5.3.3\ext\zip\lib\zip_get_archive_comment.o(zip_get_archive_comment.o)
0001:004c70c0  _zip_get_archive_comment
Module: U:\dev\php-5.3.3\ext\zip\lib\zip_get_file_comment.o(zip_get_file_comment.o)
0001:004c7110  _zip_get_file_comment
Module: U:\dev\php-5.3.3\ext\zip\lib\zip_new.o(zip_new.o)
0001:004c71b0  __zip_new
Module: U:\dev\php-5.3.3\ext\zip\lib\zip_source_file.o(zip_source_file.o)
0001:004c7260  _zip_source_file
Module: U:\dev\php-5.3.3\ext\zip\lib\zip_stat_index.o(zip_stat_index.o)
0001:004c72f0  _zip_stat_index
Module: U:\dev\php-5.3.3\ext\zip\lib\zip_set_archive_comment.o(zip_set_archive_comment.o)
0001:004c7440  _zip_set_archive_comment
Module: U:\dev\php-5.3.3\ext\zip\lib\zip_set_file_comment.o(zip_set_file_comment.o)
0001:004c74d0  _zip_set_file_comment
Module: U:\dev\php-5.3.3\ext\zip\lib\zip_unchange_archive.o(zip_unchange_archive.o)
0001:004c7590  _zip_unchange_archive
Module: U:\dev\php-5.3.3\ext\zip\lib\zip_memdup.o(zip_memdup.o)
0001:004c75d0  __zip_memdup
Module: U:\dev\php-5.3.3\ext\zip\lib\zip_stat_init.o(zip_stat_init.o)
0001:004c7630  _zip_stat_init
Module: U:\dev\php-5.3.3\ext\zip\lib\zip_add_dir.o(zip_add_dir.o)
0001:004c7680  _zip_add_dir
Module: U:\dev\php-5.3.3\ext\zip\lib\zip_error_clear.o(zip_error_clear.o)
0001:004c77b0  _zip_error_clear
Module: U:\dev\php-5.3.3\ext\zip\lib\zip_file_error_clear.o(zip_file_error_clear.o)
0001:004c77c0  _zip_file_error_clear
Module: U:\dev\php-5.3.3\ext\mysqlnd\mysqlnd.o(mysqlnd.o)
0002:000208d8  _mysqlnd_globals_id
0001:004c7938  __mysqlnd_restart_psession
0001:004c7950  __mysqlnd_end_psession
0001:004c7a23  _php_mysqlnd_conn_ssl_set_pub
0001:004c7e2d  _mysqlnd_get_client_info
0001:004c7e37  _mysqlnd_get_client_version
0001:004c7eeb  _mysqlnd_field_type_name
0001:004c7fce  __mysqlnd_init
0001:004c8084  _mysqlnd_connect
0001:004c815f  _mysqlnd_conn_get_methods
0001:004c8169  _mysqlnd_conn_set_methods
0001:004c8176  _mysqlnd_plugin_register
0001:004c8189  _mysqlnd_plugin_count
0001:004c8193  __mysqlnd_plugin_get_plugin_connection_data
0001:004c81b5  _mysqlnd_library_init
0001:004c9f38  _mysqlnd_library_end
0001:004ca31f  _php_mysqlnd_conn_list_fields_pub
0001:004cadfe  _php_mysqlnd_conn_list_method_pub
0001:004caf29  _mysqlnd_old_escape_string
0001:004ccd4f  _mysqlnd_stream_array_check_for_readiness
0001:004cceee  __mysqlnd_poll
0001:004cd14c  _mysqlnd_old_passwd
0001:004cd150  _mysqlnd_server_gone
0001:004cd154  _mysqlnd_out_of_sync
0001:004cd158  _mysqlnd_out_of_memory
0002:0001b1d0  _mysqlnd_global_stats
Module: U:\dev\php-5.3.3\ext\mysqlnd\mysqlnd_charset.o(mysqlnd_charset.o)
0001:004cd51a  _mysqlnd_find_charset_nr
0001:004ce200  _mysqlnd_charsets
0001:004cd53c  _mysqlnd_cset_escape_quotes
0001:004cd603  _mysqlnd_cset_escape_slashes
0001:004cd75e  _mysqlnd_find_charset_name
0001:004cf760  _mysqlnd_charsets60
Module: U:\dev\php-5.3.3\ext\mysqlnd\mysqlnd_wireprotocol.o(mysqlnd_wireprotocol.o)
0001:004d0a60  _php_mysqlnd_net_field_length
0001:004d0ac4  _php_mysqlnd_net_field_length_ll
0001:004d0b36  _php_mysqlnd_net_store_length
0001:004d109b  _mysqlnd_protocol_free
0001:004d10be  _mysqlnd_protocol_get_methods
0001:004d1830  _php_mysqlnd_cmd_write
0001:004d1ce0  __mysqlnd_plugin_get_plugin_protocol_data
0001:004d1d06  _mysqlnd_protocol_init
0001:004d1d5f  _php_mysqlnd_rowp_read_binary_protocol
0001:004d22ad  _php_mysqlnd_rowp_read_text_protocol
0001:004d291f  _php_mysqlnd_scramble
0001:004d65f0  _mysqlnd_empty_string
0001:004d6600  _mysqlnd_read_header_name
0001:004d6620  _mysqlnd_read_body_name
0001:004d6770  _mysqlnd_command_to_text
Module: U:\dev\php-5.3.3\ext\mysqlnd\mysqlnd_ps.o(mysqlnd_ps.o)
0001:004d6ad3  _php_mysqlnd_stmt_free_parameter_bind_pub
0001:004d6afd  _php_mysqlnd_stmt_free_result_bind_pub
0001:004d6b27  _mysqlnd_stmt_get_methods
0001:004d6b31  _mysqlnd_stmt_set_methods
0001:004d9502  _mysqlnd_fetch_stmt_row_cursor
0001:004dae22  _mysqlnd_fetch_stmt_row_buffered
0001:004dac45  __mysqlnd_init_ps_subsystem
0001:004dac5b  __mysqlnd_plugin_get_plugin_stmt_data
0001:004dac81  __mysqlnd_stmt_init
0001:004db140  _mysqlnd_not_bound_as_blob
0001:004db144  _mysqlnd_stmt_not_prepared
0002:00003630  _mysqlnd_mysqlnd_stmt_methods
Module: U:\dev\php-5.3.3\ext\mysqlnd\mysqlnd_loaddata.o(mysqlnd_loaddata.o)
0001:004db150  _mysqlnd_local_infile_default
0001:004db195  _mysqlnd_handle_local_infile
0001:004db3d1  _mysqlnd_set_local_infile_handler
Module: U:\dev\php-5.3.3\ext\mysqlnd\mysqlnd_net.o(mysqlnd_net.o)
0001:004dba69  _php_mysqlnd_net_consume_uneaten_data_pub
0001:004dbb59  _mysqlnd_net_get_methods
0001:004dc747  __mysqlnd_plugin_get_plugin_net_data
0001:004dc770  _mysqlnd_net_init
0001:004dc801  _mysqlnd_net_free
0001:004dc8a8  _php_mysqlnd_net_send_pub
Module: U:\dev\php-5.3.3\ext\mysqlnd\mysqlnd_ps_codec.o(mysqlnd_ps_codec.o)
0002:000208e8  _mysqlnd_ps_fetch_functions
0001:004dd030  __mysqlnd_init_ps_fetch_subsystem
0001:004dd4e9  _mysqlnd_stmt_execute_generate_request
0001:004de215  _ps_fetch_from_1_to_8_bytes
Module: U:\dev\php-5.3.3\ext\mysqlnd\mysqlnd_statistics.o(mysqlnd_statistics.o)
0001:004de740  _mysqlnd_stats_reset_triggers
0001:004de78a  _mysqlnd_stats_set_trigger
0001:004de7cb  _mysqlnd_stats_end
0001:004de802  _mysqlnd_stats_init
0001:004de870  _mysqlnd_fill_stats_hash
0001:004de938  __mysqlnd_get_client_stats
0001:004df730  _mysqlnd_stats_values_names
Module: U:\dev\php-5.3.3\ext\mysqlnd\mysqlnd_result.o(mysqlnd_result.o)
0001:004dff13  __mysqlnd_fetch_lengths
0001:004e0139  _mysqlnd_result_get_methods
0001:004e082f  _mysqlnd_palloc_zval_ptr_dtor
0001:004e280f  __mysqlnd_plugin_get_plugin_result_data
0001:004e2838  _mysqlnd_result_init
0001:004e289d  _php_mysqlnd_res_store_result_fetch_data_pub
0001:004e2f32  _mysqlnd_query_read_result_set_header
Module: U:\dev\php-5.3.3\ext\mysqlnd\mysqlnd_result_meta.o(mysqlnd_result_meta.o)
0001:004e3d47  _mysqlnd_result_metadata_get_methods
0001:004e3d51  __mysqlnd_plugin_get_plugin_result_metadata_data
0001:004e3d77  _mysqlnd_result_meta_init
Module: U:\dev\php-5.3.3\ext\mysqlnd\mysqlnd_debug.o(mysqlnd_debug.o)
0001:004e5688  _mysqlnd_get_backtrace
0001:004e6139  __mysqlnd_efree
0001:004e62bf  __mysqlnd_erealloc
0001:004e649e  __mysqlnd_emalloc
0001:004e665b  __mysqlnd_malloc
0001:004e6827  __mysqlnd_pemalloc
0001:004e6aa6  __mysqlnd_free
0001:004e6c2c  __mysqlnd_pefree
0001:004e6e53  __mysqlnd_realloc
0001:004e703e  __mysqlnd_perealloc
0001:004e72f5  __mysqlnd_calloc
0001:004e74bd  __mysqlnd_ecalloc
0001:004e76d7  __mysqlnd_pecalloc
0001:004e7953  _mysqlnd_debug_init
0001:004e79d0  __mysqlnd_debug
0001:004e7a42  __mysqlnd_pestrndup
0001:004e7c08  __mysqlnd_pestrdup
0002:00003810  _mysqlnd_mysqlnd_debug_methods
0002:000037d0  _mysqlnd_debug_std_no_trace_funcs
0002:00003830  _mysqlnd_allocator
Module: U:\dev\php-5.3.3\ext\mysqlnd\mysqlnd_block_alloc.o(mysqlnd_block_alloc.o)
0001:004e808c  _mysqlnd_mempool_destroy
0001:004e80bc  _mysqlnd_mempool_create
Module: U:\dev\php-5.3.3\ext\mysqlnd\php_mysqlnd.o(php_mysqlnd.o)
0001:004e8407  _mysqlnd_minfo_print_hash
0001:004e8566  _zm_info_mysqlnd
0002:00003870  _mysqlnd_module_entry
Module: U:\dev\php-5.3.3\TSRM\TSRM.o(TSRM.o)
0001:004e8d40  _tsrm_set_interpreter_context
0001:004e8d52  _tsrm_mutex_alloc
0001:004e8d59  _tsrm_mutex_unlock
0001:004e8d5e  _tsrm_set_new_thread_begin_handler
0001:004e8d71  _tsrm_set_new_thread_end_handler
0001:004e8d84  _tsrm_error_set
0001:004e8d91  _tsrm_mutex_lock
0001:004e8d9d  _tsrm_mutex_free
0001:004e8db2  _tsrm_thread_id
0001:004e8dc1  _ts_free_id
0001:004e8e8f  _ts_free_worker_threads
0001:004e8fab  _ts_free_thread
0001:004e90aa  _tsrm_free_interpreter_context
0001:004e924d  _tsrm_new_interpreter_context
0001:004e9290  _ts_resource_ex
0001:004e934b  _ts_allocate_id
0001:004e94f0  _tsrm_shutdown
0001:004e9664  _tsrm_startup
Module: U:\dev\php-5.3.3\TSRM\tsrm_strtok_r.o(tsrm_strtok_r.o)
0001:004e9750  _tsrm_strtok_r
Module: U:\dev\php-5.3.3\TSRM\tsrm_virtual_cwd.o(tsrm_virtual_cwd.o)
0002:000218e8  _cwd_globals_id
0002:000218f8  _cwd_mutex
0002:00021908  _main_cwd_state
0001:004e9800  _realpath_cache_size
0001:004e9817  _realpath_cache_max_buckets
0001:004e9821  _realpath_cache_get_buckets
0001:004e9838  _realpath
0001:004e98c4  _realpath_cache_clean
0001:004e994f  _virtual_getcwd_ex
0001:004e9a0d  _virtual_getcwd
0001:004e9af4  _virtual_chdir_file
0001:004ea5ba  _virtual_file_ex
0001:004eabdd  _tsrm_realpath
0001:004ead7c  _virtual_opendir
0001:004eae25  _virtual_rmdir
0001:004eaecd  _virtual_mkdir
0001:004eaf7c  _virtual_unlink
0001:004eb024  _virtual_lstat
0001:004eb0d3  _virtual_stat
0001:004eb182  _virtual_rename
0001:004eb2c9  _virtual_creat
0001:004eb378  _virtual_open
0001:004eb449  _virtual_chown
0001:004eb51f  _virtual_chmod
0001:004eb5ce  _virtual_utime
0001:004eb67d  _virtual_access
0001:004eb72c  _virtual_fopen
0001:004eb7eb  _virtual_filepath_ex
0001:004eb868  _virtual_filepath
0001:004eb891  _virtual_realpath
0001:004eba15  _virtual_chdir
0001:004eba52  _virtual_popen
0001:004ebae2  _realpath_cache_del
0001:004ebbc4  _virtual_cwd_shutdown
0001:004ebbe6  _virtual_cwd_startup
0001:004ebcd8  _realpath_cache_lookup
Module: U:\dev\php-5.3.3\main\main.o(main.o)
0002:00021918  _core_globals_id
0001:004ebdc1  _php_com_initialize
0001:004ebdc6  _php_module_shutdown_for_exec
0001:004ebdcb  _php_lint_script
0001:004ebe87  _php_handle_auth_data
0001:004ec00f  _php_handle_aborted_connection
0001:004ec081  _php_execute_simple_script
0001:004ec1eb  _php_execute_script
0001:004ec537  _php_module_shutdown
0001:004ec5bd  _php_module_shutdown_wrapper
0001:004ec5e3  _php_request_shutdown_for_exec
0001:004ec917  _php_write
0001:004eccb8  _php_register_extensions
0001:004ecd15  _zm_info_php_core
0001:004ecd52  _php_request_shutdown
0001:004ed26f  _php_request_shutdown_for_hook
0001:004ed62c  _php_request_startup_for_hook
0001:004ed682  _php_request_startup
0001:004ed951  _php_on_timeout
0001:004eda30  _php_stream_open_for_zend_ex
0001:004edb92  _php_html_puts
0001:004edb9e  _php_printf
0001:004edf96  _php_module_startup
0001:004eecc9  _php_verror
0001:004ef307  _php_error_docref2
0001:004ef380  _php_error_docref1
0001:004ef3b6  _php_error_docref0
0001:004ef71d  _zif_set_time_limit
0001:004ef834  _php_log_err
0002:000038d0  _php_register_internal_extensions_func
Module: U:\dev\php-5.3.3\main\snprintf.o(snprintf.o)
0001:004f2220  _ap_php_conv_10
0001:004f22bb  _ap_php_conv_p2
0001:004f231c  _ap_php_asprintf
0001:004f249e  _php_conv_fp
0001:004f3da7  _php_gcvt
0001:004f3cb7  _ap_php_vsnprintf
0001:004f3ce9  _ap_php_vasprintf
0001:004f3d6d  _ap_php_snprintf
0001:004f40a5  _ap_php_vslprintf
0001:004f40ea  _ap_php_slprintf
Module: U:\dev\php-5.3.3\main\spprintf.o(spprintf.o)
0001:004f57f1  _vspprintf
0001:004f5858  _spprintf
Module: U:\dev\php-5.3.3\main\php_sprintf.o(php_sprintf.o)
0001:004f5890  _php_sprintf
Module: U:\dev\php-5.3.3\main\safe_mode.o(safe_mode.o)
0001:004f58d1  _php_get_current_user
0001:004f5acb  _php_checkuid_ex
0001:004f5fe0  _php_checkuid
Module: U:\dev\php-5.3.3\main\fopen_wrappers.o(fopen_wrappers.o)
0001:004f6011  _php_strip_url_passwd
0001:004f60b6  _expand_filepath_ex
0001:004f62e5  _expand_filepath
0001:004f6316  _php_resolve_path
0001:004f68c3  _php_fopen_primary_script
0001:004f6dc5  _php_check_safe_mode_include_dir
0001:004f6ec7  _php_check_specific_open_basedir
0001:004f71f1  _php_check_open_basedir_ex
0001:004f72f0  _php_check_open_basedir
0001:004f73a7  _php_fopen_with_path
0001:004f7816  _OnUpdateBaseDir
Module: U:\dev\php-5.3.3\main\php_scandir.o(php_scandir.o)
0001:004f7910  _php_scandir
0001:004f7ab2  _php_alphasort
Module: U:\dev\php-5.3.3\main\php_ini.o(php_ini.o)
0001:004f7afd  _php_ini_has_per_dir_config
0001:004f7b07  _php_ini_has_per_host_config
0001:004f7b11  _php_ini_get_configuration_hash
0001:004f7b1b  _cfg_get_string
0001:004f7b6e  _cfg_get_entry
0001:004f7ba2  _cfg_get_double
0001:004f7c24  _cfg_get_long
0001:004f7ca8  _php_ini_activate_config
0001:004f7d6a  _php_ini_activate_per_host_config
0001:004f7dcf  _php_ini_activate_per_dir_config
0001:004f7e7b  _php_parse_user_ini_file
0001:004f7fd6  _php_ini_register_extensions
0001:004f806d  _php_shutdown_config
0001:004f80b9  _config_zval_dtor
0001:004f814a  _php_init_config
0001:004f8b86  _display_ini_entries
0002:0001b310  _php_ini_opened_path
0002:0001b318  _php_ini_scanned_files
0002:0001b314  _php_ini_scanned_path
Module: U:\dev\php-5.3.3\main\SAPI.o(SAPI.o)
0002:00021928  _sapi_globals_id
0002:00021938  _sapi_module
0001:004f94a0  _sapi_initialize_empty_request
0001:004f94e3  _sapi_flush
0001:004f9512  _sapi_get_fd
0001:004f9537  _sapi_force_http_10
0001:004f9556  _sapi_get_target_uid
0001:004f957b  _sapi_get_target_gid
0001:004f95a0  _sapi_terminate_process
0001:004f95b4  _sapi_get_request_time
0001:004f961c  _sapi_getenv
0001:004f96a0  _sapi_get_stat
0001:004f9703  _sapi_register_input_filter
0001:004f9760  _sapi_register_treat_data
0001:004f97b5  _sapi_register_default_post_reader
0001:004f980a  _sapi_unregister_post_entry
0001:004f9871  _sapi_register_post_entry
0001:004f98ed  _sapi_register_post_entries
0001:004f997e  _sapi_handle_post
0001:004f9a05  _sapi_free_header
0001:004f9a80  _sapi_apply_default_charset
0001:004f9d58  _sapi_header_op
0001:004fa750  _sapi_add_header_ex
0001:004fa7ac  _sapi_deactivate
0001:004fa9c8  _sapi_activate_headers_only
0001:004fab1c  _sapi_activate
0001:004fae70  _sapi_get_default_content_type
0001:004faf33  _sapi_get_default_content_type_header
0001:004fafc6  _sapi_send_headers
0001:004fb2e4  _sapi_read_standard_form_data
0001:004fb43a  _sapi_shutdown
0001:004fb446  _sapi_startup
Module: U:\dev\php-5.3.3\main\rfc1867.o(rfc1867.o)
0001:004fbd75  _destroy_uploaded_files_hash
0001:004fbe9a  _php_rfc1867_register_constants
0001:004fc40b  _rfc1867_post_handler
0002:0001b3d0  _php_rfc1867_callback
Module: U:\dev\php-5.3.3\main\php_content_types.o(php_content_types.o)
0001:004fddd0  _php_setup_sapi_content_types
0001:004fdded  _php_startup_sapi_content_types
0001:004fde3b  _php_default_post_reader
Module: U:\dev\php-5.3.3\main\mergesort.o(mergesort.o)
0001:004fe151  _php_mergesort
Module: U:\dev\php-5.3.3\main\php_variables.o(php_variables.o)
0001:004fe9d0  _php_default_input_filter
0001:004fe9ea  _php_std_auto_global_callback
0001:004fea38  _php_startup_auto_globals
0001:004ff6f4  _php_handle_special_queries
0001:004ff7f4  _php_register_variable_ex
0001:005002ac  _php_register_variable_safe
0001:00500330  _php_default_treat_data
0001:00500736  _php_std_post_handler
0001:0050085f  _php_register_variable
0001:005008a0  __php_import_environment_variables
0001:00500a44  _php_hash_environment
0002:00003970  _php_import_environment_variables
Module: U:\dev\php-5.3.3\main\php_ticks.o(php_ticks.o)
0001:00501820  _php_run_ticks
0001:0050189a  _php_remove_tick_function
0001:005018de  _php_add_tick_function
0001:0050191a  _php_shutdown_ticks
0001:0050193d  _php_deactivate_ticks
0001:00501960  _php_startup_ticks
Module: U:\dev\php-5.3.3\main\network.o(network.o)
0001:005019a0  _php_sockaddr_size
0001:005019c2  _php_any_addr
0001:00501b77  __php_emit_fd_setsize_warning
0001:00501bd7  _php_poll2
0001:00501e9a  _php_set_sock_blocking
0001:00501eeb  __php_stream_sock_open_host
0001:00501fc9  __php_stream_sock_open_from_socket
0001:005020c0  _php_socket_strerror
0001:0050227a  _php_network_populate_name_from_sockaddr
0001:00502393  _php_network_get_sock_name
0001:00502415  _php_network_get_peer_name
0001:005024b2  _php_network_parse_network_address_with_port
0001:00502676  _php_network_bind_socket_to_local_addr
0001:005027c6  _php_network_connect_socket
0001:005029fb  _php_network_connect_socket_to_host
0001:00502ce8  _php_network_accept_incoming
Module: U:\dev\php-5.3.3\main\php_open_temporary_file.o(php_open_temporary_file.o)
0001:00502e40  _php_shutdown_temporary_directory
0001:00502fd7  _php_get_temporary_directory
0001:0050305c  _php_open_temporary_fd_ex
0001:00503108  _php_open_temporary_fd
0001:0050313c  _php_open_temporary_file
Module: U:\dev\php-5.3.3\main\php_logos.o(php_logos.o)
0001:005031a0  _php_info_logos
0001:00503280  _php_shutdown_info_logos
0001:00503296  _php_unregister_info_logo
0001:005032da  _php_register_info_logo
0001:005033d4  _php_init_info_logos
Module: U:\dev\php-5.3.3\main\output.o(output.o)
0002:000219d8  _output_globals_id
0001:005080fe  _php_default_output_func
0001:00505dec  _php_output_activate
0001:0050654b  _php_ub_body_write
0001:00505e3c  _php_output_set_status
0001:00505e58  _php_body_write
0001:00505e72  _php_header_write
0001:00505ea9  _php_start_implicit_flush
0001:00505ec1  _php_end_implicit_flush
0001:00505ed9  _php_ob_get_length
0001:00505f06  _php_get_output_start_filename
0001:00505f1d  _php_get_output_start_lineno
0001:00505f37  _zif_ob_implicit_flush
0001:00505f9f  _zif_ob_get_length
0001:00505ffd  _zif_ob_get_level
0001:00506046  _zif_output_add_rewrite_var
0001:005060de  _zif_output_reset_rewrite_vars
0001:005062f7  _zif_ob_get_status
0001:005064c9  _php_ub_body_write_no_header
0001:0050665f  _php_ob_get_buffer
0001:005066a7  _zif_ob_get_contents
0001:00506752  _php_ob_handler_used
0001:00506803  _php_ob_init_conflict
0001:005068b7  _zif_ob_list_handlers
0001:0050694f  _php_end_ob_buffer
0001:00506f26  _zif_ob_get_clean
0001:00507051  _zif_ob_get_flush
0001:0050713a  _zif_ob_end_clean
0001:00507211  _zif_ob_end_flush
0001:005072e8  _zif_ob_clean
0001:00507407  _zif_ob_flush
0001:005074de  _php_end_ob_buffers
0001:00507ca1  _php_start_ob_buffer
0001:00507d83  _zif_ob_start
0001:00507e28  _php_ob_set_internal_handler
0001:00507f2c  _php_start_ob_buffer_named
0001:00508032  _php_output_register_constants
0001:005080d2  _php_output_startup
Module: U:\dev\php-5.3.3\main\getopt.o(getopt.o)
0001:0050828b  _php_getopt
0002:00003980  _php_optidx
Module: U:\dev\php-5.3.3\main\streams\streams.o(streams.o)
0001:00508710  _php_file_le_stream
0001:0050871a  _php_file_le_pstream
0001:00508724  _php_file_le_stream_filter
0001:0050872e  __php_stream_get_url_stream_wrappers_hash
0001:00508750  _php_stream_get_url_stream_wrappers_hash_global
0001:00508891  __php_stream_tell
0001:0050889f  __php_stream_set_option
0001:0050891d  __php_stream_eof
0001:00508996  __php_stream_truncate_set_size
0001:005089c7  _php_stream_notification_notify
0001:00508a08  _php_stream_dirent_alphasortr
0001:00508a24  _php_stream_dirent_alphasort
0001:00508a40  _php_unregister_url_stream_wrapper
0001:00508a81  _php_stream_context_del_link
0001:00508b8a  _php_stream_context_set_link
0001:00508c78  _php_register_url_stream_wrapper
0001:00508d22  _php_stream_context_get_link
0001:00508d87  _php_stream_context_get_option
0001:00508e00  _php_stream_context_set_option
0001:00508f90  _php_stream_notification_free
0001:00508fb3  _php_stream_tidy_wrapper_error_log
0001:0050900c  _php_stream_notification_alloc
0001:00509028  _php_stream_context_alloc
0001:005090a0  _php_stream_from_persistent_id
0001:00509136  _php_stream_context_free
0001:00509193  _php_stream_context_set
0001:005093cd  _php_stream_locate_url_wrapper
0001:00509889  __php_stream_stat_path
0001:00509a56  __php_stream_rmdir
0001:00509abc  __php_stream_mkdir
0001:00509bcb  _php_unregister_url_stream_wrapper_volatile
0001:00509c39  _php_register_url_stream_wrapper_volatile
0001:00509d14  _php_shutdown_stream_hashes
0001:00509da2  _php_shutdown_stream_wrappers
0001:00509e0a  _php_init_stream_wrappers
0001:0050a009  _php_stream_wrapper_log_error
0001:0050a0bd  __php_stream_stat
0001:0050a264  __php_stream_write
0001:0050a2d2  __php_stream_printf
0001:0050a334  __php_stream_puts
0001:0050a3b2  __php_stream_putc
0001:0050a3e9  __php_stream_flush
0001:0050a447  _php_stream_locate_eol
0001:0050a534  __php_stream_free
0001:0050a91b  _php_stream_display_wrapper_errors
0001:0050abcf  __php_stream_open_wrapper_ex
0001:0050b0e0  __php_stream_opendir
0001:0050b1d9  _zm_deactivate_streams
0001:0050b683  __php_stream_get_line
0001:0050b82f  __php_stream_read
0001:0050b955  __php_stream_readdir
0001:0050b994  __php_stream_scandir
0001:0050bad6  __php_stream_copy_to_stream_ex
0001:0050bd39  __php_stream_copy_to_stream
0001:0050bd87  __php_stream_passthru
0001:0050bec8  __php_stream_seek
0001:0050c2b5  __php_stream_getc
0001:0050c2ed  _php_stream_get_record
0001:0050c506  __php_stream_alloc
0001:0050c68d  __php_stream_copy_to_mem
Module: U:\dev\php-5.3.3\main\streams\cast.o(cast.o)
0001:0050c8f0  __php_stream_make_seekable
0001:0050ca9e  __php_stream_cast
0001:0050ce5e  __php_stream_open_wrapper_as_file
Module: U:\dev\php-5.3.3\main\streams\memory.o(memory.o)
0001:0050d04d  __php_stream_memory_get_buffer
0001:0050d6ad  __php_stream_memory_create
0001:0050d724  __php_stream_memory_open
0001:0050d79a  __php_stream_temp_create
0001:0050dee2  __php_stream_temp_open
0002:000039a0  _php_stream_memory_ops
0002:000039d0  _php_stream_temp_ops
0002:00003a00  _php_stream_rfc2397_ops
0002:00003a30  _php_stream_rfc2397_wops
0002:00003a60  _php_stream_rfc2397_wrapper
Module: U:\dev\php-5.3.3\main\streams\filter.o(filter.o)
0001:0050df80  _php_get_stream_filters_hash_global
0001:0050df8a  __php_get_stream_filters_hash
0001:0050dfac  _php_stream_bucket_prepend
0001:0050dfd8  _php_stream_bucket_append
0001:0050e003  _php_stream_bucket_unlink
0001:0050e050  _php_stream_filter_prepend_ex
0001:0050e081  __php_stream_filter_prepend
0001:0050e10c  _php_stream_filter_free
0001:0050e14c  _php_stream_filter_remove
0001:0050e1ba  _php_stream_bucket_delref
0001:0050e225  __php_stream_filter_flush
0001:0050e4df  _php_stream_filter_create
0001:0050e6ca  _php_stream_filter_register_factory_volatile
0001:0050e7c8  _php_stream_filter_register_factory
0001:0050e818  _php_stream_filter_unregister_factory
0001:0050e859  _php_stream_bucket_new
0001:0050e967  _php_stream_filter_append_ex
0001:0050ec9d  __php_stream_filter_append
0001:0050ece9  _php_stream_bucket_split
0001:0050f014  _php_stream_bucket_make_writeable
0001:0050f149  __php_stream_filter_alloc
Module: U:\dev\php-5.3.3\main\streams\plain_wrapper.o(plain_wrapper.o)
0001:00510072  _php_stream_parse_fopen_modes
0001:00510187  __php_stream_fopen_from_pipe
0001:005101fd  __php_stream_fopen_from_file
0001:0051038c  __php_stream_fopen_from_fd
0001:0051049b  __php_stream_fopen
0001:005107ef  __php_stream_fopen_with_path
0001:00510d7d  __php_stream_fopen_tmpfile
0001:00510e33  __php_stream_fopen_temporary_file
0002:00003a80  _php_stream_stdio_ops
0002:00003ab0  _php_plain_files_wrapper
Module: U:\dev\php-5.3.3\main\streams\userspace.o(userspace.o)
0001:005127b0  _zif_stream_wrapper_unregister
0001:005128c5  _zif_stream_wrapper_restore
0001:00512a98  _zif_stream_wrapper_register
0001:00514475  _zm_startup_user_streams
0002:00003b60  _php_stream_userspace_dir_ops
0002:00003b30  _php_stream_userspace_ops
Module: U:\dev\php-5.3.3\main\streams\transports.o(transports.o)
0001:00514800  _php_stream_xport_get_hash
0001:0051480a  _php_stream_xport_shutdown
0001:0051486b  _php_stream_xport_recvfrom
0001:00514922  _php_stream_xport_get_name
0001:005149c5  _php_stream_xport_accept
0001:00514a8f  _php_stream_xport_listen
0001:00514b05  _php_stream_xport_connect
0001:00514b9b  _php_stream_xport_bind
0001:00514c5a  _php_stream_xport_sendto
0001:00514d5f  _php_stream_xport_crypto_enable
0001:00514dea  _php_stream_xport_crypto_setup
0001:00514f54  __php_stream_xport_create
0001:005154ed  _php_stream_xport_unregister
0001:0051552e  _php_stream_xport_register
Module: U:\dev\php-5.3.3\main\streams\xp_socket.o(xp_socket.o)
0001:00515d73  _php_stream_generic_socket_factory
0002:00003bf0  _php_stream_socket_ops
0002:00003c20  _php_stream_udp_socket_ops
0002:00003c50  _php_stream_unix_socket_ops
0002:00003c80  _php_stream_unixdg_socket_ops
0002:00003bc0  _php_stream_generic_socket_ops
Module: U:\dev\php-5.3.3\main\streams\mmap.o(mmap.o)
0001:00516cd0  __php_stream_mmap_unmap
0001:00516d0a  __php_stream_mmap_unmap_ex
0001:00516d60  __php_stream_mmap_range
Module: U:\dev\php-5.3.3\main\streams\glob_wrapper.o(glob_wrapper.o)
0001:00516dd0  __php_glob_stream_get_count
0001:00516e99  __php_glob_stream_get_pattern
0001:00516ee5  __php_glob_stream_get_path
0002:00003cb0  _php_glob_stream_ops
0002:00003ce0  _php_glob_stream_wrapper
Module: U:\dev\php-5.3.3\main\internal_functions.o(internal_functions.o)
0001:005171f0  _php_register_internal_extensions
Module: U:\dev\php-5.3.3\Zend\zend_language_parser.o(zend_language_parser.o)
0001:005175c3  _zendparse
Module: U:\dev\php-5.3.3\Zend\zend_language_scanner.o(zend_language_scanner.o)
0002:000219e8  _language_scanner_globals_id
0001:00524a80  _zend_get_scanned_file_offset
0001:00524ff3  _lex_scan
0001:0052d639  _zend_prepare_string_for_scanning
0001:0052d74c  _open_file_for_scanning
0001:0052d901  _zend_destroy_file_handle
0001:0052d94d  _compile_filename
0001:0052db02  _shutdown_scanner
0001:0052db99  _zend_restore_lexical_state
0001:0052dc3a  _zend_save_lexical_state
0001:0052dcdb  _highlight_string
0001:0052dd94  _highlight_file
0001:0052de45  _compile_string
0001:0052e04f  _compile_file
0001:0052e226  _startup_scanner
Module: U:\dev\php-5.3.3\Zend\zend_ini_parser.o(zend_ini_parser.o)
0001:0052f045  _ini_parse
0001:0052fc43  _zend_parse_ini_string
0001:0052fccc  _zend_parse_ini_file
Module: U:\dev\php-5.3.3\Zend\zend_ini_scanner.o(zend_ini_scanner.o)
0002:000219f8  _ini_scanner_globals_id
0001:00530390  _zend_ini_scanner_get_lineno
0001:005303af  _zend_ini_scanner_get_filename
0001:005304ab  _ini_lex
0001:00536b96  _zend_ini_prepare_string_for_scanning
0001:00536bf9  _zend_ini_open_file_for_scanning
0001:00536c69  _shutdown_ini_scanner
Module: U:\dev\php-5.3.3\Zend\zend_alloc.o(zend_alloc.o)
0001:005374b5  _is_zend_mm
0001:005374cd  _zend_memory_usage
0001:00537503  _zend_memory_peak_usage
0001:00537536  _zend_mm_set_heap
0001:00537551  _zend_mm_get_storage
0001:0053755c  _zend_mm_set_custom_handlers
0001:0053757c  _start_memory_manager
0001:00537603  _zend_set_memory_limit
0001:00537747  __zend_mm_block_size
0001:00537759  __zend_mem_block_size
0001:00537786  _zend_strndup
0001:00537818  __safe_realloc
0001:005378a0  __safe_malloc
0001:00537b95  __efree
0001:00537be6  __zend_mm_free
0001:005387f9  __emalloc
0001:0053884a  __estrndup
0001:00538886  __estrdup
0001:005388c9  __safe_emalloc
0001:00538914  __ecalloc
0001:0053895e  __zend_mm_alloc
0001:0053896a  _zend_mm_shutdown
0001:00538aaa  _shutdown_memory_manager
0001:00538b50  _zend_mm_startup_ex
0001:00538e67  _zend_mm_startup
0001:0053978e  __erealloc
0001:005397e9  __safe_erealloc
0001:00539843  __zend_mm_realloc
Module: U:\dev\php-5.3.3\Zend\zend_compile.o(zend_compile.o)
0002:00021a08  _zend_compile_file
0002:00021a18  _zend_compile_string
0001:005398a0  _zend_auto_global_arm
0001:005398b3  _zend_restore_compiled_filename
0001:005398d0  _zend_get_compiled_filename
0001:005398ea  _zend_get_compiled_lineno
0001:00539904  _zend_is_compiling
0001:00539939  _zend_visibility_string
0001:00539964  _zend_do_declare_implicit_property
0001:00539969  _zend_get_compiled_variable_name
0001:005399a6  _zend_dirname
0001:00539a8e  _zend_verify_namespace
0001:00539b07  _zend_unmangle_property_name
0001:00539cae  _zend_do_verify_access_types
0001:00539e0d  _zend_check_writable_variable
0001:00539e5d  _zend_do_ticks
0001:00539ed7  _zend_do_extended_fcall_end
0001:00539f1d  _zend_do_extended_fcall_begin
0001:00539f63  _zend_do_extended_info
0001:00539fa9  _zend_do_end_silence
0001:0053a002  _zend_do_begin_silence
0001:0053a092  _zend_do_exit
0001:0053a1f5  _zend_do_include_or_eval
0001:0053a2ca  _zend_do_cast
0001:0053a37b  _zend_do_add_array_element
0001:0053a439  _zend_do_init_array
0001:0053a546  _zend_do_brk_cont
0001:0053a5e8  _zend_do_throw
0001:0053a6cc  _zend_do_clone
0001:0053a777  _zend_do_handle_exception
0001:0053a7b2  _zend_do_add_variable
0001:0053a8a6  _zend_do_add_string
0001:0053aaab  _zend_do_abstract_method
0001:0053ac03  _zend_do_echo
0001:0053ac5c  _zend_do_print
0001:0053ad07  _zend_do_unary_op
0001:0053adbb  _zend_do_binary_op
0001:0053b00c  _zend_is_auto_global
0001:0053b088  _zend_auto_global_disable_jit
0001:0053b12b  _zend_get_class_fetch_type
0001:0053b223  _do_bind_function
0001:0053b348  _zend_set_compiled_filename
0001:0053b42a  _zend_initialize_class_data
0001:0053b77d  _zend_auto_global_dtor
0001:0053b791  _zendlex
0001:0053b89b  _zend_register_auto_global
0001:0053b934  _zend_do_qm_false
0001:0053ba31  _zend_do_qm_true
0001:0053bb87  _zend_do_begin_qm_op
0001:0053bc46  _zend_do_jmp_set_else
0001:0053bd45  _zend_do_jmp_set
0001:0053be7e  _zend_do_instanceof
0001:0053bfed  _zend_do_unset
0001:0053c0c7  _zend_do_case_after_statement
0001:0053c17c  _zend_do_boolean_and_end
0001:0053c251  _zend_do_boolean_and_begin
0001:0053c341  _zend_do_boolean_or_end
0001:0053c416  _zend_do_boolean_or_begin
0001:0053c506  _zend_do_first_catch
0001:0053c531  _zend_do_if_cond
0001:0053c5cc  _zend_do_post_incdec
0001:0053c724  _zend_do_pre_incdec
0001:0053c88a  _zend_do_for_cond
0001:0053c920  _zend_do_assign_ref
0001:0053cb2d  _zend_do_binary_assign_op
0001:0053cd44  _zend_do_declare_end
0001:0053cdd4  _zend_do_default_before_statement
0001:0053cead  _zend_do_declare_begin
0001:0053cee1  _zend_do_begin_new_object
0001:0053cfb6  _zend_do_push_object
0001:0053cfe7  _zend_do_foreach_end
0001:0053d13f  _zend_do_pop_object
0001:0053d1ac  _zend_do_for_before_statement
0001:0053d292  _zend_do_if_end
0001:0053d34f  _zend_do_mark_last_catch
0001:0053d430  _zend_do_begin_variable_parse
0001:0053d483  _zend_do_new_list_end
0001:0053d4bd  _zend_do_new_list_begin
0001:0053d4ed  _zend_do_list_init
0001:0053d5ae  _zend_do_end_catch
0001:0053d66b  _zend_initialize_try_catch_element
0001:0053d773  _zend_do_if_after_statement
0001:0053d883  _zend_do_add_list_element
0001:0053d910  _zend_do_try
0001:0053d9bb  _zend_do_build_full_name
0001:0053daa8  _zend_do_shell_exec
0001:0053dc18  _zend_do_end_function_call
0001:0053ddf0  _zend_do_begin_dynamic_function_call
0001:0053e015  _zend_do_fetch_property
0001:0053e242  _fetch_array_dim
0001:0053e344  _fetch_string_offset
0001:0053e41f  _zend_do_declare_property
0001:0053e60a  _zend_mangle_property_name
0001:0053e6dd  _zend_do_halt_compiler_register
0001:0053e853  _zend_do_end_class_declaration
0001:0053eaa9  _do_bind_class
0001:0053ee28  _zend_do_end_variable_parse
0001:0053f1b5  _zend_do_foreach_begin
0001:0053f52b  _zend_do_isset_or_isempty
0001:0053f7ca  _zend_do_pass_param
0001:0053fc67  _zend_do_begin_method_call
0001:0053fe46  _fetch_simple_variable_ex
0001:00540093  _fetch_simple_variable
0001:005400c3  _fetch_array_begin
0001:00540108  _zend_do_indirect_references
0001:0054028d  _zend_do_assign
0001:0054180a  _function_add_ref
0001:005418a5  _zend_do_return
0001:00541abf  _zend_release_labels
0001:00541bb2  _zend_do_end_function_declaration
0001:00541d2d  _shutdown_compiler
0001:00541e27  _file_handle_dtor
0001:00541e52  _zend_init_compiler_data_structures
0001:00542023  _init_compiler
0001:0054212a  _zend_do_declare_class_constant
0001:005422aa  _zend_do_label
0001:00542449  _zend_do_fetch_global_variable
0001:005425aa  _zend_do_end_namespace
0001:0054269d  _zend_do_end_compilation
0001:00542717  _zend_resolve_goto_label
0001:005428c3  _zend_do_goto
0001:00542a43  _zend_do_case_before_statement
0001:00542c44  _zend_do_declare_stmt
0001:00542d85  _zend_do_inherit_interfaces
0001:00542f86  _zend_do_implement_interface
0001:005432c1  _zend_do_inheritance
0001:00543999  _do_bind_inherited_class
0001:00543ab5  _zend_do_delayed_early_binding
0001:00543ca5  _zend_do_begin_namespace
0001:005440c2  _zend_do_build_namespace_name
0001:0054420f  _zend_do_declare_constant
0001:00544494  _zend_do_begin_class_declaration
0001:00544915  _zend_resolve_non_class_name
0001:00544b82  _zend_do_begin_function_call
0001:00545003  _zend_do_begin_function_declaration
0001:00545e3c  _zend_do_begin_lambda_function_declaration
0001:00545f5b  _zend_do_free
0001:00546098  _zend_do_end_new_object
0001:00546166  _zend_do_fetch_static_variable
0001:00546445  _zend_do_fetch_lexical_variable
0001:005464d9  _zend_do_list_end
0001:005467df  _zend_do_switch_end
0001:005469ca  _zend_do_early_binding
0001:00546d1d  _zend_do_while_cond
0001:00546e69  _zend_do_foreach_cont
0001:005471ae  _zend_do_switch_cond
0001:0054727a  _zend_do_do_while_begin
0001:005472f2  _zend_do_do_while_end
0001:005473bb  _zend_do_for_end
0001:005474a8  _zend_do_while_end
0001:0054763c  _zend_do_use
0001:00547b67  _zend_resolve_class_name
0001:00547f20  _zend_do_implements_interface
0001:0054805b  _zend_do_fetch_class
0001:00548247  _zend_do_begin_catch
0001:00548384  _zend_do_fetch_static_member
0001:00548634  _zend_do_fetch_constant
0001:00548a87  _zend_do_receive_arg
0001:00548e8a  _zend_do_begin_class_member_function_call
0001:0054906b  _zend_do_add_static_array_element
Module: U:\dev\php-5.3.3\Zend\zend_constants.o(zend_constants.o)
0001:00549594  _zend_register_constant
0001:005496f6  _free_zend_constant
0001:00549734  _zend_get_constant
0001:00549a26  _zend_get_constant_ex
0001:00549f2d  _zend_register_stringl_constant
0001:00549f83  _zend_register_string_constant
0001:00549fd2  _zend_register_double_constant
0001:0054a022  _zend_register_long_constant
0001:0054a171  _zend_register_standard_constants
0001:0054a59d  _copy_zend_constant
0001:0054a5de  _clean_non_persistent_constants
0001:0054a634  _zend_shutdown_constants
0001:0054a67a  _zend_startup_constants
0001:0054a6f0  _clean_module_constants
0001:0054a728  _zend_copy_constants
Module: U:\dev\php-5.3.3\Zend\zend_dynamic_array.o(zend_dynamic_array.o)
0001:0054a760  _zend_dynamic_array_pop
0001:0054a779  _zend_dynamic_array_get_element
0001:0054a793  _zend_dynamic_array_push
0001:0054a7e1  _zend_dynamic_array_init
Module: U:\dev\php-5.3.3\Zend\zend_execute_API.o(zend_execute_API.o)
0002:00021a28  _zend_execute
0002:00021a38  _zend_execute_internal
0001:0054a8b9  _get_active_class_name
0001:0054a924  _get_active_function_name
0001:0054a97b  _zend_get_executed_filename
0001:0054a9a1  _zend_get_executed_lineno
0001:0054a9fc  _zend_is_executing
0001:0054aa69  _zend_reset_all_cv
0001:0054ab20  _zend_rebuild_symbol_table
0001:0054b490  __zval_ptr_dtor
0001:0054ada1  _zend_verify_abstract_class
0001:0054aff2  _zend_unset_timeout
0001:0054b07b  _zend_timeout
0001:0054b0ff  _zend_set_timeout
0001:0054b1c7  _execute_new_code
0001:0054b44b  __zval_internal_ptr_dtor
0001:0054b5e1  _zend_is_true
0001:0054b71b  _shutdown_executor
0001:0054bcec  _shutdown_destructors
0001:0054be10  _init_executor
0001:0054c229  _zend_eval_stringl
0001:0054c520  _zend_eval_stringl_ex
0001:0054c58c  _zend_eval_string_ex
0001:0054c5d4  _zend_eval_string
0001:0054c6a8  _zval_update_constant_ex
0001:0054d187  _zval_update_constant_inline_change
0001:0054d135  _zval_update_constant
0001:0054d15e  _zval_update_constant_no_inline_change
0001:0054d1b0  _zend_delete_global_variable
0001:0054d55f  _zend_call_function
0001:0054e346  _zend_lookup_class_ex
0001:0054ea0b  _zend_fetch_class
0001:0054ec18  _zend_lookup_class
0001:0054ec48  _call_user_function_ex
0001:0054eca9  _call_user_function
0001:0054ede0  _empty_fcall_info
0001:0054ee10  _empty_fcall_info_cache
Module: U:\dev\php-5.3.3\Zend\zend_highlight.o(zend_highlight.o)
0001:0054ee77  _zend_html_putc
0001:0054f00e  _zend_html_puts
0001:0054f05b  _zend_strip
0001:0054f207  _zend_highlight
Module: U:\dev\php-5.3.3\Zend\zend_llist.o(zend_llist.o)
0001:0054f400  _zend_llist_init
0001:0054f42e  _zend_llist_apply
0001:0054f460  _zend_llist_apply_with_argument
0001:0054f497  _zend_llist_count
0001:0054f4a2  _zend_llist_get_first_ex
0001:0054f4c3  _zend_llist_get_last_ex
0001:0054f4e5  _zend_llist_get_next_ex
0001:0054f50e  _zend_llist_get_prev_ex
0001:0054f538  _zend_llist_apply_with_arguments
0001:0054f576  _zend_llist_sort
0001:0054f635  _zend_llist_apply_with_del
0001:0054f6bb  _zend_llist_remove_tail
0001:0054f722  _zend_llist_destroy
0001:0054f778  _zend_llist_clean
0001:0054f79d  _zend_llist_del_element
0001:0054f83d  _zend_llist_add_element
0001:0054f8df  _zend_llist_copy
0001:0054f936  _zend_llist_prepend_element
Module: U:\dev\php-5.3.3\Zend\zend_opcode.o(zend_opcode.o)
0001:0054fa16  _zend_class_add_ref
0001:0054fa24  _get_next_op_number
0001:0054fa4a  _get_unary_op
0001:0054fa65  _get_binary_op
0001:0054fa9c  _print_class
0001:0054fb2f  _pass_two
0001:0054faee  _get_next_brk_cont_element
0001:0054fd56  _init_op
0001:0054fe10  _get_next_op
0001:0054feae  _destroy_op_array
0001:00550068  _destroy_zend_function
0001:0055007e  _destroy_zend_class
0001:005501b0  _zend_cleanup_class_data
0001:00550285  _zend_cleanup_function_data_full
0001:005502aa  _zend_cleanup_function_data
0001:005502d4  _zend_function_dtor
0001:005502ff  _init_op_array
Module: U:\dev\php-5.3.3\Zend\zend_operators.o(zend_operators.o)
0001:00550540  _instanceof_function
0001:00550569  _instanceof_function_ex
0001:005505f3  _zend_str_tolower_copy
0001:00550631  _zend_str_tolower
0001:00550655  _zend_binary_strcasecmp
0001:005506a2  _zend_binary_strncasecmp
0001:00550718  _zend_binary_zval_strcasecmp
0001:00550744  _zend_binary_zval_strncasecmp
0001:00550779  _zend_compare_objects
0001:005507d6  _zend_locale_sprintf_double
0001:00550831  _zend_compare_symbol_tables
0001:00550870  _zend_compare_arrays
0001:00550889  _zend_compare_symbol_tables_i
0001:00550ce5  _zend_binary_strncmp
0001:00550d44  _zend_binary_zval_strncmp
0001:00550d79  _zend_binary_strcmp
0001:00550daf  _zend_binary_zval_strcmp
0001:00550ddb  _is_identical_function
0001:00550edc  _is_not_identical_function
0001:00550f73  _zend_str_tolower_dup
0001:00550fc2  _decrement_function
0001:005510dc  _bitwise_not_function
0001:00551214  _add_string_to_string
0001:0055127c  _add_char_to_string
0001:005513f3  _convert_to_object
0001:00551470  _zend_string_to_double
0001:005515b7  _zend_atol
0001:005516c5  _zend_atoi
0001:005517d1  _convert_to_null
0001:00551949  _string_compare_function
0001:00551a0d  _string_locale_compare_function
0001:00551ae8  _concat_function
0001:00551cec  _convert_to_array
0001:00551fb7  _convert_to_double
0001:0055221c  _numeric_compare_function
0001:005522c3  _multi_convert_to_double_ex
0001:005523c0  _convert_to_long_base
0001:0055266b  _convert_to_long
0001:0055268c  _multi_convert_to_long_ex
0001:00552735  _bitwise_xor_function
0001:00552aab  _bitwise_and_function
0001:00552e1e  _bitwise_or_function
0001:005531d2  _mod_function
0001:00553557  __convert_to_string
0001:00553879  _multi_convert_to_string_ex
0001:0055392b  _convert_to_boolean
0001:00553b5d  _zval_is_true
0001:00553b7d  _boolean_xor_function
0001:00553dc5  _boolean_not_function
0001:00553ef5  _shift_right_function
0001:005541c1  _shift_left_function
0001:0055448d  _zendi_smart_strcmp
0001:00554b0d  _increment_function
0001:00554fa9  _convert_scalar_to_number
0001:005552a5  _compare_function
0001:00556050  _is_smaller_or_equal_function
0001:00556099  _is_smaller_function
0001:005560db  _is_not_equal_function
0001:00556124  _is_equal_function
0001:0055616d  _div_function
0001:00556535  _mul_function
0001:00556861  _sub_function
0001:00556b78  _add_function
Module: U:\dev\php-5.3.3\Zend\zend_ptr_stack.o(zend_ptr_stack.o)
0001:00556f50  _zend_ptr_stack_apply
0001:00556f84  _zend_ptr_stack_num_elements
0001:00556f8e  _zend_ptr_stack_clean
0001:00556fff  _zend_ptr_stack_destroy
0001:00557029  _zend_ptr_stack_n_pop
0001:0055707e  _zend_ptr_stack_n_push
0001:00557150  _zend_ptr_stack_init_ex
0001:005571db  _zend_ptr_stack_init
Module: U:\dev\php-5.3.3\Zend\zend_stack.o(zend_stack.o)
0001:00557200  _zend_stack_top
0001:00557229  _zend_stack_int_top
0001:0055724b  _zend_stack_is_empty
0001:0055725d  _zend_stack_base
0001:00557268  _zend_stack_count
0001:00557272  _zend_stack_apply
0001:005572fc  _zend_stack_apply_with_argument
0001:00557390  _zend_stack_destroy
0001:005573dc  _zend_stack_del_top
0001:00557402  _zend_stack_init
0001:0055743b  _zend_stack_push
Module: U:\dev\php-5.3.3\Zend\zend_variables.o(zend_variables.o)
0001:005574d0  _zval_add_ref
0001:005574de  _zend_print_variable
0001:005574f9  __zval_copy_ctor_func
0001:0055766a  __zval_internal_dtor
0001:005576c5  __zval_dtor_func
0001:005577a8  __zval_dtor_wrapper
Module: U:\dev\php-5.3.3\Zend\zend.o(zend.o)
0002:00021a48  _zend_uv
0002:00021a58  _executor_globals_id
0002:00021a68  _compiler_globals_id
0002:00021a78  _zval_used_for_init
0002:00021a88  _zend_vspprintf
0002:00021a98  _zend_error_cb
0002:00021aa8  _zend_printf
0002:00021ab8  _zend_write
0002:00021ac8  _zend_fopen
0002:00021ad8  _zend_stream_open_function
0002:00021ae8  _zend_block_interruptions
0002:00021af8  _zend_unblock_interruptions
0002:00021b08  _zend_ticks_function
0002:00021b18  _zend_on_timeout
0002:00021b28  _zend_getenv
0002:00021b38  _zend_resolve_path
0001:00557800  _get_zend_version
0001:00557820  _zend_message_dispatcher
0001:0055783d  _zend_get_configuration_directive
0001:00557871  _zend_output_debug_string
0001:00557876  _free_estring
0001:0055789e  _zend_make_compiled_string_description
0001:00557925  _zend_set_utility_values
0001:0055795c  _zend_execute_scripts
0001:00557c97  _zend_error
0001:00558300  _zenderror
0001:00558323  _zend_activate_modules
0001:00558346  _zend_post_deactivate_modules
0001:00558386  _zend_deactivate_modules
0001:00558400  _zend_deactivate
0001:0055858c  _zend_call_destructors
0001:005585ec  _zend_activate
0001:00558637  _zend_append_version_info
0001:005586f2  __zend_bailout
0001:00558820  _zend_shutdown
0001:00558cf5  _zend_post_startup
0001:00558e4c  _zend_register_standard_ini_entries
0001:00558f6b  _zend_startup
0001:00559473  _zend_print_flat_zval_r
0001:0055977c  _zend_make_printable_zval
0001:00559a6d  _zend_print_zval_ex
0001:00559aff  _zend_print_zval_r_ex
0001:00559fb6  _zend_print_zval_r
0001:00559fe0  _zend_print_zval
0001:00557c97  _zend_error_noreturn
0002:0001b4f0  _zend_standard_class_def
Module: U:\dev\php-5.3.3\Zend\zend_API.o(zend_API.o)
0002:00021b48  _module_registry
0001:0055a0f0  __zend_get_parameters_array_ex
0001:0055a144  _zend_get_type_by_const
0001:0055a15d  _zend_zval_type_name
0001:0055a17a  _module_registry_cleanup
0001:0055a1a5  _module_registry_unload_temp
0001:0055a1ba  _zend_next_free_module
0001:0055a1cc  _zend_fcall_info_args_save
0001:0055a1f2  _zend_save_error_handling
0001:0055a22b  _zend_restore_error_handling
0001:0055a2cb  _zend_replace_error_handling
0001:0055a39d  _zend_read_static_property
0001:0055a434  _add_assoc_function
0001:0055a48e  _zend_get_class_entry
0001:0055a4bc  _zend_get_object_classname
0001:0055a54b  _zend_read_property
0001:0055a68a  _zend_update_property
0001:0055a787  _zend_update_property_double
0001:0055a7f6  _zend_update_property_long
0001:0055a865  _zend_update_property_bool
0001:0055a8dc  _zend_update_property_null
0001:0055a931  _zend_update_property_stringl
0001:0055a9c0  _add_property_zval_ex
0001:0055aa3e  _add_property_stringl_ex
0001:0055ab1f  _add_property_double_ex
0001:0055abd8  _add_property_resource_ex
0001:0055ac8b  _add_property_null_ex
0001:0055ad39  _add_property_bool_ex
0001:0055adf2  _add_property_long_ex
0001:0055af38  _zend_update_property_string
0001:0055afd4  _add_property_string_ex
0001:0055b0c3  _zend_declare_class_constant
0001:0055b10b  _zend_declare_class_constant_stringl
0001:0055b1cb  _zend_declare_class_constant_string
0001:0055b213  _zend_declare_class_constant_double
0001:0055b29c  _zend_declare_class_constant_bool
0001:0055b330  _zend_declare_class_constant_long
0001:0055b3b9  _zend_declare_class_constant_null
0001:0055b426  _zend_unregister_functions
0001:0055b4cb  _zend_fcall_info_args_clear
0001:0055b4ff  _zend_fcall_info_args_restore
0001:0055b564  _zend_declare_property_ex
0001:0055b895  _zend_declare_property
0001:0055b8db  _zend_declare_property_stringl
0001:0055b9a7  _zend_declare_property_string
0001:0055ba83  _zend_declare_property_double
0001:0055bb1e  _zend_declare_property_long
0001:0055bbb3  _zend_declare_property_bool
0001:0055bc50  _zend_declare_property_null
0001:0055bcd8  _zend_register_class_alias_ex
0001:0055bd5b  _zend_get_module_version
0001:0055bdc9  _zend_get_module_started
0001:0055be16  _zend_fcall_info_argv
0001:0055be94  _zend_fcall_info_argn
0001:0055bec2  _zend_fcall_info_argp
0001:0055bf3f  _zend_fcall_info_args
0001:0055bfee  _zend_fcall_info_call
0001:0055d323  _zend_is_callable_ex
0001:0055d9bb  _zend_fcall_info_init
0001:0055da6d  _zend_is_callable
0001:0055db77  __array_init
0001:0055dbc2  _zif_display_disabled_function
0001:0055dbea  _zend_set_hash_symbol
0001:0055ddd2  _zend_check_magic_method_implementation
0001:0055e20d  _zend_class_implements
0001:0055e273  _module_registry_request_startup
0001:0055e2cf  _zend_get_parameters_ex
0001:0055e33b  _module_destructor
0001:0055e5c3  _zend_register_functions
0001:0055f321  _zend_disable_function
0001:0055f4dc  _zend_register_internal_interface
0001:0055f4fe  _zend_register_internal_class
0001:0055f520  _zend_disable_class
0001:0055f680  _zend_register_internal_class_ex
0001:0055f7ad  _zend_register_module_ex
0001:0055f9b7  _zend_register_internal_module
0001:0055f9df  _zend_startup_modules
0001:0055fb65  _zend_startup_module_ex
0001:0055fd22  _zend_startup_module
0001:0055fd73  _add_get_index_stringl
0001:0055fe02  _add_get_index_string
0001:0055fe9e  _add_get_index_double
0001:0055ff08  _add_get_index_long
0001:0055ff6c  _add_next_index_zval
0001:0055ffa8  _zend_copy_parameters_array
0001:0056000d  _add_next_index_stringl
0001:0056009e  _add_next_index_string
0001:0056013e  _zend_make_callable
0001:00560236  _add_next_index_double
0001:005602a2  _add_next_index_resource
0001:00560308  _add_next_index_bool
0001:00560374  _add_next_index_null
0001:005603d5  _add_next_index_long
0001:0056043b  _add_index_zval
0001:00560476  _add_index_stringl
0001:00560506  _add_index_string
0001:005605a5  _add_index_double
0001:00560610  _add_index_resource
0001:00560675  _add_index_bool
0001:005606e0  _add_index_null
0001:00560740  _add_index_long
0001:005607a5  _zend_merge_properties
0001:0056087b  _zend_wrong_param_count
0001:00560c68  _add_get_assoc_stringl_ex
0001:00560dea  _zend_update_class_constants
0001:005612c7  __object_and_properties_init
0001:005613eb  __object_init_ex
0001:00561414  __object_init
0001:00561437  __zend_get_parameters_array
0001:00561500  _zend_get_parameters
0001:005615e7  _zend_update_static_property
0001:0056173a  _zend_update_static_property_stringl
0001:005617bd  _zend_update_static_property_string
0001:0056184d  _zend_update_static_property_double
0001:005618b0  _zend_update_static_property_long
0001:00561913  _zend_update_static_property_bool
0001:0056197e  _zend_update_static_property_null
0001:005630c5  _zend_parse_method_parameters_ex
0001:00563277  _zend_parse_method_parameters
0001:005633f2  _zend_parse_parameters
0001:00563481  _zend_parse_parameters_ex
0001:00563514  _add_assoc_long_ex
0001:00563672  _add_assoc_null_ex
0001:005637c9  _add_assoc_bool_ex
0001:00563929  _add_assoc_resource_ex
0001:00563a82  _add_assoc_double_ex
0001:00563be2  _add_assoc_string_ex
0001:00563d5e  _add_assoc_stringl_ex
0001:00563ee2  _add_assoc_zval_ex
0001:0056401a  _add_get_assoc_string_ex
Module: U:\dev\php-5.3.3\Zend\zend_extensions.o(zend_extensions.o)
0002:00021b78  _zend_extensions
0001:0056426e  _zend_get_resource_handle
0001:005642ac  _zend_os2_module_error
0001:0056445f  _zend_os2_query_symbol
0001:00564493  _zend_os2_load_module
0001:005644cd  _zend_get_extension
0001:00564517  _zend_extension_dispatch_message
0001:00564561  _zend_extension_dtor
0001:0056457c  _zend_shutdown_extensions
0001:005645aa  _zend_startup_extensions
0001:00564601  _zend_startup_extensions_mechanism
0001:00564639  _zend_register_extension
0001:0056488b  _zend_load_extension
Module: U:\dev\php-5.3.3\Zend\zend_hash.o(zend_hash.o)
0001:00564ac0  _zend_hash_set_apply_protection
0001:00564ace  _zend_hash_index_find
0001:00564b0b  _zend_hash_index_exists
0001:00564b45  _zend_hash_num_elements
0001:00564b50  _zend_hash_get_pointer
0001:00564b79  _zend_hash_set_pointer
0001:00564bd1  _zend_hash_internal_pointer_reset_ex
0001:00564bed  _zend_hash_internal_pointer_end_ex
0001:00564c09  _zend_hash_move_forward_ex
0001:00564c2f  _zend_hash_move_backwards_ex
0001:00564c55  _zend_hash_get_current_key_type_ex
0001:00564c7f  _zend_hash_get_current_data_ex
0001:00564ca8  _zend_hash_minmax
0001:00564d4a  _zend_hash_next_free_element
0001:00564d55  _zend_hash_quick_exists
0001:00564de0  _zend_hash_quick_find
0001:00564eab  _zend_hash_compare
0001:005652d7  _zend_hash_reverse_apply
0001:0056536c  _zend_hash_apply_with_argument
0001:005653f5  _zend_hash_apply
0001:00565477  _zend_hash_graceful_reverse_destroy
0001:005654c1  _zend_hash_graceful_destroy
0001:00565508  _zend_hash_destroy
0001:005655f2  _zend_hash_get_current_key_ex
0001:00565674  _zend_hash_apply_with_arguments
0001:0056572f  _zend_hash_clean
0001:005657e4  _zend_hash_rehash
0001:00565845  _zend_hash_sort
0001:00565ac4  __zend_hash_init
0001:00565bae  __zend_hash_init_ex
0001:00565bed  _zend_hash_func
0001:00565d42  _zend_get_hash_value
0001:00565e96  _zend_hash_exists
0001:0056603a  _zend_hash_find
0001:005661e9  __zend_hash_index_update_or_next_insert
0001:005665b9  __zend_hash_quick_add_or_update
0001:005669ad  _zend_hash_merge_ex
0001:00566a66  __zend_hash_merge
0001:00566b65  _zend_hash_copy
0001:00566c45  __zend_hash_add_or_update
0001:00567139  _zend_hash_add_empty_element
0001:00567180  _zend_hash_del_key_or_index
0001:00567455  _zend_hash_update_current_key_ex
Module: U:\dev\php-5.3.3\Zend\zend_list.o(zend_list.o)
0002:00021b98  _le_index_ptr
0001:00567ce6  __zend_list_addref
0001:00567d2c  __zend_list_find
0001:00567d82  _zend_rsrc_list_get_rsrc_type
0001:00567dcf  _zend_destroy_rsrc_list_dtors
0001:00567de3  _zend_init_rsrc_list_dtors
0001:00567e21  _zend_init_rsrc_list
0001:005681f9  _list_entry_destructor
0001:00567e8d  _zend_fetch_list_dtor_id
0001:00567f08  _zend_register_list_destructors_ex
0001:00567f89  _zend_register_list_destructors
0001:0056800b  _zend_clean_module_rsrc_dtors
0001:0056808e  _zend_destroy_rsrc_list
0001:0056809a  _zend_init_rsrc_plist
0001:00568123  _plist_entry_destructor
0001:00568357  _zend_fetch_resource
0001:00568552  __zend_list_delete
0001:005685e4  _zend_list_insert
0001:00568675  _zend_register_resource
Module: U:\dev\php-5.3.3\Zend\zend_indent.o(zend_indent.o)
0001:0056872d  _zend_indent
Module: U:\dev\php-5.3.3\Zend\zend_builtin_functions.o(zend_builtin_functions.o)
0001:0056b1a8  _debug_print_backtrace_args
0001:0056b22a  _zend_startup_builtin_functions
0001:0056b27b  _zm_startup_core
0001:0056b8b8  _zend_fetch_debug_backtrace
0002:00003e10  _zend_builtin_module
Module: U:\dev\php-5.3.3\Zend\zend_sprintf.o(zend_sprintf.o)
0001:0056e370  _zend_sprintf
Module: U:\dev\php-5.3.3\Zend\zend_ini.o(zend_ini.o)
0001:0056e40f  _OnUpdateStringUnempty
0001:0056e44e  _OnUpdateString
0001:0056e476  _OnUpdateReal
0001:0056e4b5  _OnUpdateLongGEZero
0001:0056e4fe  _OnUpdateLong
0001:0056e548  _OnUpdateBool
0001:0056e5ef  _display_link_numbers
0001:0056e65e  _zend_ini_boolean_displayer_cb
0001:0056e76f  _zend_ini_color_displayer_cb
0001:0056e803  _zend_ini_string_ex
0001:0056e88f  _zend_ini_string
0001:0056e8d1  _zend_ini_double
0001:0056e956  _zend_ini_register_displayer
0001:0056e997  _zend_ini_long
0001:0056eb3b  _zend_restore_ini_entry
0001:0056ec4b  _zend_alter_ini_entry_ex
0001:0056ee65  _zend_alter_ini_entry
0001:0056eebb  _zend_ini_refresh_caches
0001:0056eef3  _zend_unregister_ini_entries
0001:0056ef1e  _zend_register_ini_entries
0001:0056f086  _zend_ini_sort_entries
0001:0056f117  _zend_ini_startup
0001:0056f18b  _zend_copy_ini_directives
0001:0056f253  _zend_ini_deactivate
0001:0056f2d9  _zend_ini_global_shutdown
0001:0056f2fd  _zend_ini_shutdown
Module: U:\dev\php-5.3.3\Zend\zend_qsort.o(zend_qsort.o)
0001:0056f350  _zend_qsort
Module: U:\dev\php-5.3.3\Zend\zend_ts_hash.o(zend_ts_hash.o)
0001:0056f770  _zend_ts_hash_rehash
0001:0056f82f  _zend_ts_hash_num_elements
0001:0056f85d  _zend_ts_hash_minmax
0001:0056f8a7  _zend_ts_hash_compare
0001:0056f90b  _zend_ts_hash_sort
0001:0056f95b  _zend_ts_hash_merge_ex
0001:0056f9d1  _zend_ts_hash_merge
0001:0056fa47  _zend_ts_hash_copy_to_hash
0001:0056fa9a  _zend_ts_hash_copy
0001:0056fb03  _zend_ts_hash_index_exists
0001:0056fb38  _zend_ts_hash_exists
0001:0056fb74  _zend_ts_hash_index_find
0001:0056fbb0  _zend_ts_hash_quick_find
0001:0056fbfa  _zend_ts_hash_find
0001:0056fc3d  _zend_ts_get_hash_value
0001:0056fc75  _zend_ts_hash_del_key_or_index
0001:0056fcc5  _zend_ts_hash_reverse_apply
0001:0056fd04  _zend_ts_hash_apply_with_arguments
0001:0056fd50  _zend_ts_hash_apply_with_argument
0001:0056fd9c  _zend_ts_hash_apply
0001:0056fddb  _zend_ts_hash_graceful_destroy
0001:0056fe1e  _zend_ts_hash_add_empty_element
0001:0056fe60  __zend_ts_hash_index_update_or_next_insert
0001:0056feb7  __zend_ts_hash_quick_add_or_update
0001:0056ff1c  __zend_ts_hash_add_or_update
0001:0056ff7a  _zend_ts_hash_clean
0001:0056ffae  _zend_ts_hash_destroy
0001:0056fff1  __zend_ts_hash_init_ex
0001:00570057  __zend_ts_hash_init
Module: U:\dev\php-5.3.3\Zend\zend_stream.o(zend_stream.o)
0001:00570150  _zend_compare_file_handles
0001:005701e3  _zend_file_handle_dtor
0001:005702c1  _zend_stream_open
0001:00570332  _zend_stream_fixup
Module: U:\dev\php-5.3.3\Zend\zend_iterators.o(zend_iterators.o)
0001:00570717  _zend_iterator_unwrap
0001:00570778  _zend_iterator_wrap
0001:005707f1  _zend_register_iterator_wrapper
Module: U:\dev\php-5.3.3\Zend\zend_interfaces.o(zend_interfaces.o)
0002:00021ba8  _zend_ce_traversable
0002:00021bb8  _zend_ce_aggregate
0002:00021bc8  _zend_ce_iterator
0002:00021bd8  _zend_ce_arrayaccess
0002:00021be8  _zend_ce_serializable
0001:00570927  _zend_user_it_invalidate_current
0001:005709c7  _zend_register_interfaces
0001:005720b0  _zend_funcs_aggregate
0001:005720e0  _zend_funcs_iterator
0001:00572190  _zend_funcs_arrayaccess
0001:00572200  _zend_funcs_serializable
0001:005718a1  _zend_user_serialize
0001:00571787  _zend_user_unserialize
0001:00571f9a  _zend_user_it_get_new_iterator
0001:0057133f  _zend_class_unserialize_deny
0001:005713a1  _zend_class_serialize_deny
0001:0057143f  _zend_call_method
0001:005719b6  _zend_user_it_rewind
0001:00571a31  _zend_user_it_move_forward
0001:00571af1  _zend_user_it_get_current_key
0001:00571c9d  _zend_user_it_get_current_data
0001:00571d21  _zend_user_it_valid
0001:00571ee3  _zend_user_it_new_iterator
0002:00003ee0  _zend_interface_iterator_funcs_iterator
0002:0001bc90  _zend_funcs_traversable
Module: U:\dev\php-5.3.3\Zend\zend_exceptions.o(zend_exceptions.o)
0002:00021bf8  _default_exception_ce
0002:00021c08  _error_exception_ce
0002:00021c18  _zend_throw_exception_hook
0001:00572350  _zend_exception_get_default
0001:0057235a  _zend_get_error_exception
0001:00572364  _zend_clear_exception
0001:005724cb  _zend_exception_error
0001:0057280d  _zend_spprintf
0001:00572875  _zend_register_default_exception
0001:00572e1b  _zend_exception_set_previous
0001:00572f2f  _zend_throw_exception_internal
0001:0057307f  _zend_throw_exception_object
0001:00573135  _zend_throw_exception
0001:0057323f  _zend_throw_error_exception
0001:0057329f  _zend_throw_exception_ex
0001:00573320  _zim_exception___clone
0001:00573347  _zend_exception_restore
0001:005733b5  _zend_exception_save
0001:00573496  _zim_error_exception_getSeverity
0001:005734ef  _zim_exception_getTrace
0001:00573548  _zim_exception_getCode
0001:005735a1  _zim_exception_getMessage
0001:005735fa  _zim_exception_getLine
0001:00573653  _zim_exception_getFile
0001:005736ac  _zim_exception_getPrevious
0001:005737d9  _zim_exception___toString
0001:00573c34  _zim_exception_getTraceAsString
0001:00574779  _zim_error_exception___construct
0001:005749da  _zim_exception___construct
Module: U:\dev\php-5.3.3\Zend\zend_strtod.o(zend_strtod.o)
0001:00575207  _zend_hex_strtod
0001:005752bc  _zend_oct_strtod
0001:0057538f  _zend_freedtoa
0001:00575b92  _zend_strtod
0001:00576b39  _zend_dtoa
0001:00577e85  _zend_shutdown_strtod
0001:00577f12  _zend_startup_strtod
Module: U:\dev\php-5.3.3\Zend\zend_gc.o(zend_gc.o)
0002:00021c28  _gc_globals_id
0001:00578129  _gc_globals_dtor
0001:0057812e  _gc_reset
0001:005786b8  _gc_remove_zval_from_buffer
0001:00578717  _gc_collect_cycles
0001:00578dc0  _gc_zobj_possible_root
0001:00578edd  _gc_zval_possible_root
0001:0057900b  _gc_init
0001:0057906a  _gc_globals_ctor
Module: U:\dev\php-5.3.3\Zend\zend_closures.o(zend_closures.o)
0002:00021c38  _zend_ce_closure
0001:005790d5  _zend_closure_get_closure
0001:00579125  _zend_get_closure_method_def
0001:00579142  _zend_create_closure
0001:00579334  _zim_Closure___construct
0001:0057963b  _zend_register_closure_ce
0001:00579928  _zend_get_closure_invoke_method
0001:00579a75  _zim_Closure___invoke
Module: U:\dev\php-5.3.3\Zend\zend_float.o(zend_float.o)
0001:00579f60  _zend_ensure_fpu_mode
0001:00579f7c  _zend_shutdown_fpu
0001:00579fc2  _zend_init_fpu
Module: U:\dev\php-5.3.3\Zend\zend_objects.o(zend_objects.o)
0001:0057a030  _zend_object_std_init
0001:0057a08b  _zend_objects_clone_members
0001:0057a16e  _zend_objects_get_address
0001:0057a17a  _zend_objects_new
0001:0057a62a  _zend_objects_free_object_storage
0001:0057a341  _zend_objects_destroy_object
0001:0057a1d2  _zend_objects_clone_obj
0001:0057a5e1  _zend_object_std_dtor
Module: U:\dev\php-5.3.3\Zend\zend_object_handlers.o(zend_object_handlers.o)
0001:0057a6f6  _zend_check_protected
0001:0057a733  _zend_std_object_get_class
0001:0057a74f  _zend_std_get_properties
0001:0057a76c  _zend_std_get_debug_info
0001:0057a8a8  _zend_std_get_constructor
0001:0057aa59  _zend_std_unset_static_property
0001:0057b9eb  _zend_std_call_user_call
0001:0057aaf2  _zend_std_object_get_class_name
0001:0057b7bf  _zend_std_callstatic_user_call
0001:0057abb9  _zend_std_get_closure
0001:0057ae1a  _zend_get_property_info
0001:0057b19e  _zend_std_get_static_property
0001:0057b33d  _zend_std_get_static_method
0001:0057b6c4  _zend_check_property_access
0001:0057c076  _zend_std_read_dimension
0001:0057c63b  _zend_check_private
0001:0057c7dc  _zend_std_cast_object_tostring
0001:0057cdc7  _zend_std_read_property
0002:00003f00  _std_object_handlers
Module: U:\dev\php-5.3.3\Zend\zend_objects_API.o(zend_objects_API.o)
0001:0057dcc0  _zend_objects_store_call_destructors
0001:0057dd2f  _zend_objects_store_mark_destructed
0001:0057dd5e  _zend_objects_store_free_object_storage
0001:0057de19  _zend_objects_store_get_refcount
0001:0057de3f  _zend_objects_store_add_ref
0001:0057de65  _zend_objects_store_add_ref_by_handle
0001:0057de89  _zend_object_store_get_object
0001:0057deaf  _zend_object_store_get_object_by_handle
0001:0057ded3  _zend_object_store_set_object
0001:0057defc  _zend_object_store_ctor_failed
0001:0057df27  _zend_get_std_object_handlers
0001:0057df6d  _zend_object_proxy_get
0001:0057e017  _zend_object_proxy_set
0001:0057e089  _zend_objects_proxy_clone
0001:0057e0ca  _zend_objects_proxy_free_storage
0001:0057e0f4  _zend_objects_store_destroy
0001:0057e13d  _zend_objects_store_del_ref_by_handle_ex
0001:0057e3fa  _zend_objects_store_del_ref
0001:0057e45f  _zend_objects_store_put
0001:0057e570  _zend_object_create_proxy
0001:0057e633  _zend_objects_store_clone_obj
0001:0057e704  _zend_objects_store_init
Module: U:\dev\php-5.3.3\Zend\zend_default_classes.o(zend_default_classes.o)
0001:0057e750  _zend_register_default_classes
Module: U:\dev\php-5.3.3\Zend\zend_execute.o(zend_execute.o)
0002:00021c48  _zend_opcode_handlers
0001:0057e8d2  _zend_get_compiled_variable_value
0001:0057e934  _execute_internal
0001:0057ea51  _zend_init_opcodes_handlers
0001:0057ea60  _zend_vm_set_opcode_handler
0001:0057eaa1  _zend_set_user_opcode_handler
0001:0057eaca  _zend_get_user_opcode_handler
0001:005812a4  _execute
0001:005871bc  _zend_get_zval_ptr_ptr
0001:005ab4c8  _zend_do_fcall
0001:005c9ee8  _zend_get_zval_ptr
Module: U:\usr\lib\libc_dll.lib(dllinit.obj)
0001:005ebdb0  _DLL_InitTerm
Module: U:\usr\lib\libend.lib(src/libend/386/endlink386.asm)
0002:00021cc0  _end
0002:00008910  _edata
Module: U:\usr\lib\libend.lib(src/libend/386/end.asm)
0001:00883ff0* _etext
0001:00883ff0* __etext
0000:00000000* WEAK$ZERO
0002:00021cc0  __end
0002:00008910  __edata
Module: U:\extras\lib\xml2.lib(xmlIO.obj)
0001:005ec280  ___xmlIOErr
0001:005ec7a0* _xmlIOHTTPOpenW
0001:005eca40  _xmlOutputBufferClose
0001:005ec950  _xmlAllocOutputBuffer
0001:005edc00  _xmlOutputBufferFlush
0001:005ecb10  ___xmlParserInputBufferCreateFilename
0001:005ee740* _xmlFileMatch
0001:005ee750* _xmlFileOpen
0001:005ee7b0* _xmlFileRead
0001:005ee830* _xmlFileClose
0001:005ee8e0* _xmlIOHTTPMatch
0001:005ee910* _xmlIOHTTPOpen
0001:005ee930* _xmlIOHTTPRead
0001:005ee950* _xmlIOHTTPClose
0001:005ee9a0* _xmlIOFTPOpen
0001:005ee970* _xmlIOFTPMatch
0001:005ee9b0* _xmlIOFTPRead
0001:005ee9d0* _xmlIOFTPClose
0001:005ece90  ___xmlOutputBufferCreateFilename
0001:005ed320  _xmlParserInputBufferCreateStatic
0001:005ed400  _xmlParserInputBufferPush
0001:005ed510  _xmlParserInputBufferGrow
0001:005ed700  _xmlOutputBufferWrite
0001:005ed920  _xmlOutputBufferWriteEscape
0001:005edd30  _xmlParserGetDirectory
0001:005edf90  _xmlCheckHTTPInput
0001:005ee290* _xmlResolveResourceFromCatalog
0001:005ee4e0  ___xmlLoaderErr
0001:005ee5c0* _xmlNormalizeWindowsPath
0001:005ee5d0  _xmlCleanupInputCallbacks
0001:005ee630* _xmlPopInputCallbacks
0001:005ee690  _xmlCleanupOutputCallbacks
0001:005ee6f0* _xmlCheckFilename
0001:005ee9e0* _xmlRegisterInputCallbacks
0001:005eea40* _xmlRegisterOutputCallbacks
0001:005eeaa0  _xmlRegisterDefaultInputCallbacks
0001:005eebe0  _xmlRegisterDefaultOutputCallbacks
0001:005eeca0* _xmlRegisterHTTPPostCallbacks
0001:005eed10  _xmlAllocParserInputBuffer
0001:005eedf0  _xmlFreeParserInputBuffer
0001:005eee80  _xmlParserInputBufferCreateFilename
0001:005eeeb0  _xmlOutputBufferCreateFilename
0001:005eeef0* _xmlParserInputBufferCreateFile
0001:005eef40  _xmlOutputBufferCreateFile
0001:005eef90  _xmlOutputBufferCreateBuffer
0001:005eefe0  _xmlParserInputBufferCreateFd
0001:005ef020  _xmlParserInputBufferCreateMem
0001:005ef0a0  _xmlOutputBufferCreateFd
0001:005ef0e0  _xmlParserInputBufferCreateIO
0001:005ef120  _xmlOutputBufferCreateIO
0001:005ef160  _xmlParserInputBufferCreateFilenameDefault
0001:005ef190  _xmlOutputBufferCreateFilenameDefault
0001:005ef1c0  _xmlParserInputBufferRead
0001:005ef210  _xmlOutputBufferWriteString
0001:005ef270* _xmlSetExternalEntityLoader
0001:005ef280* _xmlGetExternalEntityLoader
0001:005ef2b0  _xmlLoadExternalEntity
0001:005ef3e0* _xmlNoNetExternalEntityLoader
Module: U:\extras\lib\xml2.lib(uri.obj)
0001:005f0bd0  _xmlSaveUri
0001:005f1800* _xmlNormalizeURIPath
0001:005f1a40  _xmlURIUnescapeString
0001:005f1bf0  _xmlURIEscapeStr
0001:005f1e20  _xmlURIEscape
0001:005f2350  _xmlParseURIReference
0001:005f2d50  _xmlBuildURI
0001:005f3620  _xmlBuildRelativeURI
0001:005f3c70  _xmlCanonicPath
0001:005f40f0  _xmlCreateURI
0001:005f4140* _xmlPrintURI
0001:005f4180  _xmlFreeURI
0001:005f4260  _xmlParseURI
0001:005f4380  _xmlParseURIRaw
0001:005f44b0  _xmlPathToURI
Module: U:\extras\lib\xml2.lib(xmlstring.obj)
0001:005f5b50  _xmlStrPrintf
0001:005f5ba0  _xmlUTF8Strlen
0001:005f5c50  _xmlGetUTF8Char
0001:005f5d90  _xmlCheckUTF8
0001:005f5e80  _xmlStrndup
0001:005f5f00  _xmlStrdup
0001:005f5f90  _xmlCharStrndup
0001:005f6010  _xmlCharStrdup
0001:005f60a0  _xmlStrcmp
0001:005f60f0  _xmlStrEqual
0001:005f6130  _xmlStrQEqual
0001:005f61d0  _xmlStrncmp
0001:005f6220  _xmlStrcasecmp
0001:005f6280  _xmlStrncasecmp
0001:005f62f0  _xmlStrchr
0001:005f6330  _xmlStrstr
0001:005f63d0  _xmlStrcasestr
0001:005f64b0* _xmlStrsub
0001:005f6550  _xmlStrlen
0001:005f6580  _xmlStrncat
0001:005f6680  _xmlStrncatNew
0001:005f6870  _xmlStrcat
0001:005f6930* _xmlStrVPrintf
0001:005f6980* _xmlUTF8Size
0001:005f69e0* _xmlUTF8Charcmp
0001:005f6a70  _xmlUTF8Strsize
0001:005f6af0  _xmlUTF8Strndup
0001:005f6bb0  _xmlUTF8Strpos
0001:005f6c30  _xmlUTF8Strloc
0001:005f6d10  _xmlUTF8Strsub
Module: U:\extras\lib\xml2.lib(globals.obj)
0002:00021c60  _xmlLastError
0001:005f6dc0* _xmlInitializeGlobalState
0001:005f6fa0  _xmlInitGlobals
0001:005f6fc0  _xmlCleanupGlobals
0001:005f6ff0* _xmlThrDefSetGenericErrorFunc
0001:005f7050* _xmlThrDefSetStructuredErrorFunc
0001:005f70a0* _xmlRegisterNodeDefault
0001:005f70c0* _xmlThrDefRegisterNodeDefault
0001:005f7110* _xmlDeregisterNodeDefault
0001:005f7130* _xmlThrDefDeregisterNodeDefault
0001:005f7180* _xmlThrDefParserInputBufferCreateFilenameDefault
0001:005f71d0* _xmlThrDefOutputBufferCreateFilenameDefault
0001:005f7220* ___docbDefaultSAXHandler
0001:005f7230* ___htmlDefaultSAXHandler
0001:005f7240* ___xmlLastError
0001:005f7250* ___oldXMLWDcompatibility
0001:005f7260* ___xmlBufferAllocScheme
0001:005f7270* _xmlThrDefBufferAllocScheme
0001:005f72b0* ___xmlDefaultBufferSize
0001:005f72c0* _xmlThrDefDefaultBufferSize
0001:005f7300* ___xmlDefaultSAXHandler
0001:005f7310* ___xmlDefaultSAXLocator
0001:005f7320* ___xmlDoValidityCheckingDefaultValue
0001:005f7330* _xmlThrDefDoValidityCheckingDefaultValue
0001:005f7370* ___xmlGenericError
0001:005f7380* ___xmlStructuredError
0001:005f7390* ___xmlGenericErrorContext
0001:005f73a0* ___xmlGetWarningsDefaultValue
0001:005f73b0* _xmlThrDefGetWarningsDefaultValue
0001:005f73f0* ___xmlIndentTreeOutput
0001:005f7400* _xmlThrDefIndentTreeOutput
0001:005f7440* ___xmlTreeIndentString
0001:005f7450* _xmlThrDefTreeIndentString
0001:005f7490* ___xmlKeepBlanksDefaultValue
0001:005f74a0* _xmlThrDefKeepBlanksDefaultValue
0001:005f74e0* ___xmlLineNumbersDefaultValue
0001:005f74f0* _xmlThrDefLineNumbersDefaultValue
0001:005f7530* ___xmlLoadExtDtdDefaultValue
0001:005f7540* _xmlThrDefLoadExtDtdDefaultValue
0001:005f7580* ___xmlParserDebugEntities
0001:005f7590* _xmlThrDefParserDebugEntities
0001:005f75d0* ___xmlParserVersion
0001:005f75e0* ___xmlPedanticParserDefaultValue
0001:005f75f0* _xmlThrDefPedanticParserDefaultValue
0001:005f7630* ___xmlSaveNoEmptyTags
0001:005f7640* _xmlThrDefSaveNoEmptyTags
0001:005f7680* ___xmlSubstituteEntitiesDefaultValue
0001:005f7690* _xmlThrDefSubstituteEntitiesDefaultValue
0001:005f76d0* ___xmlRegisterNodeDefaultValue
0001:005f76e0* ___xmlDeregisterNodeDefaultValue
0001:005f76f0* ___xmlParserInputBufferCreateFilenameValue
0001:005f7700* ___xmlOutputBufferCreateFilenameValue
0002:000041e0  _xmlFree
0002:000041e4  _xmlMalloc
0002:000041e8  _xmlMallocAtomic
0002:000041ec  _xmlRealloc
0002:000041f0  _xmlMemStrdup
0002:000041f4  _xmlParserVersion
0002:000041f8  _xmlBufferAllocScheme
0002:00004200  _xmlDefaultBufferSize
0002:00004208  _xmlGetWarningsDefaultValue
0002:00004210  _xmlKeepBlanksDefaultValue
0002:00004218  _xmlGenericError
0002:00004220  _xmlIndentTreeOutput
0002:00004228  _xmlTreeIndentString
0002:00004240  _xmlDefaultSAXHandler
0002:000042b0  _xmlDefaultSAXLocator
0002:000042c0  _htmlDefaultSAXHandler
0002:00004340  _docbDefaultSAXHandler
0002:0001c410* _oldXMLWDcompatibility
0002:0001c414  _xmlParserDebugEntities
0002:0001c418  _xmlDoValidityCheckingDefaultValue
0002:0001c41c  _xmlLoadExtDtdDefaultValue
0002:0001c420  _xmlPedanticParserDefaultValue
0002:0001c424  _xmlLineNumbersDefaultValue
0002:0001c428  _xmlSubstituteEntitiesDefaultValue
0002:0001c42c  _xmlRegisterNodeDefaultValue
0002:0001c430  _xmlDeregisterNodeDefaultValue
0002:0001c434  _xmlParserInputBufferCreateFilenameValue
0002:0001c438  _xmlOutputBufferCreateFilenameValue
0002:0001c43c  _xmlStructuredError
0002:0001c440  _xmlGenericErrorContext
0002:0001c444  _xmlSaveNoEmptyTags
Module: U:\extras\lib\xml2.lib(error.obj)
0001:005f7710  _xmlGenericErrorDefaultFunc
0001:005f7770  ___xmlRaiseError
0001:005f8550  _xmlResetError
0001:005f8600  _xmlCopyError
0001:005f7d50  _xmlParserError
0001:005f7f80  _xmlParserWarning
0001:005f81c0  _xmlParserValidityError
0001:005f83b0  _xmlParserValidityWarning
0001:005f8740  _initGenericErrorDefaultFunc
0001:005f8760  _xmlSetGenericErrorFunc
0001:005f8790  _xmlSetStructuredErrorFunc
0001:005f87b0* _xmlParserPrintFileInfo
0001:005f8820* _xmlParserPrintFileContext
0001:005f8890  ___xmlSimpleError
0001:005f89e0  _xmlGetLastError
0001:005f8a00  _xmlResetLastError
0001:005f8a30* _xmlCtxtGetLastError
0001:005f8a50* _xmlCtxtResetLastError
Module: U:\extras\lib\xml2.lib(tree.obj)
0001:005f9230  _xmlStringText
0001:005f9235  _xmlStringTextNoenc
0001:005f923f  _xmlStringComment
0001:005f9260  _xmlBuildQName
0001:005f9360  _xmlSplitQName2
0001:005f9460  _xmlValidateNCName
0001:005f9850  _xmlValidateQName
0001:005f9e90  _xmlValidateName
0001:005fa2b0  _xmlValidateNMToken
0001:005fa790  _xmlNewNs
0001:005fa8f0  _xmlFreeNs
0001:005fa960  _xmlCreateIntSubset
0001:005fabb0  _xmlFreeDtd
0001:005fd550  _xmlUnlinkNode
0001:005fd260  _xmlFreeNode
0001:005fad40  _xmlFreeDoc
0001:005fcfb0  _xmlFreeNodeList
0001:005fafe0  _xmlStringLenGetNodeList
0001:005fc410* _xmlNewDocTextLen
0001:005fc5a0  _xmlAddNextSibling
0001:005ff3f0  _xmlNodeAddContentLen
0001:005fc250  _xmlNewReference
0001:005fc350  _xmlNewDocText
0001:005fb4b0  _xmlStringGetNodeList
0001:005ff600  _xmlNodeAddContent
0001:005fb920  _xmlNodeListGetString
0001:005fba60* _xmlNodeListGetRawString
0001:005fbbb0  _xmlNewDocProp
0001:005fbcd0* _xmlRemoveProp
0001:005fbe60  _xmlNewDocNode
0001:005fbfd0  _xmlNewDocNodeEatName
0001:005fc0e0* _xmlNewDocRawNode
0001:005fc170  _xmlNewTextChild
0001:005fc4d0  _xmlNewChild
0001:006032d0  _xmlSetTreeDoc
0001:005ff0d0  _xmlNodeSetContent
0001:005fc780  _xmlAddPrevSibling
0001:005fc950  _xmlAddSibling
0001:005fcb00  _xmlAddChildList
0001:005fcc90  _xmlAddChild
0001:00600580  _xmlHasNsProp
0001:005fd610  _xmlReplaceNode
0001:005fd890* _xmlCopyDtd
0001:005fdb60  _xmlCopyDoc
0001:005fdec0  _xmlGetNodePath
0001:005fe5e0  _xmlDocSetRootElement
0001:005fe740* _xmlNodeSetLang
0001:005ffa90  _xmlSearchNsByHref
0001:00600620  _xmlSetNsProp
0001:005fe7d0* _xmlNodeSetSpacePreserve
0001:005fe880  _xmlNodeSetName
0001:005fe990  _xmlNodeSetBase
0001:005feb00  _xmlNodeGetBase
0001:006005e0  _xmlGetNsProp
0001:006005b0  _xmlGetProp
0001:005fed70  _xmlNodeBufGetContent
0001:00600c90  _xmlBufferCat
0001:005fefa0  _xmlNodeGetContent
0001:00600850  _xmlBufferCreateSize
0001:00600930  _xmlBufferFree
0001:00600790  _xmlBufferCreate
0001:005ff260  _xmlNodeSetContentLen
0001:005ff640* _xmlTextMerge
0001:005ff6c0  _xmlGetNsList
0001:005ff830  _xmlSearchNs
0001:005ffe80* _xmlNewReconciliedNs
0001:005ffff0  _xmlReconciliateNs
0001:006004b0  _xmlHasProp
0001:00600980  _xmlBufferResize
0001:00600ab0  _xmlBufferAdd
0001:00600ba0  _xmlBufferAddHead
0001:00600cd0  _xmlBufferCCat
0001:00600d90  _xmlBufferWriteQuotedString
0001:00600ed0* _xmlDOMWrapRemoveNode
0001:006011f0* _xmlDOMWrapReconcileNamespaces
0001:006017c0* _xmlDOMWrapCloneNode
0001:00602230* _xmlDOMWrapAdoptNode
0001:006025e0  _xmlSplitQName3
0001:00602640* _xmlSetBufferAllocationScheme
0001:00602650* _xmlGetBufferAllocationScheme
0001:00602660  _xmlSetNs
0001:00602680  _xmlFreeNsList
0001:006026b0  _xmlNewDtd
0001:006027b0  _xmlGetIntSubset
0001:006027f0  _xmlNewDoc
0001:00602900  _xmlNewProp
0001:00602940  _xmlNewNsProp
0001:00602980  _xmlNewNsPropEatName
0001:006029c0* _xmlFreePropList
0001:00602a70  _xmlFreeProp
0001:00602b30  _xmlNewDocPI
0001:00602c10  _xmlNewPI
0001:00602c40  _xmlNewNode
0001:00602cf0* _xmlNewNodeEatName
0001:00602db0  _xmlNewDocFragment
0001:00602e40  _xmlNewText
0001:00602f10  _xmlNewCharRef
0001:00602fe0  _xmlNewTextLen
0001:006030a0  _xmlNewComment
0001:00603160  _xmlNewCDataBlock
0001:00603210  _xmlNewDocComment
0001:00603370* _xmlSetListDoc
0001:006033b0  _xmlGetLastChild
0001:006033d0* _xmlCopyNamespace
0001:00603410  _xmlCopyNamespaceList
0001:00603480* _xmlCopyProp
0001:006034b0  _xmlCopyPropList
0001:00603520  _xmlCopyNode
0001:00603550  _xmlDocCopyNode
0001:00603580  _xmlDocCopyNodeList
0001:006035b0  _xmlCopyNodeList
0001:006035e0  _xmlGetLineNo
0001:00603670  _xmlDocGetRootElement
0001:006036a0  _xmlNodeGetLang
0001:006036e0  _xmlNodeGetSpacePreserve
0001:00603780  _xmlGetNoNsProp
0001:006037c0  _xmlUnsetProp
0001:006038a0* _xmlUnsetNsProp
0001:00603980  _xmlSetProp
0001:00603aa0  _xmlNodeIsText
0001:00603ac0  _xmlIsBlankNode
0001:00603b30  _xmlTextConcat
0001:00603bf0  _xmlBufferCreateStatic
0001:00603c70* _xmlBufferSetAllocationScheme
0001:00603c90  _xmlBufferEmpty
0001:00603ce0  _xmlBufferShrink
0001:00603d50  _xmlBufferGrow
0001:00603de0* _xmlBufferDump
0001:00603e30  _xmlBufferContent
0001:00603e40  _xmlBufferLength
0001:00603e60  _xmlBufferWriteCHAR
0001:00603e80  _xmlBufferWriteChar
0001:00603ea0* _xmlGetDocCompressMode
0001:00603ec0  _xmlSetDocCompressMode
0001:00603ef0  _xmlGetCompressMode
0001:00603f00* _xmlSetCompressMode
0001:00603f50* _xmlDOMWrapNewCtxt
0001:00603fb0* _xmlDOMWrapFreeCtxt
0002:0001c540  ___xmlRegisterCallbacks
Module: U:\extras\lib\xml2.lib(valid.obj)
0001:00606fa0* _xmlValidBuildContentModel
0001:00607e60  _xmlSnprintfElementContent
0001:00607300  _xmlNewDocElementContent
0001:00607640* _xmlCopyDocElementContent
0001:00607aa0  _xmlFreeDocElementContent
0001:006082c0  _xmlAddElementDecl
0001:00608d10  _xmlDumpElementDecl
0001:00609090  _xmlAddAttributeDecl
0001:0060be50* _xmlValidateAttributeValue
0001:00613140  _xmlFreeEnumeration
0001:00609af0  _xmlDumpAttributeDecl
0001:00609e80  _xmlAddNotationDecl
0001:0060a300  _xmlAddID
0001:0060a780  _xmlIsID
0001:0060b340  _xmlGetDtdAttrDesc
0001:0060aae0  _xmlAddRef
0001:0060ae90  _xmlIsRef
0001:0060af50* _xmlRemoveRef
0001:0060b3f0* _xmlValidateNamesValue
0001:0060b860* _xmlValidateNmtokensValue
0001:0060c410  _xmlValidCtxtNormalizeAttributeValue
0001:0060c6e0  _xmlValidNormalizeAttributeValue
0001:0060ca90  _xmlValidateAttributeDecl
0001:0060d2d0  _xmlValidateElementDecl
0001:0060dca0  _xmlValidateOneAttribute
0001:0060ec00  _xmlValidateOneNamespace
0001:0060fe30  _xmlValidatePushElement
0001:00610250  _xmlValidatePushCData
0001:006104e0  _xmlValidatePopElement
0001:006109f0  _xmlValidateOneElement
0001:00611c90  _xmlValidateRoot
0001:00611f90  _xmlValidateElement
0001:00612130  _xmlValidateDtd
0001:00612240  _xmlValidateDtdFinal
0001:006123e0  _xmlValidateDocument
0001:006127f0* _xmlValidGetPotentialChildren
0001:00612970* _xmlValidGetValidElements
0001:00612d40  _xmlNewValidCtxt
0001:00612e90  _xmlFreeValidCtxt
0001:00612ee0* _xmlNewElementContent
0001:00612f10* _xmlCopyElementContent
0001:00612f30* _xmlFreeElementContent
0001:00612f50* _xmlSprintfElementContent
0001:00612f60  _xmlFreeElementTable
0001:00612f80  _xmlCopyElementTable
0001:00612fa0* _xmlDumpElementTable
0001:00612fd0  _xmlCreateEnumeration
0001:00613190* _xmlCopyEnumeration
0001:006131e0* _xmlScanAttributeDecl
0001:00613240  _xmlFreeAttributeTable
0001:00613260  _xmlCopyAttributeTable
0001:00613280* _xmlDumpAttributeTable
0001:006132b0  _xmlFreeNotationTable
0001:006132d0  _xmlCopyNotationTable
0001:00613310* _xmlDumpNotationDecl
0001:006133e0  _xmlDumpNotationTable
0001:00613410  _xmlFreeIDTable
0001:00613430  _xmlRemoveID
0001:006134e0  _xmlGetID
0001:00613530  _xmlFreeRefTable
0001:00613550* _xmlGetRefs
0001:00613580* _xmlGetDtdElementDesc
0001:00613620  _xmlGetDtdQElementDesc
0001:00613650  _xmlGetDtdQAttrDesc
0001:00613690* _xmlGetDtdNotationDesc
0001:006136e0  _xmlValidateNotationUse
0001:00613820  _xmlIsMixedElement
0001:00613980* _xmlValidateNameValue
0001:00613bd0* _xmlValidateNmtokenValue
0001:00613eb0  _xmlValidateNotationDecl
0001:00613ec0  _xmlValidateDocumentFinal
Module: U:\extras\lib\xml2.lib(relaxng.obj)
0001:0061e750  _xmlRelaxNGFreeParserCtxt
0001:00620a60  _xmlRelaxNGParse
0001:006253c0  _xmlRelaxNGFree
0001:00621da0* _xmlRelaxNGDump
0001:006227b0  _xmlRelaxNGValidatePushElement
0001:00625250  _xmlRelaxNGFreeValidCtxt
0001:006255d0* _xmlRelaxParserSetFlag
0001:00625610* _xmlRelaxNGInitTypes
0001:006256f0  _xmlRelaxNGCleanupTypes
0001:00625750  _xmlRelaxNGNewParserCtxt
0001:006258d0  _xmlRelaxNGNewMemParserCtxt
0001:00625a60* _xmlRelaxNGNewDocParserCtxt
0001:00625bf0  _xmlRelaxNGSetParserErrors
0001:00625c20* _xmlRelaxNGGetParserErrors
0001:00625c70* _xmlRelaxNGSetParserStructuredErrors
0001:00625ca0* _xmlRelaxNGDumpTree
0001:00625d20  _xmlRelaxNGValidatePushCData
0001:00625dd0  _xmlRelaxNGValidatePopElement
0001:00625ea0  _xmlRelaxNGValidateFullElement
0001:00625f70  _xmlRelaxNGNewValidCtxt
0001:00626120  _xmlRelaxNGSetValidErrors
0001:00626150  _xmlRelaxNGSetValidStructuredErrors
0001:00626180* _xmlRelaxNGGetValidErrors
0001:006261d0  _xmlRelaxNGValidateDoc
Module: U:\extras\lib\xml2.lib(parser.obj)
0001:00635bc0* _xmlHasFeature
0001:00635c70  _xmlCheckLanguageID
0001:00635dd0* _xmlSkipBlankChars
0001:00635f50  _xmlPopInput
0001:00636630  _xmlParserHandlePEReference
0001:00636060* _xmlParseCharRef
0001:00637b50* _xmlParseName
0001:00641120* _xmlParseTextDecl
0001:00636f80  _xmlStringLenDecodeEntities
0001:006436e0* _xmlParseStringPEReference
0001:00637550  _xmlStringDecodeEntities
0001:00642a20* _xmlParseStringEntityRef
0001:00637600  _xmlSplitQName
0001:00638050* _xmlParseNmtoken
0001:00638690* _xmlParseEntityValue
0001:00638c20* _xmlParseSystemLiteral
0001:00639070* _xmlParsePubidLiteral
0001:006394f0* _xmlParseCharData
0001:00639a00* _xmlParseCharDataComplex
0001:00639ff0* _xmlParseExternalID
0001:0063a570* _xmlParseComment
0001:0063adb0* _xmlParsePITarget
0001:0063b0c0* _xmlParsePI
0001:0063ba90* _xmlParseNotationDecl
0001:0063c070* _xmlParseEntityDecl
0001:0063cf90* _xmlParseDefaultDecl
0001:0063d3c0* _xmlParseNotationType
0001:0063d5c0* _xmlParseEnumerationType
0001:0063d760* _xmlParseEnumeratedType
0001:0063d930* _xmlParseAttributeType
0001:0063e030* _xmlParseAttributeListDecl
0001:0063ebb0* _xmlParseElementMixedContentDecl
0001:0063f2d0* _xmlParseElementChildrenContentDecl
0001:0063fce0* _xmlParseElementContentDecl
0001:00640000* _xmlParseElementDecl
0001:00640f40* _xmlParseMarkupDecl
0001:00642f80* _xmlParsePEReference
0001:00641600  _xmlParseExternalSubset
0001:00641a10* _xmlParseReference
0001:006423f0* _xmlParseEntityRef
0001:00643b00* _xmlParseDocTypeDecl
0001:00643e40* _xmlParseAttribute
0001:00644380* _xmlParseStartTag
0001:006450a0* _xmlParseCDSect
0001:006456a0* _xmlParseContent
0001:00645a60* _xmlParseElement
0001:006466a0* _xmlParseVersionInfo
0001:00646ac0* _xmlParseEncodingDecl
0001:00646560* _xmlParseVersionNum
0001:00646810* _xmlParseEncName
0001:00646dc0* _xmlParseSDDecl
0001:006470f0* _xmlParseXMLDecl
0001:006476e0  _xmlParseDocument
0001:0064c290  _xmlInitParser
0001:00647fc0* _xmlParseExtParsedEnt
0001:006483c0  _xmlParseChunk
0001:00648790  _xmlCreatePushParserCtxt
0001:00648af0* _xmlCreateIOParserCtxt
0001:00648c60* _xmlIOParseDTD
0001:006490c0* _xmlSAXParseDTD
0001:00649440  _xmlParseCtxtExternalEntity
0001:0064b6d0* _xmlCreateEntityParserCtxt
0001:0064bd00  _xmlCreateMemoryParserCtxt
0001:0064a900  _xmlParseInNodeContext
0001:0064c940  _xmlCtxtUseOptions
0001:0064b050* _xmlParseBalancedChunkMemoryRecover
0001:0064b630* _xmlSAXParseEntity
0001:0064b890  _xmlCreateFileParserCtxt
0001:0064b9a0* _xmlSAXParseFileWithData
0001:0064bb80* _xmlSAXUserParseFile
0001:0064bde0* _xmlSAXParseMemoryWithData
0001:0064bf70* _xmlSAXUserParseMemory
0001:0064c0f0* _xmlSAXParseDoc
0001:0064c300  _xmlCtxtReset
0001:0064c5f0* _xmlCtxtResetPush
0001:0064cb30  _inputPush
0001:0064cbc0  _inputPop
0001:0064cc10  _nodePush
0001:0064cd60  _nodePop
0001:0064cdb0* _namePush
0001:0064ce60* _namePop
0001:0064cec0  _xmlPushInput
0001:0064d020* _xmlParseAttValue
0001:0064d060* _xmlParseEndTag
0001:0064d080* _xmlParseMisc
0001:0064d140  _xmlStopParser
0001:0064d180  _xmlParseDTD
0001:0064d1b0* _xmlParseExternalEntity
0001:0064d200  _xmlParseBalancedChunkMemory
0001:0064d240* _xmlParseEntity
0001:0064d260* _xmlCreateURLParserCtxt
0001:0064d370* _xmlSAXParseFile
0001:0064d3a0* _xmlRecoverDoc
0001:0064d3d0* _xmlParseFile
0001:0064d400* _xmlRecoverFile
0001:0064d460* _xmlSetupParserForBuffer
0001:0064d560* _xmlSAXParseMemory
0001:0064d590* _xmlParseMemory
0001:0064d5c0* _xmlRecoverMemory
0001:0064d600* _xmlCreateDocParserCtxt
0001:0064d630* _xmlParseDoc
0001:0064d660* _xmlSetEntityReferenceFunc
0001:0064d670  _xmlCleanupParser
0001:0064d6d0* _xmlReadDoc
0001:0064d730  _xmlReadFile
0001:0064d780  _xmlReadMemory
0001:0064d7f0* _xmlReadFd
0001:0064d8f0* _xmlReadIO
0001:0064da10* _xmlCtxtReadDoc
0001:0064daf0  _xmlCtxtReadFile
0001:0064dbb0  _xmlCtxtReadMemory
0001:0064dcc0* _xmlCtxtReadFd
0001:0064ddd0* _xmlCtxtReadIO
0002:000043e0* _xmlParserMaxDepth
Module: U:\extras\lib\libz.lib(deflate.obj)
0001:00656ad0* _deflate_copyright
0001:00656b90  _deflateInit2_
0001:00656f40* _deflateReset
0001:00657cbc  _deflateEnd
0001:00656e04* _deflateSetDictionary
0001:00656ffc  _deflateParams
0001:006570e0  _deflate
0001:00657da0* _deflateCopy
0001:00658c44  _deflateInit_
0001:00658c68* _deflateSetHeader
0001:00658c94* _deflatePrime
0001:00658ccc* _deflateTune
0001:00658d0c* _deflateBound
Module: U:\extras\lib\libz.lib(crc32.obj)
0001:0065b070  _crc32
0001:0065b58c* _crc32_combine
0001:0065b720* _get_crc_table
Module: U:\extras\lib\libz.lib(zutil.obj)
0001:0065b7b0  _z_errmsg
0001:0065b7d8* _zlibCompileFlags
0001:0065b7e8  _zlibVersion
0001:0065b7f4  _zError
0001:0065b808  _zcalloc
0001:0065b81c  _zcfree
Module: U:\extras\lib\libz.lib(inflate.obj)
0001:0065b830  _inflateInit2_
0001:0065c41c  _inflate
0001:0065da90* _inflateSetDictionary
0001:0065db74* _inflateSync
0001:0065dd98* _inflateCopy
0001:0065dec4  _inflateReset
0001:0065df58* _inflatePrime
0001:0065dfa8  _inflateInit_
0001:0065dfc0  _inflateEnd
0001:0065e018* _inflateGetHeader
0001:0065e048* _inflateSyncPoint
Module: U:\extras\lib\libz.lib(uncompr.obj)
0001:0065e1b8  _uncompress
Module: U:\extras\lib\libz.lib(compress.obj)
0001:0065e268  _compress2
0001:0065e304  _compress
0001:0065e3a4  _compressBound
Module: U:\extras\lib\libz.lib(gzio.obj)
0001:0065e9e4  _gzread
0001:0065ec70  _gzwrite
0001:0065ed40* _gzprintf
0001:0065ed98  _gzseek
0001:0065f034  _gzrewind
0001:0065f2c8  _gzopen
0001:0065f2e8  _gzdopen
0001:0065f320* _gzsetparams
0001:0065f398* _gzgetc
0001:0065f3c4* _gzungetc
0001:0065f41c* _gzgets
0001:0065f474* _gzputc
0001:0065f4a4* _gzputs
0001:0065f4cc  _gzflush
0001:0065f50c* _gztell
0001:0065f524  _gzeof
0001:0065f554* _gzdirect
0001:0065f570  _gzclose
0001:0065f618* _gzerror
0001:0065f71c* _gzclearerr
Module: U:\extras\lib\xml2.lib(xpath.obj)
0001:0065fe40  _xmlXPathErr
0001:00660010* _xmlXPathFreeCompExpr
0001:006646e0  _xmlXPathFreeObject
0001:006603f0  _xmlXPathDebugDumpObject
0001:00661d40* _xmlXPathContextSetCache
0001:00662220* _xmlXPathPopNodeSet
0001:006622f0* _xmlXPathPopExternal
0001:006623b0* _xmlXPathOrderDocElems
0001:00662420  _xmlXPathCmpNodes
0001:006626e0* _xmlXPathNodeSetSort
0001:006627a0* _xmlXPathNodeSetCreate
0001:00662c50  _xmlXPathNodeSetContains
0001:00662d10* _xmlXPathNodeSetAddNs
0001:00663140* _xmlXPathNodeSetAdd
0001:00663510* _xmlXPathNodeSetAddUnique
0001:006638c0* _xmlXPathNodeSetMerge
0001:00663d60  _xmlXPathNewNodeSet
0001:00663ee0* _xmlXPathDistinctSorted
0001:00665610* _xmlXPathCastNodeToString
0001:00664000  _xmlXPathNewString
0001:00664180* _xmlXPathWrapString
0001:006642e0* _xmlXPathNewCString
0001:006644a0  _xmlXPathObjectCopy
0001:00665480* _xmlXPathCastBooleanToString
0001:006654d0* _xmlXPathCastNumberToString
0001:00665620* _xmlXPathCastNodeSetToString
0001:006656a0  _xmlXPathCastToString
0001:00665780* _xmlXPathConvertString
0001:00665860* _xmlXPathCastToNumber
0001:0066c790* _xmlXPathStringEvalNumber
0001:00665950* _xmlXPathCastToBoolean
0001:00665ab0* _xmlXPathEqualValues
0001:00665d50* _xmlXPathNotEqualValues
0001:00666020* _xmlXPathCompareValues
0001:0066b940* _xmlXPathNumberFunction
0001:0066b250* _xmlXPathBooleanFunction
0001:00666950* _xmlXPathDivValues
0001:00666ba0* _xmlXPathNextChild
0001:00666c50* _xmlXPathNextDescendant
0001:00666d10* _xmlXPathNextParent
0001:00666e20* _xmlXPathNextAncestor
0001:00667010* _xmlXPathNextNamespace
0001:00667120* _xmlXPathCountFunction
0001:00667580  _xmlXPathIdFunction
0001:00667c10* _xmlXPathLocalNameFunction
0001:00667ea0* _xmlXPathNamespaceURIFunction
0001:00668110* _xmlXPathStringLengthFunction
0001:006689b0* _xmlXPathConcatFunction
0001:00668dd0* _xmlXPathContainsFunction
0001:006693d0* _xmlXPathStartsWithFunction
0001:006699f0* _xmlXPathSubstringFunction
0001:0066a010* _xmlXPathSubstringBeforeFunction
0001:0066a3e0* _xmlXPathSubstringAfterFunction
0001:0066a7d0* _xmlXPathNormalizeFunction
0001:0066ac30* _xmlXPathTranslateFunction
0001:0066b460* _xmlXPathLangFunction
0001:0066c0e0* _xmlXPathSumFunction
0001:0066c480* _xmlXPathCeilingFunction
0001:0066c5a0* _xmlXPathRoundFunction
0001:00674380  _xmlXPathEvaluatePredicateResult
0001:006744b0* _xmlXPathCtxtCompile
0001:00674c60  _xmlXPathEval
0001:006755c0  _xmlXPathEvalExpression
0001:00675f90* _xmlXPathRegisterAllFunctions
0001:0067a390* _xmlXPathFalseFunction
0001:0067a450* _xmlXPathFloorFunction
0001:00679f40* _xmlXPathLastFunction
0001:0067a260* _xmlXPathNotFunction
0001:0067a010* _xmlXPathPositionFunction
0001:0067a0e0* _xmlXPathStringFunction
0001:0067a2e0* _xmlXPathTrueFunction
0001:00676e30  _xmlXPathInit
0001:00676f20  _xmlXPathIsNaN
0001:00676fb0* _xmlXPathIsInf
0001:00676ff0* _xmlXPatherror
0001:00677030* _xmlXPathDebugDumpCompExpr
0001:006770f0  _valuePop
0001:00677140  _valuePush
0001:006771d0* _xmlXPathPopBoolean
0001:00677290* _xmlXPathPopNumber
0001:00677340* _xmlXPathPopString
0001:00677400* _xmlXPathNodeSetFreeNs
0001:00677460* _xmlXPathNodeSetDel
0001:00677530* _xmlXPathNodeSetRemove
0001:006775e0* _xmlXPathFreeNodeSet
0001:006776a0* _xmlXPathNewValueTree
0001:00677820* _xmlXPathNewNodeSetList
0001:006778a0* _xmlXPathWrapNodeSet
0001:00677a00* _xmlXPathFreeNodeSetList
0001:00677a20* _xmlXPathDifference
0001:00677b00* _xmlXPathIntersection
0001:00677bc0* _xmlXPathDistinct
0001:00677c10* _xmlXPathHasSameNodes
0001:00677ca0* _xmlXPathNodeLeadingSorted
0001:00677d40* _xmlXPathNodeLeading
0001:00677df0* _xmlXPathLeadingSorted
0001:00677ec0* _xmlXPathLeading
0001:00677fd0* _xmlXPathNodeTrailingSorted
0001:00678070* _xmlXPathNodeTrailing
0001:00678120* _xmlXPathTrailingSorted
0001:006781f0* _xmlXPathTrailing
0001:006782f0  _xmlXPathRegisterFunc
0001:00678380  _xmlXPathRegisterFuncNS
0001:00678420* _xmlXPathRegisterFuncLookup
0001:00678440* _xmlXPathFunctionLookup
0001:006784e0* _xmlXPathFunctionLookupNS
0001:00678560* _xmlXPathRegisteredFuncsCleanup
0001:00678590* _xmlXPathRegisterVariable
0001:00678630* _xmlXPathRegisterVariableNS
0001:006786e0* _xmlXPathRegisterVariableLookup
0001:00678700* _xmlXPathVariableLookup
0001:006787f0* _xmlXPathVariableLookupNS
0001:006788f0* _xmlXPathRegisteredVariablesCleanup
0001:00678930  _xmlXPathRegisterNs
0001:006789d0* _xmlXPathNsLookup
0001:00678a80* _xmlXPathRegisteredNsCleanup
0001:00678ac0* _xmlXPathNewFloat
0001:00678c30  _xmlXPathNewBoolean
0001:00678da0* _xmlXPathWrapCString
0001:00678dc0* _xmlXPathWrapExternal
0001:00678f20* _xmlXPathCastBooleanToNumber
0001:00678f40* _xmlXPathCastStringToNumber
0001:00678f50* _xmlXPathCastNodeToNumber
0001:00678fa0* _xmlXPathCastNodeSetToNumber
0001:00678fe0* _xmlXPathConvertNumber
0001:00679030* _xmlXPathCastNumberToBoolean
0001:006790d0* _xmlXPathCastStringToBoolean
0001:00679100* _xmlXPathCastNodeSetToBoolean
0001:00679120* _xmlXPathConvertBoolean
0001:00679190  _xmlXPathNewContext
0001:00679360  _xmlXPathFreeContext
0001:00679400  _xmlXPathNewParserContext
0001:00679640  _xmlXPathFreeParserContext
0001:006796a0* _xmlXPathValueFlipSign
0001:00679820* _xmlXPathAddValues
0001:00679900* _xmlXPathSubValues
0001:006799e0* _xmlXPathMultValues
0001:00679ac0* _xmlXPathModValues
0001:00679bd0* _xmlXPathNextSelf
0001:00679c00* _xmlXPathNextDescendantOrSelf
0001:00679c50* _xmlXPathNextAncestorOrSelf
0001:00679c80* _xmlXPathNextFollowingSibling
0001:00679cc0* _xmlXPathNextPrecedingSibling
0001:00679d10* _xmlXPathNextFollowing
0001:00679d80* _xmlXPathNextPreceding
0001:00679e50* _xmlXPathNextAttribute
0001:00679ea0  _xmlXPathRoot
0001:0067a530  _xmlXPathParseNCName
0001:0067a600  _xmlXPathParseName
0001:0067a6e0* _xmlXPathIsNodeType
0001:0067a770* _xmlXPathEvalPredicate
0001:0067a850* _xmlXPathCompile
0001:0067a870* _xmlXPathCompiledEval
0001:0067a8b0* _xmlXPathCompiledEvalToBoolean
0001:0067a8e0  _xmlXPathEvalExpr
0002:000043f0  _xmlXPathPINF
0002:000043f8  _xmlXPathNINF
0002:0001c5a0  _xmlXPathNAN
Module: U:\extras\lib\xml2.lib(HTMLtree.obj)
0001:00686ed0  _htmlGetMetaEncoding
0001:00687190* _htmlSetMetaEncoding
0001:00687530  _htmlDocDumpMemoryFormat
0001:00687c80* _htmlDocContentDumpFormatOutput
0001:006876b0* _htmlNodeDumpFormatOutput
0001:00687d20* _htmlDocContentDumpOutput
0001:00687d50  _htmlDocDump
0001:00687e20  _htmlSaveFile
0001:00687f10  _htmlSaveFileFormat
0001:00688020  _htmlIsBooleanAttr
0001:00688070* _htmlNodeDump
0001:006880b0* _htmlNodeDumpFileFormat
0001:00688160  _htmlNodeDumpFile
0001:006881e0* _htmlDocDumpMemory
0001:00688210  _htmlNodeDumpOutput
0001:00688250* _htmlSaveFileEnc
Module: U:\extras\lib\xml2.lib(HTMLparser.obj)
0001:006905f0  _UTF8ToHtml
0001:00690810* _htmlEncodeEntities
0001:00690a50* _htmlParseEntityRef
0001:00690f00* _htmlParseCharRef
0001:00691430* _htmlParseElement
0001:00691b80  _htmlParseDocument
0001:00692800* _htmlParseChunk
0001:00692bb0* _htmlCreatePushParserCtxt
0001:00693130  _htmlCreateFileParserCtxt
0001:006933c0* _htmlCtxtReset
0001:00693660* _htmlCtxtUseOptions
0001:00693760  _htmlInitAutoClose
0001:006937f0  _htmlTagLookup
0001:00693850* _htmlAutoCloseTag
0001:006938f0* _htmlIsAutoClosed
0001:00693990* _htmlIsScriptAttribute
0001:006939f0* _htmlEntityLookup
0001:00693a50* _htmlEntityValueLookup
0001:00693ab0  _htmlNewDocNoDtD
0001:00693ca0* _htmlNewDoc
0001:00693ce0  ___htmlParseContent
0001:00693d00  _htmlFreeParserCtxt
0001:00693d10* _htmlNewParserCtxt
0001:00693ea0  _htmlCreateMemoryParserCtxt
0001:00693f30* _htmlSAXParseDoc
0001:00693fc0* _htmlParseDoc
0001:00693ff0* _htmlSAXParseFile
0001:00694070  _htmlParseFile
0001:006940a0* _htmlHandleOmittedElem
0001:006940c0* _htmlElementAllowedHere
0001:00694130* _htmlElementStatusHere
0001:006941b0* _htmlAttrAllowed
0001:00694290* _htmlNodeStatus
0001:00694570* _htmlReadDoc
0001:00694650* _htmlReadFile
0001:006946e0* _htmlReadMemory
0001:006947e0* _htmlReadFd
0001:00694920* _htmlReadIO
0001:00694a70* _htmlCtxtReadDoc
0001:00694b40* _htmlCtxtReadFile
0001:00694be0* _htmlCtxtReadMemory
0001:00694ce0* _htmlCtxtReadFd
0001:00694de0* _htmlCtxtReadIO
Module: U:\extras\lib\xml2.lib(xinclude.obj)
0001:0069fa10  _xmlXIncludeFreeContext
0001:006a0170  _xmlXIncludeSetFlags
0001:006a01d0  _xmlXIncludeNewContext
0001:006a02c0* _xmlXIncludeProcessFlagsData
0001:006a0430  _xmlXIncludeProcessFlags
0001:006a0460* _xmlXIncludeProcess
0001:006a0490* _xmlXIncludeProcessTreeFlags
0001:006a0600* _xmlXIncludeProcessTree
0001:006a0620  _xmlXIncludeProcessNode
Module: U:\extras\lib\xml2.lib(xmlsave.obj)
0001:006a64a0  _xmlAttrSerializeTxtContent
0001:006a63b0* _xmlSaveToBuffer
0001:006a6840  _xmlNodeDump
0001:006a6930  _xmlNodeDumpOutput
0001:006a6bb0* _xmlDocDumpFormatMemoryEnc
0001:006a6e70* _xmlDocFormatDump
0001:006a7010  _xmlSaveFormatFileEnc
0001:006a71e0* _xmlIsXHTML
0001:006a72e0  _xmlNsListDumpOutput
0001:006a73c0* _xmlSaveToFd
0001:006a7440* _xmlSaveToFilename
0001:006a74c0* _xmlSaveToIO
0001:006a7550* _xmlSaveDoc
0001:006a7580* _xmlSaveTree
0001:006a75b0* _xmlSaveFlush
0001:006a75e0* _xmlSaveClose
0001:006a7660* _xmlSaveSetEscape
0001:006a7680* _xmlSaveSetAttrEscape
0001:006a76a0  _xmlElemDump
0001:006a7740  _xmlDocDumpMemory
0001:006a7770  _xmlDocDumpFormatMemory
0001:006a77a0  _xmlDocDumpMemoryEnc
0001:006a77d0  _xmlDocDump
0001:006a7800* _xmlSaveFileTo
0001:006a7960  _xmlSaveFormatFileTo
0001:006a7ac0* _xmlSaveFileEnc
0001:006a7af0* _xmlSaveFormatFile
0001:006a7b20  _xmlSaveFile
Module: U:\extras\lib\xml2.lib(xmlschemas.obj)
0001:006a8fb0  _xmlSchemaFreeType
0001:006a9580  _xmlSchemaFree
0001:006b5be0  _xmlSchemaFreeParserCtxt
0001:006b7850  _xmlSchemaCheckFacet
0001:006ba560  _xmlSchemaFreeValidCtxt
0001:006ba480  _xmlSchemaNewValidCtxt
0001:006ba830  _xmlSchemaSetValidErrors
0001:006ba870  _xmlSchemaSetValidStructuredErrors
0001:006b92c0  _xmlSchemaParse
0001:006b97a0  _xmlSchemaSetParserErrors
0001:006b97e0* _xmlSchemaSetParserStructuredErrors
0001:006ba8b0  _xmlSchemaSAXPlug
0001:006bab60* _xmlSchemaValidateStream
0001:006badb0  _xmlSchemaNewFacet
0001:006badf0  _xmlSchemaFreeWildcard
0001:006bae80  _xmlSchemaFreeFacet
0001:006baf40* _xmlSchemaDump
0001:006bb0e0  _xmlSchemaNewParserCtxt
0001:006bb140  _xmlSchemaNewMemParserCtxt
0001:006bb190* _xmlSchemaNewDocParserCtxt
0001:006bb1e0* _xmlSchemaGetParserErrors
0001:006bb230  _xmlSchemaIsValid
0001:006bb250* _xmlSchemaGetValidErrors
0001:006bb2a0* _xmlSchemaSetValidOptions
0001:006bb2e0* _xmlSchemaValidCtxtGetOptions
0001:006bb300* _xmlSchemaValidateOneElement
0001:006bb380  _xmlSchemaValidateDoc
0001:006bb490  _xmlSchemaSAXUnplug
0001:006bb520* _xmlSchemaValidateFile
Module: U:\extras\lib\xml2.lib(parserInternals.obj)
0001:006f9bf0* _xmlParserInputRead
0001:006f9ca0  _xmlParserInputGrow
0001:006f9d50  _xmlParserInputShrink
0001:006f9f10  _xmlNextChar
0001:006fa460  _xmlCurrentChar
0001:006fa8c0  _xmlStringCurrentChar
0001:006fac70  _xmlCopyCharMultiByte
0001:006fae20  _xmlSwitchEncoding
0001:006fb850  _xmlSwitchToEncoding
0001:006fb4d0  _xmlSwitchInputEncoding
0001:006fbb00  _xmlNewEntityInputStream
0001:006fbfc0  _xmlNewInputFromFile
0001:006fc330* _xmlInitParserCtxt
0001:006fd0e0  _xmlInitNodeInfoSeq
0001:006fcd60  _xmlFreeParserCtxt
0001:006fd120  _xmlParserAddNodeInfo
0001:006fd510* _xmlCheckVersion
0001:006fd5e0  _xmlErrMemory
0001:006fd720  ___xmlErrEncoding
0001:006fd7f0* _xmlIsLetter
0001:006fd8a0  _xmlCopyChar
0001:006fd8d0  _xmlFreeInputStream
0001:006fd970  _xmlNewInputStream
0001:006fdb40  _xmlNewIOInputStream
0001:006fdc40  _xmlNewStringInputStream
0001:006fdf10  _xmlNewParserCtxt
0001:006fe0a0  _xmlClearParserCtxt
0001:006fe100* _xmlParserFindNodeInfo
0001:006fe1d0* _xmlClearNodeInfoSeq
0001:006fe210* _xmlParserFindNodeInfoIndex
0001:006fe2c0* _xmlPedanticParserDefault
0001:006fe2e0* _xmlLineNumbersDefault
0001:006fe300* _xmlSubstituteEntitiesDefault
0001:006fe320* _xmlKeepBlanksDefault
Module: U:\extras\lib\xml2.lib(encoding.obj)
0001:006fe350* _isolat1ToUTF8
0001:006fe450* _UTF8Toisolat1
0001:006fe5e0  _xmlDetectCharEncoding
0001:006fe7b0* _xmlAddEncodingAlias
0001:006fea60  _xmlParseCharEncoding
0001:006fef10  _xmlGetCharEncodingName
0001:006ff080* _xmlNewCharEncodingHandler
0001:006ff430* _xmlRegisterCharEncodingHandler
0001:006ff740  _xmlGetCharEncodingHandler
0001:006ffb60  _xmlFindCharEncodingHandler
0001:007000c0  _xmlCharEncFirstLine
0001:00700290  _xmlCharEncInFunc
0001:00700540  _xmlCharEncOutFunc
0001:007008f0  _xmlCharEncCloseFunc
0001:00700990  _xmlByteConsumed
0001:00700b60* _xmlCleanupEncodingAliases
0001:00700bf0* _xmlGetEncodingAlias
0001:00700ca0* _xmlDelEncodingAlias
0001:00700d60  _xmlInitCharEncodingHandlers
0001:00700f70  _xmlCleanupCharEncodingHandlers
Module: U:\extras\lib\xml2.lib(c14n.obj)
0001:00701e70* _xmlC14NExecute
0001:00702440* _xmlC14NDocDumpMemory
0001:00702920  _xmlC14NDocSaveTo
0001:007029c0* _xmlC14NDocSave
Module: U:\extras\lib\xml2.lib(hash.obj)
0001:00705950  _xmlHashFree
0001:00705ab0  _xmlHashAddEntry3
0001:00705e00* _xmlHashUpdateEntry3
0001:00706150  _xmlHashLookup3
0001:00706230* _xmlHashScanFull3
0001:00706330  _xmlHashCopy
0001:00706490* _xmlHashRemoveEntry3
0001:00706630  _xmlHashCreate
0001:007066f0  _xmlHashCreateDict
0001:007067c0  _xmlHashAddEntry
0001:007067f0  _xmlHashAddEntry2
0001:00706820  _xmlHashUpdateEntry
0001:00706860  _xmlHashUpdateEntry2
0001:007068a0  _xmlHashLookup
0001:007068d0  _xmlHashLookup2
0001:00706900* _xmlHashQLookup
0001:007069d0  _xmlHashQLookup2
0001:00706aa0* _xmlHashQLookup3
0001:00706b70  _xmlHashScan
0001:00706c30  _xmlHashScanFull
0001:00706ce0  _xmlHashScan3
0001:00706cf0  _xmlHashSize
0001:00706d10  _xmlHashRemoveEntry
0001:00706d40  _xmlHashRemoveEntry2
Module: U:\extras\lib\libssl.lib(ssl_lib.obj)
0001:0070b550  _ssl_undefined_function
0001:00707294  _SSL_clear
0001:0070bb43* _ssl_clear_cipher_ctx
0001:0070c519* _ssl_clear_hash_ctx
0001:007074bb* _SSL_CTX_set_ssl_version
0001:00707583  _SSL_new
0001:0070a305  _SSL_CTX_free
0001:007079fd* _SSL_CTX_set_session_id_context
0001:00707a6e* _SSL_set_session_id_context
0001:00707adf* _SSL_CTX_set_generate_session_id
0001:00707b40* _SSL_set_generate_session_id
0001:00707ba1  _SSL_has_matching_session_id
0001:00707ca7* _SSL_CTX_set_purpose
0001:00707cc7* _SSL_set_purpose
0001:00707ce4* _SSL_CTX_set_trust
0001:00707d04* _SSL_set_trust
0001:00707d21* _SSL_CTX_set1_param
0001:00707d41* _SSL_set1_param
0001:00707d5e* _SSL_free
0001:00708097* _SSL_set_bio
0001:0070813d  _SSL_get_rbio
0001:00708148* _SSL_get_wbio
0001:00708153* _SSL_get_fd
0001:00708166* _SSL_get_rfd
0001:007081c4* _SSL_get_wfd
0001:00708222  _SSL_set_fd
0001:007082c1* _SSL_set_wfd
0001:007083e8* _SSL_set_rfd
0001:0070850f* _SSL_get_finished
0001:0070856a* _SSL_get_peer_finished
0001:007085c5* _SSL_get_verify_mode
0001:007085d3* _SSL_get_verify_depth
0001:007085e9* _SSL_get_verify_callback
0001:007085f7* _SSL_CTX_get_verify_mode
0001:00708605* _SSL_CTX_get_verify_depth
0001:0070861e* _SSL_CTX_get_verify_callback
0001:0070862c* _SSL_set_verify
0001:0070864f* _SSL_set_verify_depth
0001:0070866c* _SSL_set_read_ahead
0001:0070867a* _SSL_get_read_ahead
0001:00708685* _SSL_pending
0001:0070869e* _SSL_get_peer_certificate
0001:00708710* _SSL_get_peer_cert_chain
0001:0070875e  _SSL_copy_session_id
0001:00708862* _SSL_CTX_check_private_key
0001:0070892d* _SSL_check_private_key
0001:00708a64* _SSL_accept
0001:0070b490* _SSL_set_accept_state
0001:00708a92  _SSL_connect
0001:0070b4f0* _SSL_set_connect_state
0001:00708ac0  _SSL_get_default_timeout
0001:00708ad3  _SSL_read
0001:00708b55  _SSL_peek
0001:00708bcd  _SSL_write
0001:00708c7b  _SSL_shutdown
0001:0070c004  _SSL_state
0001:00708cf2* _SSL_renegotiate
0001:00708d1f* _SSL_renegotiate_pending
0001:00708d32  _SSL_ctrl
0001:0070bec4  _SSL_version
0001:00708ffc* _SSL_callback_ctrl
0001:0070903b* _SSL_CTX_sessions
0001:00709046  _SSL_CTX_ctrl
0001:0070938d* _SSL_CTX_callback_ctrl
0001:007093ce* _ssl_cipher_id_cmp
0001:0070940a  _ssl_cipher_ptr_id_cmp
0001:0070944a  _SSL_get_ciphers
0001:00709497  _ssl_get_ciphers_by_id
0001:007094e4* _SSL_get_cipher_list
0001:0070954c* _SSL_CTX_set_cipher_list
0001:007095d8* _SSL_set_cipher_list
0001:0070966a* _SSL_get_shared_ciphers
0001:00709755  _ssl_cipher_list_to_bytes
0001:00709876  _ssl_bytes_to_cipher_list
0001:00709a83* _SSL_get_servername
0001:00709ac9* _SSL_get_servername_type
0001:00709c0e  _SSL_CTX_new
0001:0070a50c* _SSL_CTX_set_default_passwd_cb
0001:0070a51a* _SSL_CTX_set_default_passwd_cb_userdata
0001:0070a528* _SSL_CTX_set_cert_verify_callback
0001:0070a53f* _SSL_CTX_set_verify
0001:0070a55c* _SSL_CTX_set_verify_depth
0001:0070a58c  _ssl_set_cert_masks
0001:0070aae4  _ssl_check_srvr_ecc_cert_and_alg
0001:0070ad31* _ssl_get_server_send_cert
0001:0070aeed* _ssl_get_sign_pkey
0001:0070afab  _ssl_update_cache
0001:0070b11d* _SSL_get_ssl_method
0001:0070b128  _SSL_set_ssl_method
0001:0070b1e4* _SSL_get_error
0001:0070c168* _SSL_want
0001:0070b3f7* _SSL_do_handshake
0001:0070b589  _ssl_undefined_void_function
0001:0070b5c2  _ssl_undefined_const_function
0001:0070b5fb* _ssl_bad_method
0001:0070b640* _SSL_get_version
0001:0070b681* _SSL_dup
0001:0070bece* _SSL_get_SSL_CTX
0001:0070bff6* _SSL_get_info_callback
0001:0070bfe5* _SSL_set_info_callback
0001:0070bc19* _SSL_get_certificate
0001:0070bc3f* _SSL_get_privatekey
0001:0070bc66* _SSL_get_current_cipher
0001:0070bca1* _SSL_get_current_compression
0001:0070bcc5* _SSL_get_current_expansion
0001:0070bce9  _ssl_init_wbio_buffer
0001:0070be22  _ssl_free_wbio_buffer
0001:0070be73* _SSL_CTX_set_quiet_shutdown
0001:0070be84* _SSL_CTX_get_quiet_shutdown
0001:0070be92* _SSL_set_quiet_shutdown
0001:0070bea0* _SSL_get_quiet_shutdown
0001:0070beab* _SSL_set_shutdown
0001:0070beb9* _SSL_get_shutdown
0001:0070bedc* _SSL_set_SSL_CTX
0001:0070bfab* _SSL_CTX_set_default_verify_paths
0001:0070bfc1* _SSL_CTX_load_verify_locations
0001:0070c00f* _SSL_set_verify_result
0001:0070c020* _SSL_get_verify_result
0001:0070c02e* _SSL_get_ex_new_index
0001:0070c065* _SSL_set_ex_data
0001:0070c08c* _SSL_get_ex_data
0001:0070c0ac* _SSL_CTX_get_ex_new_index
0001:0070c0e3* _SSL_CTX_set_ex_data
0001:0070c10a* _SSL_CTX_get_ex_data
0001:0070c12a  _ssl_ok
0001:0070c134* _SSL_CTX_get_cert_store
0001:0070c13f* _SSL_CTX_set_cert_store
0001:0070c173* _SSL_CTX_set_tmp_rsa_callback
0001:0070c195* _SSL_set_tmp_rsa_callback
0001:0070c1b7* _SSL_CTX_set_tmp_dh_callback
0001:0070c1d9* _SSL_set_tmp_dh_callback
0001:0070c1fb* _SSL_CTX_set_tmp_ecdh_callback
0001:0070c21d* _SSL_set_tmp_ecdh_callback
0001:0070c23f* _SSL_CTX_use_psk_identity_hint
0001:0070c2f3* _SSL_use_psk_identity_hint
0001:0070c3f1* _SSL_get_psk_identity_hint
0001:0070c41f* _SSL_get_psk_identity
0001:0070c44d* _SSL_set_psk_client_callback
0001:0070c45e* _SSL_CTX_set_psk_client_callback
0001:0070c46f* _SSL_set_psk_server_callback
0001:0070c480* _SSL_CTX_set_psk_server_callback
0001:0070c491* _SSL_CTX_set_msg_callback
0001:0070c4b3* _SSL_set_msg_callback
0001:0070c4d5  _ssl_replace_hash
0001:0070c566  _OBJ_bsearch_ssl_cipher_id
0002:000046b0* _SSL_version_str
0002:000046c0  _ssl3_undef_enc_method
Module: U:\extras\lib\libssl.lib(s23_clnt.obj)
0001:0070c5da  _SSLv23_client_method
0001:0070c5ef* _ssl23_connect
Module: U:\usr\lib\libc_dll.lib(accept.obj)
0001:0070d890  _accept
Module: U:\usr\lib\libc_dll.lib(send.obj)
0001:0070d970  _send
Module: U:\usr\lib\libc_dll.lib(recv.obj)
0001:0070da20  _recv
Module: U:\usr\lib\libc_dll.lib(socket.obj)
0001:0070dad0  _socket
Module: U:\usr\lib\libc_dll.lib(bind.obj)
0001:0070db50  _bind
Module: U:\usr\lib\libc_dll.lib(getsockname.obj)
0001:0070dbf0  _getsockname
Module: U:\usr\lib\libc_dll.lib(listen.obj)
0001:0070dc90  _listen
Module: U:\extras\lib\xml2.lib(entities.obj)
0001:0070ddc0  _xmlAddDtdEntity
0001:0070df00  _xmlAddDocEntity
0001:0070e0e0  _xmlEncodeEntitiesReentrant
0001:0070e560  _xmlEncodeSpecialChars
0001:0070e730  _xmlDumpEntityDecl
0001:0070e960  _xmlGetPredefinedEntity
0001:0070ea20  _xmlGetParameterEntity
0001:0070ea90* _xmlGetDtdEntity
0001:0070eac0  _xmlGetDocEntity
0001:0070ebf0* _xmlCreateEntitiesTable
0001:0070ec10  _xmlFreeEntitiesTable
0001:0070ec30  _xmlCopyEntitiesTable
0001:0070ec50* _xmlDumpEntitiesTable
Module: U:\usr\lib\libc_dll.lib(shutdown.obj)
0001:0070f3b0  _shutdown
Module: U:\usr\lib\libc_dll.lib(getsockopt.obj)
0001:0070f450  _getsockopt
Module: U:\usr\lib\libc_dll.lib(sendto.obj)
0001:0070f530  _sendto
Module: U:\usr\lib\libc_dll.lib(connect.obj)
0001:0070f5e0  _connect
Module: U:\usr\lib\libc_dll.lib(socketpair.obj)
0001:0070f680  _socketpair
Module: U:\usr\lib\libc_dll.lib(getpeername.obj)
0001:0070f740  _getpeername
Module: U:\usr\lib\libc_dll.lib(recvfrom.obj)
0001:0070f7e0  _recvfrom
Module: U:\usr\lib\libc_dll.lib(setsockopt.obj)
0001:0070f8b0  _setsockopt
Module: U:\usr\lib\libc_dll.lib(syslog.obj)
0001:0070f9fc  _syslog
0001:0070fa64* _vsyslog
0001:0070fec1  _openlog
0001:0070ff10  _closelog
0001:0070ff44* _setlogmask
Module: U:\extras\lib\xml2.lib(xmlreader.obj)
0001:00710450  _xmlTextReaderRead
0001:00712640* _xmlTextReaderPreserve
0001:00710d30  _xmlTextReaderExpand
0001:00710dd0  _xmlTextReaderReadInnerXml
0001:00710fc0  _xmlNewTextReader
0001:00711270  _xmlFreeTextReader
0001:007114f0  _xmlTextReaderGetAttributeNo
0001:007115c0  _xmlTextReaderGetAttribute
0001:00711760  _xmlTextReaderGetAttributeNs
0001:007118a0* _xmlTextReaderGetRemainder
0001:00711960  _xmlTextReaderMoveToAttributeNo
0001:007119f0  _xmlTextReaderMoveToAttribute
0001:00711be0  _xmlTextReaderMoveToAttributeNs
0001:00711d30  _xmlTextReaderMoveToNextAttribute
0001:00711da0* _xmlTextReaderReadAttributeValue
0001:00711e60  _xmlTextReaderAttributeCount
0001:00711ed0  _xmlTextReaderNodeType
0001:00712050* _xmlTextReaderName
0001:007121b0  _xmlTextReaderConstName
0001:00712330* _xmlTextReaderValue
0001:00712460  _xmlTextReaderConstValue
0001:00712580  _xmlTextReaderSetParserProp
0001:007126b0* _xmlTextReaderPreservePattern
0001:00712800  _xmlTextReaderRelaxNGSetSchema
0001:00712930* _xmlTextReaderSetSchema
0001:00712b40* _xmlTextReaderRelaxNGValidate
0001:00712ee0* _xmlTextReaderSetErrorHandler
0001:00713060* _xmlTextReaderSetStructuredErrorHandler
0001:00713200  _xmlTextReaderSetup
0001:007136f0* _xmlReaderNewWalker
0001:007137a0* _xmlTextReaderReadState
0001:007137c0  _xmlTextReaderNext
0001:00713840  _xmlTextReaderReadOuterXml
0001:007138e0  _xmlTextReaderReadString
0001:00713990* _xmlTextReaderNextSibling
0001:007139f0* _xmlNewTextReaderFilename
0001:00713aa0* _xmlTextReaderClose
0001:00713b30  _xmlTextReaderLookupNamespace
0001:00713b80  _xmlTextReaderMoveToFirstAttribute
0001:00713bc0  _xmlTextReaderMoveToElement
0001:00713c00* _xmlTextReaderConstEncoding
0001:00713c60  _xmlTextReaderIsEmptyElement
0001:00713cc0* _xmlTextReaderLocalName
0001:00713d20  _xmlTextReaderConstLocalName
0001:00713da0* _xmlTextReaderPrefix
0001:00713e00  _xmlTextReaderConstPrefix
0001:00713e90* _xmlTextReaderNamespaceUri
0001:00713ee0  _xmlTextReaderConstNamespaceUri
0001:00713f60* _xmlTextReaderBaseUri
0001:00713fa0  _xmlTextReaderConstBaseUri
0001:00714010  _xmlTextReaderDepth
0001:00714060  _xmlTextReaderHasAttributes
0001:007140b0  _xmlTextReaderHasValue
0001:00714150  _xmlTextReaderIsDefault
0001:00714160* _xmlTextReaderQuoteChar
0001:00714180* _xmlTextReaderXmlLang
0001:007141b0  _xmlTextReaderConstXmlLang
0001:00714210* _xmlTextReaderConstString
0001:00714240* _xmlTextReaderNormalization
0001:00714260  _xmlTextReaderGetParserProp
0001:007142d0* _xmlTextReaderGetParserLineNumber
0001:00714300* _xmlTextReaderGetParserColumnNumber
0001:00714330* _xmlTextReaderCurrentNode
0001:00714350* _xmlTextReaderCurrentDoc
0001:00714390* _xmlTextReaderSchemaValidateCtxt
0001:007143c0  _xmlTextReaderSchemaValidate
0001:007143f0* _xmlTextReaderIsNamespaceDecl
0001:00714420* _xmlTextReaderConstXmlVersion
0001:00714480* _xmlTextReaderStandalone
0001:007144c0* _xmlTextReaderLocatorLineNumber
0001:00714520* _xmlTextReaderLocatorBaseURI
0001:00714590  _xmlTextReaderIsValid
0001:007145e0* _xmlTextReaderGetErrorHandler
0001:00714610* _xmlTextReaderByteConsumed
0001:00714640* _xmlReaderWalker
0001:007146f0* _xmlReaderForDoc
0001:00714780  _xmlReaderForFile
0001:00714860* _xmlReaderForMemory
0001:007148f0* _xmlReaderForFd
0001:00714980* _xmlReaderForIO
0001:00714a10* _xmlReaderNewDoc
0001:00714a80* _xmlReaderNewFile
0001:00714ae0* _xmlReaderNewMemory
0001:00714b60* _xmlReaderNewFd
0001:00714be0* _xmlReaderNewIO
Module: U:\extras\lib\xmlrpc.lib(xmlrpc.obj)
0001:00716350  _XMLRPC_RequestGetMethodName
0001:00716361  _XMLRPC_RequestSetRequestType
0001:00716377  _XMLRPC_RequestGetRequestType
0001:00716388  _XMLRPC_RequestGetData
0001:00716398  _XMLRPC_RequestGetError
0001:007163a9  _XMLRPC_RequestGetOutputOptions
0001:007163ba  _XMLRPC_SetValueInt
0001:007163d2  _XMLRPC_SetValueBoolean
0001:007163f0  _XMLRPC_CopyValue
0001:00716400  _XMLRPC_SetValueDouble
0001:0071641c  _XMLRPC_GetValueString
0001:00716434  _XMLRPC_GetValueStringLen
0001:00716445  _XMLRPC_GetValueInt
0001:00716461  _XMLRPC_GetValueBoolean
0001:00716479  _XMLRPC_GetValueDouble
0001:00716491  _XMLRPC_GetValueBase64
0001:007164a9  _XMLRPC_GetValueDateTime
0001:007164c1  _XMLRPC_GetValueDateTime_ISO8601
0001:007164d9  _XMLRPC_GetValueID
0001:007164f3  _XMLRPC_GetValueType
0001:00716506  _XMLRPC_GetVectorType
0001:00716521  _XMLRPC_GetValueTypeEasy
0001:007165b2  _type_to_str
0001:00716653  _XMLRPC_GetDefaultIdCase
0001:0071665d* _XMLRPC_SetDefaultIdCase
0001:0071666a  _XMLRPC_GetDefaultIdCaseComparison
0001:00716674* _XMLRPC_SetDefaultIdCaseComparison
0001:00716694  _XMLRPC_GetVersionString
0001:0071669e* _XMLRPC_Free
0001:007166b3* _XMLRPC_ServerFindMethod
0001:00716700  _find_method
0001:0071674c  _XMLRPC_ServerRegisterMethod
0001:007167b2  _XMLRPC_VectorRewind
0001:007167de  _XMLRPC_VectorNext
0001:00716807  _XMLRPC_CreateValueEmpty
0001:0071684c  _XMLRPC_RequestNew
0001:0071687d  _XMLRPC_ServerCreate
0001:007168c1* _XMLRPC_GetGlobalServer
0001:007168de  _XMLRPC_VectorSize
0001:00716907  _XMLRPC_SetIsVector
0001:007169a4  _XMLRPC_RequestSetMethodName
0001:007169d9  _XMLRPC_SetValueBase64
0001:00716a3c  _XMLRPC_SetValueString
0001:00716aa4  _XMLRPC_SetValueID_Case
0001:00716b83  _XMLRPC_CreateValueDouble
0001:00716bd5  _XMLRPC_CreateValueBase64
0001:00716c2b  _XMLRPC_CreateValueBoolean
0001:00716c7d  _XMLRPC_CreateValueInt
0001:00716cc9  _XMLRPC_CreateValueString
0001:00716d27  _XMLRPC_CreateVector
0001:00716d82  _XMLRPC_SetValueDateTime_ISO8601
0001:00716f15  _XMLRPC_CreateValueDateTime_ISO8601
0001:00716f75* _XMLRPC_SetValueDateTime
0001:00716fe3* _XMLRPC_CreateValueDateTime
0001:00717065  _XMLRPC_CleanupValue
0001:00717173  _XMLRPC_ServerDestroy
0001:00717234  _XMLRPC_RequestSetError
0001:00717273  _XMLRPC_RequestSetData
0001:007172b0  _XMLRPC_RequestFree
0001:00717386  _XMLRPC_AddValueToVector
0001:0071759b* _XMLRPC_UtilityCreateFault
0001:0071773d  _XMLRPC_ServerCallMethod
0001:007177d6  _XMLRPC_DupValueNew
0001:0071791f  _XMLRPC_VectorRemoveValue
0001:00717993  _XMLRPC_VectorGetValueWithID_Case
0001:00717a0d* _XMLRPC_GetValueFaultString
0001:00717a41* _XMLRPC_GetResponseFaultString
0001:00717a58* _XMLRPC_GetValueFaultCode
0001:00717a8c* _XMLRPC_GetResponseFaultCode
0001:00717aa3* _XMLRPC_ValueIsFault
0001:00717af3* _XMLRPC_ResponseIsFault
0001:00717b0a  _XMLRPC_AddValuesToVector
0001:00717c1f  _XMLRPC_REQUEST_FromXML
0001:00717d35* _XMLRPC_VALUE_FromXML
0001:00717d75  _XMLRPC_REQUEST_ToXML
0001:00717df3  _XMLRPC_VALUE_ToXML
0001:00717e38  _XMLRPC_RequestSetOutputOptions
Module: U:\extras\lib\xmlrpc.lib(xmlrpc_introspection.obj)
0001:00717f04* _XMLRPC_ServerSetValidationLevel
0001:00717f22* _find_named_value
0001:00717f96* _validate_scalar
0001:007180f3* _validate_value
0001:007182f4* _validate_vector
0001:007181e7* _validate_method
0001:00718272  _XMLRPC_ServerValidateRequest
0001:00718409  _XMLRPC_ServerRegisterIntrospectionCallback
0001:00718472* _describe_method
0001:00718594* _xml_element_to_method_description
0001:00718b81  _XMLRPC_IntrospectionCreateDescription
0001:00718c30  _xi_register_system_methods
0001:0071908b  _XMLRPC_ServerAddIntrospectionData
Module: U:\extras\lib\xml2.lib(xmlwriter.obj)
0001:00719390* _xmlNewTextWriter
0001:00719720* _xmlNewTextWriterDoc
0001:007199f0* _xmlNewTextWriterTree
0001:00719d60  _xmlTextWriterStartDocument
0001:0071a1b0  _xmlTextWriterEndDocument
0001:0071ae00  _xmlTextWriterEndElement
0001:0071c560  _xmlTextWriterEndPI
0001:0071ca10  _xmlTextWriterEndCDATA
0001:0071d180  _xmlTextWriterEndDTD
0001:0071a670  _xmlTextWriterEndComment
0001:0071a3b0  _xmlTextWriterStartComment
0001:0071a7e0* _xmlTextWriterWriteFormatComment
0001:0071a860* _xmlTextWriterWriteVFormatComment
0001:0071a930  _xmlTextWriterWriteComment
0001:0071b3d0  _xmlTextWriterWriteString
0001:0071a990  _xmlTextWriterStartElement
0001:0071ba50  _xmlTextWriterEndAttribute
0001:0071acf0  _xmlTextWriterStartElementNS
0001:0071bc30  _xmlTextWriterWriteAttribute
0001:0071af60  _xmlTextWriterFullEndElement
0001:0071b080* _xmlTextWriterWriteFormatRaw
0001:0071b0b0* _xmlTextWriterWriteVFormatRaw
0001:0071b300  _xmlTextWriterWriteRaw
0001:0071b190* _xmlTextWriterWriteRawLen
0001:0071b330* _xmlTextWriterWriteFormatString
0001:0071b370* _xmlTextWriterWriteVFormatString
0001:0071b4b0* _xmlTextWriterWriteBase64
0001:0071b570* _xmlTextWriterWriteBinHex
0001:0071b6c0  _xmlTextWriterStartAttribute
0001:0071b810  _xmlTextWriterStartAttributeNS
0001:0071bba0* _xmlTextWriterWriteFormatAttribute
0001:0071bbd0* _xmlTextWriterWriteVFormatAttribute
0001:0071bca0* _xmlTextWriterWriteFormatAttributeNS
0001:0071bce0* _xmlTextWriterWriteVFormatAttributeNS
0001:0071bd50  _xmlTextWriterWriteAttributeNS
0001:0071be60* _xmlTextWriterWriteFormatElement
0001:0071be90* _xmlTextWriterWriteVFormatElement
0001:0071bef0  _xmlTextWriterWriteElement
0001:0071bf60* _xmlTextWriterWriteFormatElementNS
0001:0071bfa0* _xmlTextWriterWriteVFormatElementNS
0001:0071c010  _xmlTextWriterWriteElementNS
0001:0071c180  _xmlTextWriterStartPI
0001:0071c610* _xmlTextWriterWriteFormatPI
0001:0071c640* _xmlTextWriterWriteVFormatPI
0001:0071c6a0  _xmlTextWriterWritePI
0001:0071c7a0  _xmlTextWriterStartCDATA
0001:0071caa0* _xmlTextWriterWriteFormatCDATA
0001:0071cad0* _xmlTextWriterWriteVFormatCDATA
0001:0071cb30  _xmlTextWriterWriteCDATA
0001:0071cc80  _xmlTextWriterStartDTD
0001:0071d780  _xmlTextWriterEndDTDElement
0001:0071dcb0  _xmlTextWriterEndDTDAttlist
0001:0071e1f0  _xmlTextWriterEndDTDEntity
0001:0071d2c0* _xmlTextWriterWriteFormatDTD
0001:0071d300* _xmlTextWriterWriteVFormatDTD
0001:0071d370  _xmlTextWriterWriteDTD
0001:0071d440  _xmlTextWriterStartDTDElement
0001:0071d830* _xmlTextWriterWriteFormatDTDElement
0001:0071d860* _xmlTextWriterWriteVFormatDTDElement
0001:0071d8c0  _xmlTextWriterWriteDTDElement
0001:0071d970  _xmlTextWriterStartDTDAttlist
0001:0071dd60* _xmlTextWriterWriteFormatDTDAttlist
0001:0071dd90* _xmlTextWriterWriteVFormatDTDAttlist
0001:0071ddf0  _xmlTextWriterWriteDTDAttlist
0001:0071de80  _xmlTextWriterStartDTDEntity
0001:0071e2e0* _xmlTextWriterWriteFormatDTDInternalEntity
0001:0071e320* _xmlTextWriterWriteVFormatDTDInternalEntity
0001:0071e390* _xmlTextWriterWriteDTDInternalEntity
0001:0071e5d0* _xmlTextWriterWriteDTDExternalEntityContents
0001:0071e8f0* _xmlTextWriterWriteDTDNotation
0001:0071eff0  _xmlNewTextWriterFilename
0001:0071f170  _xmlNewTextWriterMemory
0001:0071f2d0* _xmlNewTextWriterPushParser
0001:0071f430  _xmlFreeTextWriter
0001:0071f4f0  _xmlTextWriterWriteDTDEntity
0001:0071f600* _xmlTextWriterWriteDTDExternalEntity
0001:0071f6b0  _xmlTextWriterFlush
0001:0071f6e0  _xmlTextWriterSetIndent
0001:0071f710  _xmlTextWriterSetIndentString
Module: U:\usr\lib\libos2.lib(code2.obj)
0001:0071fbf4  DosGetMessage
0001:0071fbe0* __msgseg32
Module: U:\tmp\ldconv_gcc444_a_92b84c4a69841efbf0.lib(emx-ctordtor.obj)
0001:0071fc10  ___ctordtorTerm
0001:0071fc42  ___ctordtorInit
Module: U:\extras\lib\xml2.lib(nanohttp.obj)
0001:0071fc80  _xmlNanoHTTPRead
0001:0071feb0* _xmlNanoHTTPMethodRedir
0001:007206f0* _xmlNanoHTTPFetch
0001:007208e0* _xmlNanoHTTPInit
0001:00720a40* _xmlNanoHTTPCleanup
0001:00720a80* _xmlNanoHTTPScanProxy
0001:00720b60  _xmlNanoHTTPOpen
0001:00720bb0* _xmlNanoHTTPOpenRedir
0001:00720c00  _xmlNanoHTTPClose
0001:00720c20  _xmlNanoHTTPMethod
0001:00720c60* _xmlNanoHTTPSave
0001:00720d30  _xmlNanoHTTPReturnCode
0001:00720d50* _xmlNanoHTTPAuthHeader
0001:00720d70* _xmlNanoHTTPContentLength
0001:00720d90  _xmlNanoHTTPRedir
0001:00720db0  _xmlNanoHTTPEncoding
0001:00720dd0  _xmlNanoHTTPMimeType
Module: U:\extras\lib\xml2.lib(catalog.obj)
0001:007224c0* _xmlParseCatalogFile
0001:00722c00* _xmlLoadACatalog
0001:007230c0* _xmlACatalogResolve
0001:00723290* _xmlInitializeCatalog
0001:00723510* _xmlLoadCatalogs
0001:007236e0  _xmlCatalogLocalResolve
0001:007237f0* _xmlCatalogGetSystem
0001:00723930* _xmlCatalogGetPublic
0001:00723a70* _xmlFreeCatalog
0001:00723ae0* _xmlConvertSGMLCatalog
0001:00723b50* _xmlLoadSGMLSuperCatalog
0001:00723ce0* _xmlACatalogResolveSystem
0001:00723dc0* _xmlACatalogResolvePublic
0001:00723ef0* _xmlACatalogResolveURI
0001:00723fa0* _xmlACatalogDump
0001:00724040* _xmlACatalogAdd
0001:00724240* _xmlACatalogRemove
0001:007242a0* _xmlNewCatalog
0001:007244a0* _xmlCatalogIsEmpty
0001:00724510* _xmlLoadCatalog
0001:007245f0  _xmlCatalogCleanup
0001:007246f0* _xmlCatalogResolveSystem
0001:00724730* _xmlCatalogResolvePublic
0001:00724770  _xmlCatalogResolve
0001:007247b0  _xmlCatalogResolveURI
0001:00724870* _xmlCatalogDump
0001:007248d0* _xmlCatalogAdd
0001:00724ab0* _xmlCatalogRemove
0001:00724b40* _xmlCatalogConvert
0001:00724bf0  _xmlCatalogGetDefaults
0001:00724ca0* _xmlCatalogSetDefaults
0001:00724d90* _xmlCatalogSetDefaultPrefer
0001:00724e00* _xmlCatalogSetDebug
0001:00724e20  _xmlCatalogFreeLocal
0001:00724e80  _xmlCatalogAddLocal
0001:00724f30  _xmlCatalogLocalResolveURI
Module: U:\extras\lib\xml2.lib(nanoftp.obj)
0001:00728aa0* _xmlNanoFTPInit
0001:00728c60* _xmlNanoFTPScanProxy
0001:00728b60* _xmlNanoFTPUpdateURL
0001:00728e40* _xmlNanoFTPConnect
0001:00729720* _xmlNanoFTPCwd
0001:00729830* _xmlNanoFTPDele
0001:007299b0* _xmlNanoFTPGetConnection
0001:00729de0* _xmlNanoFTPCloseConnection
0001:00729f40* _xmlNanoFTPList
0001:0072a3f0* _xmlNanoFTPGetSocket
0001:0072a5d0* _xmlNanoFTPGet
0001:0072a860* _xmlNanoFTPCleanup
0001:0072a8d0* _xmlNanoFTPProxy
0001:0072a9b0* _xmlNanoFTPNewCtxt
0001:0072aab0* _xmlNanoFTPFreeCtxt
0001:0072ab40* _xmlNanoFTPGetResponse
0001:0072ab50* _xmlNanoFTPCheckResponse
0001:0072ac30* _xmlNanoFTPQuit
0001:0072ad00* _xmlNanoFTPConnectTo
0001:0072ade0  _xmlNanoFTPRead
0001:0072ae70  _xmlNanoFTPOpen
0001:0072af60  _xmlNanoFTPClose
Module: U:\extras\lib\xml2.lib(SAX2.obj)
0001:0072b990  _xmlSAX2ExternalSubset
0001:0072bc50  _xmlSAX2GetEntity
0001:0072c000  _xmlSAX2EntityDecl
0001:0072c300  _xmlSAX2AttributeDecl
0001:0072c660  _xmlSAX2UnparsedEntityDecl
0001:0072c880  _xmlSAX2StartDocument
0001:0072ca60  _xmlSAX2StartElement
0001:0072d0a0* _xmlSAX2StartElementNs
0001:0072d790  _xmlSAX2Characters
0001:0072da10  _xmlSAX2ProcessingInstruction
0001:0072daf0  _xmlSAX2Comment
0001:0072dbd0  _xmlSAXVersion
0001:0072e6a0  _xmlSAX2EndElement
0001:0072dfd0  _xmlSAX2InternalSubset
0001:0072df30  _xmlSAX2IsStandalone
0001:0072df60  _xmlSAX2HasInternalSubset
0001:0072df90  _xmlSAX2HasExternalSubset
0001:0072e0b0  _xmlSAX2ResolveEntity
0001:0072e120  _xmlSAX2GetParameterEntity
0001:0072e180  _xmlSAX2ElementDecl
0001:0072e380  _xmlSAX2NotationDecl
0001:0072e5b0  _xmlSAX2SetDocumentLocator
0001:0072e5c0  _xmlSAX2EndDocument
0001:0072e800  _xmlSAX2Reference
0001:0072e870  _xmlSAX2CDataBlock
0001:0072e750* _xmlSAX2EndElementNs
0001:0072dd00* _xmlSAX2InitHtmlDefaultSAXHandler
0001:0072e860  _xmlSAX2IgnorableWhitespace
0001:0072dde0* _xmlSAX2InitDocbDefaultSAXHandler
0001:0072dec0  _xmlSAX2GetPublicId
0001:0072ded0  _xmlSAX2GetSystemId
0001:0072def0  _xmlSAX2GetLineNumber
0001:0072df10  _xmlSAX2GetColumnNumber
0001:0072e900* _xmlSAXDefaultVersion
0001:0072e930  _xmlSAX2InitDefaultSAXHandler
0001:0072e980  _xmlDefaultSAXHandlerInit
0001:0072e9a0  _htmlDefaultSAXHandlerInit
0001:0072e9c0* _docbDefaultSAXHandlerInit
Module: U:\extras\lib\xml2.lib(threads.obj)
0001:00730940  _xmlNewMutex
0001:00730970  _xmlFreeMutex
0001:00730990  _xmlMutexLock
0001:007309a0  _xmlMutexUnlock
0001:007309b0  _xmlNewRMutex
0001:007309e0  _xmlFreeRMutex
0001:00730a00  _xmlRMutexLock
0001:00730a10  _xmlRMutexUnlock
0001:00730a20* ___xmlGlobalInitMutexLock
0001:00730a30* ___xmlGlobalInitMutexUnlock
0001:00730a40* _xmlGetGlobalState
0001:00730a50  _xmlGetThreadId
0001:00730a60* _xmlIsMainThread
0001:00730a70* _xmlLockLibrary
0001:00730a80* _xmlUnlockLibrary
0001:00730a90  _xmlInitThreads
0001:00730aa0  _xmlCleanupThreads
Module: U:\extras\lib\xml2.lib(SAX.obj)
0001:00730ab0  _initxmlDefaultSAXHandler
0001:00730b90  _inithtmlDefaultSAXHandler
0001:00730c70  _initdocbDefaultSAXHandler
Module: U:\extras\lib\xml2.lib(chvalid.obj)
0001:00730d50  _xmlIsPubidChar_tab
0001:00731164  _xmlIsBaseCharGroup
0001:00731184* _xmlIsCharGroup
0001:0073132c  _xmlIsCombiningGroup
0001:00731388  _xmlIsDigitGroup
0001:007313d8  _xmlIsExtenderGroup
0001:007313f4* _xmlIsIdeographicGroup
0001:00731410  _xmlCharInRange
0001:007314d0* _xmlIsBaseChar
0001:00731550* _xmlIsBlank
0001:00731590* _xmlIsChar
0001:00731600* _xmlIsCombining
0001:00731630* _xmlIsDigit
0001:00731670* _xmlIsExtender
0001:007316b0* _xmlIsIdeographic
0001:007316f0* _xmlIsPubidChar
Module: U:\extras\lib\xml2.lib(dict.obj)
0001:00731710  _xmlDictCreate
0001:00731800  _xmlDictFree
0001:00731970  _xmlDictLookup
0001:00731be0  _xmlDictExists
0001:00731d60  _xmlDictQLookup
0001:00731fa0  _xmlDictCleanup
0001:00731fd0* _xmlDictCreateSub
0001:00732050  _xmlDictReference
0001:007320c0  _xmlDictOwns
0001:00732110* _xmlDictSize
Module: U:\extras\lib\xml2.lib(xmlregexp.obj)
0001:00733400  _xmlRegNewExecCtxt
0001:00733660  _xmlRegFreeExecCtxt
0001:007337d0  _xmlRegExecPushString2
0001:007340e0* _xmlRegexpPrint
0001:00734440  _xmlRegexpCompile
0001:007347b0  _xmlRegexpIsDeterminist
0001:00734990  _xmlNewAutomata
0001:00734af0  _xmlFreeAutomata
0001:00734870  _xmlRegFreeRegexp
0001:00734bc0  _xmlAutomataNewTransition2
0001:00734db0  _xmlAutomataNewNegTrans
0001:00735000  _xmlAutomataNewCountTrans2
0001:007353b0* _xmlAutomataNewCountTrans
0001:007356b0  _xmlAutomataNewOnceTrans2
0001:00735a00* _xmlAutomataNewOnceTrans
0001:00735cb0* _xmlExpNewCtxt
0001:00736380* _xmlExpFree
0001:00737260* _xmlExpSubsume
0001:00737870  _xmlRegExecPushString
0001:007378a0  _xmlRegExecNextValues
0001:007378e0  _xmlRegExecErrInfo
0001:00737960  _xmlRegexpExec
0001:00737980  _xmlAutomataGetInitState
0001:007379a0  _xmlAutomataSetFinalState
0001:007379d0  _xmlAutomataNewTransition
0001:00737b30  _xmlAutomataNewState
0001:00737c20  _xmlAutomataNewEpsilon
0001:00737c70  _xmlAutomataNewAllTrans
0001:00737cd0  _xmlAutomataNewCounter
0001:00737d20  _xmlAutomataNewCountedTrans
0001:00737d70  _xmlAutomataNewCounterTrans
0001:00737dc0  _xmlAutomataCompile
0001:00737e00* _xmlAutomataIsDeterminist
0001:00737e20* _xmlExpFreeCtxt
0001:00737e60* _xmlExpRef
0001:00737e70* _xmlExpNewAtom
0001:00737ee0* _xmlExpNewOr
0001:00737f60* _xmlExpNewSeq
0001:00737fe0* _xmlExpNewRange
0001:00738060* _xmlExpGetLanguage
0001:007380b0* _xmlExpGetStart
0001:00738100* _xmlExpIsNillable
0001:00738120* _xmlExpStringDerive
0001:007381a0* _xmlExpExpDerive
0001:00738220* _xmlExpParse
0001:007382a0* _xmlExpDump
0001:007382d0* _xmlExpMaxToken
0001:007382f0* _xmlExpCtxtNbNodes
0001:00738310* _xmlExpCtxtNbCons
0002:00004a2c* _forbiddenExp
0002:00004a4c* _emptyExp
Module: U:\extras\lib\xml2.lib(list.obj)
0001:00741a90  _xmlListCreate
0001:00741b60  _xmlListSearch
0001:00741bd0* _xmlListReverseSearch
0001:00741c70  _xmlListInsert
0001:00741d00  _xmlListAppend
0001:00741d90  _xmlListDelete
0001:00741e00  _xmlListRemoveFirst
0001:00741ea0* _xmlListRemoveLast
0001:00741f40* _xmlListRemoveAll
0001:00741f80  _xmlListClear
0001:00741fe0  _xmlListEmpty
0001:00742000  _xmlListFront
0001:00742020* _xmlListEnd
0001:00742040  _xmlListSize
0001:00742070  _xmlListPopFront
0001:007420c0* _xmlListPopBack
0001:00742110  _xmlListPushFront
0001:00742180* _xmlListPushBack
0001:007421f0  _xmlLinkGetData
0001:00742210* _xmlListReverse
0001:00742250* _xmlListSort
0001:00742520  _xmlListWalk
0001:00742570* _xmlListReverseWalk
0001:007425c0* _xmlListMerge
0001:007426b0* _xmlListDup
0001:00742820* _xmlListCopy
Module: U:\extras\lib\xml2.lib(xmlschemastypes.obj)
0001:00742b30  _xmlSchemaInitTypes
0001:007433a0  _xmlSchemaIsBuiltInTypeFacet
0001:00743530  _xmlSchemaGetBuiltInType
0001:007437d0  _xmlSchemaFreeValue
0001:00743a10  _xmlSchemaCollapseString
0001:00743be0  _xmlSchemaValPredefTypeNode
0001:00743ca0  _xmlSchemaCopyValue
0001:00743f60  _xmlSchemaValidateListSimpleTypeFacet
0001:00744020  _xmlSchemaValidateFacet
0001:00744210  _xmlSchemaGetCanonValue
0001:00745140* _xmlSchemaGetCanonValueWhtsp
0001:00745340  _xmlSchemaCleanupTypes
0001:007453e0  _xmlSchemaValueAppend
0001:00745400  _xmlSchemaValueGetNext
0001:00745420  _xmlSchemaValueGetAsString
0001:00745510  _xmlSchemaValueGetAsBoolean
0001:00745530* _xmlSchemaNewStringValue
0001:00745580  _xmlSchemaNewNOTATIONValue
0001:007455e0  _xmlSchemaNewQNameValue
0001:00745630  _xmlSchemaGetPredefinedType
0001:00745680* _xmlSchemaGetBuiltInListSimpleTypeItemType
0001:007456d0  _xmlSchemaWhiteSpaceReplace
0001:00745780  _xmlSchemaValPredefTypeNodeNoNorm
0001:007457e0  _xmlSchemaValidatePredefinedType
0001:00745810  _xmlSchemaCompareValues
0001:007458a0  _xmlSchemaCompareValuesWhtsp
0001:00745900  _xmlSchemaGetFacetValueAsULong
0001:00745920* _xmlSchemaValidateLengthFacet
0001:00745970  _xmlSchemaValidateLengthFacetWhtsp
0001:00745980  _xmlSchemaValidateFacetWhtsp
0001:00745990  _xmlSchemaGetValType
Module: U:\extras\lib\xml2.lib(xmlmemory.obj)
0001:0074d530* _xmlMallocLoc
0001:0074dd40* _xmlMemoryDump
0001:0074dd70  _xmlInitMemory
0001:0074d680* _xmlMallocAtomicLoc
0001:0074d7f0* _xmlReallocLoc
0001:0074da10* _xmlMemFree
0001:0074dba0* _xmlMemStrdupLoc
0001:0074de00* _xmlMallocBreakpoint
0001:0074de40* _xmlMemMalloc
0001:0074de70* _xmlMemRealloc
0001:0074dea0* _xmlMemoryStrdup
0001:0074ded0* _xmlMemUsed
0001:0074dee0* _xmlMemBlocks
0001:0074df50* _xmlMemDisplay
0001:0074e010  _xmlMemShow
0001:0074e050  _xmlCleanupMemory
0001:0074e090* _xmlMemSetup
0001:0074e0f0* _xmlMemGet
0001:0074e150* _xmlGcMemSetup
0001:0074e1c0* _xmlGcMemGet
Module: U:\extras\lib\libz.lib(adler32.obj)
0001:0074e240  _adler32
0001:0074e4b0* _adler32_combine
Module: U:\extras\lib\libz.lib(trees.obj)
0001:0074ebc0  __dist_code
0001:0074edc0  __length_code
0001:0074efb8  __tr_stored_block
0001:0074f05c  __tr_align
0001:0074f2d0  __tr_flush_block
0001:0074fc0c  __tr_init
0001:0074fce0* __tr_tally
Module: U:\extras\lib\libz.lib(inftrees.obj)
0001:00750cc0* _inflate_copyright
0001:00750e00  _inflate_table
Module: U:\extras\lib\libz.lib(inffast.obj)
0001:00751390  _inflate_fast
Module: U:\extras\lib\xml2.lib(pattern.obj)
0001:007517d0  _xmlFreePattern
0001:00751950  _xmlPatterncompile
0001:00751d00  _xmlFreePatternList
0001:00751d30  _xmlFreeStreamCtxt
0001:00751d70  _xmlStreamPush
0001:00751da0  _xmlStreamPushNode
0001:00751db0  _xmlStreamPushAttr
0001:00751de0  _xmlStreamPop
0001:00751e30  _xmlStreamWantsAnyNode
0001:00751e60  _xmlPatternMatch
0001:00751eb0  _xmlPatternGetStreamCtxt
0001:00751fd0  _xmlPatternStreamable
0001:00752000  _xmlPatternMaxDepth
0001:00752070  _xmlPatternMinDepth
0001:007520c0  _xmlPatternFromRoot
Module: U:\extras\lib\xml2.lib(debugXML.obj)
0001:00755760* _xmlLsCountNode
0001:00755860* _xmlLsOneNode
0001:00755cc0* _xmlShellPrintXPathError
0001:00755da0* _xmlShellList
0001:00755e40* _xmlShellLoad
0001:00755f10* _xmlShellWrite
0001:00756050* _xmlShellSave
0001:00756100* _xmlShellDu
0001:00756d10* _xmlShell
0001:00758950  _xmlDebugDumpString
0001:00758a40  _xmlDebugDumpAttr
0001:00758b50* _xmlDebugDumpEntities
0001:00758d00* _xmlDebugDumpAttrList
0001:00758db0  _xmlDebugDumpOneNode
0001:00758e40* _xmlDebugDumpNode
0001:00758ee0* _xmlDebugDumpNodeList
0001:00758f80* _xmlDebugDumpDocumentHead
0001:00759030* _xmlDebugDumpDocument
0001:00759160* _xmlDebugDumpDTD
0001:00759280* _xmlDebugCheckDocument
0001:00759370* _xmlBoolToText
0001:00759390* _xmlShellPrintNode
0001:00759410* _xmlShellPrintXPathResult
0001:00759430* _xmlShellBase
0001:007594e0* _xmlShellDir
0001:007596f0* _xmlShellCat
0001:007597b0* _xmlShellValidate
0001:00759860* _xmlShellPwd
Module: U:\extras\lib\xml2.lib(xpointer.obj)
0001:0075fbd0  _xmlXPtrNewRangeNodeObject
0001:0075fdf0  _xmlXPtrLocationSetAdd
0001:00760280  _xmlXPtrEval
0001:00760670* _xmlXPtrBuildNodeList
0001:00760870* _xmlXPtrStartPointFunction
0001:00760f40* _xmlXPtrEndPointFunction
0001:00761620* _xmlXPtrRangeFunction
0001:00761b00* _xmlXPtrRangeInsideFunction
0001:00761fe0* _xmlXPtrRangeToFunction
0001:007622f0  _xmlXPtrAdvanceNode
0001:007623a0* _xmlXPtrStringRangeFunction
0001:00762ec0* _xmlXPtrEvalRangePredicate
0001:007632f0  _xmlXPtrNewRange
0001:00763400* _xmlXPtrNewRangePoints
0001:00763520* _xmlXPtrNewRangePointNode
0001:00763620* _xmlXPtrNewRangeNodePoint
0001:00763740* _xmlXPtrNewRangeNodes
0001:00763840* _xmlXPtrNewCollapsedRange
0001:00763930  _xmlXPtrLocationSetCreate
0001:00763ac0  _xmlXPtrLocationSetMerge
0001:00763b10* _xmlXPtrLocationSetDel
0001:00763b90* _xmlXPtrLocationSetRemove
0001:00763bd0  _xmlXPtrFreeLocationSet
0001:00763c30* _xmlXPtrNewLocationSetNodes
0001:00763e40* _xmlXPtrNewLocationSetNodeSet
0001:00764040  _xmlXPtrWrapLocationSet
0001:00764150  _xmlXPtrNewContext
0001:00764260* _xmlXPtrHereFunction
0001:007642d0* _xmlXPtrOriginFunction
Module: U:\extras\lib\libcrypto.lib(err.obj)
0001:00766541* _ERR_get_implementation
0001:00766553* _ERR_set_implementation
0001:00766fa6* _ERR_load_ERR_strings
0001:0076704d* _ERR_load_strings
0001:0076706c* _ERR_unload_strings
0001:007670b1* _ERR_free_strings
0001:007670c8  _ERR_put_error
0001:00767b3c* _ERR_get_state
0001:00767225  _ERR_clear_error
0001:0076730a* _ERR_get_error
0001:00767346* _ERR_get_error_line
0001:00767380  _ERR_get_error_line_data
0001:007673b8  _ERR_peek_error
0001:007673f4* _ERR_peek_error_line
0001:0076742e* _ERR_peek_error_line_data
0001:00767466  _ERR_peek_last_error
0001:007674a2* _ERR_peek_last_error_line
0001:007674dc* _ERR_peek_last_error_line_data
0001:00767767  _ERR_error_string_n
0001:0076799d* _ERR_lib_error_string
0001:007679e7* _ERR_func_error_string
0001:00767a4e* _ERR_reason_error_string
0001:00767913* _ERR_error_string
0001:00767945* _ERR_get_string_table
0001:00767962* _ERR_get_err_state_table
0001:00767980* _ERR_release_err_state_table
0001:00767ada* _ERR_remove_thread_state
0001:00767b28* _ERR_remove_state
0001:00767c79* _ERR_get_next_error_library
0001:00767c90* _ERR_set_error_data
0001:00767d35  _ERR_add_error_data
0001:00767e42  _ERR_set_mark
0001:00767e99  _ERR_pop_to_mark
Module: U:\extras\lib\libssl.lib(ssl_sess.obj)
0001:00768030  _SSL_get_session
0001:00768049* _SSL_get1_session
0001:007680c3* _SSL_SESSION_get_ex_new_index
0001:007680fa* _SSL_SESSION_set_ex_data
0001:00768121* _SSL_SESSION_get_ex_data
0001:00768141  _SSL_SESSION_new
0001:0076829f* _SSL_SESSION_get_id
0001:00768323  _ssl_get_new_session
0001:00769153  _SSL_SESSION_free
0001:007689bd* _ssl_get_prev_session
0001:00768e58  _SSL_CTX_add_session
0001:00769019  _SSL_CTX_remove_session
0001:0076934f  _SSL_set_session
0001:00769527* _SSL_SESSION_set_timeout
0001:0076954a* _SSL_SESSION_get_timeout
0001:00769565* _SSL_SESSION_get_time
0001:00769580* _SSL_SESSION_set_time
0001:007695a1* _SSL_CTX_set_timeout
0001:007695cb* _SSL_CTX_get_timeout
0001:007695e3* _SSL_set_session_secret_cb
0001:00769612* _SSL_set_session_ticket_ext_cb
0001:00769641* _SSL_set_session_ticket_ext
0001:00769825  _SSL_CTX_flush_sessions
0001:007698ce  _ssl_clear_bad_session
0001:00769b0b* _SSL_CTX_sess_set_new_cb
0001:00769b19* _SSL_CTX_sess_get_new_cb
0001:00769b24* _SSL_CTX_sess_set_remove_cb
0001:00769b32* _SSL_CTX_sess_get_remove_cb
0001:00769b3d* _SSL_CTX_sess_set_get_cb
0001:00769b4b* _SSL_CTX_sess_get_get_cb
0001:00769b56* _SSL_CTX_set_info_callback
0001:00769b67* _SSL_CTX_get_info_callback
0001:00769b75* _SSL_CTX_set_client_cert_cb
0001:00769b83* _SSL_CTX_get_client_cert_cb
0001:00769b8e* _SSL_CTX_set_client_cert_engine
0001:00769c36* _SSL_CTX_set_cookie_generate_cb
0001:00769c44* _SSL_CTX_set_cookie_verify_cb
0001:00769c69* _PEM_read_bio_SSL_SESSION
0001:00769ca2* _PEM_read_SSL_SESSION
0001:00769cdb* _PEM_write_bio_SSL_SESSION
0001:00769d2e* _PEM_write_SSL_SESSION
Module: U:\extras\lib\libcrypto.lib(buffer.obj)
0001:00769d99  _BUF_MEM_new
0001:00769e19  _BUF_MEM_free
0001:00769e6d  _BUF_MEM_grow
0001:00769fc9  _BUF_MEM_grow_clean
0001:0076a158  _BUF_strdup
0001:0076a187  _BUF_strndup
0001:0076a296  _BUF_strlcpy
0001:0076a211  _BUF_memdup
0001:0076a2e6  _BUF_strlcat
0001:0076a32b* _BUF_reverse
Module: U:\extras\lib\libssl.lib(ssl_ciph.obj)
0001:0076b371* _ssl_load_ciphers
0001:0076b708  _ssl_cipher_get_evp
0001:0076b9b7  _ssl_get_handshake_digest
0001:0076cbb1  _ssl_create_cipher_list
0001:0076d4b6* _SSL_CIPHER_description
0001:0076d953* _SSL_CIPHER_get_version
0001:0076d993* _SSL_CIPHER_get_name
0001:0076d9ab* _SSL_CIPHER_get_bits
0001:0076d9dd  _ssl3_comp_find
0001:0076da43  _SSL_COMP_get_compression_methods
0001:0076da55* _SSL_COMP_add_compression_method
0001:0076dbe6* _SSL_COMP_get_name
Module: U:\extras\lib\libcrypto.lib(stack.obj)
0001:0076dc30* _STACK_version
0001:0076dc58  _sk_set_cmp_func
0001:0076dc92  _sk_dup
0001:0076dd7f  _sk_new
0001:0076e2b5  _sk_free
0001:0076dd6b  _sk_new_null
0001:0076de45  _sk_insert
0001:0076df5e  _sk_delete_ptr
0001:0076dfaa  _sk_delete
0001:0076e369  _sk_sort
0001:0076e110  _sk_find
0001:0076e132* _sk_find_ex
0001:0076e154  _sk_push
0001:0076e177* _sk_unshift
0001:0076e199* _sk_shift
0001:0076e1d1  _sk_pop
0001:0076e20b  _sk_zero
0001:0076e257  _sk_pop_free
0001:0076e2e9  _sk_num
0001:0076e300  _sk_value
0001:0076e332  _sk_set
0001:0076e3bc  _sk_is_sorted
Module: U:\extras\lib\libcrypto.lib(mem.obj)
0001:0076e429* _CRYPTO_set_mem_functions
0001:0076e4a2* _CRYPTO_set_mem_ex_functions
0001:0076e51b* _CRYPTO_set_locked_mem_functions
0001:0076e562* _CRYPTO_set_locked_mem_ex_functions
0001:0076e5a9* _CRYPTO_set_mem_debug_functions
0001:0076e5eb* _CRYPTO_get_mem_functions
0001:0076e647* _CRYPTO_get_mem_ex_functions
0001:0076e6a3* _CRYPTO_get_locked_mem_functions
0001:0076e6dc* _CRYPTO_get_locked_mem_ex_functions
0001:0076e715* _CRYPTO_get_mem_debug_functions
0001:0076e76f  _CRYPTO_malloc_locked
0001:0076e847  _CRYPTO_free_locked
0001:0076e89b  _CRYPTO_malloc
0001:0076e973* _CRYPTO_strdup
0001:0076e9b5  _CRYPTO_realloc
0001:0076ea98  _CRYPTO_realloc_clean
0001:0076ebb3  _CRYPTO_free
0001:0076ec0d* _CRYPTO_remalloc
0001:0076ec47* _CRYPTO_set_mem_debug_options
0001:0076ec66* _CRYPTO_get_mem_debug_options
Module: U:\extras\lib\libssl.lib(ssl_cert.obj)
0001:0076ecb3  _SSL_get_ex_data_X509_STORE_CTX_idx
0001:0076edd1  _ssl_cert_new
0001:0076ee64  _ssl_cert_dup
0001:0076f305  _ssl_cert_free
0001:0076f407  _ssl_cert_inst
0001:0076f49c  _ssl_sess_cert_new
0001:0076f530  _ssl_sess_cert_free
0001:0076f627  _ssl_set_peer_cert_type
0001:0076f650  _ssl_verify_cert_chain
0001:0076f825* _SSL_dup_CA_list
0001:0076f8a8* _SSL_set_client_CA_list
0001:0076f8c8* _SSL_CTX_set_client_CA_list
0001:0076f8e8* _SSL_CTX_get_client_CA_list
0001:0076f8f6  _SSL_get_client_CA_list
0001:0076f9e7* _SSL_add_client_CA
0001:0076fa07* _SSL_CTX_add_client_CA
0001:0076fa45* _SSL_load_client_CA_file
0001:0076fc39* _SSL_add_file_cert_subjects_to_stack
0001:0076fdd5* _SSL_add_dir_cert_subjects_to_stack
Module: U:\extras\lib\libcrypto.lib(cryptlib.obj)
0001:007701bf* _CRYPTO_get_new_lockid
0001:0077028e* _CRYPTO_num_locks
0001:00770298* _CRYPTO_get_new_dynlockid
0001:0077095d  _CRYPTO_lock
0001:0077054d* _CRYPTO_destroy_dynlockid
0001:0077068b* _CRYPTO_get_dynlock_value
0001:00770743* _CRYPTO_get_dynlock_create_callback
0001:0077074d* _CRYPTO_get_dynlock_lock_callback
0001:00770757* _CRYPTO_get_dynlock_destroy_callback
0001:00770761* _CRYPTO_set_dynlock_create_callback
0001:0077076e* _CRYPTO_set_dynlock_lock_callback
0001:0077077b* _CRYPTO_set_dynlock_destroy_callback
0001:00770788* _CRYPTO_get_locking_callback
0001:00770792* _CRYPTO_get_add_lock_callback
0001:0077079c* _CRYPTO_set_locking_callback
0001:007707a9* _CRYPTO_set_add_lock_callback
0001:007707b6* _CRYPTO_THREADID_set_numeric
0001:007707ea* _CRYPTO_THREADID_set_pointer
0001:00770836* _CRYPTO_THREADID_set_callback
0001:00770858* _CRYPTO_THREADID_get_callback
0001:00770862  _CRYPTO_THREADID_current
0001:007708b8  _CRYPTO_THREADID_cmp
0001:007708da  _CRYPTO_THREADID_cpy
0001:007708fc  _CRYPTO_THREADID_hash
0001:00770907* _CRYPTO_get_id_callback
0001:00770911* _CRYPTO_set_id_callback
0001:0077091e* _CRYPTO_thread_id
0001:00770b8e  _OpenSSLDie
0001:00770a07  _CRYPTO_add_lock
0001:00770ab4* _CRYPTO_get_lock_name
0001:00770b15* _OPENSSL_ia32cap_loc
0001:00770b1f* _OPENSSL_cpuid_setup
0001:00770b24* _OPENSSL_showfatal
0001:00770b4d* _OPENSSL_isservice
0001:00770bba* _OPENSSL_stderr
0002:0001ed00* _OPENSSL_ia32cap_P
0002:0001ed04* _OPENSSL_NONPIC_relocated
Module: U:\extras\lib\libcrypto.lib(x509_vpm.obj)
0001:00770c52  _X509_VERIFY_PARAM_new
0001:00770ca2  _X509_VERIFY_PARAM_free
0001:00770cc0  _X509_VERIFY_PARAM_inherit
0001:0077100a* _X509_VERIFY_PARAM_set1_policies
0001:00770e68  _X509_VERIFY_PARAM_set1
0001:00770eab* _X509_VERIFY_PARAM_set1_name
0001:00770eee  _X509_VERIFY_PARAM_set_flags
0001:00770f26* _X509_VERIFY_PARAM_clear_flags
0001:00770f43* _X509_VERIFY_PARAM_get_flags
0001:00770f4e  _X509_VERIFY_PARAM_set_purpose
0001:00770f6b  _X509_VERIFY_PARAM_set_trust
0001:00770f88  _X509_VERIFY_PARAM_set_depth
0001:00770f96  _X509_VERIFY_PARAM_set_time
0001:00770fb5* _X509_VERIFY_PARAM_add0_policy
0001:0077110b  _X509_VERIFY_PARAM_get_depth
0001:00771287* _X509_VERIFY_PARAM_add0_table
0001:00771334  _X509_VERIFY_PARAM_lookup
0001:00771399* _X509_VERIFY_PARAM_table_cleanup
Module: U:\extras\lib\libcrypto.lib(ex_data.obj)
0001:0077143d* _CRYPTO_get_ex_data_implementation
0001:00771458* _CRYPTO_set_ex_data_implementation
0001:007721e1  _CRYPTO_get_ex_data
0001:007720fc  _CRYPTO_set_ex_data
0001:00771fcb* _CRYPTO_ex_data_new_class
0001:00771fea* _CRYPTO_cleanup_all_ex_data
0001:0077200a  _CRYPTO_get_ex_new_index
0001:00772060  _CRYPTO_new_ex_data
0001:00772094  _CRYPTO_dup_ex_data
0001:007720c8  _CRYPTO_free_ex_data
Module: U:\extras\lib\libcrypto.lib(lhash.obj)
0001:00772230* _lh_version
0001:00772260  _lh_new
0001:00772b9a  _lh_strhash
0001:007723fd  _lh_free
0001:00772471  _lh_insert
0001:0077258f  _lh_delete
0001:00772669  _lh_retrieve
0001:0077274a  _lh_doall
0001:0077277c  _lh_doall_arg
0001:00772c11  _lh_num_items
Module: U:\extras\lib\libcrypto.lib(bio_lib.obj)
0001:00772c3a  _BIO_new
0001:00772ccc  _BIO_set
0001:00772dc0  _BIO_free
0001:00772eca  _BIO_vfree
0001:00772edd  _BIO_clear_flags
0001:00772ef5  _BIO_test_flags
0001:00772f03  _BIO_set_flags
0001:00772f19* _BIO_get_callback
0001:00772f24* _BIO_set_callback
0001:00772f32* _BIO_set_callback_arg
0001:00772f40* _BIO_get_callback_arg
0001:00772f4b* _BIO_method_name
0001:00772f58  _BIO_method_type
0001:00772f64  _BIO_read
0001:007730bf  _BIO_write
0001:00773224  _BIO_puts
0001:0077337a  _BIO_gets
0001:007734c0  _BIO_indent
0001:00773518  _BIO_int_ctrl
0001:00773583  _BIO_ctrl
0001:00773546* _BIO_ptr_ctrl
0001:00773696  _BIO_callback_ctrl
0001:007737a4* _BIO_ctrl_pending
0001:007737cf* _BIO_ctrl_wpending
0001:007737fa  _BIO_push
0001:00773865  _BIO_pop
0001:007738ee* _BIO_get_retry_BIO
0001:00773948  _BIO_get_retry_reason
0001:00773953  _BIO_find_type
0001:007739bf  _BIO_next
0001:007739d7  _BIO_free_all
0001:00773a13* _BIO_dup_chain
0001:00773b4b  _BIO_copy_next_retry
0001:00773b87* _BIO_get_ex_new_index
0001:00773bbe* _BIO_set_ex_data
0001:00773be2* _BIO_get_ex_data
0001:00773bff* _BIO_number_read
0001:00773c17* _BIO_number_written
Module: U:\extras\lib\libcrypto.lib(x_exten.obj)
0001:00773ca0  _X509_EXTENSION_it
0001:00773d00  _X509_EXTENSIONS_it
0001:00773d1c* _d2i_X509_EXTENSION
0001:00773d45* _i2d_X509_EXTENSION
0001:00773d67  _X509_EXTENSION_new
0001:00773d7b  _X509_EXTENSION_free
0001:00773d96  _d2i_X509_EXTENSIONS
0001:00773dbf  _i2d_X509_EXTENSIONS
0001:00773de1  _X509_EXTENSION_dup
Module: U:\extras\lib\libcrypto.lib(ocsp_asn.obj)
0001:00773e80* _OCSP_SIGNATURE_it
0001:00773e9c* _d2i_OCSP_SIGNATURE
0001:00773ec5* _i2d_OCSP_SIGNATURE
0001:00773ee7* _OCSP_SIGNATURE_new
0001:00773efb* _OCSP_SIGNATURE_free
0001:00773fb0* _OCSP_CERTID_it
0001:00773fcc* _d2i_OCSP_CERTID
0001:00773ff5* _i2d_OCSP_CERTID
0001:00774017* _OCSP_CERTID_new
0001:0077402b* _OCSP_CERTID_free
0001:007740b0* _OCSP_ONEREQ_it
0001:007740cc* _d2i_OCSP_ONEREQ
0001:007740f5* _i2d_OCSP_ONEREQ
0001:00774117* _OCSP_ONEREQ_new
0001:0077412b* _OCSP_ONEREQ_free
0001:007741e0* _OCSP_REQINFO_it
0001:007741fc* _d2i_OCSP_REQINFO
0001:00774225* _i2d_OCSP_REQINFO
0001:00774247* _OCSP_REQINFO_new
0001:0077425b* _OCSP_REQINFO_free
0001:007742e0* _OCSP_REQUEST_it
0001:007742fc* _d2i_OCSP_REQUEST
0001:00774325* _i2d_OCSP_REQUEST
0001:00774347* _OCSP_REQUEST_new
0001:0077435b* _OCSP_REQUEST_free
0001:007743d0* _OCSP_RESPBYTES_it
0001:007743ec* _d2i_OCSP_RESPBYTES
0001:00774415* _i2d_OCSP_RESPBYTES
0001:00774437* _OCSP_RESPBYTES_new
0001:0077444b* _OCSP_RESPBYTES_free
0001:007744d0* _OCSP_RESPONSE_it
0001:007744ec* _d2i_OCSP_RESPONSE
0001:00774515* _i2d_OCSP_RESPONSE
0001:00774537* _OCSP_RESPONSE_new
0001:0077454b* _OCSP_RESPONSE_free
0001:007745c0* _OCSP_RESPID_it
0001:007745dc  _d2i_OCSP_RESPID
0001:00774605  _i2d_OCSP_RESPID
0001:00774627* _OCSP_RESPID_new
0001:0077463b  _OCSP_RESPID_free
0001:007746c0* _OCSP_REVOKEDINFO_it
0001:007746dc* _d2i_OCSP_REVOKEDINFO
0001:00774705* _i2d_OCSP_REVOKEDINFO
0001:00774727* _OCSP_REVOKEDINFO_new
0001:0077473b* _OCSP_REVOKEDINFO_free
0001:007747d0* _OCSP_CERTSTATUS_it
0001:007747ec* _d2i_OCSP_CERTSTATUS
0001:00774815* _i2d_OCSP_CERTSTATUS
0001:00774837* _OCSP_CERTSTATUS_new
0001:0077484b* _OCSP_CERTSTATUS_free
0001:00774920* _OCSP_SINGLERESP_it
0001:0077493c* _d2i_OCSP_SINGLERESP
0001:00774965* _i2d_OCSP_SINGLERESP
0001:00774987* _OCSP_SINGLERESP_new
0001:0077499b* _OCSP_SINGLERESP_free
0001:00774a70* _OCSP_RESPDATA_it
0001:00774a8c* _d2i_OCSP_RESPDATA
0001:00774ab5* _i2d_OCSP_RESPDATA
0001:00774ad7* _OCSP_RESPDATA_new
0001:00774aeb* _OCSP_RESPDATA_free
0001:00774b80* _OCSP_BASICRESP_it
0001:00774b9c* _d2i_OCSP_BASICRESP
0001:00774bc5* _i2d_OCSP_BASICRESP
0001:00774be7* _OCSP_BASICRESP_new
0001:00774bfb* _OCSP_BASICRESP_free
0001:00774c80  _OCSP_CRLID_it
0001:00774c9c* _d2i_OCSP_CRLID
0001:00774cc5* _i2d_OCSP_CRLID
0001:00774ce7* _OCSP_CRLID_new
0001:00774cfb* _OCSP_CRLID_free
0001:00774d70  _OCSP_SERVICELOC_it
0001:00774d8c* _d2i_OCSP_SERVICELOC
0001:00774db5* _i2d_OCSP_SERVICELOC
0001:00774dd7* _OCSP_SERVICELOC_new
0001:00774deb* _OCSP_SERVICELOC_free
Module: U:\extras\lib\libcrypto.lib(x_name.obj)
0001:00774ee0  _X509_NAME_ENTRY_it
0001:00774efc* _d2i_X509_NAME_ENTRY
0001:00774f25* _i2d_X509_NAME_ENTRY
0001:00774f47  _X509_NAME_ENTRY_new
0001:00774f5b  _X509_NAME_ENTRY_free
0001:00774f76  _X509_NAME_ENTRY_dup
0001:00774fd0* _X509_NAME_ENTRIES_it
0001:00775030* _X509_NAME_INTERNAL_it
0001:00775050* _x509_name_ff
0001:00775080  _X509_NAME_it
0001:0077509c  _d2i_X509_NAME
0001:007750c5  _i2d_X509_NAME
0001:007750e7  _X509_NAME_new
0001:007750fb  _X509_NAME_free
0001:00775116  _X509_NAME_dup
0001:00775bc6  _X509_NAME_set
Module: U:\extras\lib\libcrypto.lib(bss_sock.obj)
0001:00775c37  _BIO_s_socket
0001:00775c41* _BIO_new_socket
0001:00775f16* _BIO_sock_should_retry
0001:00775f46* _BIO_sock_non_fatal_error
Module: U:\extras\lib\libcrypto.lib(x509_cmp.obj)
0001:00775f70* _X509_issuer_and_serial_cmp
0001:00776246  _X509_NAME_cmp
0001:00775fc6* _X509_issuer_and_serial_hash
0001:007760cd* _X509_issuer_name_cmp
0001:007760f1  _X509_subject_name_cmp
0001:00776115  _X509_CRL_cmp
0001:00776139  _X509_CRL_match
0001:00776161  _X509_get_issuer_name
0001:0077616e* _X509_issuer_name_hash
0001:00776300  _X509_NAME_hash
0001:00776186* _X509_issuer_name_hash_old
0001:00776389* _X509_NAME_hash_old
0001:0077619e  _X509_get_subject_name
0001:007761ab  _X509_get_serialNumber
0001:007761b8* _X509_subject_name_hash
0001:007761d0* _X509_subject_name_hash_old
0001:007761e8  _X509_cmp
0001:00776415  _X509_find_by_issuer_and_serial
0001:0077649d* _X509_find_by_subject
0001:007764fe  _X509_get_pubkey
0001:0077652c  _X509_get0_pubkey_bitstr
0001:00776554  _X509_check_private_key
Module: U:\extras\lib\libssl.lib(s3_pkt.obj)
0001:00776669* _ssl3_read_n
0001:0077705a* _ssl3_do_uncompress
0001:0077891d  _ssl3_send_alert
0001:007770d8* _ssl3_do_compress
0001:00777156  _ssl3_write_bytes
0001:00777755* _ssl3_write_pending
0001:00777928  _ssl3_read_bytes
0001:007787a5* _ssl3_do_change_cipher_spec
0001:007789ec  _ssl3_dispatch_alert
Module: U:\extras\lib\libcrypto.lib(x509_lu.obj)
0001:00778b8a* _X509_LOOKUP_new
0001:00778c1f* _X509_LOOKUP_free
0001:00778c63* _X509_LOOKUP_init
0001:00778ca1* _X509_LOOKUP_shutdown
0001:00778cdf  _X509_LOOKUP_ctrl
0001:00778d39* _X509_LOOKUP_by_subject
0001:00778d96* _X509_LOOKUP_by_issuer_serial
0001:00778de9* _X509_LOOKUP_by_fingerprint
0001:00778e3c* _X509_LOOKUP_by_alias
0001:00778f18  _X509_STORE_new
0001:0077909a  _X509_STORE_free
0001:00779161  _X509_STORE_add_lookup
0001:00779205* _X509_STORE_get_by_subject
0001:007797d4* _X509_OBJECT_retrieve_by_subject
0001:007795fd* _X509_OBJECT_up_ref_count
0001:00779347  _X509_STORE_add_cert
0001:00779cb1* _X509_OBJECT_retrieve_match
0001:0077967a* _X509_OBJECT_free_contents
0001:007794a2  _X509_STORE_add_crl
0001:007797ab* _X509_OBJECT_idx_by_subject
0001:00779817  _X509_STORE_get1_certs
0001:00779a69  _X509_STORE_get1_crls
0001:00779dc1  _X509_STORE_CTX_get1_issuer
0001:00779fe0* _X509_STORE_set_flags
0001:00779ffd* _X509_STORE_set_depth
0001:0077a01f* _X509_STORE_set_purpose
0001:0077a03c* _X509_STORE_set_trust
0001:0077a059* _X509_STORE_set1_param
0001:0077a076* _X509_STORE_set_verify_cb
Module: U:\extras\lib\libcrypto.lib(names.obj)
0001:0077a090* _EVP_add_cipher
0001:0077a108* _EVP_add_digest
0001:0077a21d  _EVP_get_cipherbyname
0001:0077a23e  _EVP_get_digestbyname
0001:0077a25f* _EVP_cleanup
0001:0077a325* _EVP_CIPHER_do_all
0001:0077a354* _EVP_CIPHER_do_all_sorted
0001:0077a3fa* _EVP_MD_do_all
0001:0077a429* _EVP_MD_do_all_sorted
Module: U:\extras\lib\libcrypto.lib(rand_lib.obj)
0001:0077a460  _RAND_set_rand_method
0001:0077a495* _RAND_get_rand_method
0001:0077a4fe* _RAND_set_rand_engine
0001:0077a567* _RAND_cleanup
0001:0077a59b  _RAND_seed
0001:0077a5ce  _RAND_add
0001:0077a61d  _RAND_bytes
0001:0077a659  _RAND_pseudo_bytes
0001:0077a695  _RAND_status
Module: U:\extras\lib\libcrypto.lib(x_x509.obj)
0001:0077a810  _X509_CINF_it
0001:0077a82c* _d2i_X509_CINF
0001:0077a855* _i2d_X509_CINF
0001:0077a877* _X509_CINF_new
0001:0077a88b* _X509_CINF_free
0001:0077aab0  _X509_it
0001:0077aacc  _d2i_X509
0001:0077aaf5  _i2d_X509
0001:0077ab17* _X509_new
0001:0077ab2b  _X509_free
0001:0077ab46* _X509_dup
0001:0077ab61* _X509_get_ex_new_index
0001:0077ab98* _X509_set_ex_data
0001:0077abbc* _X509_get_ex_data
0001:0077abd9  _d2i_X509_AUX
0001:0077ac64  _i2d_X509_AUX
Module: U:\extras\lib\libcrypto.lib(eng_init.obj)
0001:0077acb0  _engine_unlocked_init
0001:0077ad16  _engine_unlocked_finish
0001:0077ae07  _ENGINE_init
0001:0077aea1  _ENGINE_finish
Module: U:\extras\lib\libcrypto.lib(rsa_lib.obj)
0001:0077af90* _RSA_version
0001:0077afb6  _RSA_new
0001:0077b083* _RSA_new_method
0001:0077afd0* _RSA_set_default_method
0001:0077afdd* _RSA_get_default_method
0001:0077affd* _RSA_get_method
0001:0077b008* _RSA_set_method
0001:0077b343  _RSA_free
0001:0077b4fc  _RSA_up_ref
0001:0077b53f* _RSA_get_ex_new_index
0001:0077b576* _RSA_set_ex_data
0001:0077b59a* _RSA_get_ex_data
0001:0077b5b7  _RSA_size
0001:0077b5da  _RSA_public_encrypt
0001:0077b60f  _RSA_private_encrypt
0001:0077b644  _RSA_private_decrypt
0001:0077b679  _RSA_public_decrypt
0001:0077b6ae  _RSA_flags
0001:0077b6c9* _RSA_blinding_off
0001:0077b715* _RSA_blinding_on
0001:0077b894  _RSA_setup_blinding
0001:0077bb1f* _RSA_memory_lock
Module: U:\extras\lib\libcrypto.lib(dh_lib.obj)
0001:0077bd10* _DH_version
0001:0077bd41* _DH_set_default_method
0001:0077bd4e* _DH_get_default_method
0001:0077bd6e* _DH_set_method
0001:0077bddf  _DH_new
0001:0077bdfc* _DH_new_method
0001:0077c070  _DH_free
0001:0077c1e1  _DH_up_ref
0001:0077c224* _DH_get_ex_new_index
0001:0077c25b* _DH_set_ex_data
0001:0077c27f* _DH_get_ex_data
0001:0077c29c  _DH_size
Module: U:\extras\lib\libcrypto.lib(p_lib.obj)
0001:0077c2c0  _EVP_PKEY_bits
0001:0077c2fd  _EVP_PKEY_size
0001:0077c33a* _EVP_PKEY_save_parameters
0001:0077c39f  _EVP_PKEY_copy_parameters
0001:0077c456  _EVP_PKEY_missing_parameters
0001:0077c48d  _EVP_PKEY_cmp_parameters
0001:0077c4e0  _EVP_PKEY_cmp
0001:0077c566  _EVP_PKEY_new
0001:0077c740  _EVP_PKEY_set_type
0001:0077c76a  _EVP_PKEY_set_type_str
0001:0077c793  _EVP_PKEY_assign
0001:0077c7cb* _EVP_PKEY_get0
0001:0077c7d6  _EVP_PKEY_set1_RSA
0001:0077c80f  _EVP_PKEY_get1_RSA
0001:0077c868  _EVP_PKEY_set1_DSA
0001:0077c8a1  _EVP_PKEY_get1_DSA
0001:0077c8fa  _EVP_PKEY_set1_EC_KEY
0001:0077c933  _EVP_PKEY_get1_EC_KEY
0001:0077c98e* _EVP_PKEY_set1_DH
0001:0077c9c7* _EVP_PKEY_get1_DH
0001:0077ca20  _EVP_PKEY_type
0001:0077ca69  _EVP_PKEY_id
0001:0077ca73* _EVP_PKEY_base_id
0001:0077ca88  _EVP_PKEY_free
0001:0077cbd8  _EVP_PKEY_print_public
0001:0077cc4c  _EVP_PKEY_print_private
0001:0077ccbf  _EVP_PKEY_print_params
0001:0077cd27  _EVP_PKEY_get_default_digest_nid
Module: U:\extras\lib\libcrypto.lib(v3_purp.obj)
0001:0077ce81  _X509_check_purpose
0001:0077d05a  _X509_PURPOSE_get_by_id
0001:0077cfbd  _X509_PURPOSE_get0
0001:0077cf3d  _X509_PURPOSE_set
0001:0077cf95* _X509_PURPOSE_get_count
0001:0077d00b* _X509_PURPOSE_get_by_sname
0001:0077d0b4* _X509_PURPOSE_add
0001:0077d32a* _X509_PURPOSE_cleanup
0001:0077d384* _X509_PURPOSE_get_id
0001:0077d38e* _X509_PURPOSE_get0_name
0001:0077d399* _X509_PURPOSE_get0_sname
0001:0077d3a4* _X509_PURPOSE_get_trust
0001:0077d41b* _X509_supported_extension
0001:0077dd0e  _X509_check_ca
0001:0077e1bb  _X509_check_issued
0001:0077e299  _X509_check_akid
Module: U:\extras\lib\libcrypto.lib(obj_dat.obj)
0001:0078d525  _OBJ_bsearch_
0001:0078c781  _check_defer
0001:0078c7a2  _OBJ_cleanup
0001:0078c82d* _OBJ_new_nid
0001:0078c857* _OBJ_add_object
0001:0078ca6f  _OBJ_nid2obj
0001:0078cb64  _OBJ_nid2sn
0001:0078cc5c  _OBJ_nid2ln
0001:0078ce16  _OBJ_obj2nid
0001:0078cebe  _OBJ_txt2obj
0001:0078d494  _OBJ_sn2nid
0001:0078d403  _OBJ_ln2nid
0001:0078d01b  _OBJ_obj2txt
0001:0078d3c9* _OBJ_txt2nid
0001:0078d55c  _OBJ_bsearch_ex_
0001:0078d65e* _OBJ_create_objects
0001:0078d82e* _OBJ_create
0002:0001ee20  _obj_cleanup_defer
Module: U:\extras\lib\libcrypto.lib(evp_enc.obj)
0001:0078d970* _EVP_version
0001:0078d996  _EVP_CIPHER_CTX_init
0001:0078d9c3* _EVP_CIPHER_CTX_new
0001:0078d9fe* _EVP_CipherInit
0001:0078dade  _EVP_CipherInit_ex
0001:0078e83a  _EVP_CIPHER_CTX_cleanup
0001:0078e9c1  _EVP_CIPHER_CTX_ctrl
0001:0078df16  _EVP_CipherUpdate
0001:0078e0ee  _EVP_EncryptUpdate
0001:0078e490  _EVP_DecryptUpdate
0001:0078df78  _EVP_CipherFinal_ex
0001:0078e35d  _EVP_EncryptFinal_ex
0001:0078e623  _EVP_DecryptFinal_ex
0001:0078dfbe* _EVP_CipherFinal
0001:0078e321* _EVP_EncryptFinal
0001:0078e5fc  _EVP_DecryptFinal
0001:0078e004* _EVP_EncryptInit
0001:0078e034  _EVP_EncryptInit_ex
0001:0078e06b* _EVP_DecryptInit
0001:0078e09b  _EVP_DecryptInit_ex
0001:0078e816* _EVP_CIPHER_CTX_free
0001:0078e8e8  _EVP_CIPHER_CTX_set_key_length
0001:0078e98d* _EVP_CIPHER_CTX_set_padding
0001:0078eaab  _EVP_CIPHER_CTX_rand_key
0001:0078eb0d  _EVP_CIPHER_CTX_copy
Module: U:\extras\lib\libcrypto.lib(comp_lib.obj)
0001:0078eccb  _COMP_CTX_new
0001:0078ed57  _COMP_CTX_free
0001:0078ed8f  _COMP_compress_block
0001:0078ee04  _COMP_expand_block
Module: U:\extras\lib\libcrypto.lib(bf_buff.obj)
0001:0078ee87  _BIO_f_buffer
Module: U:\extras\lib\libcrypto.lib(x509_d2.obj)
0001:0078fc60  _X509_STORE_set_default_paths
0001:0078fd13  _X509_STORE_load_locations
Module: U:\extras\lib\libcrypto.lib(digest.obj)
0001:0078fe00  _EVP_MD_CTX_init
0001:0078fe2c  _EVP_MD_CTX_create
0001:0078fe67  _EVP_DigestInit
0001:0078fe94  _EVP_DigestInit_ex
0001:00790160  _EVP_DigestUpdate
0001:00790184  _EVP_DigestFinal
0001:007901e0  _EVP_DigestFinal_ex
0001:00790595  _EVP_MD_CTX_cleanup
0001:00790296  _EVP_MD_CTX_copy
0001:007902bb  _EVP_MD_CTX_copy_ex
0001:007904dd  _EVP_Digest
0001:00790577  _EVP_MD_CTX_destroy
Module: U:\extras\lib\libssl.lib(s2_clnt.obj)
0001:007906aa  _SSLv2_client_method
0001:007906be* _ssl2_connect
0001:00792852* _ssl2_set_certificate
Module: U:\extras\lib\libssl.lib(s3_clnt.obj)
0001:00792c8d  _SSLv3_client_method
0001:00792ca1  _ssl3_connect
0001:00793901* _ssl3_client_hello
0001:00793d42* _ssl3_get_server_hello
0001:00798a1e* _ssl3_check_finished
0001:00794570* _ssl3_get_server_certificate
0001:00794c78* _ssl3_get_key_exchange
0001:0079857e* _ssl3_check_cert_and_algorithm
0001:00795fdf* _ssl3_get_certificate_request
0001:00796b4e* _ssl3_get_server_done
0001:00798335* _ssl3_send_client_certificate
0001:00796c02* _ssl3_send_client_key_exchange
0001:00797e8c* _ssl3_send_client_verify
0001:00796513* _ssl3_get_new_session_ticket
0001:0079688e* _ssl3_get_cert_status
0001:00798acd* _ssl_do_client_cert_cb
Module: U:\extras\lib\libssl.lib(t1_clnt.obj)
0001:00798c2d  _TLSv1_client_method
Module: U:\extras\lib\libssl.lib(s3_both.obj)
0001:00798cc0  _ssl3_do_write
0001:00798df7  _ssl3_send_finished
0001:00798fc0  _ssl3_get_finished
0001:0079920b  _ssl3_send_change_cipher_spec
0001:0079933c  _ssl3_output_cert_chain
0001:00799603  _ssl3_get_message
0001:00799b1d  _ssl_cert_type
0001:00799bd1  _ssl_verify_alarm_type
0001:00799ef5  _ssl3_setup_read_buffer
0001:0079a036  _ssl3_setup_write_buffer
0001:0079a166  _ssl3_setup_buffers
0001:0079a19f  _ssl3_release_write_buffer
0001:0079a205  _ssl3_release_read_buffer
Module: U:\extras\lib\libssl.lib(s3_enc.obj)
0001:0079a4d1  _ssl3_change_cipher_state
0001:0079abf2  _ssl3_setup_key_block
0001:0079ae26  _ssl3_cleanup_key_block
0001:0079ae98  _ssl3_enc
0001:0079b0b8  _ssl3_init_finished_mac
0001:0079b149  _ssl3_free_digest_list
0001:0079b1d2  _ssl3_finish_mac
0001:0079b266  _ssl3_digest_cached_records
0001:0079b43d  _ssl3_cert_verify_mac
0001:0079b46e  _ssl3_final_finish_mac
0001:0079b73b  _n_ssl3_mac
0001:0079b990* _ssl3_record_sequence_update
0001:0079b9c4  _ssl3_generate_master_secret
0001:0079bb58  _ssl3_alert_code
Module: U:\extras\lib\libssl.lib(s3_lib.obj)
0001:0079be50* _ssl3_version_str
0001:0079c4f8  _ssl3_default_timeout
0001:0079c502  _ssl3_num_ciphers
0001:0079c50c  _ssl3_get_cipher
0001:0079c536  _ssl3_pending
0001:0079c57c  _ssl3_new
0001:0079c62b  _ssl3_free
0001:0079c787  _ssl3_clear
0001:0079c986  _ssl3_ctrl
0001:0079d1c2  _ssl3_callback_ctrl
0001:0079d286  _ssl3_ctx_ctrl
0001:0079d8d4  _ssl3_ctx_callback_ctrl
0001:0079d969  _ssl3_get_cipher_by_char
0001:0079d9ce  _ssl3_put_cipher_by_char
0001:0079da18* _ssl3_choose_cipher
0001:0079e138* _ssl3_get_req_cert_type
0001:0079e242  _ssl3_shutdown
0001:0079e378  _ssl3_write
0001:0079e64e  _ssl3_renegotiate_check
0001:0079e5bb  _ssl3_read
0001:0079e5e4  _ssl3_peek
0001:0079e60d  _ssl3_renegotiate
0002:00004fc0* _ssl3_ciphers
0002:000060a0  _SSLv3_enc_data
Module: U:\extras\lib\libssl.lib(t1_lib.obj)
0001:0079e6f0* _tls1_version_str
0001:0079e738  _tls1_default_timeout
0001:0079e742  _tls1_new
0001:0079e776  _tls1_free
0001:0079e7a7  _tls1_clear
0001:0079e7c3  _tls1_ec_curve_id2nid
0001:0079e7e8  _tls1_ec_nid2curve_id
0001:0079ea16  _ssl_add_clienthello_tlsext
0001:0079f390* _ssl_add_serverhello_tlsext
0001:0079f83f* _ssl_parse_clienthello_tlsext
0001:007a01fd  _ssl_parse_serverhello_tlsext
0001:007a06af  _ssl_prepare_clienthello_tlsext
0001:007a08fb* _ssl_prepare_serverhello_tlsext
0001:007a0a3d* _ssl_check_clienthello_tlsext
0001:007a0c38  _ssl_check_serverhello_tlsext
0001:007a0f8a  _tls1_process_ticket
0002:000060e0  _TLSv1_enc_data
Module: U:\extras\lib\libssl.lib(s23_pkt.obj)
0001:007a15a0  _ssl23_write_bytes
0001:007a163c  _ssl23_read_bytes
Module: U:\extras\lib\libssl.lib(s2_lib.obj)
0001:007a16e0* _ssl2_version_str
0001:007a1760* _ssl2_ciphers
0001:007a18b0  _ssl2_default_timeout
0001:007a18ba  _ssl2_num_ciphers
0001:007a18c4  _ssl2_get_cipher
0001:007a18ee  _ssl2_pending
0001:007a1923  _ssl2_new
0001:007a1aa5  _ssl2_clear
0001:007a1a33  _ssl2_free
0001:007a1b1e  _ssl2_ctrl
0001:007a1b41  _ssl2_callback_ctrl
0001:007a1b4b  _ssl2_ctx_ctrl
0001:007a1b55  _ssl2_ctx_callback_ctrl
0001:007a1b5f  _ssl2_get_cipher_by_char
0001:007a1bd4  _ssl2_put_cipher_by_char
0001:007a1c96  _ssl2_generate_key_material
0001:007a1ed4  _ssl2_return_error
0001:007a1f38  _ssl2_write_error
0001:007a2044  _ssl2_shutdown
Module: U:\extras\lib\libssl.lib(s23_lib.obj)
0001:007a2060  _ssl23_default_timeout
0001:007a206a  _ssl23_num_ciphers
0001:007a2086  _ssl23_get_cipher
0001:007a20bf  _ssl23_get_cipher_by_char
0001:007a212a  _ssl23_put_cipher_by_char
0001:007a2176  _ssl23_read
0001:007a2227  _ssl23_peek
0001:007a22d8  _ssl23_write
Module: U:\extras\lib\xmlrpc.lib(queue.obj)
0001:007a2390  _Q_Init
0001:007a23c3* _Q_AtHead
0001:007a23dc* _Q_AtTail
0001:007a23f6* _Q_IsEmpty
0001:007a2410  _Q_Size
0001:007a2421  _Q_Head
0001:007a243f* _Q_Tail
0001:007a245e  _Q_Next
0001:007a2481* _Q_Previous
0001:007a24a0* _Q_Get
0001:007a24b9* _Q_Put
0001:007a24de* _Q_Find
0001:007a2656* _Q_Iter_Head
0001:007a2666* _Q_Iter_Tail
0001:007a2677* _Q_Iter_Next
0001:007a2688* _Q_Iter_Prev
0001:007a2699* _Q_Iter_Get
0001:007a26a9* _Q_Iter_Put
0001:007a26c1* _Q_PopTail
0001:007a273b* _Q_PopHead
0001:007a27b3  _Q_Destroy
0001:007a27d8  _Q_Iter_Del
0001:007a286d* _Q_DelCur
0001:007a288d* _Q_Sort
0001:007a29d5* _Q_Seek
0001:007a2a86  _Q_PushTail
0001:007a2afc* _Q_PushHead
0001:007a2b6d* _Q_Insert
Module: U:\extras\lib\xmlrpc.lib(simplestring.obj)
0001:007a2bb0  _simplestring_clear
0001:007a2bc8  _simplestring_addn
0001:007a2cba  _simplestring_add
0001:007a2cfe  _simplestring_free
0001:007a2d2d  _simplestring_init
Module: U:\extras\lib\xmlrpc.lib(system_methods.obj)
0001:007a2d78  _xsm_register
Module: U:\extras\lib\xmlrpc.lib(xml_element.obj)
0001:007a5692* _xml_elem_serialize_to_stream
0001:007a56d3  _xml_elem_serialize_to_string
0001:007a571a  _xml_elem_new
0001:007a5806  _xml_elem_free_non_recurse
0001:007a5951  _xml_elem_parse_buf
0001:007a5bc5  _xml_elem_free
Module: U:\extras\lib\xmlrpc.lib(xml_to_xmlrpc.obj)
0001:007a5c99* _XMLRPC_to_xml_element_worker
0001:007a61f8  _XMLRPC_REQUEST_to_xml_element
0001:007a631f  _XMLRPC_VALUE_to_xml_element
0001:007a634d* _xml_element_to_XMLRPC_REQUEST_worker
0001:007a6885  _xml_element_to_XMLRPC_REQUEST
0001:007a68ca* _xml_element_to_XMLRPC_VALUE
Module: U:\extras\lib\xmlrpc.lib(xml_to_soap.obj)
0001:007a6a54* _SOAP_to_xml_element_worker
0001:007a71e6  _SOAP_REQUEST_to_xml_element
0001:007a74c7* _SOAP_VALUE_to_xml_element
0001:007a75a4* _xml_element_to_SOAP_REQUEST_worker
0001:007a7d81  _xml_element_to_SOAP_REQUEST
0001:007a7dd6* _xml_element_to_SOAP_VALUE
Module: U:\extras\lib\xmlrpc.lib(xml_to_dandarpc.obj)
0001:007a7eb1* _DANDARPC_to_xml_element_worker
0001:007a8391  _DANDARPC_REQUEST_to_xml_element
0001:007a84c3* _DANDARPC_VALUE_to_xml_element
0001:007a84de* _xml_element_to_DANDARPC_REQUEST_worker
0001:007a890a  _xml_element_to_DANDARPC_REQUEST
0001:007a8947* _xml_element_to_DANDARPC_VALUE
Module: U:\tmp\ldconv_gcc444_a_92b84c4a69841efbf0.lib(emx-eh.obj)
0001:007a89a5  ___ehInit
0001:007a8970* ___ehTerm
Module: U:\extras\lib\xml2.lib(xmlunicode.obj)
0001:007abfb0* _xmlUCSIsAegeanNumbers
0001:007abfd0* _xmlUCSIsAlphabeticPresentationForms
0001:007abff0* _xmlUCSIsArabic
0001:007ac010* _xmlUCSIsArabicPresentationFormsA
0001:007ac030* _xmlUCSIsArabicPresentationFormsB
0001:007ac050* _xmlUCSIsArmenian
0001:007ac070* _xmlUCSIsArrows
0001:007ac090* _xmlUCSIsBasicLatin
0001:007ac0a0* _xmlUCSIsBengali
0001:007ac0c0* _xmlUCSIsBlockElements
0001:007ac0e0* _xmlUCSIsBopomofo
0001:007ac100* _xmlUCSIsBopomofoExtended
0001:007ac120* _xmlUCSIsBoxDrawing
0001:007ac140* _xmlUCSIsBraillePatterns
0001:007ac160* _xmlUCSIsBuhid
0001:007ac180* _xmlUCSIsByzantineMusicalSymbols
0001:007ac1a0* _xmlUCSIsCJKCompatibility
0001:007ac1c0* _xmlUCSIsCJKCompatibilityForms
0001:007ac1e0* _xmlUCSIsCJKCompatibilityIdeographs
0001:007ac200* _xmlUCSIsCJKCompatibilityIdeographsSupplement
0001:007ac220* _xmlUCSIsCJKRadicalsSupplement
0001:007ac240* _xmlUCSIsCJKSymbolsandPunctuation
0001:007ac260* _xmlUCSIsCJKUnifiedIdeographs
0001:007ac280* _xmlUCSIsCJKUnifiedIdeographsExtensionA
0001:007ac2a0* _xmlUCSIsCJKUnifiedIdeographsExtensionB
0001:007ac2c0* _xmlUCSIsCherokee
0001:007ac2e0* _xmlUCSIsCombiningDiacriticalMarks
0001:007ac300* _xmlUCSIsCombiningDiacriticalMarksforSymbols
0001:007ac320* _xmlUCSIsCombiningHalfMarks
0001:007ac340* _xmlUCSIsCombiningMarksforSymbols
0001:007ac360* _xmlUCSIsControlPictures
0001:007ac380* _xmlUCSIsCurrencySymbols
0001:007ac3a0* _xmlUCSIsCypriotSyllabary
0001:007ac3c0* _xmlUCSIsCyrillic
0001:007ac3e0* _xmlUCSIsCyrillicSupplement
0001:007ac400* _xmlUCSIsDeseret
0001:007ac420* _xmlUCSIsDevanagari
0001:007ac440* _xmlUCSIsDingbats
0001:007ac460* _xmlUCSIsEnclosedAlphanumerics
0001:007ac480* _xmlUCSIsEnclosedCJKLettersandMonths
0001:007ac4a0* _xmlUCSIsEthiopic
0001:007ac4c0* _xmlUCSIsGeneralPunctuation
0001:007ac4e0* _xmlUCSIsGeometricShapes
0001:007ac500* _xmlUCSIsGeorgian
0001:007ac520* _xmlUCSIsGothic
0001:007ac540* _xmlUCSIsGreek
0001:007ac560* _xmlUCSIsGreekExtended
0001:007ac580* _xmlUCSIsGreekandCoptic
0001:007ac5a0* _xmlUCSIsGujarati
0001:007ac5c0* _xmlUCSIsGurmukhi
0001:007ac5e0* _xmlUCSIsHalfwidthandFullwidthForms
0001:007ac600* _xmlUCSIsHangulCompatibilityJamo
0001:007ac620* _xmlUCSIsHangulJamo
0001:007ac640* _xmlUCSIsHangulSyllables
0001:007ac660* _xmlUCSIsHanunoo
0001:007ac680* _xmlUCSIsHebrew
0001:007ac6a0* _xmlUCSIsHighPrivateUseSurrogates
0001:007ac6c0* _xmlUCSIsHighSurrogates
0001:007ac6e0* _xmlUCSIsHiragana
0001:007ac700* _xmlUCSIsIPAExtensions
0001:007ac720* _xmlUCSIsIdeographicDescriptionCharacters
0001:007ac740* _xmlUCSIsKanbun
0001:007ac760* _xmlUCSIsKangxiRadicals
0001:007ac780* _xmlUCSIsKannada
0001:007ac7a0* _xmlUCSIsKatakana
0001:007ac7c0* _xmlUCSIsKatakanaPhoneticExtensions
0001:007ac7e0* _xmlUCSIsKhmer
0001:007ac800* _xmlUCSIsKhmerSymbols
0001:007ac820* _xmlUCSIsLao
0001:007ac840* _xmlUCSIsLatin1Supplement
0001:007ac860* _xmlUCSIsLatinExtendedA
0001:007ac880* _xmlUCSIsLatinExtendedB
0001:007ac8a0* _xmlUCSIsLatinExtendedAdditional
0001:007ac8c0* _xmlUCSIsLetterlikeSymbols
0001:007ac8e0* _xmlUCSIsLimbu
0001:007ac900* _xmlUCSIsLinearBIdeograms
0001:007ac920* _xmlUCSIsLinearBSyllabary
0001:007ac940* _xmlUCSIsLowSurrogates
0001:007ac960* _xmlUCSIsMalayalam
0001:007ac980* _xmlUCSIsMathematicalAlphanumericSymbols
0001:007ac9a0* _xmlUCSIsMathematicalOperators
0001:007ac9c0* _xmlUCSIsMiscellaneousMathematicalSymbolsA
0001:007ac9e0* _xmlUCSIsMiscellaneousMathematicalSymbolsB
0001:007aca00* _xmlUCSIsMiscellaneousSymbols
0001:007aca20* _xmlUCSIsMiscellaneousSymbolsandArrows
0001:007aca40* _xmlUCSIsMiscellaneousTechnical
0001:007aca60* _xmlUCSIsMongolian
0001:007aca80* _xmlUCSIsMusicalSymbols
0001:007acaa0* _xmlUCSIsMyanmar
0001:007acac0* _xmlUCSIsNumberForms
0001:007acae0* _xmlUCSIsOgham
0001:007acb00* _xmlUCSIsOldItalic
0001:007acb20* _xmlUCSIsOpticalCharacterRecognition
0001:007acb40* _xmlUCSIsOriya
0001:007acb60* _xmlUCSIsOsmanya
0001:007acb80* _xmlUCSIsPhoneticExtensions
0001:007acba0* _xmlUCSIsPrivateUse
0001:007acbe0* _xmlUCSIsPrivateUseArea
0001:007acc00* _xmlUCSIsRunic
0001:007acc20* _xmlUCSIsShavian
0001:007acc40* _xmlUCSIsSinhala
0001:007acc60* _xmlUCSIsSmallFormVariants
0001:007acc80* _xmlUCSIsSpacingModifierLetters
0001:007acca0* _xmlUCSIsSpecials
0001:007accc0* _xmlUCSIsSuperscriptsandSubscripts
0001:007acce0* _xmlUCSIsSupplementalArrowsA
0001:007acd00* _xmlUCSIsSupplementalArrowsB
0001:007acd20* _xmlUCSIsSupplementalMathematicalOperators
0001:007acd40* _xmlUCSIsSupplementaryPrivateUseAreaA
0001:007acd60* _xmlUCSIsSupplementaryPrivateUseAreaB
0001:007acd80* _xmlUCSIsSyriac
0001:007acda0* _xmlUCSIsTagalog
0001:007acdc0* _xmlUCSIsTagbanwa
0001:007acde0* _xmlUCSIsTags
0001:007ace00* _xmlUCSIsTaiLe
0001:007ace20* _xmlUCSIsTaiXuanJingSymbols
0001:007ace40* _xmlUCSIsTamil
0001:007ace60* _xmlUCSIsTelugu
0001:007ace80* _xmlUCSIsThaana
0001:007acea0* _xmlUCSIsThai
0001:007acec0* _xmlUCSIsTibetan
0001:007acee0* _xmlUCSIsUgaritic
0001:007acf00* _xmlUCSIsUnifiedCanadianAboriginalSyllabics
0001:007acf20* _xmlUCSIsVariationSelectors
0001:007acf40* _xmlUCSIsVariationSelectorsSupplement
0001:007acf60* _xmlUCSIsYiRadicals
0001:007acf80* _xmlUCSIsYiSyllables
0001:007acfa0* _xmlUCSIsYijingHexagramSymbols
0001:007ad050  _xmlUCSIsCatC
0001:007ad070  _xmlUCSIsCatCc
0001:007ad090  _xmlUCSIsCatCf
0001:007ad0b0  _xmlUCSIsCatCo
0001:007ad100* _xmlUCSIsCatCs
0001:007ad140  _xmlUCSIsCatL
0001:007ad160  _xmlUCSIsCatLl
0001:007ad180  _xmlUCSIsCatLm
0001:007ad1a0  _xmlUCSIsCatLo
0001:007ad1c0  _xmlUCSIsCatLt
0001:007ad1e0  _xmlUCSIsCatLu
0001:007ad200  _xmlUCSIsCatM
0001:007ad220  _xmlUCSIsCatMc
0001:007ad240  _xmlUCSIsCatMe
0001:007ad290  _xmlUCSIsCatMn
0001:007ad2b0  _xmlUCSIsCatN
0001:007ad2d0  _xmlUCSIsCatNd
0001:007ad2f0  _xmlUCSIsCatNl
0001:007ad350  _xmlUCSIsCatNo
0001:007ad370  _xmlUCSIsCatP
0001:007ad390  _xmlUCSIsCatPc
0001:007ad3f0  _xmlUCSIsCatPd
0001:007ad410  _xmlUCSIsCatPe
0001:007ad430  _xmlUCSIsCatPf
0001:007ad470  _xmlUCSIsCatPi
0001:007ad4c0  _xmlUCSIsCatPo
0001:007ad4e0  _xmlUCSIsCatPs
0001:007ad500  _xmlUCSIsCatS
0001:007ad520  _xmlUCSIsCatSc
0001:007ad540  _xmlUCSIsCatSk
0001:007ad560  _xmlUCSIsCatSm
0001:007ad580  _xmlUCSIsCatSo
0001:007ad5a0  _xmlUCSIsCatZ
0001:007ad5c0  _xmlUCSIsCatZl
0001:007ad5e0  _xmlUCSIsCatZp
0001:007ad600  _xmlUCSIsCatZs
0001:007acfc0  _xmlUCSIsBlock
0001:007ad660* _xmlUCSIsCat
Module: U:\extras\lib\libcrypto.lib(mem_dbg.obj)
0001:007ad74e  _CRYPTO_mem_ctrl
0001:007ad939* _CRYPTO_is_mem_check_on
0001:007ad9e0* _CRYPTO_dbg_set_options
0001:007ad9ed* _CRYPTO_dbg_get_options
0001:007adc56  _CRYPTO_push_info_
0001:007add5d  _CRYPTO_pop_info
0001:007adda0* _CRYPTO_remove_all_info
0001:007adde1* _CRYPTO_dbg_malloc
0001:007ae00f* _CRYPTO_dbg_free
0001:007ae097* _CRYPTO_dbg_realloc
0001:007ae5b7* _CRYPTO_mem_leaks
0001:007ae709* _CRYPTO_mem_leaks_fp
0001:007ae7f4* _CRYPTO_mem_leaks_cb
Module: U:\extras\lib\libcrypto.lib(b_print.obj)
0001:007afcb0  _BIO_printf
0001:007afce5* _BIO_vprintf
0001:007afdd9  _BIO_snprintf
0001:007afe0d* _BIO_vsnprintf
Module: U:\extras\lib\libcrypto.lib(mem_clr.obj)
0001:007afe80  _OPENSSL_cleanse
0002:0001eef0  _cleanse_ctr
Module: U:\extras\lib\libcrypto.lib(eng_pkey.obj)
0001:007aff10* _ENGINE_set_load_privkey_function
0001:007aff23* _ENGINE_set_load_pubkey_function
0001:007aff36* _ENGINE_set_load_ssl_client_cert_function
0001:007aff49* _ENGINE_get_load_privkey_function
0001:007aff54* _ENGINE_get_load_pubkey_function
0001:007aff5f  _ENGINE_get_ssl_client_cert_function
0001:007aff75* _ENGINE_load_private_key
0001:007b0104* _ENGINE_load_public_key
0001:007b0293  _ENGINE_load_ssl_client_cert
Module: U:\extras\lib\libssl.lib(ssl_asn1.obj)
0001:007b0400  _i2d_SSL_SESSION
0001:007b1149  _d2i_SSL_SESSION
Module: U:\extras\lib\libcrypto.lib(pem_oth.obj)
0001:007b27ca  _PEM_ASN1_read_bio
Module: U:\extras\lib\libcrypto.lib(pem_lib.obj)
0001:007b2890* _PEM_version
0001:007b290c  _PEM_def_callback
0001:007b2a5a  _PEM_proc_type
0001:007b2af3  _PEM_dek_info
0001:007b2be0  _PEM_ASN1_read
0001:007b4a85  _pem_check_suffix
0001:007b3087  _PEM_bytes_read_bio
0001:007b4273  _PEM_read_bio
0001:007b3a1e  _PEM_get_EVP_CIPHER_INFO
0001:007b37e4  _PEM_do_header
0001:007b31ea  _PEM_ASN1_write
0001:007b3305  _PEM_ASN1_write_bio
0001:007b3edf  _PEM_write_bio
0001:007b3e17* _PEM_write
0001:007b41c8* _PEM_read
Module: U:\extras\lib\libcrypto.lib(ameth_lib.obj)
0001:007b4ba0* _EVP_PKEY_asn1_get_count
0001:007b4bcb* _EVP_PKEY_asn1_get0
0001:007b4ca1  _EVP_PKEY_asn1_find
0001:007b4d17  _EVP_PKEY_asn1_find_str
0001:007b4e01* _EVP_PKEY_asn1_add0
0001:007b4e65* _EVP_PKEY_asn1_add_alias
0001:007b4f38* _EVP_PKEY_asn1_new
0001:007b4eb4  _EVP_PKEY_asn1_get0_info
0001:007b4f21* _EVP_PKEY_get0_asn1
0001:007b51b0  _EVP_PKEY_asn1_free
0001:007b50c7* _EVP_PKEY_asn1_copy
0001:007b5206* _EVP_PKEY_asn1_set_public
0001:007b5241* _EVP_PKEY_asn1_set_private
0001:007b5261* _EVP_PKEY_asn1_set_param
0001:007b529c* _EVP_PKEY_asn1_set_free
0001:007b52aa* _EVP_PKEY_asn1_set_ctrl
Module: U:\extras\lib\libcrypto.lib(evp_lib.obj)
0001:007b52c0  _EVP_CIPHER_param_to_asn1
0001:007b52fa  _EVP_CIPHER_asn1_to_param
0001:007b5351  _EVP_CIPHER_get_asn1_iv
0001:007b563b  _EVP_CIPHER_CTX_iv_length
0001:007b5403  _EVP_CIPHER_set_asn1_iv
0001:007b546a  _EVP_CIPHER_type
0001:007b565e  _EVP_CIPHER_nid
0001:007b55b0  _EVP_CIPHER_block_size
0001:007b55bb  _EVP_CIPHER_CTX_block_size
0001:007b55c8  _EVP_Cipher
0001:007b55f5  _EVP_CIPHER_CTX_cipher
0001:007b55ff* _EVP_CIPHER_flags
0001:007b560a  _EVP_CIPHER_CTX_flags
0001:007b5617* _EVP_CIPHER_CTX_get_app_data
0001:007b5622* _EVP_CIPHER_CTX_set_app_data
0001:007b5630  _EVP_CIPHER_iv_length
0001:007b5648  _EVP_CIPHER_key_length
0001:007b5653  _EVP_CIPHER_CTX_key_length
0001:007b5668* _EVP_CIPHER_CTX_nid
0001:007b5674  _EVP_MD_block_size
0001:007b567f  _EVP_MD_type
0001:007b5689  _EVP_MD_pkey_type
0001:007b5694  _EVP_MD_size
0001:007b56db* _EVP_MD_flags
0001:007b56e6  _EVP_MD_CTX_md
0001:007b56fd  _EVP_MD_CTX_set_flags
0001:007b5713  _EVP_MD_CTX_clear_flags
0001:007b572b  _EVP_MD_CTX_test_flags
0001:007b573b* _EVP_CIPHER_CTX_set_flags
0001:007b5751* _EVP_CIPHER_CTX_clear_flags
0001:007b5769* _EVP_CIPHER_CTX_test_flags
Module: U:\extras\lib\libcrypto.lib(c_zlib.obj)
0001:007b5788  _COMP_zlib
0001:007b579a* _COMP_zlib_cleanup
Module: U:\extras\lib\libcrypto.lib(e_null.obj)
0001:007b57d4  _EVP_enc_null
Module: U:\extras\lib\libcrypto.lib(x509_vfy.obj)
0001:007b5820* _X509_version
0001:007b585b  _X509_verify_cert
0001:007b85ad* _X509_get_pubkey_parameters
0001:007b81df* _X509_cmp_time
0001:007b8b2a  _X509_STORE_CTX_init
0001:007b908d* _X509_STORE_CTX_set0_param
0001:007b8efb  _X509_STORE_CTX_cleanup
0001:007b81c4* _X509_cmp_current_time
0001:007b84d4* _X509_time_adj
0001:007b84b2  _X509_gmtime_adj
0001:007b84fd* _X509_time_adj_ex
0001:007b8725  _X509_STORE_CTX_get_ex_new_index
0001:007b875c  _X509_STORE_CTX_set_ex_data
0001:007b8783* _X509_STORE_CTX_get_ex_data
0001:007b87a3* _X509_STORE_CTX_get_error
0001:007b87ae* _X509_STORE_CTX_set_error
0001:007b87bc* _X509_STORE_CTX_get_error_depth
0001:007b87c7* _X509_STORE_CTX_get_current_cert
0001:007b87d2* _X509_STORE_CTX_get_chain
0001:007b87dd* _X509_STORE_CTX_get1_chain
0001:007b886f* _X509_STORE_CTX_get0_current_issuer
0001:007b887a* _X509_STORE_CTX_get0_current_crl
0001:007b8885* _X509_STORE_CTX_get0_parent_ctx
0001:007b8890* _X509_STORE_CTX_set_cert
0001:007b889e* _X509_STORE_CTX_set_chain
0001:007b88ac* _X509_STORE_CTX_set0_crls
0001:007b88ba  _X509_STORE_CTX_set_purpose
0001:007b890e* _X509_STORE_CTX_purpose_inherit
0001:007b88e4* _X509_STORE_CTX_set_trust
0001:007b8a86* _X509_STORE_CTX_new
0001:007b8b04* _X509_STORE_CTX_free
0001:007b8ee3* _X509_STORE_CTX_trusted_stack
0001:007b8fcf* _X509_STORE_CTX_set_depth
0001:007b8fec* _X509_STORE_CTX_set_flags
0001:007b9009* _X509_STORE_CTX_set_time
0001:007b9026  _X509_STORE_CTX_set_verify_cb
0001:007b9034* _X509_STORE_CTX_get0_policy_tree
0001:007b903f* _X509_STORE_CTX_get_explicit_policy
0001:007b904a  _X509_STORE_CTX_set_default
0001:007b9082  _X509_STORE_CTX_get0_param
Module: U:\extras\lib\libcrypto.lib(dh_asn1.obj)
0001:007b9190* _DHparams_it
0001:007b91ac  _d2i_DHparams
0001:007b91d5  _i2d_DHparams
0001:007b91f7  _DHparams_dup
Module: U:\extras\lib\libcrypto.lib(bn_lib.obj)
0001:007b9220* _BN_version
0001:007b924d* _BN_set_params
0001:007b9314* _BN_get_params
0001:007b9352  _BN_value_one
0001:007b9366* _BN_options
0001:007b93b3  _BN_num_bits_word
0001:007b9424  _BN_num_bits
0001:007b946e  _BN_clear_free
0001:007b94f0  _BN_free
0001:007b9558  _BN_init
0001:007b9584  _BN_new
0001:007b97d6* _bn_dup_expand
0001:007b98c4  _BN_dup
0001:007b9865  _bn_expand2
0001:007b9919  _BN_copy
0001:007b9a52* _BN_swap
0001:007b9b0c  _BN_clear
0001:007b9b57* _BN_get_word
0001:007b9b87  _BN_set_word
0001:007b9bee  _BN_bin2bn
0001:007b9d5d  _BN_bn2bin
0001:007b9de4  _BN_ucmp
0001:007b9e70  _BN_cmp
0001:007b9f86  _BN_set_bit
0001:007ba07e* _BN_clear_bit
0001:007ba153  _BN_is_bit_set
0001:007ba1c0  _BN_mask_bits
0001:007ba2b5  _BN_set_negative
0001:007ba2e0  _bn_cmp_words
0001:007ba377  _bn_cmp_part_words
Module: U:\extras\lib\libcrypto.lib(ec_key.obj)
0001:007ba539  _EC_KEY_new
0001:007ba5eb* _EC_KEY_new_by_curve_name
0001:007ba638  _EC_KEY_free
0001:007ba6fb* _EC_KEY_copy
0001:007ba946  _EC_KEY_dup
0001:007ba98e  _EC_KEY_up_ref
0001:007ba9d1  _EC_KEY_generate_key
0001:007babc0* _EC_KEY_check_key
0001:007baefa  _EC_KEY_get0_group
0001:007baf05  _EC_KEY_set_group
0001:007baf44  _EC_KEY_get0_private_key
0001:007baf4f  _EC_KEY_set_private_key
0001:007baf8e  _EC_KEY_get0_public_key
0001:007baf99  _EC_KEY_set_public_key
0001:007bafe2  _EC_KEY_get_enc_flags
0001:007bafed  _EC_KEY_set_enc_flags
0001:007baffb  _EC_KEY_get_conv_form
0001:007bb006* _EC_KEY_set_conv_form
0001:007bb036  _EC_KEY_get_key_method_data
0001:007bb061  _EC_KEY_insert_key_method_data
0001:007bb107* _EC_KEY_set_asn1_flag
0001:007bb12e* _EC_KEY_precompute_mult
Module: U:\extras\lib\libcrypto.lib(bss_file.obj)
0001:007bb187  _BIO_new_file
0001:007bb33f  _BIO_s_file
0001:007bb2e3  _BIO_new_fp
Module: U:\extras\lib\libcrypto.lib(pem_x509.obj)
0001:007bb9bc  _PEM_read_bio_X509
0001:007bb9f5* _PEM_read_X509
0001:007bba2e  _PEM_write_bio_X509
0001:007bba81* _PEM_write_X509
Module: U:\extras\lib\libcrypto.lib(o_dir.obj)
0001:007bbae0  _OPENSSL_DIR_read
0001:007bbaf8  _OPENSSL_DIR_end
Module: U:\extras\lib\libcrypto.lib(a_object.obj)
0001:007bbb10* _i2d_ASN1_OBJECT
0001:007bbbd9  _a2d_ASN1_OBJECT
0001:007bc073  _i2t_ASN1_OBJECT
0001:007bc0ab  _i2a_ASN1_OBJECT
0001:007bc1a6  _d2i_ASN1_OBJECT
0001:007bc26c  _c2i_ASN1_OBJECT
0001:007bc477  _ASN1_OBJECT_new
0001:007bc515  _ASN1_OBJECT_free
0001:007bc5cb  _ASN1_OBJECT_create
Module: U:\extras\lib\libcrypto.lib(x509_trs.obj)
0001:007bc68c* _X509_TRUST_set_default
0001:007bc6a7  _X509_check_trust
0001:007bc787  _X509_TRUST_get_by_id
0001:007bc740* _X509_TRUST_get0
0001:007bc718* _X509_TRUST_get_count
0001:007bc7ec  _X509_TRUST_set
0001:007bc844* _X509_TRUST_add
0001:007bca83* _X509_TRUST_cleanup
0001:007bcad6* _X509_TRUST_get_flags
0001:007bcae1* _X509_TRUST_get0_name
0001:007bcaec* _X509_TRUST_get_trust
Module: U:\extras\lib\libcrypto.lib(obj_lib.obj)
0001:007bccaa  _OBJ_dup
0001:007bcf17  _OBJ_cmp
Module: U:\extras\lib\libcrypto.lib(tasn_typ.obj)
0001:007bcf80  _ASN1_INTEGER_it
0001:007bcf9c  _d2i_ASN1_INTEGER
0001:007bcfc5  _i2d_ASN1_INTEGER
0001:007bcfe7  _ASN1_INTEGER_new
0001:007bcffb  _ASN1_INTEGER_free
0001:007bd030  _ASN1_ENUMERATED_it
0001:007bd04c  _d2i_ASN1_ENUMERATED
0001:007bd075* _i2d_ASN1_ENUMERATED
0001:007bd097* _ASN1_ENUMERATED_new
0001:007bd0ab  _ASN1_ENUMERATED_free
0001:007bd0e0  _ASN1_BIT_STRING_it
0001:007bd0fc  _d2i_ASN1_BIT_STRING
0001:007bd125  _i2d_ASN1_BIT_STRING
0001:007bd147  _ASN1_BIT_STRING_new
0001:007bd15b  _ASN1_BIT_STRING_free
0001:007bd190  _ASN1_OCTET_STRING_it
0001:007bd1ac  _d2i_ASN1_OCTET_STRING
0001:007bd1d5  _i2d_ASN1_OCTET_STRING
0001:007bd1f7  _ASN1_OCTET_STRING_new
0001:007bd20b  _ASN1_OCTET_STRING_free
0001:007bd230  _ASN1_NULL_it
0001:007bd24c* _d2i_ASN1_NULL
0001:007bd275* _i2d_ASN1_NULL
0001:007bd297  _ASN1_NULL_new
0001:007bd2ab* _ASN1_NULL_free
0001:007bd2e0  _ASN1_OBJECT_it
0001:007bd310  _ASN1_UTF8STRING_it
0001:007bd32c* _d2i_ASN1_UTF8STRING
0001:007bd355* _i2d_ASN1_UTF8STRING
0001:007bd377  _ASN1_UTF8STRING_new
0001:007bd38b  _ASN1_UTF8STRING_free
0001:007bd3c0* _ASN1_PRINTABLESTRING_it
0001:007bd3dc* _d2i_ASN1_PRINTABLESTRING
0001:007bd405* _i2d_ASN1_PRINTABLESTRING
0001:007bd427* _ASN1_PRINTABLESTRING_new
0001:007bd43b* _ASN1_PRINTABLESTRING_free
0001:007bd470* _ASN1_T61STRING_it
0001:007bd48c* _d2i_ASN1_T61STRING
0001:007bd4b5* _i2d_ASN1_T61STRING
0001:007bd4d7* _ASN1_T61STRING_new
0001:007bd4eb* _ASN1_T61STRING_free
0001:007bd520  _ASN1_IA5STRING_it
0001:007bd53c* _d2i_ASN1_IA5STRING
0001:007bd565* _i2d_ASN1_IA5STRING
0001:007bd587* _ASN1_IA5STRING_new
0001:007bd59b* _ASN1_IA5STRING_free
0001:007bd5d0* _ASN1_GENERALSTRING_it
0001:007bd5ec* _d2i_ASN1_GENERALSTRING
0001:007bd615* _i2d_ASN1_GENERALSTRING
0001:007bd637* _ASN1_GENERALSTRING_new
0001:007bd64b* _ASN1_GENERALSTRING_free
0001:007bd680* _ASN1_UTCTIME_it
0001:007bd69c* _d2i_ASN1_UTCTIME
0001:007bd6c5* _i2d_ASN1_UTCTIME
0001:007bd6e7* _ASN1_UTCTIME_new
0001:007bd6fb* _ASN1_UTCTIME_free
0001:007bd730  _ASN1_GENERALIZEDTIME_it
0001:007bd74c* _d2i_ASN1_GENERALIZEDTIME
0001:007bd775* _i2d_ASN1_GENERALIZEDTIME
0001:007bd797  _ASN1_GENERALIZEDTIME_new
0001:007bd7ab* _ASN1_GENERALIZEDTIME_free
0001:007bd7e0* _ASN1_VISIBLESTRING_it
0001:007bd7fc* _d2i_ASN1_VISIBLESTRING
0001:007bd825* _i2d_ASN1_VISIBLESTRING
0001:007bd847* _ASN1_VISIBLESTRING_new
0001:007bd85b* _ASN1_VISIBLESTRING_free
0001:007bd890* _ASN1_UNIVERSALSTRING_it
0001:007bd8ac* _d2i_ASN1_UNIVERSALSTRING
0001:007bd8d5* _i2d_ASN1_UNIVERSALSTRING
0001:007bd8f7* _ASN1_UNIVERSALSTRING_new
0001:007bd90b* _ASN1_UNIVERSALSTRING_free
0001:007bd940* _ASN1_BMPSTRING_it
0001:007bd95c* _d2i_ASN1_BMPSTRING
0001:007bd985* _i2d_ASN1_BMPSTRING
0001:007bd9a7* _ASN1_BMPSTRING_new
0001:007bd9bb* _ASN1_BMPSTRING_free
0001:007bd9e0  _ASN1_ANY_it
0001:007bda10  _ASN1_SEQUENCE_it
0001:007bda2c  _d2i_ASN1_TYPE
0001:007bda55  _i2d_ASN1_TYPE
0001:007bda77  _ASN1_TYPE_new
0001:007bda8b  _ASN1_TYPE_free
0001:007bdac0  _ASN1_PRINTABLE_it
0001:007bdadc* _d2i_ASN1_PRINTABLE
0001:007bdb05* _i2d_ASN1_PRINTABLE
0001:007bdb27* _ASN1_PRINTABLE_new
0001:007bdb3b* _ASN1_PRINTABLE_free
0001:007bdb70  _DISPLAYTEXT_it
0001:007bdb8c* _d2i_DISPLAYTEXT
0001:007bdbb5* _i2d_DISPLAYTEXT
0001:007bdbd7* _DISPLAYTEXT_new
0001:007bdbeb* _DISPLAYTEXT_free
0001:007bdc20  _DIRECTORYSTRING_it
0001:007bdc3c* _d2i_DIRECTORYSTRING
0001:007bdc65* _i2d_DIRECTORYSTRING
0001:007bdc87* _DIRECTORYSTRING_new
0001:007bdc9b* _DIRECTORYSTRING_free
0001:007bdcd0  _ASN1_BOOLEAN_it
0001:007bdd00* _ASN1_TBOOLEAN_it
0001:007bdd30  _ASN1_FBOOLEAN_it
0001:007bdd70  _ASN1_OCTET_STRING_NDEF_it
0001:007bddc0* _ASN1_SEQUENCE_ANY_it
0001:007bde10* _ASN1_SET_ANY_it
0001:007bde2c  _d2i_ASN1_SEQUENCE_ANY
0001:007bde55  _i2d_ASN1_SEQUENCE_ANY
0001:007bde77* _d2i_ASN1_SET_ANY
0001:007bdea0  _i2d_ASN1_SET_ANY
Module: U:\extras\lib\libcrypto.lib(tasn_dec.obj)
0001:007bdf50  _ASN1_tag2bit
0001:007bdf72  _ASN1_item_d2i
0001:007be03b  _ASN1_item_ex_d2i
0001:007bdfe0* _ASN1_template_d2i
0001:007bf86c* _asn1_ex_c2i
Module: U:\extras\lib\libcrypto.lib(tasn_enc.obj)
0001:007c03c0  _ASN1_item_ndef_i2d
0001:007c03e9  _ASN1_item_i2d
0001:007c0504  _ASN1_item_ex_i2d
0001:007c0a2c* _ASN1_template_i2d
0001:007c1214* _asn1_ex_i2c
Module: U:\extras\lib\libcrypto.lib(tasn_new.obj)
0001:007c14c0  _ASN1_item_new
0001:007c14ef  _ASN1_item_ex_new
0001:007c1a3c* _ASN1_template_new
0001:007c1b52* _ASN1_primitive_new
Module: U:\extras\lib\libcrypto.lib(tasn_fre.obj)
0001:007c1d40  _ASN1_item_free
0001:007c1d62  _ASN1_item_ex_free
0001:007c2113  _ASN1_template_free
0001:007c21b9  _ASN1_primitive_free
Module: U:\extras\lib\libcrypto.lib(a_dup.obj)
0001:007c2308  _ASN1_dup
0001:007c23dc  _ASN1_item_dup
Module: U:\extras\lib\libcrypto.lib(x_algor.obj)
0001:007c24f0  _X509_ALGOR_it
0001:007c2540  _X509_ALGORS_it
0001:007c255c  _d2i_X509_ALGOR
0001:007c2585* _i2d_X509_ALGOR
0001:007c25a7  _X509_ALGOR_new
0001:007c25bb  _X509_ALGOR_free
0001:007c25d6* _d2i_X509_ALGORS
0001:007c25ff  _i2d_X509_ALGORS
0001:007c2621* _X509_ALGOR_dup
0001:007c263c  _X509_ALGOR_set0
0001:007c26ff  _X509_ALGOR_get0
Module: U:\extras\lib\libcrypto.lib(v3_genn.obj)
0001:007c27a0* _OTHERNAME_it
0001:007c27bc* _d2i_OTHERNAME
0001:007c27e5* _i2d_OTHERNAME
0001:007c2807  _OTHERNAME_new
0001:007c281b* _OTHERNAME_free
0001:007c2890* _EDIPARTYNAME_it
0001:007c28ac* _d2i_EDIPARTYNAME
0001:007c28d5* _i2d_EDIPARTYNAME
0001:007c28f7* _EDIPARTYNAME_new
0001:007c290b* _EDIPARTYNAME_free
0001:007c2a80  _GENERAL_NAME_it
0001:007c2a9c* _d2i_GENERAL_NAME
0001:007c2ac5* _i2d_GENERAL_NAME
0001:007c2ae7  _GENERAL_NAME_new
0001:007c2afb  _GENERAL_NAME_free
0001:007c2b60  _GENERAL_NAMES_it
0001:007c2b7c* _d2i_GENERAL_NAMES
0001:007c2ba5* _i2d_GENERAL_NAMES
0001:007c2bc7  _GENERAL_NAMES_new
0001:007c2bdb  _GENERAL_NAMES_free
0001:007c2bf6* _GENERAL_NAME_dup
0001:007c2c1b  _GENERAL_NAME_cmp
0001:007c2d3c* _OTHERNAME_cmp
0001:007c2da0* _GENERAL_NAME_set0_value
0001:007c2e26* _GENERAL_NAME_get0_value
0001:007c2ea7* _GENERAL_NAME_set0_othername
0001:007c2ef4* _GENERAL_NAME_get0_otherName
Module: U:\extras\lib\libcrypto.lib(v3_info.obj)
0001:007c2f40  _v3_info
0001:007c30f0* _AUTHORITY_INFO_ACCESS_it
0001:007c2f80  _v3_sinfo
0001:007c3010  _ACCESS_DESCRIPTION_it
0001:007c302c* _d2i_ACCESS_DESCRIPTION
0001:007c3055* _i2d_ACCESS_DESCRIPTION
0001:007c3077* _ACCESS_DESCRIPTION_new
0001:007c308b* _ACCESS_DESCRIPTION_free
0001:007c310c* _d2i_AUTHORITY_INFO_ACCESS
0001:007c3135* _i2d_AUTHORITY_INFO_ACCESS
0001:007c3157* _AUTHORITY_INFO_ACCESS_new
0001:007c316b  _AUTHORITY_INFO_ACCESS_free
0001:007c35d6* _i2a_ACCESS_DESCRIPTION
Module: U:\extras\lib\libcrypto.lib(a_strex.obj)
0001:007c446b  _X509_NAME_print_ex
0001:007c44bc* _X509_NAME_print_ex_fp
0001:007c4541  _ASN1_STRING_print_ex
0001:007c456a* _ASN1_STRING_print_ex_fp
0001:007c4593  _ASN1_STRING_to_UTF8
Module: U:\extras\lib\libcrypto.lib(asn1_lib.obj)
0001:007c4660* _ASN1_version
0001:007c46d0* _ASN1_check_infinite_end
0001:007c46ea  _ASN1_const_check_infinite_end
0001:007c470f  _ASN1_get_object
0001:007c49d4  _ASN1_put_object
0001:007c4ad4  _ASN1_put_eoc
0001:007c4b87  _ASN1_object_size
0001:007c4c61* _asn1_Finish
0001:007c4c74  _asn1_const_Finish
0001:007c4c87  _asn1_GetSequence
0001:007c4d8c  _ASN1_STRING_copy
0001:007c4e3c  _ASN1_STRING_set
0001:007c4de7  _ASN1_STRING_dup
0001:007c4f9b  _ASN1_STRING_new
0001:007c5038  _ASN1_STRING_free
0001:007c4f6a  _ASN1_STRING_set0
0001:007c4faf  _ASN1_STRING_type_new
0001:007c5079  _ASN1_STRING_cmp
0001:007c50fb  _asn1_add_error
0001:007c5171* _ASN1_STRING_length
0001:007c517b* _ASN1_STRING_length_set
0001:007c5188* _ASN1_STRING_type
0001:007c5193  _ASN1_STRING_data
Module: U:\extras\lib\libcrypto.lib(x509_obj.obj)
0001:007c51b8  _X509_NAME_oneline
Module: U:\extras\lib\libcrypto.lib(m_md5.obj)
0001:007c56ac  _EVP_md5
Module: U:\extras\lib\libcrypto.lib(m_sha1.obj)
0001:007c576c  _EVP_sha1
0001:007c583c* _EVP_sha224
0001:007c589c  _EVP_sha256
0001:007c596c* _EVP_sha384
0001:007c59cc* _EVP_sha512
Module: U:\extras\lib\libcrypto.lib(x_pubkey.obj)
0001:007c5a80  _X509_PUBKEY_it
0001:007c5a9c* _d2i_X509_PUBKEY
0001:007c5ac5* _i2d_X509_PUBKEY
0001:007c5ae7* _X509_PUBKEY_new
0001:007c5afb* _X509_PUBKEY_free
0001:007c5b21  _X509_PUBKEY_set
0001:007c5c54  _X509_PUBKEY_get
0001:007c5e32  _d2i_PUBKEY
0001:007c5ea8  _i2d_PUBKEY
0001:007c5f04  _d2i_RSA_PUBKEY
0001:007c5f8a  _i2d_RSA_PUBKEY
0001:007c6015  _d2i_DSA_PUBKEY
0001:007c609b  _i2d_DSA_PUBKEY
0001:007c6126  _d2i_EC_PUBKEY
0001:007c61ac  _i2d_EC_PUBKEY
0001:007c6237  _X509_PUBKEY_set0_param
0001:007c62d6  _X509_PUBKEY_get0_param
Module: U:\extras\lib\libcrypto.lib(x_crl.obj)
0001:007c63b0* _X509_REVOKED_it
0001:007c6510  _X509_CRL_INFO_it
0001:007c6c10  _X509_CRL_it
0001:007c6c2c* _d2i_X509_REVOKED
0001:007c6c55* _i2d_X509_REVOKED
0001:007c6c77* _X509_REVOKED_new
0001:007c6c8b* _X509_REVOKED_free
0001:007c6ca6* _d2i_X509_CRL_INFO
0001:007c6ccf* _i2d_X509_CRL_INFO
0001:007c6cf1* _X509_CRL_INFO_new
0001:007c6d05* _X509_CRL_INFO_free
0001:007c6d20  _d2i_X509_CRL
0001:007c6d49  _i2d_X509_CRL
0001:007c6d6b* _X509_CRL_new
0001:007c6d7f  _X509_CRL_free
0001:007c6d9a* _X509_CRL_dup
0001:007c6ddf* _X509_CRL_add0_revoked
0001:007c6e73  _X509_CRL_verify
0001:007c6ea7* _X509_CRL_get0_by_serial
0001:007c6eea  _X509_CRL_get0_by_cert
0001:007c718e* _X509_CRL_set_default_method
0001:007c71ad* _X509_CRL_METHOD_new
0001:007c7211* _X509_CRL_METHOD_free
0001:007c7233* _X509_CRL_set_meth_data
0001:007c7241* _X509_CRL_get_meth_data
Module: U:\extras\lib\libcrypto.lib(o_names.obj)
0001:007c728f* _OBJ_NAME_init
0001:007c72ef* _OBJ_NAME_new_index
0001:007c757e  _OBJ_NAME_get
0001:007c7629  _OBJ_NAME_add
0001:007c774e* _OBJ_NAME_remove
0001:007c785f  _OBJ_NAME_do_all
0001:007c7906  _OBJ_NAME_do_all_sorted
0001:007c7a2a  _OBJ_NAME_cleanup
Module: U:\extras\lib\libcrypto.lib(evp_pbe.obj)
0001:007c7c65  _EVP_PBE_CipherInit
0001:007c8086  _EVP_PBE_find
0001:007c7f5c* _EVP_PBE_alg_add_type
0001:007c801c* _EVP_PBE_alg_add
0001:007c816a  _EVP_PBE_cleanup
Module: U:\extras\lib\libcrypto.lib(obj_xref.obj)
0002:00021ca0+ _sig_app
0002:00021cb0+ _sigx_app
0001:007c8492  _OBJ_find_sigid_algs
0001:007c8530  _OBJ_find_sigid_by_algs
0001:007c85e1* _OBJ_add_sigid
0001:007c8709  _OBJ_sigid_free
Module: U:\extras\lib\libcrypto.lib(tb_rand.obj)
0001:007c8764* _ENGINE_unregister_RAND
0001:007c8793* _ENGINE_register_RAND
0001:007c87df* _ENGINE_register_all_RAND
0001:007c8810* _ENGINE_set_default_RAND
0001:007c885c  _ENGINE_get_default_RAND
0001:007c8879  _ENGINE_get_RAND
0001:007c8884* _ENGINE_set_RAND
Module: U:\extras\lib\libcrypto.lib(md_rand.obj)
0001:007c88a0* _RAND_version
0001:007c88c7  _RAND_SSLeay
0002:00006b70* _rand_ssleay_meth
Module: U:\extras\lib\libcrypto.lib(x_val.obj)
0001:007c9560  _X509_VAL_it
0001:007c957c* _d2i_X509_VAL
0001:007c95a5* _i2d_X509_VAL
0001:007c95c7* _X509_VAL_new
0001:007c95db* _X509_VAL_free
Module: U:\extras\lib\libcrypto.lib(x_x509a.obj)
0001:007c96a0* _X509_CERT_AUX_it
0001:007c96bc  _d2i_X509_CERT_AUX
0001:007c96e5  _i2d_X509_CERT_AUX
0001:007c9707* _X509_CERT_AUX_new
0001:007c971b  _X509_CERT_AUX_free
0001:007c9777* _X509_alias_set1
0001:007c982e* _X509_keyid_set1
0001:007c98e5* _X509_alias_get0
0001:007c992a* _X509_keyid_get0
0001:007c996f* _X509_add1_trust_object
0001:007c99e6* _X509_add1_reject_object
0001:007c9a61* _X509_trust_clear
0001:007c9aa4* _X509_reject_clear
0001:007c9b40* _X509_CERT_PAIR_it
0001:007c9b5c  _d2i_X509_CERT_PAIR
0001:007c9b85  _i2d_X509_CERT_PAIR
0001:007c9ba7* _X509_CERT_PAIR_new
0001:007c9bbb* _X509_CERT_PAIR_free
Module: U:\extras\lib\libcrypto.lib(v3_akeya.obj)
0001:007c9c50  _AUTHORITY_KEYID_it
0001:007c9c6c* _d2i_AUTHORITY_KEYID
0001:007c9c95* _i2d_AUTHORITY_KEYID
0001:007c9cb7  _AUTHORITY_KEYID_new
0001:007c9ccb  _AUTHORITY_KEYID_free
Module: U:\extras\lib\libcrypto.lib(v3_crld.obj)
0001:007c9cf0  _v3_crld
0001:007caa60* _CRL_DIST_POINTS_it
0001:007c9d30  _v3_freshest_crl
0001:007ca8f7* _DIST_POINT_NAME_new
0001:007ca9e7* _DIST_POINT_new
0001:007ca9fb* _DIST_POINT_free
0001:007ca890* _DIST_POINT_NAME_it
0001:007ca8ac* _d2i_DIST_POINT_NAME
0001:007ca8d5* _i2d_DIST_POINT_NAME
0001:007ca90b* _DIST_POINT_NAME_free
0001:007ca980* _DIST_POINT_it
0001:007ca99c* _d2i_DIST_POINT
0001:007ca9c5* _i2d_DIST_POINT
0001:007caa7c* _d2i_CRL_DIST_POINTS
0001:007caaa5* _i2d_CRL_DIST_POINTS
0001:007caac7* _CRL_DIST_POINTS_new
0001:007caadb  _CRL_DIST_POINTS_free
0001:007cabc0* _ISSUING_DIST_POINT_it
0001:007cabdc* _d2i_ISSUING_DIST_POINT
0001:007cac05* _i2d_ISSUING_DIST_POINT
0001:007cac27* _ISSUING_DIST_POINT_new
0001:007cac3b  _ISSUING_DIST_POINT_free
0001:007cac60  _v3_idp
0001:007cb3ae  _DIST_POINT_set_dpname
Module: U:\extras\lib\libcrypto.lib(pcy_cache.obj)
0001:007cb8e6  _policy_cache_free
0001:007cb939  _policy_cache_set
0001:007cb9a4  _policy_cache_find_data
Module: U:\extras\lib\libcrypto.lib(v3_ncons.obj)
0001:007cba50  _v3_name_constraints
0001:007cbb70* _NAME_CONSTRAINTS_it
0001:007cbaf0* _GENERAL_SUBTREE_it
0001:007cbb8c* _GENERAL_SUBTREE_new
0001:007cbba0* _GENERAL_SUBTREE_free
0001:007cbbbb* _NAME_CONSTRAINTS_new
0001:007cbbcf  _NAME_CONSTRAINTS_free
0001:007cc13d  _NAME_CONSTRAINTS_check
Module: U:\extras\lib\libcrypto.lib(eng_lib.obj)
0001:007cc84a  _ENGINE_new
0001:007cc8ef* _engine_set_all_null
0001:007cc99d  _engine_free_util
0001:007cca9a  _ENGINE_free
0001:007ccb30  _engine_cleanup_add_first
0001:007ccb7b  _engine_cleanup_add_last
0001:007ccbd8* _ENGINE_cleanup
0001:007ccc1c* _ENGINE_get_ex_new_index
0001:007ccc53* _ENGINE_set_ex_data
0001:007ccc77* _ENGINE_get_ex_data
0001:007ccc94* _ENGINE_set_id
0001:007ccce2* _ENGINE_set_name
0001:007ccd31* _ENGINE_set_destroy_function
0001:007ccd44* _ENGINE_set_init_function
0001:007ccd57* _ENGINE_set_finish_function
0001:007ccd6a* _ENGINE_set_ctrl_function
0001:007ccd7d* _ENGINE_set_flags
0001:007ccd90* _ENGINE_set_cmd_defns
0001:007ccda3* _ENGINE_get_id
0001:007ccdad* _ENGINE_get_name
0001:007ccdb8* _ENGINE_get_destroy_function
0001:007ccdc3* _ENGINE_get_init_function
0001:007ccdce* _ENGINE_get_finish_function
0001:007ccdd9* _ENGINE_get_ctrl_function
0001:007ccde4* _ENGINE_get_flags
0001:007ccdef* _ENGINE_get_cmd_defns
0001:007ccdfa* _ENGINE_get_static_state
Module: U:\extras\lib\libcrypto.lib(rsa_eay.obj)
0001:007cce28  _RSA_PKCS1_SSLeay
Module: U:\extras\lib\libcrypto.lib(tb_rsa.obj)
0001:007ceee4* _ENGINE_unregister_RSA
0001:007cef13* _ENGINE_register_RSA
0001:007cef5f* _ENGINE_register_all_RSA
0001:007cef90* _ENGINE_set_default_RSA
0001:007cefdc  _ENGINE_get_default_RSA
0001:007ceff9  _ENGINE_get_RSA
0001:007cf004* _ENGINE_set_RSA
Module: U:\extras\lib\libcrypto.lib(bn_blind.obj)
0001:007cf02b* _BN_BLINDING_new
0001:007cf167  _BN_BLINDING_free
0001:007cf1e1* _BN_BLINDING_update
0001:007cf565  _BN_BLINDING_create_param
0001:007cf345* _BN_BLINDING_convert
0001:007cf36e  _BN_BLINDING_convert_ex
0001:007cf423* _BN_BLINDING_invert
0001:007cf44c  _BN_BLINDING_invert_ex
0001:007cf528* _BN_BLINDING_get_thread_id
0001:007cf533* _BN_BLINDING_set_thread_id
0001:007cf541  _BN_BLINDING_thread_id
0001:007cf54c* _BN_BLINDING_get_flags
0001:007cf557* _BN_BLINDING_set_flags
Module: U:\extras\lib\libcrypto.lib(bn_ctx.obj)
0001:007cf7d0* _BN_CTX_init
0001:007cf818  _BN_CTX_new
0001:007cf8b2  _BN_CTX_free
0001:007cf8e7  _BN_CTX_start
0001:007cf96b  _BN_CTX_end
0001:007cf9d7  _BN_CTX_get
Module: U:\extras\lib\libcrypto.lib(bn_add.obj)
0001:007cfeb0  _BN_add
0001:007d0119  _BN_usub
0001:007cff8b  _BN_uadd
0001:007d0332  _BN_sub
Module: U:\extras\lib\libcrypto.lib(bn_mul.obj)
0001:007d04a0* _bn_sub_part_words
0001:007d07e4* _bn_add_part_words
0001:007d0c2c* _bn_mul_recursive
0001:007d2915* _bn_mul_normal
0001:007d135a* _bn_mul_part_recursive
0001:007d1b93* _bn_mul_low_recursive
0001:007d2ab8* _bn_mul_low_normal
0001:007d1d74* _bn_mul_high
0001:007d24aa  _BN_mul
Module: U:\extras\lib\libcrypto.lib(bn_gcd.obj)
0001:007d2bd0  _BN_gcd
0001:007d2ec0  _BN_mod_inverse
Module: U:\extras\lib\libcrypto.lib(dh_key.obj)
0001:007d3b40  _DH_generate_key
0001:007d3b59  _DH_compute_key
0001:007d3b92  _DH_OpenSSL
Module: U:\extras\lib\libcrypto.lib(tb_dh.obj)
0001:007d4134* _ENGINE_unregister_DH
0001:007d4163* _ENGINE_register_DH
0001:007d41af* _ENGINE_register_all_DH
0001:007d41e0* _ENGINE_set_default_DH
0001:007d422c  _ENGINE_get_default_DH
0001:007d4249  _ENGINE_get_DH
0001:007d4254* _ENGINE_set_DH
Module: U:\extras\lib\libcrypto.lib(dsa_lib.obj)
0001:007d4270* _DSA_version
0001:007d4296* _DSA_set_default_method
0001:007d42a3* _DSA_get_default_method
0001:007d42c3  _DSA_new
0001:007d4352* _DSA_new_method
0001:007d42d7* _DSA_set_method
0001:007d45b2  _DSA_free
0001:007d470b  _DSA_up_ref
0001:007d474e  _DSA_size
0001:007d47ca* _DSA_get_ex_new_index
0001:007d4801* _DSA_set_ex_data
0001:007d4825* _DSA_get_ex_data
0001:007d4842* _DSA_dup_DH
Module: U:\extras\lib\libcrypto.lib(x_attrib.obj)
0001:007d49c0* _X509_ATTRIBUTE_SET_it
0001:007d4a20  _X509_ATTRIBUTE_it
0001:007d4a3c* _d2i_X509_ATTRIBUTE
0001:007d4a65* _i2d_X509_ATTRIBUTE
0001:007d4a87  _X509_ATTRIBUTE_new
0001:007d4a9b  _X509_ATTRIBUTE_free
0001:007d4ab6  _X509_ATTRIBUTE_dup
0001:007d4ad1  _X509_ATTRIBUTE_create
Module: U:\extras\lib\libcrypto.lib(x509_v3.obj)
0001:007d4bb0  _X509v3_get_ext_count
0001:007d4bd0  _X509v3_get_ext_by_NID
0001:007d4c0c  _X509v3_get_ext_by_OBJ
0001:007d4c83  _X509v3_get_ext_by_critical
0001:007d4d02  _X509v3_get_ext
0001:007d4d3f  _X509v3_delete_ext
0001:007d4d8c  _X509v3_add_ext
0001:007d4ec5  _X509_EXTENSION_create_by_NID
0001:007d4f4b  _X509_EXTENSION_create_by_OBJ
0001:007d5036* _X509_EXTENSION_set_object
0001:007d5073* _X509_EXTENSION_set_critical
0001:007d50a2* _X509_EXTENSION_set_data
0001:007d50ed  _X509_EXTENSION_get_object
0001:007d5104  _X509_EXTENSION_get_data
0001:007d511c  _X509_EXTENSION_get_critical
Module: U:\extras\lib\libcrypto.lib(x509_ext.obj)
0001:007d5150* _X509_CRL_get_ext_count
0001:007d5168  _X509_CRL_get_ext_by_NID
0001:007d518e* _X509_CRL_get_ext_by_OBJ
0001:007d51b4* _X509_CRL_get_ext_by_critical
0001:007d51da  _X509_CRL_get_ext
0001:007d51f9* _X509_CRL_delete_ext
0001:007d5218  _X509_CRL_get_ext_d2i
0001:007d5245* _X509_CRL_add1_ext_i2d
0001:007d5279* _X509_CRL_add_ext
0001:007d52a7  _X509_get_ext_count
0001:007d52bf  _X509_get_ext_by_NID
0001:007d52e5* _X509_get_ext_by_OBJ
0001:007d530b* _X509_get_ext_by_critical
0001:007d5331  _X509_get_ext
0001:007d5350* _X509_delete_ext
0001:007d536f* _X509_add_ext
0001:007d539d  _X509_get_ext_d2i
0001:007d53ca* _X509_add1_ext_i2d
0001:007d53fe* _X509_REVOKED_get_ext_count
0001:007d5414* _X509_REVOKED_get_ext_by_NID
0001:007d5438* _X509_REVOKED_get_ext_by_OBJ
0001:007d545c* _X509_REVOKED_get_ext_by_critical
0001:007d5480* _X509_REVOKED_get_ext
0001:007d549d* _X509_REVOKED_delete_ext
0001:007d54ba* _X509_REVOKED_add_ext
0001:007d54e6  _X509_REVOKED_get_ext_d2i
0001:007d5511* _X509_REVOKED_add1_ext_i2d
Module: U:\extras\lib\libcrypto.lib(x_all.obj)
0001:007d5550  _X509_verify
0001:007d558d* _X509_REQ_verify
0001:007d55ca* _NETSCAPE_SPKI_verify
0001:007d5607* _X509_sign
0001:007d5659  _X509_REQ_sign
0001:007d56a5* _X509_CRL_sign
0001:007d5703* _NETSCAPE_SPKI_sign
0001:007d574f* _d2i_X509_fp
0001:007d5771* _i2d_X509_fp
0001:007d5793  _d2i_X509_bio
0001:007d57b5* _i2d_X509_bio
0001:007d57d7* _d2i_X509_CRL_fp
0001:007d57f9* _i2d_X509_CRL_fp
0001:007d581b  _d2i_X509_CRL_bio
0001:007d583d* _i2d_X509_CRL_bio
0001:007d585f* _d2i_PKCS7_fp
0001:007d5881* _i2d_PKCS7_fp
0001:007d58a3* _d2i_PKCS7_bio
0001:007d58c5* _i2d_PKCS7_bio
0001:007d58e7* _d2i_X509_REQ_fp
0001:007d5909* _i2d_X509_REQ_fp
0001:007d592b* _d2i_X509_REQ_bio
0001:007d594d* _i2d_X509_REQ_bio
0001:007d596f* _d2i_RSAPrivateKey_fp
0001:007d5991* _i2d_RSAPrivateKey_fp
0001:007d59b3* _d2i_RSAPublicKey_fp
0001:007d59d5* _d2i_RSA_PUBKEY_fp
0001:007d5a01* _i2d_RSAPublicKey_fp
0001:007d5a23* _i2d_RSA_PUBKEY_fp
0001:007d5a46  _d2i_RSAPrivateKey_bio
0001:007d5a68* _i2d_RSAPrivateKey_bio
0001:007d5a8a* _d2i_RSAPublicKey_bio
0001:007d5aac* _d2i_RSA_PUBKEY_bio
0001:007d5ad8* _i2d_RSAPublicKey_bio
0001:007d5afa* _i2d_RSA_PUBKEY_bio
0001:007d5b1d* _d2i_DSAPrivateKey_fp
0001:007d5b49* _i2d_DSAPrivateKey_fp
0001:007d5b6c* _d2i_DSA_PUBKEY_fp
0001:007d5b98* _i2d_DSA_PUBKEY_fp
0001:007d5bbb* _d2i_DSAPrivateKey_bio
0001:007d5be7* _i2d_DSAPrivateKey_bio
0001:007d5c0a* _d2i_DSA_PUBKEY_bio
0001:007d5c36* _i2d_DSA_PUBKEY_bio
0001:007d5c59* _d2i_EC_PUBKEY_fp
0001:007d5c85* _i2d_EC_PUBKEY_fp
0001:007d5ca8* _d2i_ECPrivateKey_fp
0001:007d5cd4* _i2d_ECPrivateKey_fp
0001:007d5cf7* _d2i_EC_PUBKEY_bio
0001:007d5d23* _i2d_EC_PUBKEY_bio
0001:007d5d46* _d2i_ECPrivateKey_bio
0001:007d5d72* _i2d_ECPrivateKey_bio
0001:007d5d95* _X509_pubkey_digest
0001:007d5dee  _X509_digest
0001:007d5e1e  _X509_CRL_digest
0001:007d5e4e* _X509_REQ_digest
0001:007d5e7e* _X509_NAME_digest
0001:007d5eae* _PKCS7_ISSUER_AND_SERIAL_digest
0001:007d5ede* _d2i_PKCS8_fp
0001:007d5f0a* _i2d_PKCS8_fp
0001:007d5f2d  _d2i_PKCS8_bio
0001:007d5f59  _i2d_PKCS8_bio
0001:007d5f7c* _d2i_PKCS8_PRIV_KEY_INFO_fp
0001:007d5fa8* _i2d_PKCS8_PRIV_KEY_INFO_fp
0001:007d5fcb* _i2d_PKCS8PrivateKeyInfo_fp
0001:007d6011* _i2d_PrivateKey_fp
0001:007d6034* _d2i_PrivateKey_fp
0001:007d6060* _i2d_PUBKEY_fp
0001:007d6083* _d2i_PUBKEY_fp
0001:007d60af* _d2i_PKCS8_PRIV_KEY_INFO_bio
0001:007d60db  _i2d_PKCS8_PRIV_KEY_INFO_bio
0001:007d60fe* _i2d_PKCS8PrivateKeyInfo_bio
0001:007d6144* _i2d_PrivateKey_bio
0001:007d6167  _d2i_PrivateKey_bio
0001:007d6193* _i2d_PUBKEY_bio
0001:007d61b6* _d2i_PUBKEY_bio
Module: U:\extras\lib\libcrypto.lib(a_int.obj)
0001:007d61f0* _ASN1_INTEGER_dup
0001:007d6203  _ASN1_INTEGER_cmp
0001:007d6262  _i2c_ASN1_INTEGER
0001:007d6434  _c2i_ASN1_INTEGER
0001:007d6666  _d2i_ASN1_UINTEGER
0001:007d6838  _ASN1_INTEGER_set
0001:007d6974  _ASN1_INTEGER_get
0001:007d6a1e  _BN_to_ASN1_INTEGER
0001:007d6b8f  _ASN1_INTEGER_to_BN
Module: U:\extras\lib\libcrypto.lib(v3_bcons.obj)
0001:007d6c10  _v3_bcons
0001:007d6ca0* _BASIC_CONSTRAINTS_it
0001:007d6cbc* _d2i_BASIC_CONSTRAINTS
0001:007d6ce5* _i2d_BASIC_CONSTRAINTS
0001:007d6d07* _BASIC_CONSTRAINTS_new
0001:007d6d1b  _BASIC_CONSTRAINTS_free
Module: U:\extras\lib\libcrypto.lib(v3_pcia.obj)
0001:007d6f90* _PROXY_POLICY_it
0001:007d6fac* _d2i_PROXY_POLICY
0001:007d6fd5* _i2d_PROXY_POLICY
0001:007d6ff7* _PROXY_POLICY_new
0001:007d700b* _PROXY_POLICY_free
0001:007d70a0  _PROXY_CERT_INFO_EXTENSION_it
0001:007d70bc* _d2i_PROXY_CERT_INFO_EXTENSION
0001:007d70e5* _i2d_PROXY_CERT_INFO_EXTENSION
0001:007d7107  _PROXY_CERT_INFO_EXTENSION_new
0001:007d711b  _PROXY_CERT_INFO_EXTENSION_free
Module: U:\extras\lib\libcrypto.lib(a_octet.obj)
0001:007d7140  _ASN1_OCTET_STRING_dup
0001:007d7153  _ASN1_OCTET_STRING_cmp
0001:007d716d  _ASN1_OCTET_STRING_set
Module: U:\extras\lib\libcrypto.lib(bn_word.obj)
0001:007d7190  _BN_mod_word
0001:007d7214  _BN_div_word
0001:007d7334  _BN_add_word
0001:007d748c  _BN_sub_word
0001:007d7606  _BN_mul_word
Module: U:\extras\lib\libcrypto.lib(bn_shift.obj)
0001:007d76e0  _BN_lshift1
0001:007d77fa  _BN_rshift1
0001:007d793b  _BN_lshift
0001:007d7b20  _BN_rshift
Module: U:\extras\lib\libcrypto.lib(bn_print.obj)
0001:007d7d8c* _BN_bn2hex
0001:007d7ec0  _BN_bn2dec
0001:007d8143  _BN_hex2bn
0001:007d83bb  _BN_dec2bn
0001:007d85f0  _BN_asc2bn
0001:007d867f* _BN_print_fp
0001:007d86ed* _BN_print
Module: U:\extras\lib\libcrypto.lib(tb_cipher.obj)
0001:007d8800* _ENGINE_unregister_ciphers
0001:007d882f* _ENGINE_register_ciphers
0001:007d88a7* _ENGINE_register_all_ciphers
0001:007d88d8* _ENGINE_set_default_ciphers
0001:007d8950  _ENGINE_get_cipher_engine
0001:007d8977  _ENGINE_get_cipher
0001:007d89ee* _ENGINE_get_ciphers
0001:007d89f9* _ENGINE_set_ciphers
Module: U:\extras\lib\libcrypto.lib(by_file.obj)
0001:007d8a25  _X509_LOOKUP_file
0001:007d8fbf* _X509_load_cert_crl_file
0001:007d8b51  _X509_load_cert_file
0001:007d8d87  _X509_load_crl_file
0002:00006c00* _x509_file_lookup
Module: U:\extras\lib\libcrypto.lib(by_dir.obj)
0001:007d9175  _X509_LOOKUP_hash_dir
0002:00006c30* _x509_dir_lookup
Module: U:\extras\lib\libcrypto.lib(tb_digest.obj)
0001:007d9c20* _ENGINE_unregister_digests
0001:007d9c4f* _ENGINE_register_digests
0001:007d9cc7* _ENGINE_register_all_digests
0001:007d9cf8* _ENGINE_set_default_digests
0001:007d9d70  _ENGINE_get_digest_engine
0001:007d9d97  _ENGINE_get_digest
0001:007d9e0e* _ENGINE_get_digests
0001:007d9e19* _ENGINE_set_digests
Module: U:\extras\lib\libcrypto.lib(pmeth_lib.obj)
0001:007d9ea0* _EVP_PKEY_meth_find
0001:007da4f5  _EVP_PKEY_CTX_free
0001:007da141* _EVP_PKEY_meth_new
0001:007da28b  _EVP_PKEY_meth_free
0001:007da2b1  _EVP_PKEY_CTX_new
0001:007da2d3  _EVP_PKEY_CTX_new_id
0001:007da2f5  _EVP_PKEY_CTX_dup
0001:007da491* _EVP_PKEY_meth_add0
0001:007da57e  _EVP_PKEY_CTX_ctrl
0001:007da6dd* _EVP_PKEY_CTX_ctrl_str
0001:007da7f0* _EVP_PKEY_CTX_get_operation
0001:007da7fb* _EVP_PKEY_CTX_set0_keygen_info
0001:007da812* _EVP_PKEY_CTX_set_data
0001:007da820* _EVP_PKEY_CTX_get_data
0001:007da82b* _EVP_PKEY_CTX_get0_pkey
0001:007da836* _EVP_PKEY_CTX_get0_peerkey
0001:007da841* _EVP_PKEY_CTX_set_app_data
0001:007da84f* _EVP_PKEY_CTX_get_app_data
0001:007da85a* _EVP_PKEY_meth_set_init
0001:007da868* _EVP_PKEY_meth_set_copy
0001:007da876* _EVP_PKEY_meth_set_cleanup
0001:007da884* _EVP_PKEY_meth_set_paramgen
0001:007da89b* _EVP_PKEY_meth_set_keygen
0001:007da8b2* _EVP_PKEY_meth_set_sign
0001:007da8c9* _EVP_PKEY_meth_set_verify
0001:007da8e0* _EVP_PKEY_meth_set_verify_recover
0001:007da8f7* _EVP_PKEY_meth_set_signctx
0001:007da90e* _EVP_PKEY_meth_set_verifyctx
0001:007da925* _EVP_PKEY_meth_set_encrypt
0001:007da93c* _EVP_PKEY_meth_set_decrypt
0001:007da953* _EVP_PKEY_meth_set_derive
0001:007da96a* _EVP_PKEY_meth_set_ctrl
0002:0001f500* _app_pkey_methods
Module: U:\extras\lib\libssl.lib(s2_enc.obj)
0001:007daa06  _ssl2_enc_init
0001:007dad25  _ssl2_enc
0001:007dadba  _ssl2_mac
Module: U:\extras\lib\libssl.lib(s2_pkt.obj)
0001:007db593  _ssl2_read
0001:007db5bc  _ssl2_peek
0001:007db8c0  _ssl2_write
0001:007dbf75  _ssl2_part_read
0001:007dc051  _ssl2_do_write
Module: U:\extras\lib\libssl.lib(ssl_rsa.obj)
0001:007dc19a  _SSL_use_certificate
0001:007dc23a* _SSL_use_certificate_file
0001:007dc3f3* _SSL_use_certificate_ASN1
0001:007dc474* _SSL_use_RSAPrivateKey
0001:007dc72a* _SSL_use_RSAPrivateKey_file
0001:007dc8dd* _SSL_use_RSAPrivateKey_ASN1
0001:007dc964  _SSL_use_PrivateKey
0001:007dca0a* _SSL_use_PrivateKey_file
0001:007dcbbd* _SSL_use_PrivateKey_ASN1
0001:007dcc4b* _SSL_CTX_use_certificate
0001:007dcedb* _SSL_CTX_use_certificate_file
0001:007dd088* _SSL_CTX_use_certificate_ASN1
0001:007dd109* _SSL_CTX_use_RSAPrivateKey
0001:007dd226* _SSL_CTX_use_RSAPrivateKey_file
0001:007dd3cd* _SSL_CTX_use_RSAPrivateKey_ASN1
0001:007dd454* _SSL_CTX_use_PrivateKey
0001:007dd4f4* _SSL_CTX_use_PrivateKey_file
0001:007dd69b* _SSL_CTX_use_PrivateKey_ASN1
0001:007dd729* _SSL_CTX_use_certificate_chain_file
Module: U:\extras\lib\libcrypto.lib(p_sign.obj)
0001:007dd979  _EVP_SignFinal
Module: U:\extras\lib\libcrypto.lib(ec_curve.obj)
0001:007e1cf4  _EC_GROUP_new_by_curve_name
0001:007e1da9* _EC_get_builtin_curves
Module: U:\extras\lib\libcrypto.lib(ec_lib.obj)
0001:007e1e5e  _EC_GROUP_new
0001:007e1fce  _EC_GROUP_free
0001:007e2f72  _EC_EX_DATA_free_all_data
0001:007e312b  _EC_POINT_free
0001:007e2064  _EC_GROUP_clear_free
0001:007e2fc6* _EC_EX_DATA_clear_free_all_data
0001:007e3163  _EC_POINT_clear_free
0001:007e2143  _EC_GROUP_copy
0001:007e2d1d  _EC_EX_DATA_set_data
0001:007e301a  _EC_POINT_new
0001:007e31cc  _EC_POINT_copy
0001:007e2443  _EC_GROUP_dup
0001:007e24c4  _EC_GROUP_method_of
0001:007e24ce  _EC_METHOD_get_field_type
0001:007e24d8  _EC_GROUP_set_generator
0001:007e25f1  _EC_GROUP_get0_generator
0001:007e25fc  _EC_GROUP_get_order
0001:007e2632  _EC_GROUP_get_cofactor
0001:007e2668  _EC_GROUP_set_curve_name
0001:007e2676  _EC_GROUP_get_curve_name
0001:007e2681  _EC_GROUP_set_asn1_flag
0001:007e268f  _EC_GROUP_get_asn1_flag
0001:007e269a  _EC_GROUP_set_point_conversion_form
0001:007e26a8  _EC_GROUP_get_point_conversion_form
0001:007e26b3  _EC_GROUP_set_seed
0001:007e2756  _EC_GROUP_get0_seed
0001:007e2761  _EC_GROUP_get_seed_len
0001:007e276c  _EC_GROUP_set_curve_GFp
0001:007e27df  _EC_GROUP_get_curve_GFp
0001:007e2852  _EC_GROUP_set_curve_GF2m
0001:007e28c5  _EC_GROUP_get_curve_GF2m
0001:007e2938  _EC_GROUP_get_degree
0001:007e298f* _EC_GROUP_check_discriminant
0001:007e29ed  _EC_GROUP_cmp
0001:007e3e19  _EC_POINT_cmp
0001:007e2e18  _EC_EX_DATA_get_data
0001:007e2e64  _EC_EX_DATA_free_data
0001:007e2eeb* _EC_EX_DATA_clear_free_data
0001:007e327a  _EC_POINT_dup
0001:007e32da* _EC_POINT_method_of
0001:007e32e4  _EC_POINT_set_to_infinity
0001:007e3383  _EC_POINT_set_Jprojective_coordinates_GFp
0001:007e343e* _EC_POINT_get_Jprojective_coordinates_GFp
0001:007e34f9  _EC_POINT_set_affine_coordinates_GFp
0001:007e35ad  _EC_POINT_set_affine_coordinates_GF2m
0001:007e3661  _EC_POINT_get_affine_coordinates_GFp
0001:007e3715  _EC_POINT_get_affine_coordinates_GF2m
0001:007e37c9  _EC_POINT_set_compressed_coordinates_GFp
0001:007e387d  _EC_POINT_set_compressed_coordinates_GF2m
0001:007e3931  _EC_POINT_point2oct
0001:007e39ec  _EC_POINT_oct2point
0001:007e3aa0  _EC_POINT_add
0001:007e3b73  _EC_POINT_dbl
0001:007e3c2e  _EC_POINT_invert
0001:007e3cd4  _EC_POINT_is_at_infinity
0001:007e3d73  _EC_POINT_is_on_curve
0001:007e3ed4  _EC_POINT_make_affine
0001:007e3f7a  _EC_POINTs_make_affine
0001:007e4046* _EC_POINTs_mul
0001:007e40cb  _EC_POINT_mul
0001:007e4129  _EC_GROUP_precompute_mult
0001:007e417b  _EC_GROUP_have_precompute_mult
Module: U:\extras\lib\libcrypto.lib(rsa_sign.obj)
0001:007e41cb  _RSA_sign
0001:007e44dd  _int_rsa_verify
0001:007e4959  _RSA_verify
Module: U:\extras\lib\libcrypto.lib(m_dss1.obj)
0001:007e4a9c  _EVP_dss1
Module: U:\extras\lib\libcrypto.lib(p_verify.obj)
0001:007e4abb  _EVP_VerifyFinal
Module: U:\extras\lib\libcrypto.lib(m_ecdsa.obj)
0001:007e4d8c  _EVP_ecdsa
Module: U:\extras\lib\libcrypto.lib(ech_key.obj)
0001:007e4da0  _ECDH_compute_key
Module: U:\extras\lib\libcrypto.lib(pmeth_fn.obj)
0001:007e4dfb  _EVP_PKEY_sign_init
0001:007e4e94  _EVP_PKEY_sign
0001:007e4fcc  _EVP_PKEY_verify_init
0001:007e5065  _EVP_PKEY_verify
0001:007e5125* _EVP_PKEY_verify_recover_init
0001:007e51be* _EVP_PKEY_verify_recover
0001:007e52f6  _EVP_PKEY_encrypt_init
0001:007e538f  _EVP_PKEY_encrypt
0001:007e54c9  _EVP_PKEY_decrypt_init
0001:007e5562  _EVP_PKEY_decrypt
0001:007e569c* _EVP_PKEY_derive_init
0001:007e5735  _EVP_PKEY_derive_set_peer
0001:007e59cf* _EVP_PKEY_derive
Module: U:\extras\lib\libcrypto.lib(dsa_sign.obj)
0001:007e5b00* _DSA_do_sign
0001:007e5b27  _DSA_sign
0001:007e5b9c  _DSA_sign_setup
Module: U:\extras\lib\libcrypto.lib(ecs_sign.obj)
0001:007e5bd0* _ECDSA_do_sign
0001:007e5c01* _ECDSA_do_sign_ex
0001:007e5c51  _ECDSA_sign
0001:007e5c97* _ECDSA_sign_ex
0001:007e5d1a  _ECDSA_sign_setup
Module: U:\extras\lib\libcrypto.lib(x509type.obj)
0001:007e5d70  _X509_certificate_type
Module: U:\extras\lib\libcrypto.lib(bss_mem.obj)
0001:007e5eae  _BIO_s_mem
0001:007e5ec2  _BIO_new_mem_buf
Module: U:\extras\lib\libcrypto.lib(rsa_asn1.obj)
0001:007e6650  _RSAPrivateKey_it
0001:007e66c0  _RSAPublicKey_it
0001:007e66dc  _d2i_RSAPrivateKey
0001:007e6705  _i2d_RSAPrivateKey
0001:007e6727  _d2i_RSAPublicKey
0001:007e6750  _i2d_RSAPublicKey
0001:007e6772* _RSAPublicKey_dup
0001:007e678d  _RSAPrivateKey_dup
Module: U:\extras\lib\libssl.lib(t1_enc.obj)
0001:007e6eef  _tls1_change_cipher_state
0001:007e777a  _tls1_setup_key_block
0001:007e7a4a  _tls1_enc
0001:007e7e26  _tls1_cert_verify_mac
0001:007e7f4d  _tls1_final_finish_mac
0001:007e8165  _tls1_mac
0001:007e8437  _tls1_generate_master_secret
0001:007e8507  _tls1_alert_code
Module: U:\extras\lib\libssl.lib(t1_reneg.obj)
0001:007e880b  _ssl_add_clienthello_renegotiate_ext
0001:007e88c3  _ssl_parse_clienthello_renegotiate_ext
0001:007e8a3c  _ssl_add_serverhello_renegotiate_ext
0001:007e8bd9  _ssl_parse_serverhello_renegotiate_ext
Module: U:\extras\lib\libcrypto.lib(hmac.obj)
0001:007e8ea9  _HMAC_Init_ex
0001:007e915e* _HMAC_Init
0001:007e9273  _HMAC_CTX_init
0001:007e91a5  _HMAC_Update
0001:007e91c9  _HMAC_Final
0001:007e92a5  _HMAC_CTX_copy
0001:007e934a  _HMAC_CTX_cleanup
0001:007e9397  _HMAC
0001:007e9443* _HMAC_CTX_set_flags
Module: U:\extras\lib\libcrypto.lib(e_aes.obj)
0001:007e9724  _EVP_aes_128_cbc
0001:007e9764* _EVP_aes_128_cfb128
0001:007e97a4* _EVP_aes_128_ofb
0001:007e97e4* _EVP_aes_128_ecb
0001:007e9a84* _EVP_aes_192_cbc
0001:007e9ac4* _EVP_aes_192_cfb128
0001:007e9b04* _EVP_aes_192_ofb
0001:007e9b44* _EVP_aes_192_ecb
0001:007e9de4* _EVP_aes_256_cbc
0001:007e9e24* _EVP_aes_256_cfb128
0001:007e9e64* _EVP_aes_256_ofb
0001:007e9ea4* _EVP_aes_256_ecb
0001:007e9fa4* _EVP_aes_128_cfb1
0001:007ea0a4* _EVP_aes_192_cfb1
0001:007ea1a4* _EVP_aes_256_cfb1
0001:007ea284* _EVP_aes_128_cfb8
0001:007ea364* _EVP_aes_192_cfb8
0001:007ea444* _EVP_aes_256_cfb8
Module: U:\extras\lib\xmlrpc.lib(encodings.obj)
0001:007ea65c  _utf8_decode
0001:007ea67e* _utf8_encode
Module: U:\extras\lib\expat.lib(xmlparse.obj)
0001:007ea6d3* _XML_UseParserAsHandlerArg
0001:007ea6de* _XML_UseForeignDTD
0001:007ea708* _XML_SetReturnNSTriplet
0001:007ea72c  _XML_SetUserData
0001:007ea747* _XML_GetBase
0001:007ea755* _XML_GetSpecifiedAttributeCount
0001:007ea763* _XML_GetIdAttributeIndex
0001:007ea771  _XML_SetElementHandler
0001:007ea785* _XML_SetStartElementHandler
0001:007ea793* _XML_SetEndElementHandler
0001:007ea7a1  _XML_SetCharacterDataHandler
0001:007ea7af* _XML_SetProcessingInstructionHandler
0001:007ea7bd* _XML_SetCommentHandler
0001:007ea7cb* _XML_SetCdataSectionHandler
0001:007ea7df* _XML_SetStartCdataSectionHandler
0001:007ea7ed* _XML_SetEndCdataSectionHandler
0001:007ea7fb* _XML_SetDefaultHandler
0001:007ea810* _XML_SetDefaultHandlerExpand
0001:007ea825* _XML_SetDoctypeDeclHandler
0001:007ea839* _XML_SetStartDoctypeDeclHandler
0001:007ea847* _XML_SetEndDoctypeDeclHandler
0001:007ea855* _XML_SetUnparsedEntityDeclHandler
0001:007ea863* _XML_SetNotationDeclHandler
0001:007ea871* _XML_SetNamespaceDeclHandler
0001:007ea885* _XML_SetStartNamespaceDeclHandler
0001:007ea893* _XML_SetEndNamespaceDeclHandler
0001:007ea8a1* _XML_SetNotStandaloneHandler
0001:007ea8af* _XML_SetExternalEntityRefHandler
0001:007ea8bd* _XML_SetExternalEntityRefHandlerArg
0001:007ea8d4* _XML_SetSkippedEntityHandler
0001:007ea8e2* _XML_SetUnknownEncodingHandler
0001:007ea8f9* _XML_SetElementDeclHandler
0001:007ea90a* _XML_SetAttlistDeclHandler
0001:007ea91b* _XML_SetEntityDeclHandler
0001:007ea92c* _XML_SetXmlDeclHandler
0001:007ea93d* _XML_SetParamEntityParsing
0001:007ea967* _XML_ParseBuffer
0001:007eaa98* _XML_StopParser
0001:007eab0f* _XML_ResumeParser
0001:007eabf8  _XML_GetErrorCode
0001:007eac06  _XML_GetCurrentByteIndex
0001:007eac25  _XML_GetCurrentByteCount
0001:007eac47* _XML_GetInputContext
0001:007eac78  _XML_GetCurrentLineNumber
0001:007eacd1  _XML_GetCurrentColumnNumber
0001:007ead27* _XML_FreeContentModel
0001:007ead3c* _XML_MemMalloc
0001:007ead51* _XML_MemRealloc
0001:007ead6c* _XML_MemFree
0001:007ead81  _XML_ErrorString
0001:007eada6* _XML_ExpatVersion
0001:007eadb0* _XML_ExpatVersionInfo
0001:007eadce* _XML_GetFeatureList
0001:007eaec6* _XML_DefaultCurrent
0001:007eb689  _XML_ParserFree
0001:007ebada* _XML_GetParsingStatus
0001:007ebb20* _XML_GetBuffer
0001:007ebca2  _XML_Parse
0001:007ebff5* _XML_SetBase
0001:007ec03f* _XML_SetEncoding
0001:007edaaa* _XML_ExternalEntityParserCreate
0001:007ee0cd* _XML_ParserReset
0001:007ee421* _XML_ParserCreate_MM
0001:007ee46e* _XML_ParserCreateNS
0001:007ee496  _XML_ParserCreate
Module: U:\extras\lib\xmlrpc.lib(base64.obj)
0001:007f3c50  _buffer_delete
0001:007f3c85* _buffer_add
0001:007f3cd6* _buffer_new
0001:007f3d08  _base64_decode
0001:007f3e92  _base64_encode
Module: U:\extras\lib\libcrypto.lib(evp_key.obj)
0001:007f4020* _EVP_set_pw_prompt
0001:007f4059  _EVP_get_pw_prompt
0001:007f4073* _EVP_read_pw_string
0001:007f40a3  _EVP_read_pw_string_min
0001:007f41c6  _EVP_BytesToKey
Module: U:\extras\lib\libcrypto.lib(encode.obj)
0001:007f44e0  _EVP_EncodeInit
0001:007f4537  _EVP_EncodeUpdate
0001:007f475e  _EVP_EncodeBlock
0001:007f46f9  _EVP_EncodeFinal
0001:007f48a2  _EVP_DecodeInit
0001:007f48ef  _EVP_DecodeUpdate
0001:007f4b9f  _EVP_DecodeBlock
0001:007f4d1b  _EVP_DecodeFinal
Module: U:\extras\lib\libcrypto.lib(rsa_ameth.obj)
0001:007f5790  _rsa_asn1_meths
Module: U:\extras\lib\libcrypto.lib(dh_ameth.obj)
0001:007f65d7* _DHparams_print
0001:007f6630  _dh_asn1_meth
Module: U:\extras\lib\libcrypto.lib(dsa_ameth.obj)
0001:007f7950  _dsa_asn1_meths
Module: U:\extras\lib\libcrypto.lib(ec_ameth.obj)
0001:007f8ea0  _eckey_asn1_meth
Module: U:\extras\lib\libcrypto.lib(hm_ameth.obj)
0001:007f9090  _hmac_asn1_meth
Module: U:\extras\lib\libcrypto.lib(tb_asnmth.obj)
0001:007f90f0* _ENGINE_unregister_pkey_asn1_meths
0001:007f911f* _ENGINE_register_pkey_asn1_meths
0001:007f9197* _ENGINE_register_all_pkey_asn1_meths
0001:007f91c8* _ENGINE_set_default_pkey_asn1_meths
0001:007f9240  _ENGINE_get_pkey_asn1_meth_engine
0001:007f9267  _ENGINE_get_pkey_asn1_meth
0001:007f92de* _ENGINE_get_pkey_asn1_meths
0001:007f92e9* _ENGINE_set_pkey_asn1_meths
0001:007f92fc  _engine_pkey_asn1_meths_free
0001:007f9387* _ENGINE_get_pkey_asn1_meth_str
0001:007f952e  _ENGINE_pkey_asn1_find_str
Module: U:\extras\lib\libcrypto.lib(evp_asn1.obj)
0001:007f95d0  _ASN1_TYPE_set_octetstring
0001:007f9642  _ASN1_TYPE_get_octetstring
0001:007f96da* _ASN1_TYPE_set_int_octetstring
0001:007f9847* _ASN1_TYPE_get_int_octetstring
Module: U:\extras\lib\libcrypto.lib(pcy_tree.obj)
0001:007fa7cf  _X509_policy_tree_free
0001:007fa8b4  _X509_policy_check
Module: U:\extras\lib\libcrypto.lib(a_utctm.obj)
0001:007faa70  _ASN1_UTCTIME_check
0001:007facb8* _ASN1_UTCTIME_set_string
0001:007fad2a* _ASN1_UTCTIME_set
0001:007fad78  _ASN1_UTCTIME_adj
0001:007faf4b* _ASN1_UTCTIME_cmp_time_t
Module: U:\extras\lib\libcrypto.lib(a_gentm.obj)
0001:007fb390  _ASN1_GENERALIZEDTIME_check
0001:007fb630* _ASN1_GENERALIZEDTIME_set_string
0001:007fb6a2* _ASN1_GENERALIZEDTIME_set
0001:007fb6f0  _ASN1_GENERALIZEDTIME_adj
Module: U:\extras\lib\libcrypto.lib(a_time.obj)
0001:007fb910  _ASN1_TIME_it
0001:007fb92c* _d2i_ASN1_TIME
0001:007fb955* _i2d_ASN1_TIME
0001:007fb977* _ASN1_TIME_new
0001:007fb98b  _ASN1_TIME_free
0001:007fb9a6* _ASN1_TIME_set
0001:007fb9d9  _ASN1_TIME_adj
0001:007fbabc  _ASN1_TIME_check
0001:007fbaff* _ASN1_TIME_to_generalizedtime
0001:007fbc40* _ASN1_TIME_set_string
Module: U:\extras\lib\libcrypto.lib(x_bignum.obj)
0001:007fbcd0  _BIGNUM_it
0001:007fbcf0  _CBIGNUM_it
Module: U:\extras\lib\libcrypto.lib(x_long.obj)
0001:007fbe80  _LONG_it
0001:007fbeb0  _ZLONG_it
Module: U:\extras\lib\libcrypto.lib(bn_rand.obj)
0001:007fc3e5  _BN_rand
0001:007fc415  _BN_pseudo_rand
0001:007fc445* _BN_bntest_rand
0001:007fc6d3  _BN_rand_range
0001:007fc6f5  _BN_pseudo_rand_range
Module: U:\extras\lib\libcrypto.lib(tasn_utl.obj)
0001:007fc720  _asn1_get_choice_selector
0001:007fc740  _asn1_set_choice_selector
0001:007fc779  _asn1_do_lock
0001:007fc869  _asn1_enc_init
0001:007fc8a9  _asn1_enc_free
0001:007fc8ff  _asn1_enc_save
0001:007fc9a4  _asn1_enc_restore
0001:007fca28  _asn1_get_field_ptr
0001:007fca59  _asn1_do_adb
Module: U:\extras\lib\libcrypto.lib(a_type.obj)
0001:007fcb70  _ASN1_TYPE_get
0001:007fcb95  _ASN1_TYPE_set
0001:007fcbf1  _ASN1_TYPE_set1
0001:007fcc9b  _ASN1_TYPE_cmp
Module: U:\extras\lib\libcrypto.lib(a_bitstr.obj)
0001:007fcd20  _ASN1_BIT_STRING_set
0001:007fcd41  _i2c_ASN1_BIT_STRING
0001:007fcf01  _c2i_ASN1_BIT_STRING
0001:007fd0cd  _ASN1_BIT_STRING_set_bit
0001:007fd2af  _ASN1_BIT_STRING_get_bit
0001:007fd324* _ASN1_BIT_STRING_check
Module: U:\extras\lib\libcrypto.lib(v3_alt.obj)
0001:007fd3a0  _v3_alt
0001:007fd448  _i2v_GENERAL_NAMES
0001:007fd525  _i2v_GENERAL_NAME
0001:007fd8b0  _GENERAL_NAME_print
0001:007fe259  _v2i_GENERAL_NAME
0001:007fe182  _v2i_GENERAL_NAMES
0001:007fe605  _v2i_GENERAL_NAME_ex
0001:007fe291* _a2i_GENERAL_NAME
Module: U:\extras\lib\libcrypto.lib(a_utf8.obj)
0001:007fe9e0  _UTF8_getc
0001:007fee90  _UTF8_putc
Module: U:\extras\lib\libcrypto.lib(asn1_par.obj)
0001:007fff1c  _ASN1_tag2str
0001:007ff2ee* _ASN1_parse
0001:007ff32e  _ASN1_parse_dump
Module: U:\extras\lib\libcrypto.lib(x509name.obj)
0001:00800140* _X509_NAME_get_text_by_NID
0001:00800183* _X509_NAME_get_text_by_OBJ
0001:00800277* _X509_NAME_get_index_by_OBJ
0001:008002f6  _X509_NAME_get_entry
0001:00800ab1  _X509_NAME_ENTRY_get_data
0001:00800219  _X509_NAME_entry_count
0001:0080023b  _X509_NAME_get_index_by_NID
0001:00800337  _X509_NAME_delete_entry
0001:00800426* _X509_NAME_add_entry_by_OBJ
0001:00800882* _X509_NAME_ENTRY_create_by_OBJ
0001:00800584  _X509_NAME_add_entry
0001:00800497* _X509_NAME_add_entry_by_NID
0001:008007fb* _X509_NAME_ENTRY_create_by_NID
0001:00800508  _X509_NAME_add_entry_by_txt
0001:00800751* _X509_NAME_ENTRY_create_by_txt
0001:00800936* _X509_NAME_ENTRY_set_object
0001:008009a7* _X509_NAME_ENTRY_set_data
0001:00800a9a  _X509_NAME_ENTRY_get_object
Module: U:\extras\lib\libcrypto.lib(t_x509.obj)
0001:00800ad0* _X509_print_fp
0001:00800b03* _X509_print_ex_fp
0001:00800d41* _X509_print_ex
0001:00800ba7* _X509_print
0001:00801849* _ASN1_TIME_print
0001:00801626* _X509_signature_print
0001:00801418* _X509_ocspid_print
0001:00801749  _ASN1_STRING_print
0001:00801c7d  _ASN1_UTCTIME_print
0001:00801903  _ASN1_GENERALIZEDTIME_print
0001:00801f15  _X509_NAME_print
Module: U:\extras\lib\libcrypto.lib(a_mbstr.obj)
0001:00802090  _ASN1_mbstring_copy
0001:008020ef  _ASN1_mbstring_ncopy
Module: U:\extras\lib\libcrypto.lib(md5_dgst.obj)
0001:00802ab0  _MD5_Update
0001:00802e55* _md5_block_data_order
0001:00802c67* _MD5_Transform
0001:00802c89  _MD5_Final
0001:00802de0* _MD5_version
0001:00802e06  _MD5_Init
Module: U:\extras\lib\libcrypto.lib(sha1dgst.obj)
0001:00803af0* _SHA1_version
0001:00803b17  _SHA1_Update
0001:00803cce* _SHA1_Transform
0001:00803cf0  _SHA1_Final
0001:00803ebe  _SHA1_Init
Module: U:\extras\lib\libcrypto.lib(sha256.obj)
0001:00806680* _SHA256_version
0001:008066aa  _SHA224_Init
0001:0080672b  _SHA256_Init
0001:008067ac* _SHA224
0001:008068af  _SHA256_Update
0001:00806a88  _SHA256_Final
0001:00806810* _SHA256
0001:00806874* _SHA224_Update
0001:00806895* _SHA224_Final
0001:00806a66* _SHA256_Transform
Module: U:\extras\lib\libcrypto.lib(sha512.obj)
0001:008090b0* _SHA512_version
0001:008090da  _SHA384_Init
0001:008091a7  _SHA512_Init
0001:00809274  _SHA512_Final
0001:00809686* _SHA384_Final
0001:008096a0  _SHA512_Update
0001:00809859* _SHA384_Update
0001:0080987a* _SHA512_Transform
0001:0080989c* _SHA384
0001:0080990c* _SHA512
Module: U:\extras\lib\libcrypto.lib(a_enum.obj)
0001:0080a579* _ASN1_ENUMERATED_set
0001:0080a6b5  _ASN1_ENUMERATED_get
0001:0080a75f* _BN_to_ASN1_ENUMERATED
0001:0080a8b5  _ASN1_ENUMERATED_to_BN
Module: U:\extras\lib\libcrypto.lib(a_verify.obj)
0001:0080a94b* _ASN1_verify
0001:0080ab11  _ASN1_item_verify
Module: U:\extras\lib\libcrypto.lib(p5_crpt.obj)
0001:0080ad80* _PKCS5_PBE_add
0001:0080adeb  _PKCS5_PBE_keyivgen
Module: U:\extras\lib\libcrypto.lib(p12_crpt.obj)
0001:0080b160* _PKCS12_PBE_add
0001:0080b170  _PKCS12_PBE_keyivgen
Module: U:\extras\lib\libcrypto.lib(p5_crpt2.obj)
0001:0080b400* _PKCS5_PBKDF2_HMAC
0001:0080b5ed* _PKCS5_PBKDF2_HMAC_SHA1
0001:0080b653  _PKCS5_v2_PBE_keyivgen
Module: U:\extras\lib\libcrypto.lib(eng_table.obj)
0001:0080bb90* _ENGINE_get_table_flags
0001:0080bb9a* _ENGINE_set_table_flags
0001:0080bc67  _engine_table_register
0001:0080bf28  _engine_table_unregister
0001:0080c005  _engine_table_cleanup
0001:0080c089  _engine_table_select
0001:0080c2ab  _engine_table_doall
Module: U:\extras\lib\libcrypto.lib(eng_list.obj)
0001:0080c952* _ENGINE_remove
0001:0080c5e3  _ENGINE_get_first
0001:0080c653* _ENGINE_get_last
0001:0080c6c3  _ENGINE_get_next
0001:0080c77f* _ENGINE_get_prev
0001:0080c83b* _ENGINE_add
0001:0080cb68* _ENGINE_by_id
0001:0080cdd3* _ENGINE_up_ref
Module: U:\extras\lib\libcrypto.lib(rand_os2.obj)
0001:0080ce64  _RAND_poll
0002:0001f690* _hDoscalls
Module: U:\extras\lib\libcrypto.lib(v3_conf.obj)
0001:0080d07b* _X509V3_EXT_nconf
0001:0080d167* _X509V3_EXT_nconf_nid
0001:0080d633  _X509V3_EXT_i2d
0001:0080da11* _X509V3_EXT_add_nconf_sk
0001:0080dad9* _X509V3_EXT_add_nconf
0001:0080db19* _X509V3_EXT_CRL_add_nconf
0001:0080db59* _X509V3_EXT_REQ_add_nconf
0001:0080dbdb* _X509V3_get_string
0001:0080dc6a  _X509V3_get_section
0001:0080dcf5* _X509V3_string_free
0001:0080dd2e  _X509V3_section_free
0001:0080dda2  _X509V3_set_nconf
0001:0080ddba* _X509V3_set_ctx
0001:0080ddeb* _X509V3_EXT_conf
0001:0080de25* _X509V3_EXT_conf_nid
0001:0080de9a* _X509V3_set_conf_lhash
0001:0080deb2* _X509V3_EXT_add_conf
0001:0080deec* _X509V3_EXT_CRL_add_conf
0001:0080df26* _X509V3_EXT_REQ_add_conf
Module: U:\extras\lib\libcrypto.lib(v3_utl.obj)
0001:0080dfeb  _X509V3_add_value
0001:0080e132  _X509V3_add_value_uchar
0001:0080e153  _X509V3_conf_free
0001:0080e1c0  _X509V3_add_value_bool
0001:0080e204* _X509V3_add_value_bool_nf
0001:0080e233  _i2s_ASN1_ENUMERATED
0001:0080e2c0  _i2s_ASN1_INTEGER
0001:0080e34d  _s2i_ASN1_INTEGER
0001:0080e4fd  _X509V3_add_value_int
0001:0080e598  _X509V3_get_value_bool
0001:0080e75d  _X509V3_get_value_int
0001:0080e7d9  _X509V3_parse_list
0001:0080eb48  _hex_to_string
0001:0080ec2c  _string_to_hex
0001:0080ee80  _name_cmp
0001:0080eefe* _X509_get1_email
0001:0080ef60* _X509_get1_ocsp
0001:0080f021* _X509_REQ_get1_email
0001:0080f26d* _X509_email_free
0001:0080f289  _a2i_IPADDRESS
0001:0080f428* _a2i_ipadd
0001:0080f2fa  _a2i_IPADDRESS_NC
0001:0080f8cb  _X509V3_NAME_from_section
Module: U:\extras\lib\libcrypto.lib(pcy_data.obj)
0001:0080fa00  _policy_data_free
0001:0080fa66  _policy_data_new
Module: U:\extras\lib\libcrypto.lib(v3_cpols.obj)
0001:0080fb90  _v3_cpols
0001:0080fc00* _CERTIFICATEPOLICIES_it
0001:0080fcf0* _POLICYINFO_it
0001:0080fc1c* _d2i_CERTIFICATEPOLICIES
0001:0080fc45* _i2d_CERTIFICATEPOLICIES
0001:0080fc67* _CERTIFICATEPOLICIES_new
0001:0080fc7b* _CERTIFICATEPOLICIES_free
0001:0080fe60* _POLICYQUALINFO_it
0001:0080fd0c* _d2i_POLICYINFO
0001:0080fd35* _i2d_POLICYINFO
0001:0080fd57* _POLICYINFO_new
0001:0080fd6b  _POLICYINFO_free
0001:0080ff50* _USERNOTICE_it
0001:0080fe7c* _d2i_POLICYQUALINFO
0001:0080fea5* _i2d_POLICYQUALINFO
0001:0080fec7* _POLICYQUALINFO_new
0001:0080fedb  _POLICYQUALINFO_free
0001:00810040* _NOTICEREF_it
0001:0080ff6c* _d2i_USERNOTICE
0001:0080ff95* _i2d_USERNOTICE
0001:0080ffb7* _USERNOTICE_new
0001:0080ffcb* _USERNOTICE_free
0001:0081005c* _d2i_NOTICEREF
0001:00810085* _i2d_NOTICEREF
0001:008100a7* _NOTICEREF_new
0001:008100bb* _NOTICEREF_free
0001:008111ba* _X509_POLICY_NODE_print
Module: U:\extras\lib\libcrypto.lib(pcy_map.obj)
0001:008112b0  _policy_cache_set_mapping
Module: U:\extras\lib\libcrypto.lib(v3_pcons.obj)
0001:00811480  _v3_policy_constraints
0001:00811530* _POLICY_CONSTRAINTS_it
0001:0081154c* _POLICY_CONSTRAINTS_new
0001:00811560  _POLICY_CONSTRAINTS_free
Module: U:\extras\lib\libcrypto.lib(tb_pkmeth.obj)
0001:008117e0* _ENGINE_unregister_pkey_meths
0001:0081180f* _ENGINE_register_pkey_meths
0001:00811887* _ENGINE_register_all_pkey_meths
0001:008118b8* _ENGINE_set_default_pkey_meths
0001:00811930  _ENGINE_get_pkey_meth_engine
0001:00811957  _ENGINE_get_pkey_meth
0001:008119ce* _ENGINE_get_pkey_meths
0001:008119d9* _ENGINE_set_pkey_meths
0001:008119ec  _engine_pkey_meths_free
Module: U:\extras\lib\libcrypto.lib(bn_exp.obj)
0001:00811a89* _BN_exp
0001:00811c49  _BN_mod_exp
0001:00812ea9  _BN_mod_exp_mont_word
0001:008121f0  _BN_mod_exp_mont
0001:00811d33* _BN_mod_exp_recp
0001:0081292f* _BN_mod_exp_mont_consttime
0001:008133d2* _BN_mod_exp_simple
Module: U:\extras\lib\libcrypto.lib(rsa_pk1.obj)
0001:008137ea  _RSA_padding_add_PKCS1_type_1
0001:0081389b  _RSA_padding_check_PKCS1_type_1
0001:00813a3b  _RSA_padding_add_PKCS1_type_2
0001:00813b33  _RSA_padding_check_PKCS1_type_2
Module: U:\extras\lib\libcrypto.lib(rsa_oaep.obj)
0001:00813cab  _RSA_padding_add_PKCS1_OAEP
0001:00813f35  _RSA_padding_check_PKCS1_OAEP
0001:00814246  _PKCS1_MGF1
Module: U:\extras\lib\libcrypto.lib(rsa_ssl.obj)
0001:008143da  _RSA_padding_add_SSLv23
0001:008144f4  _RSA_padding_check_SSLv23
Module: U:\extras\lib\libcrypto.lib(rsa_none.obj)
0001:008146cb  _RSA_padding_add_none
0001:00814767  _RSA_padding_check_none
Module: U:\extras\lib\libcrypto.lib(bn_mont.obj)
0001:00814800  _BN_mod_mul_montgomery
0001:00814d93  _BN_from_montgomery
0001:00814e0b  _BN_MONT_CTX_new
0001:00814e57* _BN_MONT_CTX_init
0001:00814eb2  _BN_MONT_CTX_free
0001:00814f05  _BN_MONT_CTX_set
0001:00815179  _BN_MONT_CTX_copy
0001:0081521f  _BN_MONT_CTX_set_locked
Module: U:\extras\lib\libcrypto.lib(rsa_x931.obj)
0001:0081535b  _RSA_padding_add_X931
0001:00815429  _RSA_padding_check_X931
0001:008155b6  _RSA_X931_hash_id
Module: U:\extras\lib\libcrypto.lib(bn_div.obj)
0001:00815619  _BN_div
Module: U:\extras\lib\libcrypto.lib(bn_mod.obj)
0001:00816360  _BN_nnmod
0001:008163d8  _BN_mod_add
0001:00816424  _BN_mod_add_quick
0001:00816486* _BN_mod_sub
0001:008164d2  _BN_mod_sub_quick
0001:00816528  _BN_mod_mul
0001:008165e6  _BN_mod_sqr
0001:0081663a* _BN_mod_lshift1
0001:0081667f  _BN_mod_lshift1_quick
0001:008166da* _BN_mod_lshift
0001:0081678e  _BN_mod_lshift_quick
Module: U:\extras\lib\libcrypto.lib(bn_asm.obj)
0001:008168e0  _bn_mul_add_words
0001:00816db0  _bn_mul_words
0001:008171cd  _bn_sqr_words
0001:00817424  _bn_div_words
0001:008175b1  _bn_add_words
0001:00817763  _bn_sub_words
0001:0081790a  _bn_mul_comba8
0001:0081d14c  _bn_mul_comba4
0001:0081e5de  _bn_sqr_comba8
0001:00821b7c  _bn_sqr_comba4
Module: U:\extras\lib\libcrypto.lib(dh_check.obj)
0001:00822780* _DH_check
0001:0082295d  _DH_check_pub_key
Module: U:\extras\lib\libcrypto.lib(dsa_ossl.obj)
0001:00822a53  _DSA_OpenSSL
Module: U:\extras\lib\libcrypto.lib(tb_dsa.obj)
0001:008235c4* _ENGINE_unregister_DSA
0001:008235f3* _ENGINE_register_DSA
0001:0082363f* _ENGINE_register_all_DSA
0001:00823670* _ENGINE_set_default_DSA
0001:008236bc  _ENGINE_get_default_DSA
0001:008236d9  _ENGINE_get_DSA
0001:008236e4* _ENGINE_set_DSA
Module: U:\extras\lib\libcrypto.lib(v3_lib.obj)
0001:00823709* _X509V3_EXT_add
0001:00823828  _X509V3_EXT_get_nid
0001:008238bc  _X509V3_EXT_get
0001:008238ec* _X509V3_EXT_add_list
0001:0082391f* _X509V3_EXT_add_alias
0001:00823a0b* _X509V3_EXT_cleanup
0001:00823a53* _X509V3_add_standard_extensions
0001:00823a5d  _X509V3_EXT_d2i
0001:00823ae3  _X509V3_get_d2i
0001:00823c0b  _X509V3_add1_i2d
Module: U:\extras\lib\libcrypto.lib(x_req.obj)
0001:00823ee0  _X509_REQ_INFO_it
0001:00823efc* _d2i_X509_REQ_INFO
0001:00823f25* _i2d_X509_REQ_INFO
0001:00823f47* _X509_REQ_INFO_new
0001:00823f5b* _X509_REQ_INFO_free
0001:00824010  _X509_REQ_it
0001:0082402c  _d2i_X509_REQ
0001:00824055  _i2d_X509_REQ
0001:00824077  _X509_REQ_new
0001:0082408b  _X509_REQ_free
0001:008240a6* _X509_REQ_dup
Module: U:\extras\lib\libcrypto.lib(x_spki.obj)
0001:00824130  _NETSCAPE_SPKAC_it
0001:0082414c* _d2i_NETSCAPE_SPKAC
0001:00824175* _i2d_NETSCAPE_SPKAC
0001:00824197* _NETSCAPE_SPKAC_new
0001:008241ab* _NETSCAPE_SPKAC_free
0001:00824230* _NETSCAPE_SPKI_it
0001:0082424c* _d2i_NETSCAPE_SPKI
0001:00824275* _i2d_NETSCAPE_SPKI
0001:00824297* _NETSCAPE_SPKI_new
0001:008242ab* _NETSCAPE_SPKI_free
Module: U:\extras\lib\libcrypto.lib(a_sign.obj)
0001:008242d9* _ASN1_sign
0001:00824644  _ASN1_item_sign
Module: U:\extras\lib\libcrypto.lib(a_d2i_fp.obj)
0001:008249cb  _ASN1_d2i_fp
0001:00824a6f  _ASN1_d2i_bio
0001:00824add  _ASN1_item_d2i_bio
0001:00824b52  _ASN1_item_d2i_fp
Module: U:\extras\lib\libcrypto.lib(a_i2d_fp.obj)
0001:00824f5b  _ASN1_i2d_fp
0001:00824ff8  _ASN1_i2d_bio
0001:008250e6  _ASN1_item_i2d_fp
0001:00825183  _ASN1_item_i2d_bio
Module: U:\extras\lib\libcrypto.lib(pk7_asn1.obj)
0001:00825620* _PKCS7_SIGNED_it
0001:008259e0* _PKCS7_ENVELOPE_it
0001:00825d80* _PKCS7_SIGN_ENVELOPE_it
0001:00825f60* _PKCS7_DIGEST_it
0001:00825e60* _PKCS7_ENCRYPT_it
0001:00825480  _PKCS7_it
0001:0082549c  _d2i_PKCS7
0001:008254c5  _i2d_PKCS7
0001:008254e7  _PKCS7_new
0001:008254fb  _PKCS7_free
0001:00825516* _i2d_PKCS7_NDEF
0001:00825538* _PKCS7_dup
0001:008257f0* _PKCS7_SIGNER_INFO_it
0001:0082563c* _d2i_PKCS7_SIGNED
0001:00825665* _i2d_PKCS7_SIGNED
0001:00825687  _PKCS7_SIGNED_new
0001:0082569b  _PKCS7_SIGNED_free
0001:008258e0  _PKCS7_ISSUER_AND_SERIAL_it
0001:0082580c* _d2i_PKCS7_SIGNER_INFO
0001:00825835* _i2d_PKCS7_SIGNER_INFO
0001:00825857  _PKCS7_SIGNER_INFO_new
0001:0082586b  _PKCS7_SIGNER_INFO_free
0001:008258fc* _d2i_PKCS7_ISSUER_AND_SERIAL
0001:00825925* _i2d_PKCS7_ISSUER_AND_SERIAL
0001:00825947* _PKCS7_ISSUER_AND_SERIAL_new
0001:0082595b* _PKCS7_ISSUER_AND_SERIAL_free
0001:00825b40* _PKCS7_RECIP_INFO_it
0001:00825c40* _PKCS7_ENC_CONTENT_it
0001:008259fc* _d2i_PKCS7_ENVELOPE
0001:00825a25* _i2d_PKCS7_ENVELOPE
0001:00825a47  _PKCS7_ENVELOPE_new
0001:00825a5b* _PKCS7_ENVELOPE_free
0001:00825b5c* _d2i_PKCS7_RECIP_INFO
0001:00825b85* _i2d_PKCS7_RECIP_INFO
0001:00825ba7  _PKCS7_RECIP_INFO_new
0001:00825bbb  _PKCS7_RECIP_INFO_free
0001:00825c5c* _d2i_PKCS7_ENC_CONTENT
0001:00825c85* _i2d_PKCS7_ENC_CONTENT
0001:00825ca7* _PKCS7_ENC_CONTENT_new
0001:00825cbb* _PKCS7_ENC_CONTENT_free
0001:00825d9c* _d2i_PKCS7_SIGN_ENVELOPE
0001:00825dc5* _i2d_PKCS7_SIGN_ENVELOPE
0001:00825de7  _PKCS7_SIGN_ENVELOPE_new
0001:00825dfb* _PKCS7_SIGN_ENVELOPE_free
0001:00825e7c* _d2i_PKCS7_ENCRYPT
0001:00825ea5* _i2d_PKCS7_ENCRYPT
0001:00825ec7  _PKCS7_ENCRYPT_new
0001:00825edb* _PKCS7_ENCRYPT_free
0001:00825f7c* _d2i_PKCS7_DIGEST
0001:00825fa5* _i2d_PKCS7_DIGEST
0001:00825fc7  _PKCS7_DIGEST_new
0001:00825fdb* _PKCS7_DIGEST_free
0001:00826040  _PKCS7_ATTR_SIGN_it
0001:00826090  _PKCS7_ATTR_VERIFY_it
0001:008260ac* _PKCS7_print_ctx
Module: U:\extras\lib\libcrypto.lib(dsa_asn1.obj)
0001:008261d0* _DSA_SIG_it
0001:008261ec  _d2i_DSA_SIG
0001:00826215  _i2d_DSA_SIG
0001:00826237  _DSA_SIG_new
0001:0082624b  _DSA_SIG_free
0001:00826380* _DSAPrivateKey_it
0001:0082639c  _d2i_DSAPrivateKey
0001:008263c5  _i2d_DSAPrivateKey
0001:00826450* _DSAparams_it
0001:0082646c  _d2i_DSAparams
0001:00826495  _i2d_DSAparams
0001:00826510* _dsa_pub_internal_it
0001:00826580* _DSAPublicKey_it
0001:0082659c* _d2i_DSAPublicKey
0001:008265c5  _i2d_DSAPublicKey
0001:008265e7* _DSAparams_dup
Module: U:\extras\lib\libcrypto.lib(ec_asn1.obj)
0001:00826610  _EC_GROUP_get_basis_type
0001:00826680* _EC_GROUP_get_trinomial_basis
0001:00826713* _EC_GROUP_get_pentanomial_basis
0001:00826840* _X9_62_PENTANOMIAL_it
0001:0082685c* _X9_62_PENTANOMIAL_new
0001:00826870* _X9_62_PENTANOMIAL_free
0001:008269b0* _X9_62_CHARACTERISTIC_TWO_it
0001:008269cc* _X9_62_CHARACTERISTIC_TWO_new
0001:008269e0* _X9_62_CHARACTERISTIC_TWO_free
0001:00826ad0* _X9_62_FIELDID_it
0001:00826b50* _X9_62_CURVE_it
0001:00826c30* _ECPARAMETERS_it
0001:00826c4c* _ECPARAMETERS_new
0001:00826c60* _ECPARAMETERS_free
0001:00826d10* _ECPKPARAMETERS_it
0001:00826d2c* _d2i_UC_ECPKPARAMETERS
0001:00826d55* _i2d_UC_ECPKPARAMETERS
0001:00826d77* _ECPKPARAMETERS_new
0001:00826d8b* _ECPKPARAMETERS_free
0001:00826e30* _EC_PRIVATEKEY_it
0001:00826e4c* _d2i_EC_PRIVATEKEY
0001:00826e75* _i2d_EC_PRIVATEKEY
0001:00826e97* _EC_PRIVATEKEY_new
0001:00826eab* _EC_PRIVATEKEY_free
0001:00828ac2  _d2i_ECPKParameters
0001:00828bb8  _i2d_ECPKParameters
0001:00828c7d  _d2i_ECPrivateKey
0001:00829004  _i2d_ECPrivateKey
0001:008294ae  _i2d_ECParameters
0001:00829504  _d2i_ECParameters
0001:00829612  _o2i_ECPublicKey
0001:0082976b  _i2o_ECPublicKey
Module: U:\extras\lib\libcrypto.lib(a_digest.obj)
0001:0082993b* _ASN1_digest
0001:00829a07  _ASN1_item_digest
Module: U:\extras\lib\libcrypto.lib(x_sig.obj)
0001:00829ad0  _X509_SIG_it
0001:00829aec  _d2i_X509_SIG
0001:00829b15  _i2d_X509_SIG
0001:00829b37  _X509_SIG_new
0001:00829b4b  _X509_SIG_free
Module: U:\extras\lib\libcrypto.lib(p8_pkey.obj)
0001:00829c70  _PKCS8_PRIV_KEY_INFO_it
0001:00829c8c  _d2i_PKCS8_PRIV_KEY_INFO
0001:00829cb5  _i2d_PKCS8_PRIV_KEY_INFO
0001:00829cd7  _PKCS8_PRIV_KEY_INFO_new
0001:00829ceb  _PKCS8_PRIV_KEY_INFO_free
0001:00829d06  _PKCS8_pkey_set0
0001:00829dee  _PKCS8_pkey_get0
Module: U:\extras\lib\libcrypto.lib(evp_pkey.obj)
0001:00829ec1  _EVP_PKCS82PKEY
0001:0082a06c  _EVP_PKEY2PKCS8
0001:0082a087* _EVP_PKEY2PKCS8_broken
0001:0082a1f1* _PKCS8_set_broken
0001:0082a260* _EVP_PKEY_get_attr_count
0001:0082a276* _EVP_PKEY_get_attr_by_NID
0001:0082a29a* _EVP_PKEY_get_attr_by_OBJ
0001:0082a2be* _EVP_PKEY_get_attr
0001:0082a2db* _EVP_PKEY_delete_attr
0001:0082a2f8* _EVP_PKEY_add1_attr
0001:0082a325* _EVP_PKEY_add1_attr_by_OBJ
0001:0082a367* _EVP_PKEY_add1_attr_by_NID
0001:0082a3a9* _EVP_PKEY_add1_attr_by_txt
Module: U:\extras\lib\libcrypto.lib(i2d_pr.obj)
0001:0082a3f9  _i2d_PrivateKey
Module: U:\extras\lib\libcrypto.lib(d2i_pr.obj)
0001:0082a4b9  _d2i_PrivateKey
0001:0082a681  _d2i_AutoPrivateKey
Module: U:\extras\lib\libcrypto.lib(x509_def.obj)
0001:0082a7e0* _X509_get_default_private_dir
0001:0082a7f2  _X509_get_default_cert_area
0001:0082a80a  _X509_get_default_cert_dir
0001:0082a825  _X509_get_default_cert_file
0001:0082a83c  _X509_get_default_cert_dir_env
0001:0082a854  _X509_get_default_cert_file_env
Module: U:\extras\lib\libcrypto.lib(pem_xaux.obj)
0001:0082a874  _PEM_read_bio_X509_AUX
0001:0082a8ad* _PEM_read_X509_AUX
0001:0082a8e6* _PEM_write_bio_X509_AUX
0001:0082a939* _PEM_write_X509_AUX
0001:0082a99d* _PEM_read_bio_X509_CERT_PAIR
0001:0082a9d6* _PEM_read_X509_CERT_PAIR
0001:0082aa0f* _PEM_write_bio_X509_CERT_PAIR
0001:0082aa62* _PEM_write_X509_CERT_PAIR
Module: U:\extras\lib\libcrypto.lib(pem_all.obj)
0001:0082aad4* _PEM_read_bio_X509_REQ
0001:0082ab0d* _PEM_read_X509_REQ
0001:0082ab46* _PEM_write_bio_X509_REQ
0001:0082ab99* _PEM_write_X509_REQ
0001:0082ac04* _PEM_write_bio_X509_REQ_NEW
0001:0082ac57* _PEM_write_X509_REQ_NEW
0001:0082acb3  _PEM_read_bio_X509_CRL
0001:0082acec* _PEM_read_X509_CRL
0001:0082ad25* _PEM_write_bio_X509_CRL
0001:0082ad78* _PEM_write_X509_CRL
0001:0082add1* _PEM_read_bio_PKCS7
0001:0082ae0a* _PEM_read_PKCS7
0001:0082ae43* _PEM_write_bio_PKCS7
0001:0082ae96* _PEM_write_PKCS7
0001:0082aef5* _PEM_read_bio_NETSCAPE_CERT_SEQUENCE
0001:0082af2e* _PEM_read_NETSCAPE_CERT_SEQUENCE
0001:0082af67* _PEM_write_bio_NETSCAPE_CERT_SEQUENCE
0001:0082afba* _PEM_write_NETSCAPE_CERT_SEQUENCE
0001:0082b066  _PEM_read_bio_RSAPrivateKey
0001:0082b0a4* _PEM_read_RSAPrivateKey
0001:0082b0f2  _PEM_write_bio_RSAPrivateKey
0001:0082b140* _PEM_write_RSAPrivateKey
0001:0082b19d* _PEM_read_bio_RSAPublicKey
0001:0082b1d6* _PEM_read_RSAPublicKey
0001:0082b20f* _PEM_write_bio_RSAPublicKey
0001:0082b262* _PEM_write_RSAPublicKey
0001:0082b2c0* _PEM_read_bio_RSA_PUBKEY
0001:0082b2f9* _PEM_read_RSA_PUBKEY
0001:0082b332* _PEM_write_bio_RSA_PUBKEY
0001:0082b385* _PEM_write_RSA_PUBKEY
0001:0082b431* _PEM_read_bio_DSAPrivateKey
0001:0082b47f* _PEM_write_bio_DSAPrivateKey
0001:0082b4cd* _PEM_write_DSAPrivateKey
0001:0082b51b* _PEM_read_bio_DSA_PUBKEY
0001:0082b554* _PEM_read_DSA_PUBKEY
0001:0082b58d* _PEM_write_bio_DSA_PUBKEY
0001:0082b5e0* _PEM_write_DSA_PUBKEY
0001:0082b633* _PEM_read_DSAPrivateKey
0001:0082b680* _PEM_read_bio_DSAparams
0001:0082b6b9* _PEM_read_DSAparams
0001:0082b6f2* _PEM_write_bio_DSAparams
0001:0082b745* _PEM_write_DSAparams
0001:0082b7f1* _PEM_read_bio_ECPrivateKey
0001:0082b83d* _PEM_read_bio_ECPKParameters
0001:0082b876* _PEM_read_ECPKParameters
0001:0082b8af* _PEM_write_bio_ECPKParameters
0001:0082b902* _PEM_write_ECPKParameters
0001:0082b964* _PEM_write_bio_ECPrivateKey
0001:0082b9b2* _PEM_write_ECPrivateKey
0001:0082ba00* _PEM_read_bio_EC_PUBKEY
0001:0082ba39* _PEM_read_EC_PUBKEY
0001:0082ba72* _PEM_write_bio_EC_PUBKEY
0001:0082bac5* _PEM_write_EC_PUBKEY
0001:0082bb18* _PEM_read_ECPrivateKey
0001:0082bb64* _PEM_read_bio_DHparams
0001:0082bb9d* _PEM_read_DHparams
0001:0082bbd6* _PEM_write_bio_DHparams
0001:0082bc29* _PEM_write_DHparams
0001:0082bc7c* _PEM_read_bio_PUBKEY
0001:0082bcb5* _PEM_read_PUBKEY
0001:0082bcee* _PEM_write_bio_PUBKEY
0001:0082bd41* _PEM_write_PUBKEY
Module: U:\extras\lib\libcrypto.lib(pem_info.obj)
0001:0082bdab* _PEM_X509_INFO_read
0001:0082beb8  _PEM_X509_INFO_read_bio
0001:0082c60d* _PEM_X509_INFO_write_bio
Module: U:\extras\lib\libcrypto.lib(x_info.obj)
0001:0082c8b9  _X509_INFO_new
0001:0082c968  _X509_INFO_free
Module: U:\extras\lib\libcrypto.lib(rsa_pmeth.obj)
0001:0082daf0  _rsa_pkey_meth
Module: U:\extras\lib\libcrypto.lib(dh_pmeth.obj)
0001:0082dfa0  _dh_pkey_meth
Module: U:\extras\lib\libcrypto.lib(dsa_pmeth.obj)
0001:0082e710  _dsa_pkey_meth
Module: U:\extras\lib\libcrypto.lib(ec_pmeth.obj)
0001:0082ee90  _ec_pkey_meth
Module: U:\extras\lib\libcrypto.lib(hm_pmeth.obj)
0001:0082f380  _hmac_pkey_meth
Module: U:\extras\lib\libcrypto.lib(pem_pkey.obj)
0001:0082f42d  _PEM_read_bio_PrivateKey
0001:0082f752* _PEM_write_bio_PrivateKey
0001:0082f823* _PEM_read_bio_Parameters
0001:0082f9a6* _PEM_write_bio_Parameters
0001:0082fa45  _PEM_read_PrivateKey
0001:0082fae9* _PEM_write_PrivateKey
Module: U:\extras\lib\libcrypto.lib(ec_cvt.obj)
0001:0082fb90  _EC_GROUP_new_curve_GFp
0001:0082fca3  _EC_GROUP_new_curve_GF2m
Module: U:\extras\lib\libcrypto.lib(ec_mult.obj)
0001:00830328  _ec_wNAF_mul
0001:0083110a  _ec_wNAF_precompute_mult
0001:00831741  _ec_wNAF_have_precompute_mult
Module: U:\extras\lib\libcrypto.lib(dsa_vrf.obj)
0001:00831780* _DSA_do_verify
0001:008317ae  _DSA_verify
Module: U:\extras\lib\libcrypto.lib(ecs_vrf.obj)
0001:00831830* _ECDSA_do_verify
0001:00831879  _ECDSA_verify
Module: U:\extras\lib\libcrypto.lib(ech_lib.obj)
0001:008318f0* _ECDH_version
0001:00831917* _ECDH_set_default_method
0001:00831924* _ECDH_get_default_method
0001:00831944* _ECDH_set_method
0001:00831b77  _ecdh_check
0001:00831bf5* _ECDH_get_ex_new_index
0001:00831c2c* _ECDH_set_ex_data
0001:00831c6b* _ECDH_get_ex_data
Module: U:\extras\lib\libcrypto.lib(ecs_lib.obj)
0001:00831cb0* _ECDSA_version
0001:00831cd8* _ECDSA_set_default_method
0001:00831ce5* _ECDSA_get_default_method
0001:00831d05* _ECDSA_set_method
0001:00831f38  _ecdsa_check
0001:00831fb6  _ECDSA_size
0001:008320b7* _ECDSA_get_ex_new_index
0001:008320ee* _ECDSA_set_ex_data
0001:0083212d* _ECDSA_get_ex_data
Module: U:\extras\lib\libcrypto.lib(ecs_asn1.obj)
0001:008321c0* _ECDSA_SIG_it
0001:008321dc  _d2i_ECDSA_SIG
0001:00832205  _i2d_ECDSA_SIG
0001:00832227  _ECDSA_SIG_new
0001:0083223b  _ECDSA_SIG_free
Module: U:\extras\lib\libcrypto.lib(pmeth_gn.obj)
0001:0083226b* _EVP_PKEY_paramgen_init
0001:00832304* _EVP_PKEY_paramgen
0001:008323f6* _EVP_PKEY_keygen_init
0001:0083248f* _EVP_PKEY_keygen
0001:00832581* _EVP_PKEY_CTX_set_cb
0001:0083258f* _EVP_PKEY_CTX_get_cb
0001:008325d2  _evp_pkey_set_cb_translate
0001:008325fc* _EVP_PKEY_CTX_get_keygen_info
0001:00832637  _EVP_PKEY_new_mac_key
Module: U:\extras\lib\libcrypto.lib(m_sigver.obj)
0001:008328df  _EVP_DigestSignInit
0001:00832916  _EVP_DigestVerifyInit
0001:0083294d  _EVP_DigestSignFinal
0001:00832aeb  _EVP_DigestVerifyFinal
Module: U:\extras\lib\libcrypto.lib(aes_cbc.obj)
0001:00832be0  _AES_cbc_encrypt
Module: U:\extras\lib\libcrypto.lib(aes_cfb.obj)
0001:00832c50  _AES_cfb128_encrypt
0001:00832c96  _AES_cfb1_encrypt
0001:00832cdc  _AES_cfb8_encrypt
Module: U:\extras\lib\libcrypto.lib(aes_ecb.obj)
0001:00832d30  _AES_ecb_encrypt
Module: U:\extras\lib\libcrypto.lib(aes_ofb.obj)
0001:00832d80  _AES_ofb128_encrypt
Module: U:\extras\lib\libcrypto.lib(aes_core.obj)
0001:00834ee8  _AES_set_encrypt_key
0001:00835585  _AES_set_decrypt_key
0001:00835948  _AES_encrypt
0001:00835fa7  _AES_decrypt
Module: U:\extras\lib\expat.lib(xmlrole.obj)
0001:00837f70  _XmlPrologStateInit
0001:00837f93  _XmlPrologStateInitExternalEntity
Module: U:\extras\lib\expat.lib(xmltok.obj)
0001:00846f8f  _XmlUtf8Encode
0001:0084702f* _XmlUtf16Encode
0001:00847077  _XmlSizeOfUnknownEncoding
0001:008472ac  _XmlInitUnknownEncoding
0001:008477d2  _XmlGetUtf8InternalEncoding
0001:008477dc* _XmlGetUtf16InternalEncoding
0001:00847843  _XmlInitEncoding
0001:00847935  _XmlParseXmlDecl
0001:00847985  _XmlGetUtf8InternalEncodingNS
0001:0084798f* _XmlGetUtf16InternalEncodingNS
0001:008479f6  _XmlInitEncodingNS
0001:00847ae8  _XmlParseXmlDeclNS
0001:00847b38  _XmlInitUnknownEncodingNS
Module: U:\extras\lib\libcrypto.lib(ui_lib.obj)
0001:00849a40  _UI_new
0001:00849a5d* _UI_new_method
0001:0084aa9a* _UI_get_default_method
0001:00849b77  _UI_free
0001:00849ef4  _UI_add_input_string
0001:00849f42* _UI_dup_input_string
0001:00849fe4  _UI_add_verify_string
0001:0084a031* _UI_dup_verify_string
0001:0084a0d2* _UI_add_input_boolean
0001:0084a11f* _UI_dup_input_boolean
0001:0084a2fc* _UI_add_info_string
0001:0084a34e* _UI_dup_info_string
0001:0084a3f4* _UI_add_error_string
0001:0084a446* _UI_dup_error_string
0001:0084a4f5* _UI_construct_prompt
0001:0084a660* _UI_add_user_data
0001:0084a67d* _UI_get0_user_data
0001:0084a688* _UI_get0_result
0001:0084ad1f  _UI_get0_result_string
0001:0084a78f  _UI_process
0001:0084a939* _UI_ctrl
0001:0084aa15* _UI_get_ex_new_index
0001:0084aa4c* _UI_set_ex_data
0001:0084aa70* _UI_get_ex_data
0001:0084aa8d* _UI_set_default_method
0001:0084aaba* _UI_get_method
0001:0084aac4* _UI_set_method
0001:0084aad6* _UI_create_method
0001:0084ab31* _UI_destroy_method
0001:0084ab5a* _UI_method_set_opener
0001:0084ab7a* _UI_method_set_writer
0001:0084ab9a* _UI_method_set_flusher
0001:0084abba* _UI_method_set_reader
0001:0084abda* _UI_method_set_closer
0001:0084abfa* _UI_method_set_prompt_constructor
0001:0084ac1a* _UI_method_get_opener
0001:0084ac32* _UI_method_get_writer
0001:0084ac4a* _UI_method_get_flusher
0001:0084ac62* _UI_method_get_reader
0001:0084ac7a* _UI_method_get_closer
0001:0084ac92* _UI_method_get_prompt_constructor
0001:0084acaa  _UI_get_string_type
0001:0084acc1  _UI_get_input_flags
0001:0084acd9  _UI_get0_output_string
0001:0084acf1  _UI_get0_action_string
0001:0084ad49  _UI_get0_test_string
0001:0084ad72* _UI_get_result_minsize
0001:0084ad9c* _UI_get_result_maxsize
0001:0084adec  _UI_set_result
Module: U:\extras\lib\libcrypto.lib(t_pkey.obj)
0001:0084b0f9  _ASN1_bn_print
Module: U:\extras\lib\libcrypto.lib(pk7_lib.obj)
0001:0084b34a  _PKCS7_ctrl
0001:0084b4cb* _PKCS7_content_new
0001:0084b5f1  _PKCS7_set_type
0001:0084b538* _PKCS7_set_content
0001:0084b88d* _PKCS7_set0_type_other
0001:0084b8b4* _PKCS7_add_signer
0001:0084ba7d* _PKCS7_add_certificate
0001:0084bba5* _PKCS7_add_crl
0001:0084bccd* _PKCS7_SIGNER_INFO_set
0001:0084be82* _PKCS7_add_signature
0001:0084bf68* _PKCS7_set_digest
0001:0084c03f* _PKCS7_get_signer_info
0001:0084c088  _PKCS7_SIGNER_INFO_get0_algs
0001:0084c0c0  _PKCS7_RECIP_INFO_get0_alg
0001:0084c0d6* _PKCS7_add_recipient
0001:0084c1d1* _PKCS7_RECIP_INFO_set
0001:0084c13a* _PKCS7_add_recipient_info
0001:0084c3bf* _PKCS7_cert_from_signer_info
0001:0084c40b* _PKCS7_set_cipher
0001:0084c4e3  _PKCS7_stream
Module: U:\extras\lib\libcrypto.lib(cms_sd.obj)
0001:0084c71c* _CMS_SignedData_init
0001:0084d2f7* _CMS_get0_SignerInfos
0001:0084ca58  _cms_set1_SignerIdentifier
0001:0084cbc0  _cms_SignerIdentifier_get0_signer_id
0001:0084cc24  _cms_SignerIdentifier_cert_cmp
0001:0084ccd9* _CMS_add1_signer
0001:0084e22f* _CMS_add_standard_smimecap
0001:0084e051* _CMS_add_smimecap
0001:0084d902* _CMS_SignerInfo_sign
0001:0084d320* _CMS_get0_signers
0001:0084d3c1* _CMS_SignerInfo_set1_signer_cert
0001:0084d447* _CMS_SignerInfo_get0_signer_id
0001:0084d472* _CMS_SignerInfo_cert_cmp
0001:0084d48f* _CMS_set1_signers_certs
0001:0084d604  _CMS_SignerInfo_get0_algs
0001:0084d882  _cms_SignedData_final
0001:0084dbb6* _CMS_SignerInfo_verify
0001:0084dd54  _cms_SignedData_init_bio
0001:0084de23* _CMS_SignerInfo_verify_content
0001:0084e0bc* _CMS_add_simple_smimecap
Module: U:\extras\lib\libcrypto.lib(cms_env.obj)
0001:0084e4ad* _CMS_get0_RecipientInfos
0001:0084e4d6* _CMS_RecipientInfo_type
0001:0084e4e0* _CMS_EnvelopedData_create
0001:0084e581* _CMS_add1_recipient_cert
0001:0084e818  _CMS_RecipientInfo_ktri_get0_algs
0001:0084e89d* _CMS_RecipientInfo_ktri_get0_signer_id
0001:0084e90d* _CMS_RecipientInfo_ktri_cert_cmp
0001:0084e969* _CMS_RecipientInfo_set0_pkey
0001:0084ee3c* _CMS_RecipientInfo_kekri_id_cmp
0001:0084eef2* _CMS_add0_recipient_key
0001:0084f198* _CMS_RecipientInfo_kekri_get0_id
0001:0084f277* _CMS_RecipientInfo_set0_key
0001:0084f737* _CMS_RecipientInfo_decrypt
0001:0084f7a8  _cms_EnvelopedData_init_bio
Module: U:\extras\lib\libcrypto.lib(ec_print.obj)
0001:0084f94b  _EC_POINT_point2bn
0001:0084fa36* _EC_POINT_bn2point
0001:0084fb6b* _EC_POINT_point2hex
0001:0084fcda* _EC_POINT_hex2point
Module: U:\extras\lib\libcrypto.lib(eck_prn.obj)
0001:0084fd4a* _ECPKParameters_print_fp
0001:0085004c  _ECPKParameters_print
0001:0084fde7* _EC_KEY_print_fp
0001:0084ff1a* _EC_KEY_print
0001:0084fe84* _ECParameters_print_fp
0001:0084ff7f* _ECParameters_print
Module: U:\extras\lib\libcrypto.lib(a_bytes.obj)
0001:00850a3a* _d2i_ASN1_type_bytes
0001:00850c2e  _i2d_ASN1_bytes
0001:00850d1a* _d2i_ASN1_bytes
Module: U:\extras\lib\libcrypto.lib(pcy_node.obj)
0001:008511c8  _policy_node_cmp_new
0001:008511dd  _tree_find_sk
0001:00851225  _level_find_node
0001:0085129f  _level_add_node
0001:008513d4  _policy_node_free
0001:008513e7  _policy_node_match
Module: U:\extras\lib\libcrypto.lib(pcy_lib.obj)
0001:008514a0* _X509_policy_tree_level_count
0001:008514b8* _X509_policy_tree_get0_level
0001:008514e8* _X509_policy_tree_get0_policies
0001:00851500  _X509_policy_tree_get0_user_policies
0001:0085152d* _X509_policy_level_node_count
0001:0085157a* _X509_policy_level_get0_node
0001:008515bf* _X509_policy_node_get0_policy
0001:008515d9* _X509_policy_node_get0_qualifiers
0001:008515f3* _X509_policy_node_get0_parent
Module: U:\extras\lib\libcrypto.lib(o_time.obj)
0001:00851610  _OPENSSL_gmtime
0001:0085165d  _OPENSSL_gmtime_adj
Module: U:\extras\lib\libcrypto.lib(asn1_gen.obj)
0001:00851b30* _ASN1_generate_nconf
0001:00851b82  _ASN1_generate_v3
Module: U:\extras\lib\libcrypto.lib(a_bool.obj)
0001:00853520* _i2d_ASN1_BOOLEAN
0001:008535a5  _d2i_ASN1_BOOLEAN
Module: U:\extras\lib\libcrypto.lib(b_dump.obj)
0001:00853680* _BIO_dump_cb
0001:008536e3* _BIO_dump_indent_cb
0001:00853a99* _BIO_dump_fp
0001:00853ac2* _BIO_dump_indent_fp
0001:00853b13* _BIO_dump
0001:00853b3c  _BIO_dump_indent
Module: U:\extras\lib\libcrypto.lib(a_strnid.obj)
0001:00853b70* _ASN1_STRING_set_default_mask
0001:00853b7d* _ASN1_STRING_get_default_mask
0001:00853bab* _ASN1_STRING_set_default_mask_asc
0001:00853cb7  _ASN1_STRING_set_by_NID
0001:00853f91* _ASN1_STRING_TABLE_get
0001:0085401b* _ASN1_STRING_TABLE_add
0001:00854167* _ASN1_STRING_TABLE_cleanup
Module: U:\extras\lib\libcrypto.lib(a_print.obj)
0001:008541c0  _ASN1_PRINTABLE_type
0001:008542ce* _ASN1_UNIVERSALSTRING_to_string
Module: U:\extras\lib\libcrypto.lib(err_prn.obj)
0001:008543e2  _ERR_print_errors_cb
0001:00854555* _ERR_print_errors_fp
0001:00854591  _ERR_print_errors
Module: U:\extras\lib\libcrypto.lib(v3_prn.obj)
0001:008545c9* _X509V3_EXT_val_prn
0001:0085473a* _X509V3_EXT_print
0001:008549b0  _X509V3_extensions_print
0001:00854c89* _X509V3_EXT_print_fp
Module: U:\extras\lib\libcrypto.lib(t_x509a.obj)
0001:00854d6f  _X509_CERT_AUX_print
Module: U:\extras\lib\libcrypto.lib(p5_pbe.obj)
0001:008550c0* _PBEPARAM_it
0001:008550dc  _d2i_PBEPARAM
0001:00855105* _i2d_PBEPARAM
0001:00855127* _PBEPARAM_new
0001:0085513b  _PBEPARAM_free
0001:0085515f* _PKCS5_pbe_set0_algor
0001:00855374  _PKCS5_pbe_set
Module: U:\extras\lib\libcrypto.lib(p12_key.obj)
0001:0085540a  _PKCS12_key_gen_asc
0001:008554fb* _PKCS12_key_gen_uni
Module: U:\extras\lib\libcrypto.lib(p5_pbev2.obj)
0001:00855a20* _PBE2PARAM_it
0001:00855a3c  _d2i_PBE2PARAM
0001:00855a65* _i2d_PBE2PARAM
0001:00855a87* _PBE2PARAM_new
0001:00855a9b  _PBE2PARAM_free
0001:00855b30* _PBKDF2PARAM_it
0001:00855b4c  _d2i_PBKDF2PARAM
0001:00855b75* _i2d_PBKDF2PARAM
0001:00855b97* _PBKDF2PARAM_new
0001:00855bab  _PBKDF2PARAM_free
0001:00855bd1* _PKCS5_pbe2_set_iv
0001:0085610d  _PKCS5_pbe2_set
Module: U:\extras\lib\libcrypto.lib(eng_ctrl.obj)
0001:00856582* _ENGINE_ctrl
0001:0085676b* _ENGINE_cmd_is_executable
0001:00856803* _ENGINE_ctrl_cmd
0001:00856906  _ENGINE_ctrl_cmd_string
Module: U:\extras\lib\libcrypto.lib(conf_lib.obj)
0001:00856c80* _CONF_version
0001:00856ca7  _CONF_set_nconf
0001:00856cdb* _CONF_set_default_method
0001:00856cfb* _CONF_load
0001:00856e04* _CONF_load_bio
0001:00856d83* _CONF_load_fp
0001:008571a6* _NCONF_load_bio
0001:00856e4a  _CONF_get_section
0001:00857205  _NCONF_get_section
0001:00856e83  _CONF_get_string
0001:0085729f  _NCONF_get_string
0001:00856ed8* _CONF_get_number
0001:00857365* _NCONF_get_number_e
0001:00856f56  _CONF_free
0001:008570a5* _NCONF_free_data
0001:00856f7b* _CONF_dump_fp
0001:00856ff5* _CONF_dump_bio
0001:008574b8* _NCONF_dump_bio
0001:00857021  _NCONF_new
0001:00857084  _NCONF_free
0001:008570c6  _NCONF_load
0001:00857125* _NCONF_load_fp
0001:0085743e* _NCONF_dump_fp
Module: U:\extras\lib\libcrypto.lib(x509_req.obj)
0001:0085751b* _X509_to_X509_REQ
0001:00857651* _X509_REQ_get_pubkey
0001:0085767f* _X509_REQ_check_private_key
0001:008577f4* _X509_REQ_extension_nid
0001:00857836* _X509_REQ_get_extension_nids
0001:00857840* _X509_REQ_set_extension_nids
0001:0085784d  _X509_REQ_get_extensions
0001:00857ae5* _X509_REQ_get_attr_by_NID
0001:00857b31* _X509_REQ_get_attr
0001:00857967* _X509_REQ_add_extensions_nid
0001:00857aab  _X509_REQ_add_extensions
0001:00857acd* _X509_REQ_get_attr_count
0001:00857b0b* _X509_REQ_get_attr_by_OBJ
0001:00857b50* _X509_REQ_delete_attr
0001:00857b6f* _X509_REQ_add1_attr
0001:00857b9e* _X509_REQ_add1_attr_by_OBJ
0001:00857be2* _X509_REQ_add1_attr_by_NID
0001:00857c26* _X509_REQ_add1_attr_by_txt
Module: U:\extras\lib\libcrypto.lib(conf_mod.obj)
0001:00857ccf* _CONF_modules_load
0001:00857df0* _CONF_modules_load_file
0001:00858777* _CONF_get1_default_config_file
0001:00858521* _CONF_modules_unload
0001:008585fb* _CONF_modules_finish
0001:0085869f* _CONF_module_add
0001:008586d8* _CONF_modules_free
0001:008586f1* _CONF_imodule_get_name
0001:008586fc* _CONF_imodule_get_value
0001:00858707* _CONF_imodule_get_usr_data
0001:00858712* _CONF_imodule_set_usr_data
0001:00858720* _CONF_imodule_get_module
0001:0085872a* _CONF_imodule_get_flags
0001:00858735* _CONF_imodule_set_flags
0001:00858743* _CONF_module_get_usr_data
0001:0085874e* _CONF_module_set_usr_data
0001:00858848  _CONF_parse_list
Module: U:\extras\lib\libcrypto.lib(v3_pmaps.obj)
0001:008589a0  _v3_policy_mappings
0001:00858a90* _POLICY_MAPPINGS_it
0001:00858a40* _POLICY_MAPPING_it
0001:00858aac* _POLICY_MAPPING_new
0001:00858ac0  _POLICY_MAPPING_free
Module: U:\extras\lib\libcrypto.lib(bn_sqr.obj)
0001:00858e10  _BN_sqr
0001:008590b3* _bn_sqr_normal
0001:008591e2* _bn_sqr_recursive
Module: U:\extras\lib\libcrypto.lib(bn_recp.obj)
0001:00859490  _BN_RECP_CTX_init
0001:008594cf* _BN_RECP_CTX_new
0001:0085951b  _BN_RECP_CTX_free
0001:0085955d  _BN_RECP_CTX_set
0001:008595b8  _BN_mod_mul_reciprocal
0001:0085968b* _BN_div_recp
0001:008599b6* _BN_reciprocal
Module: U:\extras\lib\libcrypto.lib(bn_prime.obj)
0001:0085aa50  _BN_GENCB_call
0001:0085aad0  _BN_generate_prime_ex
0001:0085ae24  _BN_is_prime_fasttest_ex
0001:0085adf4  _BN_is_prime_ex
Module: U:\extras\lib\libcrypto.lib(bn_exp2.obj)
0001:0085b8da  _BN_mod_exp2_mont
Module: U:\extras\lib\libcrypto.lib(v3_bitst.obj)
0001:0085c250  _v3_nscert
0001:0085c2c8* _i2v_ASN1_BIT_STRING
0001:0085c344* _v2i_ASN1_BIT_STRING
0001:0085c290  _v3_key_usage
Module: U:\extras\lib\libcrypto.lib(v3_ia5.obj)
0001:0085c520  _v3_ns_ia5_list
Module: U:\extras\lib\libcrypto.lib(v3_skey.obj)
0001:0085c860  _v3_skey_id
0001:0085c898* _i2s_ASN1_OCTET_STRING
0001:0085c8c1* _s2i_ASN1_OCTET_STRING
Module: U:\extras\lib\libcrypto.lib(v3_pku.obj)
0001:0085cb40  _v3_pkey_usage_period
0001:0085cbd0* _PKEY_USAGE_PERIOD_it
0001:0085cbec* _d2i_PKEY_USAGE_PERIOD
0001:0085cc15* _i2d_PKEY_USAGE_PERIOD
0001:0085cc37* _PKEY_USAGE_PERIOD_new
0001:0085cc4b* _PKEY_USAGE_PERIOD_free
Module: U:\extras\lib\libcrypto.lib(v3_int.obj)
0001:0085cd50  _v3_crl_num
0001:0085cd90  _v3_delta_crl
0001:0085cdf0  _v3_inhibit_anyp
Module: U:\extras\lib\libcrypto.lib(v3_akey.obj)
0001:0085ce30  _v3_akey_id
Module: U:\extras\lib\libcrypto.lib(v3_extku.obj)
0001:0085d320  _v3_ext_ku
0001:0085d3d0* _EXTENDED_KEY_USAGE_it
0001:0085d360  _v3_ocsp_accresp
0001:0085d3ec* _d2i_EXTENDED_KEY_USAGE
0001:0085d415* _i2d_EXTENDED_KEY_USAGE
0001:0085d437* _EXTENDED_KEY_USAGE_new
0001:0085d44b* _EXTENDED_KEY_USAGE_free
Module: U:\extras\lib\libcrypto.lib(v3_enum.obj)
0001:0085d7a0  _v3_crl_reason
0001:0085d7d8* _i2s_ASN1_ENUMERATED_TABLE
Module: U:\extras\lib\libcrypto.lib(v3_ocsp.obj)
0001:0085d840  _v3_ocsp_crlid
0001:0085d880  _v3_ocsp_acutoff
0001:0085d8c0  _v3_crl_invdate
0001:0085d900  _v3_crl_hold
0001:0085d940  _v3_ocsp_nonce
0001:0085d980  _v3_ocsp_nocheck
0001:0085d9c0  _v3_ocsp_serviceloc
Module: U:\extras\lib\libcrypto.lib(v3_sxnet.obj)
0001:0085df50  _v3_sxnet
0001:0085e0b0* _SXNET_it
0001:0085dfd0* _SXNETID_it
0001:0085dfec* _d2i_SXNETID
0001:0085e015* _i2d_SXNETID
0001:0085e037* _SXNETID_new
0001:0085e04b* _SXNETID_free
0001:0085e0cc* _d2i_SXNET
0001:0085e0f5* _i2d_SXNET
0001:0085e117* _SXNET_new
0001:0085e12b* _SXNET_free
0001:0085e2e0* _SXNET_add_id_asc
0001:0085e3f6* _SXNET_add_id_INTEGER
0001:0085e35e* _SXNET_add_id_ulong
0001:0085e71d* _SXNET_get_id_INTEGER
0001:0085e601* _SXNET_get_id_asc
0001:0085e682* _SXNET_get_id_ulong
Module: U:\extras\lib\libcrypto.lib(v3_pci.obj)
0001:0085e790  _v3_pci
Module: U:\extras\lib\libcrypto.lib(pk7_doit.obj)
0001:0085fd53  _PKCS7_dataInit
0001:00860346* _PKCS7_dataDecode
0001:00861b00  _PKCS7_get_signed_attribute
0001:0086124d* _PKCS7_SIGNER_INFO_sign
0001:00860c9f  _PKCS7_dataFinal
0001:008614c4* _PKCS7_dataVerify
0001:0086168c* _PKCS7_signatureVerify
0001:00861bef* _PKCS7_digest_from_attributes
0001:00861a68* _PKCS7_get_issuer_and_serial
0001:00861b1d* _PKCS7_get_attribute
0001:00861c20* _PKCS7_set_signed_attributes
0001:00861ccc* _PKCS7_set_attributes
0001:00861d78  _PKCS7_add_signed_attribute
0001:00861da3* _PKCS7_add_attribute
Module: U:\extras\lib\libcrypto.lib(tasn_prn.obj)
0001:00861f3b* _ASN1_PCTX_new
0001:00861fcf* _ASN1_PCTX_free
0001:00861fe2* _ASN1_PCTX_get_flags
0001:00861fec* _ASN1_PCTX_set_flags
0001:00861ff9* _ASN1_PCTX_get_nm_flags
0001:00862004* _ASN1_PCTX_set_nm_flags
0001:00862012* _ASN1_PCTX_get_cert_flags
0001:0086201d* _ASN1_PCTX_set_cert_flags
0001:0086202b* _ASN1_PCTX_get_oid_flags
0001:00862036* _ASN1_PCTX_set_oid_flags
0001:00862044* _ASN1_PCTX_get_str_flags
0001:0086204f* _ASN1_PCTX_set_str_flags
0001:0086205d  _ASN1_item_print
0001:008626b0* _asn1_template_print_ctx
0002:00008270* _default_pctx
Module: U:\extras\lib\libcrypto.lib(ec2_smpl.obj)
0001:00863040  _EC_GF2m_simple_method
0001:0086304a* _ec_GF2m_simple_group_init
0001:00863083* _ec_GF2m_simple_group_finish
0001:008630b7* _ec_GF2m_simple_group_clear_finish
0001:00863127* _ec_GF2m_simple_group_copy
0001:0086332e  _ec_GF2m_simple_group_set_curve
0001:00863548* _ec_GF2m_simple_group_get_curve
0001:008635cd* _ec_GF2m_simple_group_get_degree
0001:008635e4* _ec_GF2m_simple_group_check_discriminant
0001:008636c5* _ec_GF2m_simple_point_init
0001:008636fc* _ec_GF2m_simple_point_finish
0001:0086372e* _ec_GF2m_simple_point_clear_finish
0001:0086376a* _ec_GF2m_simple_point_copy
0001:008637ec* _ec_GF2m_simple_point_set_to_infinity
0001:00863819* _ec_GF2m_simple_point_set_affine_coordinates
0001:0086391a* _ec_GF2m_simple_point_get_affine_coordinates
0001:00863a37* _ec_GF2m_simple_set_compressed_coordinates
0001:00863d87* _ec_GF2m_simple_point2oct
0001:008641d2* _ec_GF2m_simple_oct2point
0001:0086465c* _ec_GF2m_simple_add
0001:00864bf6* _ec_GF2m_simple_dbl
0001:00864c25* _ec_GF2m_simple_invert
0001:00864c9a* _ec_GF2m_simple_is_at_infinity
0001:00864cad* _ec_GF2m_simple_is_on_curve
0001:00864ec8* _ec_GF2m_simple_cmp
0001:008650a0* _ec_GF2m_simple_make_affine
0001:008651e7* _ec_GF2m_simple_points_make_affine
0001:00865239* _ec_GF2m_simple_field_mul
0001:0086526b* _ec_GF2m_simple_field_sqr
0001:00865296* _ec_GF2m_simple_field_div
Module: U:\extras\lib\libcrypto.lib(x509_att.obj)
0001:00865370  _X509at_get_attr_count
0001:00865383  _X509at_get_attr_by_NID
0001:008653bf  _X509at_get_attr_by_OBJ
0001:00865436  _X509at_get_attr
0001:00865473  _X509at_delete_attr
0001:008654c1  _X509at_add1_attr
0001:008655c9  _X509at_add1_attr_by_OBJ
0001:0086582f* _X509_ATTRIBUTE_create_by_OBJ
0001:0086562c  _X509at_add1_attr_by_NID
0001:008657a2* _X509_ATTRIBUTE_create_by_NID
0001:0086568f  _X509at_add1_attr_by_txt
0001:00865915* _X509_ATTRIBUTE_create_by_txt
0001:008656f2  _X509at_get0_data_by_OBJ
0001:00865bdd* _X509_ATTRIBUTE_count
0001:00865c2c* _X509_ATTRIBUTE_get0_data
0001:008659bf* _X509_ATTRIBUTE_set1_object
0001:008659fc* _X509_ATTRIBUTE_set1_data
0001:00865c15* _X509_ATTRIBUTE_get0_object
0001:00865c9f* _X509_ATTRIBUTE_get0_type
Module: U:\extras\lib\libcrypto.lib(nsseq.obj)
0001:00865da0* _NETSCAPE_CERT_SEQUENCE_it
0001:00865dbc  _d2i_NETSCAPE_CERT_SEQUENCE
0001:00865de5  _i2d_NETSCAPE_CERT_SEQUENCE
0001:00865e07* _NETSCAPE_CERT_SEQUENCE_new
0001:00865e1b* _NETSCAPE_CERT_SEQUENCE_free
Module: U:\extras\lib\libcrypto.lib(x_pkey.obj)
0001:00865e40* _i2d_X509_PKEY
0001:00865e53* _d2i_X509_PKEY
0001:008660e3  _X509_PKEY_new
0001:008661fb  _X509_PKEY_free
Module: U:\extras\lib\libcrypto.lib(rsa_pss.obj)
0001:008662d2  _RSA_verify_PKCS1_PSS
0001:00866723  _RSA_padding_add_PKCS1_PSS
Module: U:\extras\lib\libcrypto.lib(rsa_gen.obj)
0001:00866a50  _RSA_generate_key_ex
Module: U:\extras\lib\libcrypto.lib(dh_gen.obj)
0001:008672d0  _DH_generate_parameters_ex
Module: U:\extras\lib\libcrypto.lib(dsa_gen.obj)
0001:008675d0* _DSA_generate_parameters_ex
0001:008676a9  _dsa_builtin_paramgen
Module: U:\extras\lib\libcrypto.lib(dsa_key.obj)
0001:00867ff0  _DSA_generate_key
Module: U:\extras\lib\libcrypto.lib(p12_p8d.obj)
0001:008681f0  _PKCS8_decrypt
Module: U:\extras\lib\libcrypto.lib(pem_pk8.obj)
0001:00868230* _PEM_write_bio_PKCS8PrivateKey_nid
0001:0086827d  _PEM_write_bio_PKCS8PrivateKey
0001:008682ca* _i2d_PKCS8PrivateKey_bio
0001:00868317* _i2d_PKCS8PrivateKey_nid_bio
0001:008689c5* _PEM_write_bio_PKCS8
0001:00868ae9* _PEM_write_bio_PKCS8_PRIV_KEY_INFO
0001:00868574* _d2i_PKCS8PrivateKey_bio
0001:008686d6* _i2d_PKCS8PrivateKey_fp
0001:00868723* _i2d_PKCS8PrivateKey_nid_fp
0001:00868770* _PEM_write_PKCS8PrivateKey_nid
0001:008687bd* _PEM_write_PKCS8PrivateKey
0001:008688b5* _d2i_PKCS8PrivateKey_fp
0001:00868953* _PEM_read_bio_PKCS8
0001:0086898c* _PEM_read_PKCS8
0001:00868a18* _PEM_write_PKCS8
0001:00868a77* _PEM_read_bio_PKCS8_PRIV_KEY_INFO
0001:00868ab0* _PEM_read_PKCS8_PRIV_KEY_INFO
0001:00868b3c* _PEM_write_PKCS8_PRIV_KEY_INFO
Module: U:\extras\lib\libcrypto.lib(ecp_nist.obj)
0001:00868b90  _EC_GFp_nist_method
0001:00868b9a* _ec_GFp_nist_group_copy
0001:00868bd1* _ec_GFp_nist_group_set_curve
0001:00868d71* _ec_GFp_nist_field_mul
0001:00868e5c* _ec_GFp_nist_field_sqr
Module: U:\extras\lib\libcrypto.lib(ecp_mont.obj)
0001:00868fe0  _EC_GFp_mont_method
0001:00868fea* _ec_GFp_mont_group_init
0001:0086901d* _ec_GFp_mont_group_finish
0001:00869086* _ec_GFp_mont_group_clear_finish
0001:008690ef* _ec_GFp_mont_group_copy
0001:0086923d* _ec_GFp_mont_group_set_curve
0001:00869446* _ec_GFp_mont_field_mul
0001:008694bb* _ec_GFp_mont_field_sqr
0001:00869530* _ec_GFp_mont_field_encode
0001:008695ae* _ec_GFp_mont_field_decode
0001:0086961c* _ec_GFp_mont_field_set_to_one
Module: U:\extras\lib\libcrypto.lib(ech_ossl.obj)
0001:00869744  _ECDH_OpenSSL
Module: U:\extras\lib\libcrypto.lib(tb_ecdh.obj)
0001:00869be4* _ENGINE_unregister_ECDH
0001:00869c13* _ENGINE_register_ECDH
0001:00869c5f* _ENGINE_register_all_ECDH
0001:00869c90* _ENGINE_set_default_ECDH
0001:00869cdc  _ENGINE_get_default_ECDH
0001:00869cf9  _ENGINE_get_ECDH
0001:00869d04* _ENGINE_set_ECDH
Module: U:\extras\lib\libcrypto.lib(ecs_ossl.obj)
0001:00869d35  _ECDSA_OpenSSL
Module: U:\extras\lib\libcrypto.lib(tb_ecdsa.obj)
0001:0086ad74* _ENGINE_unregister_ECDSA
0001:0086ada3* _ENGINE_register_ECDSA
0001:0086adef* _ENGINE_register_all_ECDSA
0001:0086ae20* _ENGINE_set_default_ECDSA
0001:0086ae6c  _ENGINE_get_default_ECDSA
0001:0086ae89  _ENGINE_get_ECDSA
0001:0086ae94* _ENGINE_set_ECDSA
Module: U:\extras\lib\libcrypto.lib(cbc128.obj)
0001:0086aeb0  _CRYPTO_cbc128_encrypt
0001:0086afdc  _CRYPTO_cbc128_decrypt
Module: U:\extras\lib\libcrypto.lib(cfb128.obj)
0001:0086b1a0  _CRYPTO_cfb128_encrypt
0001:0086b5a0  _CRYPTO_cfb128_1_encrypt
0001:0086b67d  _CRYPTO_cfb128_8_encrypt
Module: U:\extras\lib\libcrypto.lib(ofb128.obj)
0001:0086b6e0  _CRYPTO_ofb128_encrypt
Module: U:\extras\lib\libcrypto.lib(ui_openssl.obj)
0001:0086b80f  _UI_OpenSSL
Module: U:\extras\lib\libcrypto.lib(cms_asn1.obj)
0001:0086bff0  _CMS_IssuerAndSerialNumber_it
0001:0086c080* _CMS_OtherCertificateFormat_it
0001:0086c170  _CMS_CertificateChoices_it
0001:0086c200* _CMS_SignerIdentifier_it
0001:0086c290* _CMS_EncapsulatedContentInfo_it
0001:0086c410  _CMS_SignerInfo_it
0001:0086c4a0* _CMS_OtherRevocationInfoFormat_it
0001:0086c520  _CMS_RevocationInfoChoice_it
0001:0086c610  _CMS_SignedData_it
0001:0086c670* _CMS_OriginatorInfo_it
0001:0086c730* _CMS_EncryptedContentInfo_it
0001:0086c7f0  _CMS_KeyTransRecipientInfo_it
0001:0086c860  _CMS_OtherKeyAttribute_it
0001:0086c900* _CMS_RecipientKeyIdentifier_it
0001:0086c980* _CMS_KeyAgreeRecipientIdentifier_it
0001:0086c9f0* _CMS_RecipientEncryptedKey_it
0001:0086ca60* _CMS_OriginatorPublicKey_it
0001:0086caf0* _CMS_OriginatorIdentifierOrKey_it
0001:0086cbc0* _CMS_KeyAgreeRecipientInfo_it
0001:0086cc40* _CMS_KEKIdentifier_it
0001:0086cce0  _CMS_KEKRecipientInfo_it
0001:0086cd90* _CMS_PasswordRecipientInfo_it
0001:0086ce00* _CMS_OtherRecipientInfo_it
0001:0086cf90  _CMS_RecipientInfo_it
0001:0086d070  _CMS_EnvelopedData_it
0001:0086d110  _CMS_DigestedData_it
0001:0086d180  _CMS_EncryptedData_it
0001:0086d2a0* _CMS_AuthenticatedData_it
0001:0086d330* _CMS_CompressedData_it
0001:0086d5c0  _CMS_ContentInfo_it
0001:0086d620  _CMS_Attributes_Sign_it
0001:0086d670  _CMS_Attributes_Verify_it
0001:0086d6f0* _CMS_ReceiptsFrom_it
0001:0086d790* _CMS_ReceiptRequest_it
0001:0086d830* _CMS_Receipt_it
Module: U:\extras\lib\libcrypto.lib(cms_att.obj)
0001:0086d850  _CMS_signed_get_attr_count
0001:0086d866  _CMS_signed_get_attr_by_NID
0001:0086d88a* _CMS_signed_get_attr_by_OBJ
0001:0086d8ae* _CMS_signed_get_attr
0001:0086d8cb* _CMS_signed_delete_attr
0001:0086d8e8* _CMS_signed_add1_attr
0001:0086d915* _CMS_signed_add1_attr_by_OBJ
0001:0086d957  _CMS_signed_add1_attr_by_NID
0001:0086d999* _CMS_signed_add1_attr_by_txt
0001:0086d9db  _CMS_signed_get0_data_by_OBJ
0001:0086da06* _CMS_unsigned_get_attr_count
0001:0086da1c* _CMS_unsigned_get_attr_by_NID
0001:0086da40* _CMS_unsigned_get_attr_by_OBJ
0001:0086da64* _CMS_unsigned_get_attr
0001:0086da81* _CMS_unsigned_delete_attr
0001:0086da9e* _CMS_unsigned_add1_attr
0001:0086dacb* _CMS_unsigned_add1_attr_by_OBJ
0001:0086db0d* _CMS_unsigned_add1_attr_by_NID
0001:0086db4f* _CMS_unsigned_add1_attr_by_txt
0001:0086db91* _CMS_unsigned_get0_data_by_OBJ
Module: U:\extras\lib\libcrypto.lib(cms_lib.obj)
0001:0086dbc0  _d2i_CMS_ContentInfo
0001:0086dbe9  _i2d_CMS_ContentInfo
0001:0086dc0b  _CMS_ContentInfo_new
0001:0086dc1f  _CMS_ContentInfo_free
0001:0086dc3a* _CMS_ContentInfo_print_ctx
0001:0086dc6a* _CMS_get0_type
0001:0086dc74* _priv_cms_Data_create
0001:0086e2a3* _CMS_set_detached
0001:0086dcb1* _cms_content_bio
0001:0086e038  _CMS_get0_content
0001:0086dd36  _CMS_dataInit
0001:0086de79  _CMS_dataFinal
0001:0086e1de  _CMS_get0_eContentType
0001:0086e206* _CMS_set1_eContentType
0001:0086e26b* _CMS_is_detached
0001:0086e35c  _cms_DigestAlgorithm_set
0001:0086e3b2  _cms_DigestAlgorithm_init_bio
0001:0086e4ba  _cms_DigestAlgorithm_find_ctx
0001:0086e627* _CMS_add0_CertificateChoices
0001:0086e6c0* _CMS_add0_cert
0001:0086e7b6  _CMS_add1_cert
0001:0086e875* _CMS_add0_RevocationInfoChoice
0001:0086e90e* _CMS_add0_crl
0001:0086e948* _CMS_add1_crl
0001:0086e99c* _CMS_get1_certs
0001:0086ea98* _CMS_get1_crls
Module: U:\extras\lib\libcrypto.lib(cms_enc.obj)
0001:0086ebaa  _cms_EncryptedContent_init_bio
0001:0086f05f  _cms_EncryptedContent_init
0001:0086f0eb* _CMS_EncryptedData_set1_key
0001:0086f21f  _cms_EncryptedData_init_bio
Module: U:\extras\lib\libcrypto.lib(aes_wrap.obj)
0001:0086f268  _AES_wrap_key
0001:0086f3e0  _AES_unwrap_key
Module: U:\extras\lib\libcrypto.lib(asn_pack.obj)
0001:0086f59b* _ASN1_seq_unpack
0001:0086f619* _ASN1_seq_pack
0001:0086f73f* _ASN1_unpack_string
0001:0086f7a4* _ASN1_pack_string
0001:0086f8e6  _ASN1_item_pack
0001:0086fa1b  _ASN1_item_unpack
Module: U:\extras\lib\libcrypto.lib(p12_utl.obj)
0001:0086fa9a  _OPENSSL_asc2uni
0001:0086fb53* _OPENSSL_uni2asc
0001:0086fbe3* _i2d_PKCS12_bio
0001:0086fc05* _i2d_PKCS12_fp
0001:0086fc27* _d2i_PKCS12_bio
0001:0086fc49* _d2i_PKCS12_fp
0001:0086fc6b* _PKCS12_x5092certbag
0001:0086fc96* _PKCS12_x509crl2certbag
0001:0086fcc1* _PKCS12_certbag2x509
0001:0086fd1b* _PKCS12_certbag2x509crl
Module: U:\extras\lib\libcrypto.lib(conf_def.obj)
0001:0086fd80* _CONF_def_version
0001:0086fdc1  _NCONF_default
0001:0086fdcb* _NCONF_WIN32
Module: U:\extras\lib\libcrypto.lib(conf_api.obj)
0001:008713bf  __CONF_get_section
0001:00871402  __CONF_get_section_values
0001:00871432  __CONF_add_string
0001:008714d9  __CONF_get_string
0001:008716b3  __CONF_new_data
0001:00871704  __CONF_free_data
0001:00871843  __CONF_new_section
Module: U:\extras\lib\libcrypto.lib(x509rset.obj)
0001:00871960* _X509_REQ_set_version
0001:0087198c  _X509_REQ_set_subject_name
0001:008719c1  _X509_REQ_set_pubkey
Module: U:\extras\lib\libcrypto.lib(dso_lib.obj)
0001:00871a00* _DSO_new
0001:00871a5a* _DSO_new_method
0001:00871a14* _DSO_set_default_method
0001:00871a21* _DSO_get_default_method
0001:00871a2b* _DSO_get_method
0001:00871a35* _DSO_set_method
0001:00871b9a  _DSO_free
0001:00871d16* _DSO_flags
0001:00871d2e* _DSO_up_ref
0001:00871da2  _DSO_load
0001:00872192* _DSO_ctrl
0001:00872332* _DSO_set_filename
0001:00871fc6* _DSO_bind_var
0001:008720ac  _DSO_bind_func
0001:0087228b* _DSO_set_name_converter
0001:008722eb* _DSO_get_filename
0001:00872464* _DSO_merge
0001:0087251a* _DSO_convert_filename
0001:00872696* _DSO_get_loaded_filename
0001:008726dd* _DSO_pathbyaddr
0001:00872754* _DSO_global_lookup
Module: U:\extras\lib\libcrypto.lib(f_int.obj)
0001:008727c8  _i2a_ASN1_INTEGER
0001:00872936* _a2i_ASN1_INTEGER
Module: U:\extras\lib\libcrypto.lib(f_string.obj)
0001:00872d45  _i2a_ASN1_STRING
0001:00872e7c* _a2i_ASN1_STRING
Module: U:\extras\lib\libcrypto.lib(bio_md.obj)
0001:0087326f  _BIO_f_md
Module: U:\extras\lib\libcrypto.lib(bio_enc.obj)
0001:00873707  _BIO_f_cipher
0001:0087404a* _BIO_set_cipher
Module: U:\extras\lib\libcrypto.lib(bss_null.obj)
0001:00874135  _BIO_s_null
Module: U:\extras\lib\libcrypto.lib(pk7_attr.obj)
0001:0087423b* _PKCS7_add_attrib_smimecap
0001:008742c8* _PKCS7_get_smimecap
0001:00874330* _PKCS7_simple_smimecap
0001:008744a7* _PKCS7_add_attrib_content_type
0001:00874504  _PKCS7_add0_attrib_signing_time
0001:00874584  _PKCS7_add1_attrib_digest
Module: U:\extras\lib\libcrypto.lib(bn_gf2m.obj)
0001:008748c1  _BN_GF2m_add
0001:00874a06  _BN_GF2m_mod_arr
0001:00874e70* _BN_GF2m_mod
0001:008762bb  _BN_GF2m_poly2arr
0001:00874f47  _BN_GF2m_mod_mul_arr
0001:008752b3  _BN_GF2m_mod_sqr_arr
0001:008751ca* _BN_GF2m_mod_mul
0001:008754f7* _BN_GF2m_mod_sqr
0001:008755d5* _BN_GF2m_mod_inv
0001:0087580d* _BN_GF2m_mod_inv_arr
0001:00876377* _BN_GF2m_arr2poly
0001:00875888  _BN_GF2m_mod_div
0001:0087592a* _BN_GF2m_mod_div_arr
0001:008759ac* _BN_GF2m_mod_exp_arr
0001:00875b17* _BN_GF2m_mod_exp
0001:00875c00  _BN_GF2m_mod_sqrt_arr
0001:00875ca8* _BN_GF2m_mod_sqrt
0001:00875d86  _BN_GF2m_mod_solve_quad_arr
0001:008761dd* _BN_GF2m_mod_solve_quad
Module: U:\extras\lib\libcrypto.lib(ec2_mult.obj)
0001:00877006  _ec_GF2m_simple_mul
0001:0087727f  _ec_GF2m_precompute_mult
0001:00877299  _ec_GF2m_have_precompute_mult
Module: U:\extras\lib\libcrypto.lib(p12_decr.obj)
0001:008772bb* _PKCS12_pbe_crypt
0001:0087746d  _PKCS12_item_decrypt_d2i
0001:00877575  _PKCS12_item_i2d_encrypt
Module: U:\extras\lib\libcrypto.lib(p12_p8e.obj)
0001:008776da  _PKCS8_encrypt
Module: U:\extras\lib\libcrypto.lib(ecp_smpl.obj)
0001:00877860* _EC_GFp_simple_method
0001:0087786a  _ec_GFp_simple_group_init
0001:008778b0  _ec_GFp_simple_group_finish
0001:008778e4  _ec_GFp_simple_group_clear_finish
0001:00877918  _ec_GFp_simple_group_copy
0001:008779b0  _ec_GFp_simple_group_set_curve
0001:00877c1b  _ec_GFp_simple_group_get_curve
0001:00877d7e  _ec_GFp_simple_group_get_degree
0001:00877d94  _ec_GFp_simple_group_check_discriminant
0001:00878075  _ec_GFp_simple_point_init
0001:008780b6  _ec_GFp_simple_point_finish
0001:008780e8  _ec_GFp_simple_point_clear_finish
0001:00878124  _ec_GFp_simple_point_copy
0001:008781a6  _ec_GFp_simple_point_set_to_infinity
0001:008781d3  _ec_GFp_simple_set_Jprojective_coordinates_GFp
0001:00878426  _ec_GFp_simple_get_Jprojective_coordinates_GFp
0001:008785ad  _ec_GFp_simple_point_set_affine_coordinates
0001:00878624  _ec_GFp_simple_point_get_affine_coordinates
0001:00878a58  _ec_GFp_simple_set_compressed_coordinates
0001:0087907b  _ec_GFp_simple_point2oct
0001:0087947d  _ec_GFp_simple_oct2point
0001:008798be  _ec_GFp_simple_add
0001:0087a0cb  _ec_GFp_simple_dbl
0001:0087a77c  _ec_GFp_simple_invert
0001:0087a7cd  _ec_GFp_simple_is_at_infinity
0001:0087a7e0  _ec_GFp_simple_is_on_curve
0001:0087ac2e  _ec_GFp_simple_cmp
0001:0087afbe  _ec_GFp_simple_make_affine
0001:0087b110  _ec_GFp_simple_points_make_affine
0001:0087b80f* _ec_GFp_simple_field_mul
0001:0087b841* _ec_GFp_simple_field_sqr
Module: U:\extras\lib\libcrypto.lib(bn_nist.obj)
0001:0087bdb4  _BN_get0_nist_prime_192
0001:0087bdbe  _BN_get0_nist_prime_224
0001:0087bdc8  _BN_get0_nist_prime_256
0001:0087bdd2  _BN_get0_nist_prime_384
0001:0087bddc  _BN_get0_nist_prime_521
0001:0087be7b  _BN_nist_mod_192
0001:0087c18a  _BN_nist_mod_224
0001:0087c5b4  _BN_nist_mod_256
0001:0087cb4c  _BN_nist_mod_384
0001:0087d1ea  _BN_nist_mod_521
Module: U:\extras\lib\libcrypto.lib(cms_io.obj)
0001:0087d539  _CMS_stream
0001:0087d5e6* _d2i_CMS_bio
0001:0087d608* _i2d_CMS_bio
0001:0087d62e* _PEM_read_bio_CMS
0001:0087d667* _PEM_read_CMS
0001:0087d6a0* _PEM_write_bio_CMS
0001:0087d6f3* _PEM_write_CMS
0001:0087d746* _BIO_new_CMS
0001:0087d768* _i2d_CMS_bio_stream
0001:0087d798* _PEM_write_bio_CMS_stream
0001:0087d7d0* _SMIME_write_CMS
0001:0087d856* _SMIME_read_CMS
Module: U:\extras\lib\libcrypto.lib(cms_dd.obj)
0001:0087d880* _cms_DigestedData_create
0001:0087d91f  _cms_DigestedData_init_bio
0001:0087d947  _cms_DigestedData_do_final
Module: U:\extras\lib\libcrypto.lib(a_set.obj)
0001:0087db0c  _i2d_ASN1_SET
0001:0087de37  _d2i_ASN1_SET
Module: U:\extras\lib\libcrypto.lib(p12_asn.obj)
0001:0087e290* _PKCS12_MAC_DATA_it
0001:0087e190  _PKCS12_it
0001:0087e1ac* _d2i_PKCS12
0001:0087e1d5* _i2d_PKCS12
0001:0087e1f7* _PKCS12_new
0001:0087e20b* _PKCS12_free
0001:0087e2ac* _d2i_PKCS12_MAC_DATA
0001:0087e2d5* _i2d_PKCS12_MAC_DATA
0001:0087e2f7* _PKCS12_MAC_DATA_new
0001:0087e30b* _PKCS12_MAC_DATA_free
0001:0087e430* _PKCS12_BAGS_it
0001:0087e44c* _d2i_PKCS12_BAGS
0001:0087e475* _i2d_PKCS12_BAGS
0001:0087e497  _PKCS12_BAGS_new
0001:0087e4ab* _PKCS12_BAGS_free
0001:0087e630* _PKCS12_SAFEBAG_it
0001:0087e64c* _d2i_PKCS12_SAFEBAG
0001:0087e675* _i2d_PKCS12_SAFEBAG
0001:0087e697  _PKCS12_SAFEBAG_new
0001:0087e6ab* _PKCS12_SAFEBAG_free
0001:0087e700  _PKCS12_SAFEBAGS_it
0001:0087e750  _PKCS12_AUTHSAFES_it
Module: U:\extras\lib\libcrypto.lib(p12_add.obj)
0001:0087e77a  _PKCS12_item_pack_safebag
0001:0087e886* _PKCS12_MAKE_KEYBAG
0001:0087e8ec* _PKCS12_MAKE_SHKEYBAG
0001:0087e9ee* _PKCS12_pack_p7data
0001:0087eaf2* _PKCS12_unpack_p7data
0001:0087eb56* _PKCS12_pack_p7encdata
0001:0087ed44* _PKCS12_unpack_p7encdata
0001:0087eda8* _PKCS12_decrypt_skey
0001:0087edcc* _PKCS12_pack_authsafes
0001:0087ee04* _PKCS12_unpack_authsafes
Module: U:\extras\lib\libcrypto.lib(dso_openssl.obj)
0001:0087ee70  _DSO_METHOD_openssl
Module: U:\extras\lib\libcrypto.lib(bn_sqrt.obj)
0001:0087ee8a  _BN_mod_sqrt
Module: U:\extras\lib\libcrypto.lib(bn_kron.obj)
0001:0087f9f0  _BN_kronecker
Module: U:\extras\lib\libcrypto.lib(bio_ndef.obj)
0001:0087fd7b  _BIO_new_NDEF
Module: U:\extras\lib\libcrypto.lib(asn_mime.obj)
0001:0088026d  _i2d_ASN1_bio_stream
0001:008815d4* _SMIME_crlf_copy
0001:00880452  _PEM_write_bio_ASN1_stream
0001:00880a2d  _SMIME_write_ASN1
0001:00881054  _SMIME_read_ASN1
0001:0088175c* _SMIME_text
Module: U:\extras\lib\libcrypto.lib(dso_null.obj)
0001:008823bb  _DSO_METHOD_null
Module: U:\extras\lib\libcrypto.lib(bio_asn1.obj)
0001:008823d5  _BIO_f_asn1
0001:00882d1b  _BIO_asn1_set_prefix
0001:00882d44* _BIO_asn1_get_prefix
0001:00882d6d  _BIO_asn1_set_suffix
0001:00882d96* _BIO_asn1_get_suffix
Module: U:\extras\lib\libcrypto.lib(bio_b64.obj)
0001:00882dd0  _BIO_f_base64


                        +----------------------+
                        |   Imported Symbols   |
                        +----------------------+

Symbol                              Module
======                              ======

___libc_ForkRegisterModule          libc063
___init_dll                         libc063
___libc_Back_termDll                libc063
___libc_ForkDeregisterModule        libc063
__atfork_callback                   libc063
___moddi3                           libc063
___divdi3                           libc063
___libc_GLocaleCtype                libc063
___umoddi3                          libc063
_strlcat                            libc063
__alloca                            libc063
___udivdi3                          libc063
DosQueryMutexSem                    doscalls
DosReleaseMutexSem                  doscalls
DosRequestMutexSem                  doscalls
DosCloseMutexSem                    doscalls
DosCreateMutexSem                   doscalls
DosGetInfoBlocks                    doscalls
DosSleep                            doscalls
UniFreeUconvObject                  uconv
DosGetDateTime                      doscalls
DosQuerySysInfo                     doscalls
DosFreeModule                       doscalls
DosQueryProcAddr                    doscalls
DosSetFileLocks                     doscalls
DosQueryFileInfo                    doscalls
DosResetBuffer                      doscalls
DosSetFileSize                      doscalls
DosSetFilePtr                       doscalls
DosWrite                            doscalls
DosRead                             doscalls
DosClose                            doscalls
DosForceDelete                      doscalls
UniCreateUconvObject                uconv
UniStrToUcs                         uconv
UniStrFromUcs                       uconv
DosLoadModule                       doscalls
DosQueryPathInfo                    doscalls
DosDelete                           doscalls
DosOpen                             doscalls
DosScanEnv                          doscalls
DosQueryCurrentDisk                 doscalls
___fixunsdfdi                       libc063
___stderrp                          libc063
__errno                             libc063
_strlcpy                            libc063
_initgroups                         libc063
_getpwuid_r                         libc063
_getpwnam_r                         libc063
_getgrgid_r                         libc063
_getgrnam_r                         libc063
_hstrerror                          tcpip32
_inet_aton                          tcpip32
_gethostbyname                      tcpip32
_tcp_h_errno1                       tcpip32
_getprotobyname                     tcpip32
_inet_ntoa                          tcpip32
_getprotobynumber                   tcpip32
_getservbyport                      tcpip32
_getservbyname                      tcpip32
_inet_ntop                          tcpip32
_inet_pton                          tcpip32
_inet_addr                          tcpip32
_gethostbyaddr                      tcpip32
_gethostname                        tcpip32
DosQueryFSInfo                      doscalls
___stdinp                           libc063
___stdoutp                          libc063
__exit                              libc063
___threadid                         libc063
DosFreeThreadLocalMemory            doscalls
DosAllocThreadLocalMemory           doscalls
_isspace                            libc063
___flt_rounds                       libc063
__CRT_term                          libc063
__CRT_init                          libc063
__std_strdup                        libc063
__std_strnicmp                      libc063
__std_memcpy                        libc063
__std_floor                         libc063
__std_malloc                        libc063
__std_time                          libc063
__std_getenv                        libc063
__std_strftime                      libc063
__std_free                          libc063
__std_sin                           libc063
__std_cos                           libc063
__std_sqrt                          libc063
__std_atan2                         libc063
__std_acos                          libc063
__std_stricmp                       libc063
__std_strchr                        libc063
__std_calloc                        libc063
__std_strtoll                       libc063
__std_strtol                        libc063
__std_realloc                       libc063
__std_pow                           libc063
__std_strtod                        libc063
__std_memset                        libc063
__std_setlocale                     libc063
__std_printf                        libc063
__std_putchar                       libc063
__std_strcmp                        libc063
__std_strncat                       libc063
__std_strcpy                        libc063
__std_strncmp                       libc063
__std_memmove                       libc063
__std_memcmp                        libc063
__std_strncpy                       libc063
__std_sprintf                       libc063
__std_atoi                          libc063
__std_localtime                     libc063
__std_qsort                         libc063
__std_memchr                        libc063
__std_dup                           libc063
__std_fwrite                        libc063
__std_exit                          libc063
___signbit                          libc063
__std_stat                          libc063
__std_fputc                         libc063
__std_fprintf                       libc063
__std_strtoull                      libc063
__std_abort                         libc063
__std_strstr                        libc063
__std_opendir                       libc063
__std_readdir                       libc063
__std_closedir                      libc063
__std_lseek                         libc063
__std_read                          libc063
__std_mktime                        libc063
__std_write                         libc063
__std_mkstemp                       libc063
__std_unlink                        libc063
__std_dup2                          libc063
__std_close                         libc063
__std_strerror                      libc063
__std_utimes                        libc063
__std_access                        libc063
__std_gmtime                        libc063
__std_asctime                       libc063
__std_strcspn                       libc063
__std_ctime                         libc063
__std_vasprintf                     libc063
__std_strpbrk                       libc063
___libc_FH                          libc063
__libsocket_set_errno               tcpip32
__libsocket_accept                  tcpip32
___libc_TcpipAllocFH44              libc063
__libsocket_soclose                 tcpip32
__libsocket_sock_errno              tcpip32
__libsocket_send                    tcpip32
__libsocket_recv                    tcpip32
__std_sscanf                        libc063
__std_gmtime_r                      libc063
__libsocket_socket                  tcpip32
__libsocket_bind                    tcpip32
__libsocket_getsockname             tcpip32
__libsocket_listen                  tcpip32
__std_strrchr                       libc063
__std_localtime_r                   libc063
__std_getuid                        libc063
__std_getgid                        libc063
__std_getgroups                     libc063
__std_sigsetjmp                     libc063
__std_strtok_r                      libc063
__std_strtok                        libc063
__std_getrlimit                     libc063
__std_sysconf                       libc063
__std_mknod                         libc063
__std_mkfifo                        libc063
__std_isatty                        libc063
__std_ttyname                       libc063
__std_times                         libc063
__std_uname                         libc063
__std_getsid                        libc063
__std_getpgid                       libc063
__std_setpgid                       libc063
__std_setsid                        libc063
__std_getpgrp                       libc063
__std_getlogin                      libc063
__std_setegid                       libc063
__std_seteuid                       libc063
__std_setgid                        libc063
__std_setuid                        libc063
__std_getegid                       libc063
__std_geteuid                       libc063
__std_getppid                       libc063
__std_getpid                        libc063
__std_kill                          libc063
__std_gettimeofday                  libc063
__std_readdir_r                     libc063
__std_fstat                         libc063
__std_flock                         libc063
__std_fcntl                         libc063
__std_pwrite                        libc063
__std_ftruncate                     libc063
__std_pread                         libc063
__std_timezone                      libc063
__std_strcat                        libc063
__std_open                          libc063
__libsocket_shutdown                tcpip32
__libsocket_getsockopt              tcpip32
__libsocket_sendto                  tcpip32
__libsocket_connect                 tcpip32
__std_select                        libc063
__libsocket_socketpair              tcpip32
___libc_FHClose                     libc063
__libsocket_getpeername             tcpip32
__libsocket_recvfrom                tcpip32
__libsocket_setsockopt              tcpip32
__std_readlink                      libc063
__std_strtoul                       libc063
__std_getloadavg                    libc063
__std_umask                         libc063
__std_nanosleep                     libc063
__std_usleep                        libc063
__std_sleep                         libc063
__std_environ                       libc063
__std_putenv                        libc063
__std_tzset                         libc063
__std_unsetenv                      libc063
__std_strptime                      libc063
__std_glob                          libc063
__std_globfree                      libc063
__std_dlopen                        libc063
__std_dlsym                         libc063
__std_dlclose                       libc063
__std_dlerror                       libc063
__std_nice                          libc063
__std_mblen                         libc063
__std_fnmatch                       libc063
__std_fclose                        libc063
__std_localeconv                    libc063
__std_nl_langinfo                   libc063
__std_getc                          libc063
__std_fileno                        libc063
__std_link                          libc063
__std_symlink                       libc063
__std_popen                         libc063
__std_pclose                        libc063
__std_fmod                          libc063
__std_hypot                         libc063
__std_log10                         libc063
__std_log                           libc063
__std_log1p                         libc063
__std_expm1                         libc063
__std_exp                           libc063
__std_atanh                         libc063
__std_acosh                         libc063
__std_asinh                         libc063
__std_tanh                          libc063
__std_cosh                          libc063
__std_sinh                          libc063
__std_atan                          libc063
__std_asin                          libc063
__std_tan                           libc063
__std_ceil                          libc063
__std_rand_r                        libc063
__std_strcoll                       libc063
__std_ctime_r                       libc063
__getprogname                       libc063
__std_vsnprintf                     libc063
__std_writev                        libc063
__std_strspn                        libc063
__std_ftok                          libc063
__std_waitpid                       libc063
__std_fork                          libc063
__std_pipe                          libc063
__std_chdir                         libc063
__std_execle                        libc063
__std_perror                        libc063
__std_execl                         libc063
__std_fseek                         libc063
__std_fopen                         libc063
__std_ftell                         libc063
__std_clearerr                      libc063
__std_fread                         libc063
__std_remove                        libc063
__std_fdopen                        libc063
__std_rename                        libc063
__std_chmod                         libc063
__std_putc                          libc063
__std_atol                          libc063
__std_atof                          libc063
__std_lstat                         libc063
__std_rmdir                         libc063
__std_mkdir                         libc063
__std_creat                         libc063
__std_chown                         libc063
__std_lchown                        libc063
__std_utime                         libc063
__std_getcwd                        libc063
__std_asctime_r                     libc063
__std_fputs                         libc063
___strnlen                          libc063
__std_vsprintf                      libc063
__std_setmode                       libc063
__std_rewind                        libc063
__std_rewinddir                     libc063
__std_setvbuf                       libc063
__std_fflush                        libc063
__std_setitimer                     libc063
__std_signal                        libc063
__std_sigemptyset                   libc063
__std_sigaddset                     libc063
__std_sigprocmask                   libc063
__std_siglongjmp                    libc063
__std_snprintf                      libc063
DosTrueGetMessage                   msg
___ctordtorTerm1                    libc063
___ctordtorInit1                    libc063
__std_strlen                        libc063
__std_vfprintf                      libc063
__std_isinf                         libc063
__std_iconv_open                    libc063
__std_iconv_close                   libc063
__std_iconv                         libc063
__std_puts                          libc063
___deregister_frame                 libc063
___register_frame_table             libc063
__assert                            libc063
__std_ferror                        libc063
__std_feof                          libc063
__std_fgets                         libc063
DosTmrQueryTime                     doscalls
DosPerfSysCall                      doscalls
DosQuerySysState                    doscalls
__std_tcgetattr                     libc063
__std_tcsetattr                     libc063
__std_sigaction                     libc063


                        +--------------------+
                        |   Libraries Used   |
                        +--------------------+

U:\extras\lib\libz.lib
U:\extras\lib\xmlrpc.lib
U:\extras\lib\libssl.lib
U:\extras\lib\libcrypto.lib
U:\extras\lib\expat.lib
U:\extras\lib\xml2.lib
U:\usr\lib\libc_alias.lib
U:\usr\lib\libc_dll.lib
U:\usr\lib\libos2.lib
U:\tmp\ldconv_gcc444_a_92b84c4a69841efbf0.lib
U:\usr\lib\libend.lib


                        +-----------------------+
                        |   Linker Statistics   |
                        +-----------------------+

Stack size:  0000 (0.)
Memory size:  008a5cb0 (9067696.)
Link time: 00:02.63
